Archive member included to satisfy reference by file (symbol)

..\..\..\..\Libraries\libs\libplatform.a(audio.o)
                              Output\obj\Libraries\bsp\bsp_sys.o (adpll_init)
..\..\..\..\Libraries\libs\libplatform.a(cm.o)
                              Output\obj\Libraries\bsp\bsp_param.o (cm_sync)
..\..\..\..\Libraries\libs\libplatform.a(os_flash.o)
                              ..\..\..\..\Libraries\libs\libplatform.a(cm.o) (os_spiflash_read)
..\..\..\..\Libraries\libs\libplatform.a(xcfg.o)
                              Output\obj\Libraries\bsp\bsp_sys.o (xcfg_init)
..\..\..\..\Libraries\libs\libplatform.a(device.o)
                              Output\obj\Libraries\bsp\bsp_sys.o (dev_init)
..\..\..\..\Libraries\libs\libplatform.a(main.o)
                              Output\obj\Libraries\BT\spp\hid.o (delay_5ms)
..\..\..\..\Libraries\libs\libplatform.a(interrupt.o)
                              Output\obj\Libraries\bsp\bsp_fot.o (tick_get)
..\..\..\..\Libraries\libs\libplatform.a(startup.o)
                              ..\..\..\..\Libraries\libs\libplatform.a(interrupt.o) (user_timer_isr_en)
..\..\..\..\Libraries\libs\libplatform.a(sys_hook.o)
                              ..\..\..\..\Libraries\libs\libplatform.a(startup.o) (sys_hook_init)
..\..\..\..\Libraries\libs\libplatform.a(reset.o)
                              (_start)
..\..\..\..\Libraries\libs\libplatform.a(spiflash.o)
                              ..\..\..\..\Libraries\libs\libplatform.a(os_flash.o) (spiflash_program)
..\..\..\..\Libraries\libs\libplatform.a(debug.o)
                              ..\..\..\..\Libraries\libs\libplatform.a(main.o) (debug_set)
..\..\..\..\Libraries\libs\libplatform.a(fot_update.o)
                              ..\..\..\..\Libraries\libs\libplatform.a(xcfg.o) (get_spiloader_offset)
..\..\..\..\Libraries\libs\libplatform.a(lock.o)
                              ..\..\..\..\Libraries\libs\libplatform.a(main.o) (lock_init)
..\..\..\..\Libraries\libs\libplatform.a(patch.o)
                              ..\..\..\..\Libraries\libs\libplatform.a(main.o) (patch_init)
..\..\..\..\Libraries\libs\libplatform.a(power.o)
                              Output\obj\Libraries\bsp\bsp_sys.o (pmu_init)
..\..\..\..\Libraries\libs\libplatform.a(rc.o)
                              ..\..\..\..\Libraries\libs\libplatform.a(main.o) (rc_compile)
..\..\..\..\Libraries\libs\libplatform.a(s_sys.o)
                              ..\..\..\..\Libraries\libs\libplatform.a(main.o) (s_bcnt)
..\..\..\..\Libraries\libs\libplatform.a(sys.o)
                              ..\..\..\..\Libraries\libs\libplatform.a(main.o) (sys_get_rc2m_clkhz)
..\..\..\..\Libraries\libs\libplatform.a(sys_clk.o)
                              Output\obj\Libraries\BT\ble\ble.o (get_cur_sysclk)
..\..\..\..\Libraries\libs\libplatform.a(voltage_trim.o)
                              ..\..\..\..\Libraries\libs\libplatform.a(main.o) (voltage_trim_value_init)
..\..\..\..\Libraries\libs\libplatform.a(weak_symbol.o)
                              ..\..\..\..\Libraries\libs\libplatform.a(main.o) (update_complete)
..\..\..\..\Libraries\libs\libplatform.a(huart.o)
                              ..\..\..\..\Libraries\libs\libplatform.a(interrupt.o) (huart_isr)
..\..\..\..\Libraries\libs\libplatform.a(usb.o)
                              ..\..\..\..\Libraries\libs\libplatform.a(startup.o) (thread_usb_entry)
..\..\..\..\Libraries\libs\libplatform.a(bt.o)
                              ..\..\..\..\Libraries\libs\libplatform.a(reset.o) (bthw_txrx_isr)
..\..\..\..\Libraries\libs\libbtstack.a(nanos.o)
                              ..\..\..\..\Libraries\libs\libplatform.a(startup.o) (nanos_var_init)
..\..\..\..\Libraries\libs\libbtstack.a(patch.o)
                              ..\..\..\..\Libraries\libs\libplatform.a(patch.o) (bb_patch_init)
..\..\..\..\Libraries\libs\libbtstack.a(platform.o)
                              ..\..\..\..\Libraries\libs\libplatform.a(interrupt.o) (timer_sync_init)
..\..\..\..\Libraries\libs\libbtstack.a(bt_sco.o)
                              ..\..\..\..\Libraries\libs\libplatform.a(interrupt.o) (bt_codec_isr)
..\..\..\..\Libraries\libs\libbtstack.a(bt_acl.o)
                              ..\..\..\..\Libraries\libs\libbtstack.a(patch.o) (bt_acl_env)
..\..\..\..\Libraries\libs\libbtstack.a(ble_con.o)
                              ..\..\..\..\Libraries\libs\libbtstack.a(patch.o) (ble_con_evt_prio_check)
..\..\..\..\Libraries\libs\libbtstack.a(bb_utils.o)
                              ..\..\..\..\Libraries\libs\libbtstack.a(ble_con.o) (bb_sca2ppm)
..\..\..\..\Libraries\libs\libbtstack.a(bb_int.o)
                              ..\..\..\..\Libraries\libs\libplatform.a(bt.o) (bb_hal_isr)
..\..\..\..\Libraries\libs\libbtstack.a(bb.o)
                              ..\..\..\..\Libraries\libs\libbtstack.a(nanos.o) (bb_get_heap_info)
..\..\..\..\Libraries\libs\libbtstack.a(platform.o)
                              ..\..\..\..\Libraries\libs\libbtstack.a(bb.o) (dummy_void)
..\..\..\..\Libraries\libs\libbtstack.a(extern_tws.o)
                              ..\..\..\..\Libraries\libs\libbtstack.a(bb_int.o) (cfg_bt_tws_limit_pair_time)
..\..\..\..\Libraries\libs\libbtstack.a(extern_bt.o)
                              ..\..\..\..\Libraries\libs\libbtstack.a(bb_int.o) (cfg_bt_sniff_clk_sel)
..\..\..\..\Libraries\libs\libbtstack.a(extern.o)
                              ..\..\..\..\Libraries\libs\libplatform.a(reset.o) (ext_aubuf_isr)
..\..\..\..\Libraries\libs\libbtstack.a(spp.o)
                              Output\obj\Libraries\bsp\bsp_fot.o (bt_spp_tx)
..\..\..\..\Libraries\libs\libbtstack.a(sdp_util.o)
                              ..\..\..\..\Libraries\libs\libbtstack.a(spp.o) (mfi_search_uuid128)
..\..\..\..\Libraries\libs\libbtstack.a(sdp_tbl.o)
                              Output\obj\Libraries\BT\spp\profile.o (sdp_spp_service_record)
..\..\..\..\Libraries\libs\libbtstack.a(sdp_server.o)
                              Output\obj\Libraries\BT\spp\profile.o (sdp_add_service)
..\..\..\..\Libraries\libs\libbtstack.a(sdp_client.o)
                              ..\..\..\..\Libraries\libs\libbtstack.a(sdp_server.o) (sdp_client_init)
..\..\..\..\Libraries\libs\libbtstack.a(rfcomm.o)
                              ..\..\..\..\Libraries\libs\libbtstack.a(spp.o) (rfcomm_can_send_packet_now)
..\..\..\..\Libraries\libs\libbtstack.a(btstack_link_key_db.o)
                              Output\obj\Libraries\BT\spp\bt.o (link_info_page_size)
..\..\..\..\Libraries\libs\libbtstack.a(btstack_util.o)
                              ..\..\..\..\Libraries\libs\libbtstack.a(rfcomm.o) (bd_addr_cmp)
..\..\..\..\Libraries\libs\libbtstack.a(btstack_txpkt.o)
                              Output\obj\Libraries\BT\ble\ab_link\app.o (txpkt_init)
..\..\..\..\Libraries\libs\libbtstack.a(btstack_run_loop.o)
                              ..\..\..\..\Libraries\libs\libbtstack.a(rfcomm.o) (btstack_run_loop_set_timer_handler)
..\..\..\..\Libraries\libs\libbtstack.a(btstack_memory.o)
                              ..\..\..\..\Libraries\libs\libbtstack.a(rfcomm.o) (btstack_memory_rfcomm_multiplexer_get)
..\..\..\..\Libraries\libs\libbtstack.a(btstack_linked_list.o)
                              ..\..\..\..\Libraries\libs\libbtstack.a(rfcomm.o) (btstack_linked_list_empty)
..\..\..\..\Libraries\libs\libbtstack.a(btstack_link_ctrl.o)
                              ..\..\..\..\Libraries\libs\libbtstack.a(spp.o) (provide_link_ctrl_context_for_bd_addr)
..\..\..\..\Libraries\libs\libbtstack.a(gatt_server.o)
                              Output\obj\Libraries\BT\ble\ab_link\app.o (ble_init_att_for_handle)
..\..\..\..\Libraries\libs\libbtstack.a(gatt_profile.o)
                              Output\obj\Libraries\BT\ble\ab_link\app.o (ble_gatts_service_add)
..\..\..\..\Libraries\libs\libbtstack.a(att_server.o)
                              ..\..\..\..\Libraries\libs\libbtstack.a(gatt_server.o) (att_server_request_can_send_now_event)
..\..\..\..\Libraries\libs\libbtstack.a(att_dispatch.o)
                              ..\..\..\..\Libraries\libs\libbtstack.a(att_server.o) (att_dispatch_register_server)
..\..\..\..\Libraries\libs\libbtstack.a(att_db.o)
                              ..\..\..\..\Libraries\libs\libbtstack.a(gatt_server.o) (att_uuid_for_handle)
..\..\..\..\Libraries\libs\libbtstack.a(ad_parser.o)
                              ..\..\..\..\Libraries\libs\libbtstack.a(gatt_server.o) (ad_param)
..\..\..\..\Libraries\libs\libbtstack.a(btstack_main.o)
                              ..\..\..\..\Libraries\libs\libbtstack.a(gatt_server.o) (scan_data)
..\..\..\..\Libraries\libs\libbtstack.a(btstack_hal.o)
                              ..\..\..\..\Libraries\libs\libbtstack.a(btstack_run_loop.o) (hal_tick_init)
..\..\..\..\Libraries\libs\libbtstack.a(btstack_api.o)
                              ..\..\..\..\Libraries\libs\libplatform.a(startup.o) (btstack_var_init)
..\..\..\..\Libraries\libs\libbtstack.a(bt_api.o)
                              Output\obj\Libraries\BT\spp\hid.o (bt_hid_send_key)
..\..\..\..\Libraries\libs\libbtstack.a(ble_api.o)
                              ..\..\..\..\Libraries\libs\libbtstack.a(gatt_server.o) (ble_get_status)
..\..\..\..\Libraries\libs\libbtstack.a(bb_sche.o)
                              ..\..\..\..\Libraries\libs\libbtstack.a(ble_con.o) (bb_sche_frag_ble_dur_set)
..\..\..\..\Libraries\libs\libbtstack.a(patch_asm.o)
                              ..\..\..\..\Libraries\libs\libbtstack.a(patch.o) (bb_v1_patch0)
..\..\..\..\Libraries\libs\libbtstack.a(bb_dbg.o)
                              ..\..\..\..\Libraries\libs\libbtstack.a(bb.o) (bb_dbg_init)
..\..\..\..\Libraries\libs\libbtstack.a(bb_clk.o)
                              ..\..\..\..\Libraries\libs\libbtstack.a(bb.o) (bb_clk_init)
..\..\..\..\Libraries\libs\libbtstack.a(aes.o)
                              ..\..\..\..\Libraries\libs\libbtstack.a(bb.o) (aes_init)
..\..\..\..\Libraries\libs\libbtstack.a(vs_proc.o)
                              ..\..\..\..\Libraries\libs\libbtstack.a(btstack_api.o) (bt_fcc_test_ctrl)
..\..\..\..\Libraries\libs\libbtstack.a(vs_fcc.o)
                              ..\..\..\..\Libraries\libs\libbtstack.a(vs_proc.o) (vs_fcc_test_cmd_do)
..\..\..\..\Libraries\libs\libbtstack.a(vs.o)
                              ..\..\..\..\Libraries\libs\libbtstack.a(bb.o) (vs_init)
..\..\..\..\Libraries\libs\libbtstack.a(rf_smart.o)
                              ..\..\..\..\Libraries\libs\libbtstack.a(vs_fcc.o) (rfphy_pll_afc)
..\..\..\..\Libraries\libs\libbtstack.a(rf.o)
                              ..\..\..\..\Libraries\libs\libbtstack.a(bt_acl.o) (rf_txpwr_get_dbm)
..\..\..\..\Libraries\libs\libbtstack.a(bt_hook.o)
                              ..\..\..\..\Libraries\libs\libbtstack.a(bb.o) (bt_isr_hook)
..\..\..\..\Libraries\libs\libbtstack.a(ble_hook.o)
                              ..\..\..\..\Libraries\libs\libbtstack.a(bb.o) (ble_isr_hook)
..\..\..\..\Libraries\libs\libbtstack.a(hct_tl.o)
                              ..\..\..\..\Libraries\libs\libbtstack.a(bb_int.o) (hct_queue_is_empty)
..\..\..\..\Libraries\libs\libbtstack.a(hct_msg.o)
                              ..\..\..\..\Libraries\libs\libbtstack.a(hct_tl.o) (hci_look_for_cmd_desc)
..\..\..\..\Libraries\libs\libbtstack.a(hct_fc.o)
                              ..\..\..\..\Libraries\libs\libbtstack.a(hct_tl.o) (hci_fc_acl_packet_sent)
..\..\..\..\Libraries\libs\libbtstack.a(hct.o)
                              ..\..\..\..\Libraries\libs\libbtstack.a(vs_proc.o) (hci_send_2_host)
..\..\..\..\Libraries\libs\libbtstack.a(tws_sco.o)
                              ..\..\..\..\Libraries\libs\libbtstack.a(bt_hook.o) (bt_sco_get_index)
..\..\..\..\Libraries\libs\libbtstack.a(tws_acl.o)
                              ..\..\..\..\Libraries\libs\libbtstack.a(patch_asm.o) (tws_switch_acl_is_pause)
..\..\..\..\Libraries\libs\libbtstack.a(lm.o)
                              ..\..\..\..\Libraries\libs\libbtstack.a(btstack_main.o) (lm_set_scan_int)
..\..\..\..\Libraries\libs\libbtstack.a(bt_hal.o)
                              ..\..\..\..\Libraries\libs\libbtstack.a(bt_hook.o) (bt_channel_assess)
..\..\..\..\Libraries\libs\libbtstack.a(bt21.o)
                              ..\..\..\..\Libraries\libs\libbtstack.a(bb.o) (bt_buf_acl_rx_free)
..\..\..\..\Libraries\libs\libbtstack.a(bc.o)
                              ..\..\..\..\Libraries\libs\libbtstack.a(bt21.o) (bc_init)
..\..\..\..\Libraries\libs\libbtstack.a(ble_hal.o)
                              ..\..\..\..\Libraries\libs\libbtstack.a(ble_con.o) (ble_channel_assess)
..\..\..\..\Libraries\libs\libbtstack.a(ble_adv.o)
                              ..\..\..\..\Libraries\libs\libbtstack.a(ble_hal.o) (ble_adv_init)
..\..\..\..\Libraries\libs\libbtstack.a(ble.o)
                              ..\..\..\..\Libraries\libs\libbtstack.a(bb.o) (ble_var_init)
..\..\..\..\Libraries\libs\libbtstack.a(extern_ble.o)
                              ..\..\..\..\Libraries\libs\libbtstack.a(gatt_server.o) (ble_client_cfg_callback)
..\..\..\..\Libraries\libs\libbtstack.a(l2cap_test.o)
                              ..\..\..\..\Libraries\libs\libbtstack.a(btstack_main.o) (l2cap_vd_acl_init)
..\..\..\..\Libraries\libs\libbtstack.a(l2cap.o)
                              ..\..\..\..\Libraries\libs\libbtstack.a(btstack_main.o) (l2cap_init)
..\..\..\..\Libraries\libs\libbtstack.a(hci_sco.o)
                              ..\..\..\..\Libraries\libs\libbtstack.a(btstack_api.o) (sco_init_var)
..\..\..\..\Libraries\libs\libbtstack.a(hci_dump.o)
                              ..\..\..\..\Libraries\libs\libbtstack.a(btstack_api.o) (hci_dump_open)
..\..\..\..\Libraries\libs\libbtstack.a(hci_cmd.o)
                              ..\..\..\..\Libraries\libs\libbtstack.a(l2cap.o) (hci_create_connection_cancel)
..\..\..\..\Libraries\libs\libbtstack.a(hci.o)
                              ..\..\..\..\Libraries\libs\libbtstack.a(l2cap.o) (gap_get_connection_parameter_range)
..\..\..\..\Libraries\libs\libbtstack.a(hid_usage.o)
                              ..\..\..\..\Libraries\libs\libbtstack.a(bt_api.o) (hid_report_set)
..\..\..\..\Libraries\libs\libbtstack.a(hid_device.o)
                              ..\..\..\..\Libraries\libs\libbtstack.a(bt_api.o) (bt_hid_is_connected)
..\..\..\..\Libraries\libs\libbtstack.a(hfp_hf.o)
                              ..\..\..\..\Libraries\libs\libbtstack.a(btstack_api.o) (hfp_hf_get_siri_status)
..\..\..\..\Libraries\libs\libbtstack.a(hfp.o)
                              ..\..\..\..\Libraries\libs\libbtstack.a(btstack_main.o) (hfp_var_init)
..\..\..\..\Libraries\libs\libbtstack.a(avdtp.o)
                              ..\..\..\..\Libraries\libs\libbtstack.a(bt_hook.o) (a2dp_get_play_index)
..\..\..\..\Libraries\libs\libbtstack.a(a2dp.o)
                              ..\..\..\..\Libraries\libs\libbtstack.a(btstack_api.o) (a2dp_is_playing)
..\..\..\..\Libraries\libs\libbtstack.a(btstack_memory_pool.o)
                              ..\..\..\..\Libraries\libs\libbtstack.a(btstack_memory.o) (btstack_memory_pool_get)
..\..\..\..\Libraries\libs\libbtstack.a(btstack_adv0.o)
                              ..\..\..\..\Libraries\libs\libbtstack.a(btstack_api.o) (btstack_adv0_ctrl)
..\..\..\..\Libraries\libs\libbtstack.a(sm.o)
                              ..\..\..\..\Libraries\libs\libbtstack.a(att_server.o) (sm_cmac_ready)
..\..\..\..\Libraries\libs\libbtstack.a(le_device_db_memory.o)
                              ..\..\..\..\Libraries\libs\libbtstack.a(btstack_main.o) (le_device_db_init)
..\..\..\..\Libraries\libs\libbtstack.a(hci_transport_hcic.o)
                              ..\..\..\..\Libraries\libs\libbtstack.a(hci.o) (hcic_rx_flush)
..\..\..\..\Libraries\libs\libbtstack.a(btstack_chipset_inner.o)
                              ..\..\..\..\Libraries\libs\libbtstack.a(btstack_api.o) (btstack_chipset_inner_instance)
..\..\..\..\Libraries\libs\libbtstack.a(lm_hook.o)
                              ..\..\..\..\Libraries\libs\libbtstack.a(lm.o) (lm_init_hook)
..\..\..\..\Libraries\libs\libbtstack.a(lm_sp.o)
                              ..\..\..\..\Libraries\libs\libbtstack.a(lm.o) (lm_oob_f1)
..\..\..\..\Libraries\libs\libbtstack.a(lm_proc.o)
                              ..\..\..\..\Libraries\libs\libbtstack.a(lm.o) (lm_msg_env)
..\..\..\..\Libraries\libs\libbtstack.a(lm_key.o)
                              ..\..\..\..\Libraries\libs\libbtstack.a(lm.o) (lm_e22)
..\..\..\..\Libraries\libs\libbtstack.a(lc.o)
                              ..\..\..\..\Libraries\libs\libbtstack.a(bt21.o) (lc_init)
..\..\..\..\Libraries\libs\libbtstack.a(mgr.o)
                              ..\..\..\..\Libraries\libs\libbtstack.a(ble.o) (mgr_init)
..\..\..\..\Libraries\libs\libbtstack.a(ll.o)
                              ..\..\..\..\Libraries\libs\libbtstack.a(ble.o) (ll_init)
..\..\..\..\Libraries\libs\libbtstack.a(ble_test.o)
                              ..\..\..\..\Libraries\libs\libbtstack.a(ble_hal.o) (ble_test_init)
..\..\..\..\Libraries\libs\libbtstack.a(ble_scan.o)
                              ..\..\..\..\Libraries\libs\libbtstack.a(ble.o) (ble_get_scan_var)
..\..\..\..\Libraries\libs\libbtstack.a(ble_per_adv.o)
                              ..\..\..\..\Libraries\libs\libbtstack.a(ble.o) (ble_get_per_adv_var)
..\..\..\..\Libraries\libs\libbtstack.a(ble_init.o)
                              ..\..\..\..\Libraries\libs\libbtstack.a(ble_hal.o) (ble_init_init)
..\..\..\..\Libraries\libs\libbtstack.a(ble_buf.o)
                              ..\..\..\..\Libraries\libs\libbtstack.a(ble.o) (ble_buf_init)
..\..\..\..\Libraries\libs\libbtstack.a(ble_adv0.o)
                              ..\..\..\..\Libraries\libs\libbtstack.a(ble.o) (ble_adv0_init)
..\..\..\..\Libraries\libs\libbtstack.a(extern_hfhs.o)
                              ..\..\..\..\Libraries\libs\libbtstack.a(hfp.o) (hfp_notice_network_time)
..\..\..\..\Libraries\libs\libbtstack.a(l2cap_signaling.o)
                              ..\..\..\..\Libraries\libs\libbtstack.a(l2cap.o) (l2cap_next_sig_id)
..\..\..\..\Libraries\libs\libbtstack.a(lc_hook.o)
                              ..\..\..\..\Libraries\libs\libbtstack.a(lm_proc.o) (lc_auto_sniff_step_set)
..\..\..\..\Libraries\libs\libbtstack.a(lm_sco.o)
                              ..\..\..\..\Libraries\libs\libbtstack.a(lc.o) (lm_init_sync)
..\..\..\..\Libraries\libs\libbtstack.a(lc_util.o)
                              ..\..\..\..\Libraries\libs\libbtstack.a(lc.o) (lc_compute_pkt_types)
..\..\..\..\Libraries\libs\libbtstack.a(lc_sniff.o)
                              ..\..\..\..\Libraries\libs\libbtstack.a(lc.o) (lc_sniff_init)
..\..\..\..\Libraries\libs\libbtstack.a(lc_sco.o)
                              ..\..\..\..\Libraries\libs\libbtstack.a(lc.o) (lc_sco_init)
..\..\..\..\Libraries\libs\libbtstack.a(lc_proc.o)
                              ..\..\..\..\Libraries\libs\libbtstack.a(lc.o) (lc_msg_env)
..\..\..\..\Libraries\libs\libbtstack.a(lc_lmppdu.o)
                              ..\..\..\..\Libraries\libs\libbtstack.a(lc_proc.o) (lmp_estab_allowed)
..\..\..\..\Libraries\libs\libbtstack.a(mgr_proc.o)
                              ..\..\..\..\Libraries\libs\libbtstack.a(mgr.o) (mgr_msg_env)
..\..\..\..\Libraries\libs\libbtstack.a(mgr_init.o)
                              ..\..\..\..\Libraries\libs\libbtstack.a(mgr_proc.o) (ble_init_end_ind_func)
..\..\..\..\Libraries\libs\libbtstack.a(mgr_hci.o)
                              ..\..\..\..\Libraries\libs\libbtstack.a(mgr_proc.o) (hci_command_mgr_func)
..\..\..\..\Libraries\libs\libbtstack.a(ll_scan.o)
                              ..\..\..\..\Libraries\libs\libbtstack.a(mgr_hci.o) (hci_le_set_scan_param_cmd_func)
..\..\..\..\Libraries\libs\libbtstack.a(ll_adv.o)
                              ..\..\..\..\Libraries\libs\libbtstack.a(mgr_hci.o) (hci_le_rd_adv_ch_tx_pw_cmd_func)
..\..\..\..\Libraries\libs\libbtstack.a(ll_proc.o)
                              ..\..\..\..\Libraries\libs\libbtstack.a(ll.o) (ll_msg_env)
..\..\..\..\Libraries\libs\libbtstack.a(ll_ping.o)
                              ..\..\..\..\Libraries\libs\libbtstack.a(ll_proc.o) (hci_rd_auth_payl_to_cmd_func)
..\..\..\..\Libraries\libs\libbtstack.a(ll_phy_upd.o)
                              ..\..\..\..\Libraries\libs\libbtstack.a(ll_proc.o) (hci_le_rd_phy_cmd_func)
..\..\..\..\Libraries\libs\libbtstack.a(ll_past.o)
                              ..\..\..\..\Libraries\libs\libbtstack.a(ll_proc.o) (hci_le_per_adv_set_info_transf_cmd_func)
..\..\..\..\Libraries\libs\libbtstack.a(ll_length.o)
                              ..\..\..\..\Libraries\libs\libbtstack.a(ll_proc.o) (hci_le_set_data_len_cmd_func)
..\..\..\..\Libraries\libs\libbtstack.a(ll_feature.o)
                              ..\..\..\..\Libraries\libs\libbtstack.a(ll_proc.o) (hci_le_rd_rem_feats_cmd_func)
..\..\..\..\Libraries\libs\libbtstack.a(ll_encrypt.o)
                              ..\..\..\..\Libraries\libs\libbtstack.a(ll_proc.o) (hci_le_en_enc_cmd_func)
..\..\..\..\Libraries\libs\libbtstack.a(ll_disconnect.o)
                              ..\..\..\..\Libraries\libs\libbtstack.a(ll_proc.o) (ble_disc_ind_func)
..\..\..\..\Libraries\libs\libbtstack.a(ll_con_upd.o)
                              ..\..\..\..\Libraries\libs\libbtstack.a(ll_proc.o) (hci_le_con_upd_cmd_func)
..\..\..\..\Libraries\libs\libbtstack.a(ll_cntl.o)
                              ..\..\..\..\Libraries\libs\libbtstack.a(ll.o) (ll_cntl_tx_check)
..\..\..\..\Libraries\libs\libbtstack.a(ll_clk_acc.o)
                              ..\..\..\..\Libraries\libs\libbtstack.a(ll_cntl.o) (ll_clk_acc_req_func)
..\..\..\..\Libraries\libs\libbtstack.a(ll_chmap_upd.o)
                              ..\..\..\..\Libraries\libs\libbtstack.a(ll_cntl.o) (ll_channel_map_ind_func)
..\..\..\..\Libraries\libs\libbtstack.a(aes_rpa.o)
                              ..\..\..\..\Libraries\libs\libbtstack.a(ll_adv.o) (aes_rpa_gen)
..\..\..\..\Libraries\libs\libbtstack.a(scan_hook.o)
                              ..\..\..\..\Libraries\libs\libbtstack.a(ll_scan.o) (ble_scan_end_ind_hook)
..\..\..\..\Libraries\libs\libbtstack.a(adv_hook.o)
                              ..\..\..\..\Libraries\libs\libbtstack.a(ll_adv.o) (ble_adv_end_ind_hook)
..\..\..\..\Libraries\libs\libbtstack.a(ll_version.o)
                              ..\..\..\..\Libraries\libs\libbtstack.a(ll_proc.o) (ll_op_ver_exch_ind_func)
..\..\..\..\Libraries\libs\libbtstack.a(ll_pwr.o)
                              ..\..\..\..\Libraries\libs\libbtstack.a(ll_proc.o) (hci_rd_tx_pwr_lvl_cmd_func)
..\..\..\..\Libraries\libs\libdrivers.a(usb_device_hid.o)
                              Output\obj\Libraries\bsp\bsp_sys.o (ude_tmr_isr)
..\..\..\..\Libraries\libs\libdrivers.a(usb_device_printer.o)
                              ..\..\..\..\Libraries\libs\libplatform.a(usb.o) (ude_bulk_tx_process)
..\..\..\..\Libraries\libs\libdrivers.a(usb_device_run_loop.o)
                              ..\..\..\..\Libraries\libs\libdrivers.a(usb_device_hid.o) (ude_cfgval_get)
..\..\..\..\Libraries\libs\libdrivers.a(usb_host_manage.o)
                              ..\..\..\..\Libraries\libs\libplatform.a(device.o) (usb_host_init)
..\..\..\..\Libraries\libs\libdrivers.a(usb_host_storage.o)
                              ..\..\..\..\Libraries\libs\libdrivers.a(usb_host_manage.o) (uhs_start)
..\..\..\..\Libraries\libs\libdrivers.a(usb_comm.o)
                              ..\..\..\..\Libraries\libs\libdrivers.a(usb_host_storage.o) (usb_interrupt_disable)
..\..\..\..\Libraries\libs\libdrivers.a(usb_detect.o)
                              ..\..\..\..\Libraries\libs\libdrivers.a(usb_host_manage.o) (usbchk_switch_otg_device)
..\..\..\..\Libraries\libs\libdrivers.a(usb_device_desc.o)
                              ..\..\..\..\Libraries\libs\libdrivers.a(usb_device_run_loop.o) (usb_get_hid_config_descriptor)
..\..\..\..\Libraries\libs\libdrivers.a(usb_device_enum.o)
                              ..\..\..\..\Libraries\libs\libdrivers.a(usb_device_run_loop.o) (ude_run_loop_execute)
..\..\..\..\Libraries\libs\libdrivers.a(usb_device_ep.o)
                              ..\..\..\..\Libraries\libs\libdrivers.a(usb_device_hid.o) (usb_set_cur_ep)
..\..\..\..\Libraries\libs\libdrivers.a(usb_host_enum.o)
                              ..\..\..\..\Libraries\libs\libdrivers.a(usb_host_manage.o) (uhe_start)
..\..\..\..\Libraries\libs\libdrivers.a(weak_symbol.o)
                              ..\..\..\..\Libraries\libs\libdrivers.a(usb_host_enum.o) (iphone_power_set)
..\..\..\..\Libraries\libs\libdrivers.a(usb_device_audio.o)
                              ..\..\..\..\Libraries\libs\libdrivers.a(usb_device_enum.o) (uda_get_spk_mute)

Allocating common symbols
Common symbol       size              file

fot_var             0x22              Output\obj\Libraries\bsp\bsp_fot.o
ticks_50ms          0x4               Output\obj\Libraries\bsp\bsp_sys.o
xcfg_cb             0xae              Output\obj\Libraries\bsp\bsp_sys.o

Discarded input sections

 .text          0x0000000000000000        0x0 Output\obj\Libraries\bsp\bsp_cm.o
 .data          0x0000000000000000        0x0 Output\obj\Libraries\bsp\bsp_cm.o
 .bss           0x0000000000000000        0x0 Output\obj\Libraries\bsp\bsp_cm.o
 .text          0x0000000000000000        0x0 Output\obj\Libraries\bsp\bsp_fot.o
 .data          0x0000000000000000        0x0 Output\obj\Libraries\bsp\bsp_fot.o
 .bss           0x0000000000000000        0x0 Output\obj\Libraries\bsp\bsp_fot.o
 .text          0x0000000000000000        0x0 Output\obj\Libraries\bsp\bsp_param.o
 .data          0x0000000000000000        0x0 Output\obj\Libraries\bsp\bsp_param.o
 .bss           0x0000000000000000        0x0 Output\obj\Libraries\bsp\bsp_param.o
 .text          0x0000000000000000        0x0 Output\obj\Libraries\bsp\bsp_sys.o
 .data          0x0000000000000000        0x0 Output\obj\Libraries\bsp\bsp_sys.o
 .bss           0x0000000000000000        0x0 Output\obj\Libraries\bsp\bsp_sys.o
 .text.bsp_get_bat_level
                0x0000000000000000        0x6 Output\obj\Libraries\bsp\bsp_sys.o
 .rodata        0x0000000000000000       0x20 Output\obj\Libraries\bsp\bsp_sys.o
 .text          0x0000000000000000        0x0 Output\obj\Libraries\BT\ble\ab_link\app.o
 .data          0x0000000000000000        0x0 Output\obj\Libraries\BT\ble\ab_link\app.o
 .bss           0x0000000000000000        0x0 Output\obj\Libraries\BT\ble\ab_link\app.o
 .text.gatt_callback_fota
                0x0000000000000000       0x2c Output\obj\Libraries\BT\ble\ab_link\app.o
 .text.gatt_callback_app
                0x0000000000000000       0x1a Output\obj\Libraries\BT\ble\ab_link\app.o
 .text.ble_get_scan_data
                0x0000000000000000       0x68 Output\obj\Libraries\BT\ble\ab_link\app.o
 .text.ble_get_adv_data
                0x0000000000000000       0x6a Output\obj\Libraries\BT\ble\ab_link\app.o
 .text.ble_txpkt_init
                0x0000000000000000       0x3c Output\obj\Libraries\BT\ble\ab_link\app.o
 .text.ble_send_packet1
                0x0000000000000000       0x28 Output\obj\Libraries\BT\ble\ab_link\app.o
 .text.ble_send_packet2
                0x0000000000000000       0x28 Output\obj\Libraries\BT\ble\ab_link\app.o
 .text.ble_read_value
                0x0000000000000000       0x24 Output\obj\Libraries\BT\ble\ab_link\app.o
 .text.bsp_ble_process
                0x0000000000000000        0x2 Output\obj\Libraries\BT\ble\ab_link\app.o
 .text.ble_app_gatts_service_init
                0x0000000000000000      0x168 Output\obj\Libraries\BT\ble\ab_link\app.o
 .text.ble_app_init
                0x0000000000000000        0x8 Output\obj\Libraries\BT\ble\ab_link\app.o
 .rodata        0x0000000000000000       0xbc Output\obj\Libraries\BT\ble\ab_link\app.o
 .ble_tx_buff.att
                0x0000000000000000      0x840 Output\obj\Libraries\BT\ble\ab_link\app.o
 .rodata.str1.4
                0x0000000000000000        0xe Output\obj\Libraries\BT\ble\ab_link\app.o
 .text          0x0000000000000000        0x0 Output\obj\Libraries\BT\ble\adv0.o
 .data          0x0000000000000000        0x0 Output\obj\Libraries\BT\ble\adv0.o
 .bss           0x0000000000000000        0x0 Output\obj\Libraries\BT\ble\adv0.o
 .text          0x0000000000000000        0x0 Output\obj\Libraries\BT\ble\ble.o
 .data          0x0000000000000000        0x0 Output\obj\Libraries\BT\ble\ble.o
 .bss           0x0000000000000000        0x0 Output\obj\Libraries\BT\ble\ble.o
 .text.ble_enter_transmit
                0x0000000000000000       0x3a Output\obj\Libraries\BT\ble\ble.o
 .text.ble_exit_transmit
                0x0000000000000000       0x32 Output\obj\Libraries\BT\ble\ble.o
 .text.ble_get_bat_level
                0x0000000000000000        0x8 Output\obj\Libraries\BT\ble\ble.o
 .text.ble_init_att
                0x0000000000000000        0x8 Output\obj\Libraries\BT\ble\ble.o
 .sbss          0x0000000000000000        0x1 Output\obj\Libraries\BT\ble\ble.o
 .text          0x0000000000000000        0x0 Output\obj\Libraries\BT\spp\bt.o
 .data          0x0000000000000000        0x0 Output\obj\Libraries\BT\spp\bt.o
 .bss           0x0000000000000000        0x0 Output\obj\Libraries\BT\spp\bt.o
 .text.bt_clr_master_addr
                0x0000000000000000        0x2 Output\obj\Libraries\BT\spp\bt.o
 .text.bt_save_master_addr
                0x0000000000000000        0x2 Output\obj\Libraries\BT\spp\bt.o
 .text.bt_get_master_addr
                0x0000000000000000        0x4 Output\obj\Libraries\BT\spp\bt.o
 .text.bt_clr_all_link_info
                0x0000000000000000        0x8 Output\obj\Libraries\BT\spp\bt.o
 .text.bt_tws_clr_link_info
                0x0000000000000000        0x2 Output\obj\Libraries\BT\spp\bt.o
 .text.bt_get_rand_seed
                0x0000000000000000        0xa Output\obj\Libraries\BT\spp\bt.o
 .rodata        0x0000000000000000        0xa Output\obj\Libraries\BT\spp\bt.o
 .text          0x0000000000000000        0x0 Output\obj\Libraries\BT\spp\hid.o
 .data          0x0000000000000000        0x0 Output\obj\Libraries\BT\spp\hid.o
 .bss           0x0000000000000000        0x0 Output\obj\Libraries\BT\spp\hid.o
 .text.bsp_bt_hid_photo
                0x0000000000000000        0x4 Output\obj\Libraries\BT\spp\hid.o
 .text.bsp_bt_hid_vol_change
                0x0000000000000000        0x4 Output\obj\Libraries\BT\spp\hid.o
 .text.bsp_bt_hid_screen_left
                0x0000000000000000       0x32 Output\obj\Libraries\BT\spp\hid.o
 .text.bsp_bt_hid_screen_right
                0x0000000000000000       0x32 Output\obj\Libraries\BT\spp\hid.o
 .comment       0x0000000000000000       0x12 Output\obj\Libraries\BT\spp\hid.o
 .text          0x0000000000000000        0x0 Output\obj\Libraries\BT\spp\profile.o
 .bss           0x0000000000000000        0x0 Output\obj\Libraries\BT\spp\profile.o
 .text          0x0000000000000000        0x0 Output\obj\Libraries\BT\spp\spp.o
 .data          0x0000000000000000        0x0 Output\obj\Libraries\BT\spp\spp.o
 .bss           0x0000000000000000        0x0 Output\obj\Libraries\BT\spp\spp.o
 .text.bsp_spp_process
                0x0000000000000000        0x2 Output\obj\Libraries\BT\spp\spp.o
 .text          0x0000000000000000        0x0 Output\obj\Libraries\Device\Source\gw3323_clk.o
 .data          0x0000000000000000        0x0 Output\obj\Libraries\Device\Source\gw3323_clk.o
 .bss           0x0000000000000000        0x0 Output\obj\Libraries\Device\Source\gw3323_clk.o
 .text.clock_gate0_cmd
                0x0000000000000000       0x16 Output\obj\Libraries\Device\Source\gw3323_clk.o
 .text.clock_gate2_cmd
                0x0000000000000000       0x16 Output\obj\Libraries\Device\Source\gw3323_clk.o
 .text          0x0000000000000000        0x0 Output\obj\Libraries\Device\Source\gw3323_gpio.o
 .data          0x0000000000000000        0x0 Output\obj\Libraries\Device\Source\gw3323_gpio.o
 .bss           0x0000000000000000        0x0 Output\obj\Libraries\Device\Source\gw3323_gpio.o
 .text.gpio_pic_config_reset
                0x0000000000000000        0xa Output\obj\Libraries\Device\Source\gw3323_gpio.o
 .text.gpio_pic_config
                0x0000000000000000       0x88 Output\obj\Libraries\Device\Source\gw3323_gpio.o
 .com_text.isr  0x0000000000000000       0x28 Output\obj\Libraries\Device\Source\gw3323_gpio.o
 .text          0x0000000000000000        0x0 Output\obj\Libraries\Device\Source\gw3323_tmr.o
 .data          0x0000000000000000        0x0 Output\obj\Libraries\Device\Source\gw3323_tmr.o
 .bss           0x0000000000000000        0x0 Output\obj\Libraries\Device\Source\gw3323_tmr.o
 .text          0x0000000000000000        0x0 Output\obj\Libraries\libs\strong_symbol.o
 .data          0x0000000000000000        0x0 Output\obj\Libraries\libs\strong_symbol.o
 .bss           0x0000000000000000        0x0 Output\obj\Libraries\libs\strong_symbol.o
 .text.aac_dec_init
                0x0000000000000000        0x2 Output\obj\Libraries\libs\strong_symbol.o
 .text.aac_decode_init
                0x0000000000000000        0x2 Output\obj\Libraries\libs\strong_symbol.o
 .text.aac_dec_frame
                0x0000000000000000        0x4 Output\obj\Libraries\libs\strong_symbol.o
 .text.aac_nor_dec_frame
                0x0000000000000000        0x4 Output\obj\Libraries\libs\strong_symbol.o
 .text.aac_tws_dec_frame
                0x0000000000000000        0x4 Output\obj\Libraries\libs\strong_symbol.o
 .text.aac_cache_free_do
                0x0000000000000000        0x2 Output\obj\Libraries\libs\strong_symbol.o
 .text.aac_cache_read_do
                0x0000000000000000        0x4 Output\obj\Libraries\libs\strong_symbol.o
 .text.tws_pack_aac
                0x0000000000000000        0x4 Output\obj\Libraries\libs\strong_symbol.o
 .com_text.aac.obuf
                0x0000000000000000        0x2 Output\obj\Libraries\libs\strong_symbol.o
 .aacdec.text   0x0000000000000000        0x2 Output\obj\Libraries\libs\strong_symbol.o
 .text.btstack_tws_init
                0x0000000000000000        0x2 Output\obj\Libraries\libs\strong_symbol.o
 .text.a2dp_play_init
                0x0000000000000000        0x2 Output\obj\Libraries\libs\strong_symbol.o
 .bcom_text.sbc.play
                0x0000000000000000       0x28 Output\obj\Libraries\libs\strong_symbol.o
 .bcom_text.sbc_cache
                0x0000000000000000        0xc Output\obj\Libraries\libs\strong_symbol.o
 .sbcdec.code   0x0000000000000000        0x6 Output\obj\Libraries\libs\strong_symbol.o
 .com_text.bb.tws
                0x0000000000000000        0x2 Output\obj\Libraries\libs\strong_symbol.o
 .bcom_text.bb.btisr
                0x0000000000000000       0x12 Output\obj\Libraries\libs\strong_symbol.o
 .text.bt_tws_set_spr
                0x0000000000000000        0x4 Output\obj\Libraries\libs\strong_symbol.o
 .com_text.sbc.play
                0x0000000000000000        0x2 Output\obj\Libraries\libs\strong_symbol.o
 .bcom_text.sbc.send
                0x0000000000000000        0x2 Output\obj\Libraries\libs\strong_symbol.o
 .bcom_text.lc.tws
                0x0000000000000000        0x4 Output\obj\Libraries\libs\strong_symbol.o
 .bcom_text.a2dp.lost
                0x0000000000000000        0x4 Output\obj\Libraries\libs\strong_symbol.o
 .bcom_text.sbc
                0x0000000000000000        0x2 Output\obj\Libraries\libs\strong_symbol.o
 .bcom_text.bb.tws_switch
                0x0000000000000000        0x4 Output\obj\Libraries\libs\strong_symbol.o
 .bcom_text.bb.bttx
                0x0000000000000000        0x6 Output\obj\Libraries\libs\strong_symbol.o
 .text.tws_set_snoop_ticks
                0x0000000000000000        0x4 Output\obj\Libraries\libs\strong_symbol.o
 .text.ble_test_start
                0x0000000000000000        0x4 Output\obj\Libraries\libs\strong_symbol.o
 .text.ble_test_stop
                0x0000000000000000        0x4 Output\obj\Libraries\libs\strong_symbol.o
 .text.huart_init
                0x0000000000000000        0x2 Output\obj\Libraries\libs\strong_symbol.o
 .com_text.bt_rec
                0x0000000000000000        0x2 Output\obj\Libraries\libs\strong_symbol.o
 .text.bt_sco_fill_remote_buf
                0x0000000000000000        0x2 Output\obj\Libraries\libs\strong_symbol.o
 .text.btstack_pbap
                0x0000000000000000        0x2 Output\obj\Libraries\libs\strong_symbol.o
 .text.bsp_charge_ctrl_process
                0x0000000000000000        0x2 Output\obj\Libraries\libs\strong_symbol.o
 .text.usb_dev_isr
                0x0000000000000000        0x2 Output\obj\Libraries\libs\strong_symbol.o
 .text.ude_isoc_tx_process
                0x0000000000000000        0x2 Output\obj\Libraries\libs\strong_symbol.o
 .text.ude_isoc_rx_process
                0x0000000000000000        0x2 Output\obj\Libraries\libs\strong_symbol.o
 .text.lock_code_usbdev
                0x0000000000000000        0x2 Output\obj\Libraries\libs\strong_symbol.o
 .text.unlock_code_usbdev
                0x0000000000000000        0x2 Output\obj\Libraries\libs\strong_symbol.o
 .text.dac_get_max_anl_vol
                0x0000000000000000        0x4 Output\obj\Libraries\libs\strong_symbol.o
 .com_text.dac  0x0000000000000000        0x2 Output\obj\Libraries\libs\strong_symbol.o
 .text.bsp.dac  0x0000000000000000        0x2 Output\obj\Libraries\libs\strong_symbol.o
 .text          0x0000000000000000        0x0 Output\obj\Examples\TIMER\TIM_Capture\Source\timer_capture.o
 .data          0x0000000000000000        0x0 Output\obj\Examples\TIMER\TIM_Capture\Source\timer_capture.o
 .bss           0x0000000000000000        0x0 Output\obj\Examples\TIMER\TIM_Capture\Source\timer_capture.o
 .text          0x0000000000000000        0x0 Output\obj\Examples\TIMER\TIM_Capture\Source\timer_pwm.o
 .data          0x0000000000000000        0x0 Output\obj\Examples\TIMER\TIM_Capture\Source\timer_pwm.o
 .bss           0x0000000000000000        0x0 Output\obj\Examples\TIMER\TIM_Capture\Source\timer_pwm.o
 .text          0x0000000000000000        0x0 Output\obj\Examples\TIMER\TIM_Capture\Project\config.o
 .data          0x0000000000000000        0x0 Output\obj\Examples\TIMER\TIM_Capture\Project\config.o
 .bss           0x0000000000000000        0x0 Output\obj\Examples\TIMER\TIM_Capture\Project\config.o
 .text          0x0000000000000000        0x0 Output\obj\Examples\TIMER\TIM_Capture\Project\main.o
 .data          0x0000000000000000        0x0 Output\obj\Examples\TIMER\TIM_Capture\Project\main.o
 .bss           0x0000000000000000        0x0 Output\obj\Examples\TIMER\TIM_Capture\Project\main.o
 .text          0x0000000000000000        0x0 ..\..\..\..\Libraries\libs\libplatform.a(audio.o)
 .data          0x0000000000000000        0x0 ..\..\..\..\Libraries\libs\libplatform.a(audio.o)
 .bss           0x0000000000000000        0x0 ..\..\..\..\Libraries\libs\libplatform.a(audio.o)
 .com_text.dac  0x0000000000000000       0x66 ..\..\..\..\Libraries\libs\libplatform.a(audio.o)
 .text.spires   0x0000000000000000       0x40 ..\..\..\..\Libraries\libs\libplatform.a(audio.o)
 .text          0x0000000000000000        0x0 ..\..\..\..\Libraries\libs\libplatform.a(cm.o)
 .data          0x0000000000000000        0x0 ..\..\..\..\Libraries\libs\libplatform.a(cm.o)
 .text.cm_move_allpages
                0x0000000000000000      0x140 ..\..\..\..\Libraries\libs\libplatform.a(cm.o)
 .text.cm_get_startaddr
                0x0000000000000000        0xa ..\..\..\..\Libraries\libs\libplatform.a(cm.o)
 .text.cm_get_area
                0x0000000000000000       0x14 ..\..\..\..\Libraries\libs\libplatform.a(cm.o)
 .text.cm_release_all
                0x0000000000000000       0x90 ..\..\..\..\Libraries\libs\libplatform.a(cm.o)
 .text.cm_read8
                0x0000000000000000       0x28 ..\..\..\..\Libraries\libs\libplatform.a(cm.o)
 .text.cm_read16
                0x0000000000000000       0x28 ..\..\..\..\Libraries\libs\libplatform.a(cm.o)
 .text.cm_read32
                0x0000000000000000       0x24 ..\..\..\..\Libraries\libs\libplatform.a(cm.o)
 .text.cm_write8
                0x0000000000000000       0x28 ..\..\..\..\Libraries\libs\libplatform.a(cm.o)
 .text.cm_write16
                0x0000000000000000       0x28 ..\..\..\..\Libraries\libs\libplatform.a(cm.o)
 .text.cm_write32
                0x0000000000000000       0x24 ..\..\..\..\Libraries\libs\libplatform.a(cm.o)
 .text.cm_clear
                0x0000000000000000       0x60 ..\..\..\..\Libraries\libs\libplatform.a(cm.o)
 .text          0x0000000000000000        0x0 ..\..\..\..\Libraries\libs\libplatform.a(os_flash.o)
 .data          0x0000000000000000        0x0 ..\..\..\..\Libraries\libs\libplatform.a(os_flash.o)
 .bss           0x0000000000000000        0x0 ..\..\..\..\Libraries\libs\libplatform.a(os_flash.o)
 .text          0x0000000000000000        0x0 ..\..\..\..\Libraries\libs\libplatform.a(xcfg.o)
 .data          0x0000000000000000        0x0 ..\..\..\..\Libraries\libs\libplatform.a(xcfg.o)
 .bss           0x0000000000000000        0x0 ..\..\..\..\Libraries\libs\libplatform.a(xcfg.o)
 .text          0x0000000000000000        0x0 ..\..\..\..\Libraries\libs\libplatform.a(device.o)
 .data          0x0000000000000000        0x0 ..\..\..\..\Libraries\libs\libplatform.a(device.o)
 .bss           0x0000000000000000        0x0 ..\..\..\..\Libraries\libs\libplatform.a(device.o)
 .text.sd_disable
                0x0000000000000000       0x18 ..\..\..\..\Libraries\libs\libplatform.a(device.o)
 .text.sd_disable_user
                0x0000000000000000       0x46 ..\..\..\..\Libraries\libs\libplatform.a(device.o)
 .text.sd_enable_user
                0x0000000000000000       0x2c ..\..\..\..\Libraries\libs\libplatform.a(device.o)
 .com_text.device
                0x0000000000000000       0x10 ..\..\..\..\Libraries\libs\libplatform.a(device.o)
 .com_text.device.udisk
                0x0000000000000000        0xe ..\..\..\..\Libraries\libs\libplatform.a(device.o)
 .com_text.device.filter
                0x0000000000000000       0xe0 ..\..\..\..\Libraries\libs\libplatform.a(device.o)
 .text.device   0x0000000000000000       0x40 ..\..\..\..\Libraries\libs\libplatform.a(device.o)
 .text.dev_is_invalid
                0x0000000000000000        0xe ..\..\..\..\Libraries\libs\libplatform.a(device.o)
 .com_text.sd.api
                0x0000000000000000       0x3c ..\..\..\..\Libraries\libs\libplatform.a(device.o)
 .text.fs_lock  0x0000000000000000       0x14 ..\..\..\..\Libraries\libs\libplatform.a(device.o)
 .text.fs_unlock
                0x0000000000000000       0x12 ..\..\..\..\Libraries\libs\libplatform.a(device.o)
 .sbss          0x0000000000000000        0x4 ..\..\..\..\Libraries\libs\libplatform.a(device.o)
 .text          0x0000000000000000        0x0 ..\..\..\..\Libraries\libs\libplatform.a(main.o)
 .data          0x0000000000000000        0x0 ..\..\..\..\Libraries\libs\libplatform.a(main.o)
 .com_text.exception.do
                0x0000000000000000       0x5a ..\..\..\..\Libraries\libs\libplatform.a(main.o)
 .com_text.ledseg
                0x0000000000000000       0x40 ..\..\..\..\Libraries\libs\libplatform.a(main.o)
 .text.uart0_mapping_sel
                0x0000000000000000       0x18 ..\..\..\..\Libraries\libs\libplatform.a(main.o)
 .text.compiler
                0x0000000000000000       0x20 ..\..\..\..\Libraries\libs\libplatform.a(main.o)
 .com_text.ledseg.table
                0x0000000000000000        0xc ..\..\..\..\Libraries\libs\libplatform.a(main.o)
 .text          0x0000000000000000        0x0 ..\..\..\..\Libraries\libs\libplatform.a(interrupt.o)
 .data          0x0000000000000000        0x0 ..\..\..\..\Libraries\libs\libplatform.a(interrupt.o)
 .bss           0x0000000000000000        0x0 ..\..\..\..\Libraries\libs\libplatform.a(interrupt.o)
 .text.timer1_irq_init
                0x0000000000000000       0x38 ..\..\..\..\Libraries\libs\libplatform.a(interrupt.o)
 .com_text.tws.isr
                0x0000000000000000       0x22 ..\..\..\..\Libraries\libs\libplatform.a(interrupt.o)
 .text.huart_irq_init
                0x0000000000000000       0x3a ..\..\..\..\Libraries\libs\libplatform.a(interrupt.o)
 .rodata.str1.4
                0x0000000000000000       0x19 ..\..\..\..\Libraries\libs\libplatform.a(interrupt.o)
 .text.watch_point_set
                0x0000000000000000       0x48 ..\..\..\..\Libraries\libs\libplatform.a(interrupt.o)
 .text.wdt_init
                0x0000000000000000       0x3a ..\..\..\..\Libraries\libs\libplatform.a(interrupt.o)
 .text          0x0000000000000000        0x0 ..\..\..\..\Libraries\libs\libplatform.a(startup.o)
 .data          0x0000000000000000        0x0 ..\..\..\..\Libraries\libs\libplatform.a(startup.o)
 .com_text.sndp.api
                0x0000000000000000       0x26 ..\..\..\..\Libraries\libs\libplatform.a(startup.o)
 .text          0x0000000000000000        0x0 ..\..\..\..\Libraries\libs\libplatform.a(sys_hook.o)
 .data          0x0000000000000000        0x0 ..\..\..\..\Libraries\libs\libplatform.a(sys_hook.o)
 .bss           0x0000000000000000        0x0 ..\..\..\..\Libraries\libs\libplatform.a(sys_hook.o)
 .text          0x0000000000000000        0x0 ..\..\..\..\Libraries\libs\libplatform.a(reset.o)
 .data          0x0000000000000000        0x0 ..\..\..\..\Libraries\libs\libplatform.a(reset.o)
 .bss           0x0000000000000000        0x0 ..\..\..\..\Libraries\libs\libplatform.a(reset.o)
 .text          0x0000000000000000        0x0 ..\..\..\..\Libraries\libs\libplatform.a(spiflash.o)
 .data          0x0000000000000000        0x0 ..\..\..\..\Libraries\libs\libplatform.a(spiflash.o)
 .bss           0x0000000000000000        0x0 ..\..\..\..\Libraries\libs\libplatform.a(spiflash.o)
 .text          0x0000000000000000        0x0 ..\..\..\..\Libraries\libs\libplatform.a(debug.o)
 .data          0x0000000000000000        0x0 ..\..\..\..\Libraries\libs\libplatform.a(debug.o)
 .bss           0x0000000000000000        0x0 ..\..\..\..\Libraries\libs\libplatform.a(debug.o)
 .text.debug_dump_info_nanos_schedule
                0x0000000000000000        0x2 ..\..\..\..\Libraries\libs\libplatform.a(debug.o)
 .text.debug_dump_info_nanos_timer
                0x0000000000000000        0x2 ..\..\..\..\Libraries\libs\libplatform.a(debug.o)
 .text          0x0000000000000000        0x0 ..\..\..\..\Libraries\libs\libplatform.a(fot_update.o)
 .data          0x0000000000000000        0x0 ..\..\..\..\Libraries\libs\libplatform.a(fot_update.o)
 .text.param_fot_head_info_write
                0x0000000000000000        0x2 ..\..\..\..\Libraries\libs\libplatform.a(fot_update.o)
 .text.param_fot_head_info_read
                0x0000000000000000        0x2 ..\..\..\..\Libraries\libs\libplatform.a(fot_update.o)
 .text.param_fot_addr_write
                0x0000000000000000        0x2 ..\..\..\..\Libraries\libs\libplatform.a(fot_update.o)
 .text.param_fot_addr_read
                0x0000000000000000        0x2 ..\..\..\..\Libraries\libs\libplatform.a(fot_update.o)
 .text.is_fot_update_en
                0x0000000000000000        0x4 ..\..\..\..\Libraries\libs\libplatform.a(fot_update.o)
 .text.fot_head_crc_get
                0x0000000000000000       0x9c ..\..\..\..\Libraries\libs\libplatform.a(fot_update.o)
 .text.fot_get_info
                0x0000000000000000       0x50 ..\..\..\..\Libraries\libs\libplatform.a(fot_update.o)
 .text          0x0000000000000000        0x0 ..\..\..\..\Libraries\libs\libplatform.a(lock.o)
 .data          0x0000000000000000        0x0 ..\..\..\..\Libraries\libs\libplatform.a(lock.o)
 .text.unlock_whcode
                0x0000000000000000       0x3c ..\..\..\..\Libraries\libs\libplatform.a(lock.o)
 .text.lock_whcode
                0x0000000000000000       0x58 ..\..\..\..\Libraries\libs\libplatform.a(lock.o)
 .text.unlock_dcode
                0x0000000000000000       0x54 ..\..\..\..\Libraries\libs\libplatform.a(lock.o)
 .text.lock_dcode
                0x0000000000000000       0x58 ..\..\..\..\Libraries\libs\libplatform.a(lock.o)
 .text.lock_code_bt_sleep
                0x0000000000000000       0x54 ..\..\..\..\Libraries\libs\libplatform.a(lock.o)
 .text.unlock_code_bt_sleep
                0x0000000000000000       0x38 ..\..\..\..\Libraries\libs\libplatform.a(lock.o)
 .text.lock_code_pwrsave
                0x0000000000000000       0x3c ..\..\..\..\Libraries\libs\libplatform.a(lock.o)
 .text.unlock_code_pwrsave
                0x0000000000000000       0x38 ..\..\..\..\Libraries\libs\libplatform.a(lock.o)
 .text.lock_code_charge
                0x0000000000000000       0x3c ..\..\..\..\Libraries\libs\libplatform.a(lock.o)
 .text.unlock_code_charge
                0x0000000000000000        0x8 ..\..\..\..\Libraries\libs\libplatform.a(lock.o)
 .text.unlock_code_bt_voice
                0x0000000000000000       0x38 ..\..\..\..\Libraries\libs\libplatform.a(lock.o)
 .text.lock_code_usbdev
                0x0000000000000000       0x54 ..\..\..\..\Libraries\libs\libplatform.a(lock.o)
 .text.unlock_code_usbdev
                0x0000000000000000       0x38 ..\..\..\..\Libraries\libs\libplatform.a(lock.o)
 .text.load_code_btdec
                0x0000000000000000       0x54 ..\..\..\..\Libraries\libs\libplatform.a(lock.o)
 .text.unlock_code_btdec
                0x0000000000000000       0x38 ..\..\..\..\Libraries\libs\libplatform.a(lock.o)
 .text.load_code_bt_voice
                0x0000000000000000       0x5c ..\..\..\..\Libraries\libs\libplatform.a(lock.o)
 .text.lock_code_bt_comm
                0x0000000000000000        0x2 ..\..\..\..\Libraries\libs\libplatform.a(lock.o)
 .text.unlock_code_bt_comm
                0x0000000000000000        0x2 ..\..\..\..\Libraries\libs\libplatform.a(lock.o)
 .text.lock_ram_mp3enc
                0x0000000000000000       0x4c ..\..\..\..\Libraries\libs\libplatform.a(lock.o)
 .text.unlock_ram_mp3enc
                0x0000000000000000       0x38 ..\..\..\..\Libraries\libs\libplatform.a(lock.o)
 .text.lock_code_sniff
                0x0000000000000000       0x4c ..\..\..\..\Libraries\libs\libplatform.a(lock.o)
 .text.unlock_code_sniff
                0x0000000000000000       0x38 ..\..\..\..\Libraries\libs\libplatform.a(lock.o)
 .text.unlock_code_huart
                0x0000000000000000        0x8 ..\..\..\..\Libraries\libs\libplatform.a(lock.o)
 .text.lock_code_huart
                0x0000000000000000       0x54 ..\..\..\..\Libraries\libs\libplatform.a(lock.o)
 .text.lock_code_bb_test
                0x0000000000000000       0x54 ..\..\..\..\Libraries\libs\libplatform.a(lock.o)
 .text.unlock_code_bb_test
                0x0000000000000000       0x38 ..\..\..\..\Libraries\libs\libplatform.a(lock.o)
 .text.unlock_code_fota
                0x0000000000000000       0x38 ..\..\..\..\Libraries\libs\libplatform.a(lock.o)
 .text          0x0000000000000000        0x0 ..\..\..\..\Libraries\libs\libplatform.a(patch.o)
 .data          0x0000000000000000        0x0 ..\..\..\..\Libraries\libs\libplatform.a(patch.o)
 .bss           0x0000000000000000        0x0 ..\..\..\..\Libraries\libs\libplatform.a(patch.o)
 .text          0x0000000000000000        0x0 ..\..\..\..\Libraries\libs\libplatform.a(power.o)
 .data          0x0000000000000000        0x0 ..\..\..\..\Libraries\libs\libplatform.a(power.o)
 .bss           0x0000000000000000        0x0 ..\..\..\..\Libraries\libs\libplatform.a(power.o)
 .com_text.voltage.trim
                0x0000000000000000        0xa ..\..\..\..\Libraries\libs\libplatform.a(power.o)
 .text          0x0000000000000000        0x0 ..\..\..\..\Libraries\libs\libplatform.a(rc.o)
 .data          0x0000000000000000        0x0 ..\..\..\..\Libraries\libs\libplatform.a(rc.o)
 .bss           0x0000000000000000        0x0 ..\..\..\..\Libraries\libs\libplatform.a(rc.o)
 .text.compiler
                0x0000000000000000        0x2 ..\..\..\..\Libraries\libs\libplatform.a(rc.o)
 .text          0x0000000000000000        0x0 ..\..\..\..\Libraries\libs\libplatform.a(s_sys.o)
 .data          0x0000000000000000        0x0 ..\..\..\..\Libraries\libs\libplatform.a(s_sys.o)
 .bss           0x0000000000000000        0x0 ..\..\..\..\Libraries\libs\libplatform.a(s_sys.o)
 .text          0x0000000000000000        0x0 ..\..\..\..\Libraries\libs\libplatform.a(sys.o)
 .data          0x0000000000000000        0x0 ..\..\..\..\Libraries\libs\libplatform.a(sys.o)
 .bss           0x0000000000000000        0x0 ..\..\..\..\Libraries\libs\libplatform.a(sys.o)
 .text.dbg_clk_out
                0x0000000000000000       0x44 ..\..\..\..\Libraries\libs\libplatform.a(sys.o)
 .text.sys_clk_output
                0x0000000000000000      0x136 ..\..\..\..\Libraries\libs\libplatform.a(sys.o)
 .text.__divdi3
                0x0000000000000000       0x5c ..\..\..\..\Libraries\libs\libplatform.a(sys.o)
 .text.__umoddi3
                0x0000000000000000       0x30 ..\..\..\..\Libraries\libs\libplatform.a(sys.o)
 .text.get_random
                0x0000000000000000       0x26 ..\..\..\..\Libraries\libs\libplatform.a(sys.o)
 .text.random_init
                0x0000000000000000        0xa ..\..\..\..\Libraries\libs\libplatform.a(sys.o)
 .text.convert_uni2gbk
                0x0000000000000000       0x8a ..\..\..\..\Libraries\libs\libplatform.a(sys.o)
 .text.lrc      0x0000000000000000       0x58 ..\..\..\..\Libraries\libs\libplatform.a(sys.o)
 .text.utf8_convert_to_unicode
                0x0000000000000000       0x72 ..\..\..\..\Libraries\libs\libplatform.a(sys.o)
 .com_text.sys  0x0000000000000000       0x1e ..\..\..\..\Libraries\libs\libplatform.a(sys.o)
 .text.sw_reset_source_get
                0x0000000000000000       0x2a ..\..\..\..\Libraries\libs\libplatform.a(sys.o)
 .sleep_text.sleep
                0x0000000000000000      0x128 ..\..\..\..\Libraries\libs\libplatform.a(sys.o)
 .text.sys.power
                0x0000000000000000       0x96 ..\..\..\..\Libraries\libs\libplatform.a(sys.o)
 .text          0x0000000000000000        0x0 ..\..\..\..\Libraries\libs\libplatform.a(sys_clk.o)
 .data          0x0000000000000000        0x0 ..\..\..\..\Libraries\libs\libplatform.a(sys_clk.o)
 .bss           0x0000000000000000        0x0 ..\..\..\..\Libraries\libs\libplatform.a(sys_clk.o)
 .com_text.sys  0x0000000000000000        0x4 ..\..\..\..\Libraries\libs\libplatform.a(sys_clk.o)
 .text.sys_clk.aec
                0x0000000000000000      0x200 ..\..\..\..\Libraries\libs\libplatform.a(sys_clk.o)
 .text.set_uart0_baud
                0x0000000000000000       0x38 ..\..\..\..\Libraries\libs\libplatform.a(sys_clk.o)
 .text.set_uart1_baud
                0x0000000000000000       0x38 ..\..\..\..\Libraries\libs\libplatform.a(sys_clk.o)
 .text.set_uart1_baud_rc2m_clk
                0x0000000000000000       0x24 ..\..\..\..\Libraries\libs\libplatform.a(sys_clk.o)
 .text.sys_clk_get
                0x0000000000000000        0xa ..\..\..\..\Libraries\libs\libplatform.a(sys_clk.o)
 .text.sys_clk_req
                0x0000000000000000       0x5e ..\..\..\..\Libraries\libs\libplatform.a(sys_clk.o)
 .text.sys_clk_free
                0x0000000000000000       0x5c ..\..\..\..\Libraries\libs\libplatform.a(sys_clk.o)
 .text.sys_clk_free_all
                0x0000000000000000       0x50 ..\..\..\..\Libraries\libs\libplatform.a(sys_clk.o)
 .text          0x0000000000000000        0x0 ..\..\..\..\Libraries\libs\libplatform.a(voltage_trim.o)
 .data          0x0000000000000000        0x0 ..\..\..\..\Libraries\libs\libplatform.a(voltage_trim.o)
 .text          0x0000000000000000        0x0 ..\..\..\..\Libraries\libs\libplatform.a(weak_symbol.o)
 .data          0x0000000000000000        0x0 ..\..\..\..\Libraries\libs\libplatform.a(weak_symbol.o)
 .bss           0x0000000000000000        0x0 ..\..\..\..\Libraries\libs\libplatform.a(weak_symbol.o)
 .text.music_eq_get_bass_tbl
                0x0000000000000000        0x4 ..\..\..\..\Libraries\libs\libplatform.a(weak_symbol.o)
 .text.music_eq_get_treble_tbl
                0x0000000000000000        0x4 ..\..\..\..\Libraries\libs\libplatform.a(weak_symbol.o)
 .text.mic_eq_get_bass_tbl
                0x0000000000000000        0x4 ..\..\..\..\Libraries\libs\libplatform.a(weak_symbol.o)
 .text.mic_eq_get_treble_tbl
                0x0000000000000000        0x4 ..\..\..\..\Libraries\libs\libplatform.a(weak_symbol.o)
 .text.music_eq_get_tbl
                0x0000000000000000        0x4 ..\..\..\..\Libraries\libs\libplatform.a(weak_symbol.o)
 .text.bass_treble_get_coef_tbl
                0x0000000000000000        0x4 ..\..\..\..\Libraries\libs\libplatform.a(weak_symbol.o)
 .text.stream   0x0000000000000000        0x8 ..\..\..\..\Libraries\libs\libplatform.a(weak_symbol.o)
 .com_text.rec  0x0000000000000000        0x2 ..\..\..\..\Libraries\libs\libplatform.a(weak_symbol.o)
 .text.update   0x0000000000000000        0x4 ..\..\..\..\Libraries\libs\libplatform.a(weak_symbol.o)
 .text.qtest    0x0000000000000000       0x1a ..\..\..\..\Libraries\libs\libplatform.a(weak_symbol.o)
 .text.dacr_is_output
                0x0000000000000000        0x4 ..\..\..\..\Libraries\libs\libplatform.a(weak_symbol.o)
 .text.sd_is_online
                0x0000000000000000        0x4 ..\..\..\..\Libraries\libs\libplatform.a(weak_symbol.o)
 .sbss          0x0000000000000000        0x1 ..\..\..\..\Libraries\libs\libplatform.a(weak_symbol.o)
 .text          0x0000000000000000        0x0 ..\..\..\..\Libraries\libs\libplatform.a(huart.o)
 .data          0x0000000000000000        0x0 ..\..\..\..\Libraries\libs\libplatform.a(huart.o)
 .bss           0x0000000000000000        0x0 ..\..\..\..\Libraries\libs\libplatform.a(huart.o)
 .com_huart.text
                0x0000000000000000      0x1b2 ..\..\..\..\Libraries\libs\libplatform.a(huart.o)
 .text.huart_tx_done
                0x0000000000000000        0x2 ..\..\..\..\Libraries\libs\libplatform.a(huart.o)
 .text.lock_code_huart
                0x0000000000000000        0x2 ..\..\..\..\Libraries\libs\libplatform.a(huart.o)
 .text.huart_irq_init
                0x0000000000000000        0x2 ..\..\..\..\Libraries\libs\libplatform.a(huart.o)
 .text.huart.huart_init_do
                0x0000000000000000      0x194 ..\..\..\..\Libraries\libs\libplatform.a(huart.o)
 .text.huart.huart_exit
                0x0000000000000000       0x12 ..\..\..\..\Libraries\libs\libplatform.a(huart.o)
 .text.huart.huart_setbaudrate
                0x0000000000000000       0x36 ..\..\..\..\Libraries\libs\libplatform.a(huart.o)
 .com_text.huart.huart_getchar
                0x0000000000000000       0x2e ..\..\..\..\Libraries\libs\libplatform.a(huart.o)
 .com_huart.rodata
                0x0000000000000000       0x58 ..\..\..\..\Libraries\libs\libplatform.a(huart.o)
 .sbss          0x0000000000000000        0xc ..\..\..\..\Libraries\libs\libplatform.a(huart.o)
 .comment       0x0000000000000000       0x13 ..\..\..\..\Libraries\libs\libplatform.a(huart.o)
 .riscv.attributes
                0x0000000000000000       0x32 ..\..\..\..\Libraries\libs\libplatform.a(huart.o)
 .text          0x0000000000000000        0x0 ..\..\..\..\Libraries\libs\libplatform.a(usb.o)
 .data          0x0000000000000000        0x0 ..\..\..\..\Libraries\libs\libplatform.a(usb.o)
 .bss           0x0000000000000000        0x0 ..\..\..\..\Libraries\libs\libplatform.a(usb.o)
 .text          0x0000000000000000        0x0 ..\..\..\..\Libraries\libs\libplatform.a(bt.o)
 .data          0x0000000000000000        0x0 ..\..\..\..\Libraries\libs\libplatform.a(bt.o)
 .bss           0x0000000000000000        0x0 ..\..\..\..\Libraries\libs\libplatform.a(bt.o)
 .com_text.isr.txrx
                0x0000000000000000        0x2 ..\..\..\..\Libraries\libs\libplatform.a(bt.o)
 .text.update   0x0000000000000000        0x4 ..\..\..\..\Libraries\libs\libplatform.a(bt.o)
 .bt_voice.plc  0x0000000000000000       0x48 ..\..\..\..\Libraries\libs\libplatform.a(bt.o)
 .rodata.str1.4
                0x0000000000000000        0xd ..\..\..\..\Libraries\libs\libplatform.a(bt.o)
 .com_text.btstack.uart
                0x0000000000000000       0x26 ..\..\..\..\Libraries\libs\libplatform.a(bt.o)
 .data          0x0000000000000000        0x0 ..\..\..\..\Libraries\libs\libbtstack.a(nanos.o)
 .bss           0x0000000000000000        0x0 ..\..\..\..\Libraries\libs\libbtstack.a(nanos.o)
 .com_text.md.nanos
                0x0000000000000000       0x3c ..\..\..\..\Libraries\libs\libbtstack.a(nanos.o)
 .data          0x0000000000000000        0x0 ..\..\..\..\Libraries\libs\libbtstack.a(patch.o)
 .bss           0x0000000000000000        0x0 ..\..\..\..\Libraries\libs\libbtstack.a(patch.o)
 .data          0x0000000000000000        0x0 ..\..\..\..\Libraries\libs\libbtstack.a(platform.o)
 .bss           0x0000000000000000        0x0 ..\..\..\..\Libraries\libs\libbtstack.a(platform.o)
 .com_text.bb.isr.timer
                0x0000000000000000        0x2 ..\..\..\..\Libraries\libs\libbtstack.a(platform.o)
 .data          0x0000000000000000        0x0 ..\..\..\..\Libraries\libs\libbtstack.a(bt_sco.o)
 .bss           0x0000000000000000        0x0 ..\..\..\..\Libraries\libs\libbtstack.a(bt_sco.o)
 .bt_voice.bb.cvsd
                0x0000000000000000        0x2 ..\..\..\..\Libraries\libs\libbtstack.a(bt_sco.o)
 .bt_voice.plc  0x0000000000000000        0x2 ..\..\..\..\Libraries\libs\libbtstack.a(bt_sco.o)
 .data          0x0000000000000000        0x0 ..\..\..\..\Libraries\libs\libbtstack.a(bt_acl.o)
 .bss           0x0000000000000000        0x0 ..\..\..\..\Libraries\libs\libbtstack.a(bt_acl.o)
 .data          0x0000000000000000        0x0 ..\..\..\..\Libraries\libs\libbtstack.a(ble_con.o)
 .bss           0x0000000000000000        0x0 ..\..\..\..\Libraries\libs\libbtstack.a(ble_con.o)
 .data          0x0000000000000000        0x0 ..\..\..\..\Libraries\libs\libbtstack.a(bb_utils.o)
 .bss           0x0000000000000000        0x0 ..\..\..\..\Libraries\libs\libbtstack.a(bb_utils.o)
 .srodata       0x0000000000000000        0x5 ..\..\..\..\Libraries\libs\libbtstack.a(bb_utils.o)
 .data          0x0000000000000000        0x0 ..\..\..\..\Libraries\libs\libbtstack.a(bb_int.o)
 .bss           0x0000000000000000        0x0 ..\..\..\..\Libraries\libs\libbtstack.a(bb_int.o)
 .com_text.bb.isr.timer
                0x0000000000000000       0x48 ..\..\..\..\Libraries\libs\libbtstack.a(bb_int.o)
 .text.bb.timer.init
                0x0000000000000000       0x76 ..\..\..\..\Libraries\libs\libbtstack.a(bb_int.o)
 .text.bb.timer.kill
                0x0000000000000000       0x22 ..\..\..\..\Libraries\libs\libbtstack.a(bb_int.o)
 .com_text.bb.timer.get
                0x0000000000000000       0x24 ..\..\..\..\Libraries\libs\libbtstack.a(bb_int.o)
 .sleep_text.bb
                0x0000000000000000      0x232 ..\..\..\..\Libraries\libs\libbtstack.a(bb_int.o)
 .com_text.bb.sleep
                0x0000000000000000       0x4c ..\..\..\..\Libraries\libs\libbtstack.a(bb_int.o)
 .data          0x0000000000000000        0x0 ..\..\..\..\Libraries\libs\libbtstack.a(bb.o)
 .text.update   0x0000000000000000       0x1a ..\..\..\..\Libraries\libs\libbtstack.a(bb.o)
 .data          0x0000000000000000        0x0 ..\..\..\..\Libraries\libs\libbtstack.a(platform.o)
 .bss           0x0000000000000000        0x0 ..\..\..\..\Libraries\libs\libbtstack.a(platform.o)
 .com_text.cpu.sfr
                0x0000000000000000       0x3c ..\..\..\..\Libraries\libs\libbtstack.a(platform.o)
 .com_text.sco  0x0000000000000000        0x8 ..\..\..\..\Libraries\libs\libbtstack.a(platform.o)
 .data          0x0000000000000000        0x0 ..\..\..\..\Libraries\libs\libbtstack.a(extern_tws.o)
 .bss           0x0000000000000000        0x0 ..\..\..\..\Libraries\libs\libbtstack.a(extern_tws.o)
 .sdata         0x0000000000000000        0x7 ..\..\..\..\Libraries\libs\libbtstack.a(extern_tws.o)
 .data          0x0000000000000000        0x0 ..\..\..\..\Libraries\libs\libbtstack.a(extern_bt.o)
 .bss           0x0000000000000000        0x0 ..\..\..\..\Libraries\libs\libbtstack.a(extern_bt.o)
 .com_text.bt_rec
                0x0000000000000000        0x2 ..\..\..\..\Libraries\libs\libbtstack.a(extern_bt.o)
 .com_text.aec  0x0000000000000000        0x4 ..\..\..\..\Libraries\libs\libbtstack.a(extern_bt.o)
 .bt_voice.sco  0x0000000000000000        0x2 ..\..\..\..\Libraries\libs\libbtstack.a(extern_bt.o)
 .bt_voice.bb.cvsd
                0x0000000000000000        0x2 ..\..\..\..\Libraries\libs\libbtstack.a(extern_bt.o)
 .text          0x0000000000000000       0x28 ..\..\..\..\Libraries\libs\libbtstack.a(extern.o)
 .data          0x0000000000000000        0x0 ..\..\..\..\Libraries\libs\libbtstack.a(extern.o)
 .bss           0x0000000000000000        0x0 ..\..\..\..\Libraries\libs\libbtstack.a(extern.o)
 .text.huart    0x0000000000000000        0x2 ..\..\..\..\Libraries\libs\libbtstack.a(extern.o)
 .com_text.huart
                0x0000000000000000        0xe ..\..\..\..\Libraries\libs\libbtstack.a(extern.o)
 .com_text.ticks
                0x0000000000000000        0x4 ..\..\..\..\Libraries\libs\libbtstack.a(extern.o)
 .sbss          0x0000000000000000        0x1 ..\..\..\..\Libraries\libs\libbtstack.a(extern.o)
 .data          0x0000000000000000        0x0 ..\..\..\..\Libraries\libs\libbtstack.a(spp.o)
 .bss           0x0000000000000000        0x0 ..\..\..\..\Libraries\libs\libbtstack.a(spp.o)
 .sbss          0x0000000000000000        0x1 ..\..\..\..\Libraries\libs\libbtstack.a(spp.o)
 .text          0x0000000000000000        0x0 ..\..\..\..\Libraries\libs\libbtstack.a(sdp_util.o)
 .data          0x0000000000000000        0x0 ..\..\..\..\Libraries\libs\libbtstack.a(sdp_util.o)
 .bss           0x0000000000000000        0x0 ..\..\..\..\Libraries\libs\libbtstack.a(sdp_util.o)
 .text          0x0000000000000000        0x0 ..\..\..\..\Libraries\libs\libbtstack.a(sdp_tbl.o)
 .data          0x0000000000000000        0x0 ..\..\..\..\Libraries\libs\libbtstack.a(sdp_tbl.o)
 .bss           0x0000000000000000        0x0 ..\..\..\..\Libraries\libs\libbtstack.a(sdp_tbl.o)
 .rodata.sdp.tbl.avctp_controller
                0x0000000000000000       0x44 ..\..\..\..\Libraries\libs\libbtstack.a(sdp_tbl.o)
 .rodata.sdp.tbl.avctp_target2
                0x0000000000000000       0x41 ..\..\..\..\Libraries\libs\libbtstack.a(sdp_tbl.o)
 .rodata.sdp.tbl.avdtp
                0x0000000000000000       0x41 ..\..\..\..\Libraries\libs\libbtstack.a(sdp_tbl.o)
 .rodata.sdp.tbl.hfp
                0x0000000000000000       0x50 ..\..\..\..\Libraries\libs\libbtstack.a(sdp_tbl.o)
 .rodata.sdp.tbl.hid_consumer
                0x0000000000000000       0xd2 ..\..\..\..\Libraries\libs\libbtstack.a(sdp_tbl.o)
 .rodata.sdp.tbl.hid_did
                0x0000000000000000       0x40 ..\..\..\..\Libraries\libs\libbtstack.a(sdp_tbl.o)
 .rodata.sdp.tbl.hid_keyboard
                0x0000000000000000      0x115 ..\..\..\..\Libraries\libs\libbtstack.a(sdp_tbl.o)
 .rodata.sdp.tbl.hid_tscreen
                0x0000000000000000      0x110 ..\..\..\..\Libraries\libs\libbtstack.a(sdp_tbl.o)
 .rodata.sdp.tbl.hid_tscreen_ext
                0x0000000000000000      0x119 ..\..\..\..\Libraries\libs\libbtstack.a(sdp_tbl.o)
 .rodata.sdp.tbl.spp_dueros
                0x0000000000000000       0x51 ..\..\..\..\Libraries\libs\libbtstack.a(sdp_tbl.o)
 .data          0x0000000000000000        0x0 ..\..\..\..\Libraries\libs\libbtstack.a(sdp_server.o)
 .bss           0x0000000000000000        0x0 ..\..\..\..\Libraries\libs\libbtstack.a(sdp_server.o)
 .text.stack.sdp.server_rmv
                0x0000000000000000       0x2c ..\..\..\..\Libraries\libs\libbtstack.a(sdp_server.o)
 .data          0x0000000000000000        0x0 ..\..\..\..\Libraries\libs\libbtstack.a(sdp_client.o)
 .bss           0x0000000000000000        0x0 ..\..\..\..\Libraries\libs\libbtstack.a(sdp_client.o)
 .data          0x0000000000000000        0x0 ..\..\..\..\Libraries\libs\libbtstack.a(rfcomm.o)
 .bss           0x0000000000000000        0x0 ..\..\..\..\Libraries\libs\libbtstack.a(rfcomm.o)
 .text          0x0000000000000000        0x0 ..\..\..\..\Libraries\libs\libbtstack.a(btstack_link_key_db.o)
 .sbss          0x0000000000000000        0x1 ..\..\..\..\Libraries\libs\libbtstack.a(btstack_link_key_db.o)
 .data          0x0000000000000000        0x0 ..\..\..\..\Libraries\libs\libbtstack.a(btstack_util.o)
 .bss           0x0000000000000000        0x0 ..\..\..\..\Libraries\libs\libbtstack.a(btstack_util.o)
 .data          0x0000000000000000        0x0 ..\..\..\..\Libraries\libs\libbtstack.a(btstack_txpkt.o)
 .bss           0x0000000000000000        0x0 ..\..\..\..\Libraries\libs\libbtstack.a(btstack_txpkt.o)
 .text          0x0000000000000000        0x0 ..\..\..\..\Libraries\libs\libbtstack.a(btstack_run_loop.o)
 .bss           0x0000000000000000        0x0 ..\..\..\..\Libraries\libs\libbtstack.a(btstack_run_loop.o)
 .text          0x0000000000000000       0x22 ..\..\..\..\Libraries\libs\libbtstack.a(btstack_memory.o)
 .data          0x0000000000000000        0x0 ..\..\..\..\Libraries\libs\libbtstack.a(btstack_memory.o)
 .text          0x0000000000000000       0x54 ..\..\..\..\Libraries\libs\libbtstack.a(btstack_linked_list.o)
 .data          0x0000000000000000        0x0 ..\..\..\..\Libraries\libs\libbtstack.a(btstack_linked_list.o)
 .bss           0x0000000000000000        0x0 ..\..\..\..\Libraries\libs\libbtstack.a(btstack_linked_list.o)
 .com_text.fifo.search
                0x0000000000000000       0x28 ..\..\..\..\Libraries\libs\libbtstack.a(btstack_linked_list.o)
 .com_text.fifo.add
                0x0000000000000000       0x5e ..\..\..\..\Libraries\libs\libbtstack.a(btstack_linked_list.o)
 .btdec.a2dp.list
                0x0000000000000000      0x1be ..\..\..\..\Libraries\libs\libbtstack.a(btstack_linked_list.o)
 .data          0x0000000000000000        0x0 ..\..\..\..\Libraries\libs\libbtstack.a(btstack_link_ctrl.o)
 .bss           0x0000000000000000        0x0 ..\..\..\..\Libraries\libs\libbtstack.a(btstack_link_ctrl.o)
 .sbss          0x0000000000000000        0x1 ..\..\..\..\Libraries\libs\libbtstack.a(btstack_link_ctrl.o)
 .data          0x0000000000000000        0x0 ..\..\..\..\Libraries\libs\libbtstack.a(gatt_server.o)
 .bss           0x0000000000000000        0x0 ..\..\..\..\Libraries\libs\libbtstack.a(gatt_server.o)
 .com_text.ble_frame1
                0x0000000000000000       0x2a ..\..\..\..\Libraries\libs\libbtstack.a(gatt_server.o)
 .text.ble.notify_handle
                0x0000000000000000       0x54 ..\..\..\..\Libraries\libs\libbtstack.a(gatt_server.o)
 .com_text.ble.send_kick
                0x0000000000000000        0xe ..\..\..\..\Libraries\libs\libbtstack.a(gatt_server.o)
 .sbss          0x0000000000000000        0x1 ..\..\..\..\Libraries\libs\libbtstack.a(gatt_server.o)
 .data          0x0000000000000000        0x0 ..\..\..\..\Libraries\libs\libbtstack.a(gatt_profile.o)
 .bss           0x0000000000000000        0x0 ..\..\..\..\Libraries\libs\libbtstack.a(gatt_profile.o)
 .data          0x0000000000000000        0x0 ..\..\..\..\Libraries\libs\libbtstack.a(att_server.o)
 .bss           0x0000000000000000        0x0 ..\..\..\..\Libraries\libs\libbtstack.a(att_server.o)
 .data          0x0000000000000000        0x0 ..\..\..\..\Libraries\libs\libbtstack.a(att_dispatch.o)
 .bss           0x0000000000000000        0x0 ..\..\..\..\Libraries\libs\libbtstack.a(att_dispatch.o)
 .data          0x0000000000000000        0x0 ..\..\..\..\Libraries\libs\libbtstack.a(att_db.o)
 .bss           0x0000000000000000        0x0 ..\..\..\..\Libraries\libs\libbtstack.a(att_db.o)
 .text          0x0000000000000000      0x1ea ..\..\..\..\Libraries\libs\libbtstack.a(ad_parser.o)
 .data          0x0000000000000000        0x0 ..\..\..\..\Libraries\libs\libbtstack.a(ad_parser.o)
 .bss           0x0000000000000000        0x0 ..\..\..\..\Libraries\libs\libbtstack.a(ad_parser.o)
 .data          0x0000000000000000        0x0 ..\..\..\..\Libraries\libs\libbtstack.a(btstack_main.o)
 .bss           0x0000000000000000        0x0 ..\..\..\..\Libraries\libs\libbtstack.a(btstack_main.o)
 .text.stack.ble.sm
                0x0000000000000000       0x38 ..\..\..\..\Libraries\libs\libbtstack.a(btstack_main.o)
 .data          0x0000000000000000        0x0 ..\..\..\..\Libraries\libs\libbtstack.a(btstack_hal.o)
 .bss           0x0000000000000000        0x0 ..\..\..\..\Libraries\libs\libbtstack.a(btstack_hal.o)
 .com_text.stack.uart_isr
                0x0000000000000000       0x7e ..\..\..\..\Libraries\libs\libbtstack.a(btstack_hal.o)
 .text.stack.hal
                0x0000000000000000       0xa2 ..\..\..\..\Libraries\libs\libbtstack.a(btstack_hal.o)
 .com_text.stack.util
                0x0000000000000000       0x12 ..\..\..\..\Libraries\libs\libbtstack.a(btstack_hal.o)
 .sbss          0x0000000000000000        0x9 ..\..\..\..\Libraries\libs\libbtstack.a(btstack_hal.o)
 .data          0x0000000000000000        0x0 ..\..\..\..\Libraries\libs\libbtstack.a(btstack_api.o)
 .com_text.bb.sleep
                0x0000000000000000       0x34 ..\..\..\..\Libraries\libs\libbtstack.a(btstack_api.o)
 .sleep_text.sleep
                0x0000000000000000        0x8 ..\..\..\..\Libraries\libs\libbtstack.a(btstack_api.o)
 .com_text.sco  0x0000000000000000       0x44 ..\..\..\..\Libraries\libs\libbtstack.a(btstack_api.o)
 .sbss          0x0000000000000000        0x7 ..\..\..\..\Libraries\libs\libbtstack.a(btstack_api.o)
 .data          0x0000000000000000        0x0 ..\..\..\..\Libraries\libs\libbtstack.a(bt_api.o)
 .bss           0x0000000000000000        0x0 ..\..\..\..\Libraries\libs\libbtstack.a(bt_api.o)
 .text.stack.api
                0x0000000000000000      0x1da ..\..\..\..\Libraries\libs\libbtstack.a(bt_api.o)
 .text.stack.sleep
                0x0000000000000000       0xc0 ..\..\..\..\Libraries\libs\libbtstack.a(bt_api.o)
 .text.stack.api.hid_con
                0x0000000000000000       0x3a ..\..\..\..\Libraries\libs\libbtstack.a(bt_api.o)
 .text.stack.api.hid_disc
                0x0000000000000000       0x34 ..\..\..\..\Libraries\libs\libbtstack.a(bt_api.o)
 .text.stack.api.hid_send
                0x0000000000000000       0xa6 ..\..\..\..\Libraries\libs\libbtstack.a(bt_api.o)
 .com_text.timer
                0x0000000000000000       0x1a ..\..\..\..\Libraries\libs\libbtstack.a(bt_api.o)
 .sbss          0x0000000000000000        0x1 ..\..\..\..\Libraries\libs\libbtstack.a(bt_api.o)
 .data          0x0000000000000000        0x0 ..\..\..\..\Libraries\libs\libbtstack.a(ble_api.o)
 .bss           0x0000000000000000        0x0 ..\..\..\..\Libraries\libs\libbtstack.a(ble_api.o)
 .text.stack.le.api
                0x0000000000000000       0xa6 ..\..\..\..\Libraries\libs\libbtstack.a(ble_api.o)
 .sbss          0x0000000000000000        0x1 ..\..\..\..\Libraries\libs\libbtstack.a(ble_api.o)
 .data          0x0000000000000000        0x0 ..\..\..\..\Libraries\libs\libbtstack.a(bb_sche.o)
 .text          0x0000000000000000        0x0 ..\..\..\..\Libraries\libs\libbtstack.a(patch_asm.o)
 .data          0x0000000000000000        0x0 ..\..\..\..\Libraries\libs\libbtstack.a(patch_asm.o)
 .bss           0x0000000000000000        0x0 ..\..\..\..\Libraries\libs\libbtstack.a(patch_asm.o)
 .data          0x0000000000000000        0x0 ..\..\..\..\Libraries\libs\libbtstack.a(bb_dbg.o)
 .bss           0x0000000000000000        0x0 ..\..\..\..\Libraries\libs\libbtstack.a(bb_dbg.o)
 .com_text.bb.putc
                0x0000000000000000       0x60 ..\..\..\..\Libraries\libs\libbtstack.a(bb_dbg.o)
 .data          0x0000000000000000        0x0 ..\..\..\..\Libraries\libs\libbtstack.a(bb_clk.o)
 .bss           0x0000000000000000        0x0 ..\..\..\..\Libraries\libs\libbtstack.a(bb_clk.o)
 .text          0x0000000000000000        0x0 ..\..\..\..\Libraries\libs\libbtstack.a(aes.o)
 .data          0x0000000000000000        0x0 ..\..\..\..\Libraries\libs\libbtstack.a(aes.o)
 .data          0x0000000000000000        0x0 ..\..\..\..\Libraries\libs\libbtstack.a(vs_proc.o)
 .bss           0x0000000000000000        0x0 ..\..\..\..\Libraries\libs\libbtstack.a(vs_proc.o)
 .data          0x0000000000000000        0x0 ..\..\..\..\Libraries\libs\libbtstack.a(vs_fcc.o)
 .bss           0x0000000000000000        0x0 ..\..\..\..\Libraries\libs\libbtstack.a(vs_fcc.o)
 .text.bb.vs.fcc_ble.do
                0x0000000000000000       0x7a ..\..\..\..\Libraries\libs\libbtstack.a(vs_fcc.o)
 .data          0x0000000000000000        0x0 ..\..\..\..\Libraries\libs\libbtstack.a(vs.o)
 .bss           0x0000000000000000        0x0 ..\..\..\..\Libraries\libs\libbtstack.a(vs.o)
 .data          0x0000000000000000        0x0 ..\..\..\..\Libraries\libs\libbtstack.a(rf_smart.o)
 .bss           0x0000000000000000        0x0 ..\..\..\..\Libraries\libs\libbtstack.a(rf_smart.o)
 .text.update   0x0000000000000000       0x44 ..\..\..\..\Libraries\libs\libbtstack.a(rf_smart.o)
 .data          0x0000000000000000        0x0 ..\..\..\..\Libraries\libs\libbtstack.a(rf.o)
 .bss           0x0000000000000000        0x0 ..\..\..\..\Libraries\libs\libbtstack.a(rf.o)
 .sleep_text.bb
                0x0000000000000000       0x30 ..\..\..\..\Libraries\libs\libbtstack.a(rf.o)
 .data          0x0000000000000000        0x0 ..\..\..\..\Libraries\libs\libbtstack.a(bt_hook.o)
 .bss           0x0000000000000000        0x0 ..\..\..\..\Libraries\libs\libbtstack.a(bt_hook.o)
 .com_text.bt21.test.fcc
                0x0000000000000000       0xa0 ..\..\..\..\Libraries\libs\libbtstack.a(bt_hook.o)
 .data          0x0000000000000000        0x0 ..\..\..\..\Libraries\libs\libbtstack.a(ble_hook.o)
 .bss           0x0000000000000000        0x0 ..\..\..\..\Libraries\libs\libbtstack.a(ble_hook.o)
 .data          0x0000000000000000        0x0 ..\..\..\..\Libraries\libs\libbtstack.a(hct_tl.o)
 .com_text.bb.sleep
                0x0000000000000000       0x34 ..\..\..\..\Libraries\libs\libbtstack.a(hct_tl.o)
 .data          0x0000000000000000        0x0 ..\..\..\..\Libraries\libs\libbtstack.a(hct_msg.o)
 .bss           0x0000000000000000        0x0 ..\..\..\..\Libraries\libs\libbtstack.a(hct_msg.o)
 .data          0x0000000000000000        0x0 ..\..\..\..\Libraries\libs\libbtstack.a(hct_fc.o)
 .bss           0x0000000000000000        0x0 ..\..\..\..\Libraries\libs\libbtstack.a(hct_fc.o)
 .data          0x0000000000000000        0x0 ..\..\..\..\Libraries\libs\libbtstack.a(hct.o)
 .bss           0x0000000000000000        0x0 ..\..\..\..\Libraries\libs\libbtstack.a(hct.o)
 .text          0x0000000000000000        0x0 ..\..\..\..\Libraries\libs\libbtstack.a(tws_sco.o)
 .data          0x0000000000000000        0x0 ..\..\..\..\Libraries\libs\libbtstack.a(tws_sco.o)
 .bss           0x0000000000000000        0x0 ..\..\..\..\Libraries\libs\libbtstack.a(tws_sco.o)
 .text          0x0000000000000000        0x0 ..\..\..\..\Libraries\libs\libbtstack.a(tws_acl.o)
 .data          0x0000000000000000        0x0 ..\..\..\..\Libraries\libs\libbtstack.a(tws_acl.o)
 .bss           0x0000000000000000        0x0 ..\..\..\..\Libraries\libs\libbtstack.a(tws_acl.o)
 .data          0x0000000000000000        0x0 ..\..\..\..\Libraries\libs\libbtstack.a(lm.o)
 .bss           0x0000000000000000        0x0 ..\..\..\..\Libraries\libs\libbtstack.a(lm.o)
 .data          0x0000000000000000        0x0 ..\..\..\..\Libraries\libs\libbtstack.a(bt_hal.o)
 .bss           0x0000000000000000        0x0 ..\..\..\..\Libraries\libs\libbtstack.a(bt_hal.o)
 .com_rodata.bb.tbl
                0x0000000000000000       0x2a ..\..\..\..\Libraries\libs\libbtstack.a(bt_hal.o)
 .data          0x0000000000000000        0x0 ..\..\..\..\Libraries\libs\libbtstack.a(bt21.o)
 .bss           0x0000000000000000        0x0 ..\..\..\..\Libraries\libs\libbtstack.a(bt21.o)
 .com_text.bb.sleep
                0x0000000000000000       0x4e ..\..\..\..\Libraries\libs\libbtstack.a(bt21.o)
 .data          0x0000000000000000        0x0 ..\..\..\..\Libraries\libs\libbtstack.a(bc.o)
 .data          0x0000000000000000        0x0 ..\..\..\..\Libraries\libs\libbtstack.a(ble_hal.o)
 .bss           0x0000000000000000        0x0 ..\..\..\..\Libraries\libs\libbtstack.a(ble_hal.o)
 .data          0x0000000000000000        0x0 ..\..\..\..\Libraries\libs\libbtstack.a(ble_adv.o)
 .bss           0x0000000000000000        0x0 ..\..\..\..\Libraries\libs\libbtstack.a(ble_adv.o)
 .data          0x0000000000000000        0x0 ..\..\..\..\Libraries\libs\libbtstack.a(ble.o)
 .bss           0x0000000000000000        0x0 ..\..\..\..\Libraries\libs\libbtstack.a(ble.o)
 .data          0x0000000000000000        0x0 ..\..\..\..\Libraries\libs\libbtstack.a(extern_ble.o)
 .bss           0x0000000000000000        0x0 ..\..\..\..\Libraries\libs\libbtstack.a(extern_ble.o)
 .sbss          0x0000000000000000        0x1 ..\..\..\..\Libraries\libs\libbtstack.a(extern_ble.o)
 .srodata       0x0000000000000000        0x2 ..\..\..\..\Libraries\libs\libbtstack.a(extern_ble.o)
 .data          0x0000000000000000        0x0 ..\..\..\..\Libraries\libs\libbtstack.a(l2cap_test.o)
 .data          0x0000000000000000        0x0 ..\..\..\..\Libraries\libs\libbtstack.a(l2cap.o)
 .bss           0x0000000000000000        0x0 ..\..\..\..\Libraries\libs\libbtstack.a(l2cap.o)
 .sbss          0x0000000000000000        0x1 ..\..\..\..\Libraries\libs\libbtstack.a(l2cap.o)
 .text          0x0000000000000000        0x4 ..\..\..\..\Libraries\libs\libbtstack.a(hci_sco.o)
 .data          0x0000000000000000        0x0 ..\..\..\..\Libraries\libs\libbtstack.a(hci_sco.o)
 .bss           0x0000000000000000        0x0 ..\..\..\..\Libraries\libs\libbtstack.a(hci_sco.o)
 .sbss          0x0000000000000000        0x1 ..\..\..\..\Libraries\libs\libbtstack.a(hci_sco.o)
 .text          0x0000000000000000       0x18 ..\..\..\..\Libraries\libs\libbtstack.a(hci_dump.o)
 .data          0x0000000000000000        0xc ..\..\..\..\Libraries\libs\libbtstack.a(hci_dump.o)
 .bss           0x0000000000000000        0x0 ..\..\..\..\Libraries\libs\libbtstack.a(hci_dump.o)
 .rodata.str1.4
                0x0000000000000000       0x12 ..\..\..\..\Libraries\libs\libbtstack.a(hci_dump.o)
 .text.stack.util
                0x0000000000000000       0x82 ..\..\..\..\Libraries\libs\libbtstack.a(hci_dump.o)
 .text          0x0000000000000000        0x0 ..\..\..\..\Libraries\libs\libbtstack.a(hci_cmd.o)
 .data          0x0000000000000000        0x0 ..\..\..\..\Libraries\libs\libbtstack.a(hci_cmd.o)
 .bss           0x0000000000000000        0x0 ..\..\..\..\Libraries\libs\libbtstack.a(hci_cmd.o)
 .data          0x0000000000000000        0x0 ..\..\..\..\Libraries\libs\libbtstack.a(hci.o)
 .bss           0x0000000000000000        0x0 ..\..\..\..\Libraries\libs\libbtstack.a(hci.o)
 .com_text.timer
                0x0000000000000000        0xe ..\..\..\..\Libraries\libs\libbtstack.a(hci.o)
 .com_text.sco  0x0000000000000000        0xe ..\..\..\..\Libraries\libs\libbtstack.a(hci.o)
 .rodata.stack.hci_init
                0x0000000000000000       0x11 ..\..\..\..\Libraries\libs\libbtstack.a(hci.o)
 .data          0x0000000000000000        0x0 ..\..\..\..\Libraries\libs\libbtstack.a(hid_usage.o)
 .bss           0x0000000000000000        0x0 ..\..\..\..\Libraries\libs\libbtstack.a(hid_usage.o)
 .text.stack.api.hid_touch
                0x0000000000000000        0xa ..\..\..\..\Libraries\libs\libbtstack.a(hid_usage.o)
 .srodata       0x0000000000000000        0xe ..\..\..\..\Libraries\libs\libbtstack.a(hid_usage.o)
 .data          0x0000000000000000        0x0 ..\..\..\..\Libraries\libs\libbtstack.a(hid_device.o)
 .bss           0x0000000000000000        0x0 ..\..\..\..\Libraries\libs\libbtstack.a(hid_device.o)
 .sbss          0x0000000000000000        0x1 ..\..\..\..\Libraries\libs\libbtstack.a(hid_device.o)
 .data          0x0000000000000000        0x0 ..\..\..\..\Libraries\libs\libbtstack.a(hfp_hf.o)
 .bss           0x0000000000000000        0x0 ..\..\..\..\Libraries\libs\libbtstack.a(hfp_hf.o)
 .data          0x0000000000000000        0x0 ..\..\..\..\Libraries\libs\libbtstack.a(hfp.o)
 .bss           0x0000000000000000        0x0 ..\..\..\..\Libraries\libs\libbtstack.a(hfp.o)
 .sbss          0x0000000000000000        0x1 ..\..\..\..\Libraries\libs\libbtstack.a(hfp.o)
 .text          0x0000000000000000        0x0 ..\..\..\..\Libraries\libs\libbtstack.a(avdtp.o)
 .data          0x0000000000000000        0x0 ..\..\..\..\Libraries\libs\libbtstack.a(avdtp.o)
 .bss           0x0000000000000000        0x0 ..\..\..\..\Libraries\libs\libbtstack.a(avdtp.o)
 .com_text.acl.pend
                0x0000000000000000        0x4 ..\..\..\..\Libraries\libs\libbtstack.a(avdtp.o)
 .sbss          0x0000000000000000        0x1 ..\..\..\..\Libraries\libs\libbtstack.a(avdtp.o)
 .data          0x0000000000000000        0x0 ..\..\..\..\Libraries\libs\libbtstack.a(a2dp.o)
 .bss           0x0000000000000000        0x0 ..\..\..\..\Libraries\libs\libbtstack.a(a2dp.o)
 .sbss          0x0000000000000000        0x1 ..\..\..\..\Libraries\libs\libbtstack.a(a2dp.o)
 .text          0x0000000000000000        0x0 ..\..\..\..\Libraries\libs\libbtstack.a(btstack_memory_pool.o)
 .data          0x0000000000000000        0x0 ..\..\..\..\Libraries\libs\libbtstack.a(btstack_memory_pool.o)
 .bss           0x0000000000000000        0x0 ..\..\..\..\Libraries\libs\libbtstack.a(btstack_memory_pool.o)
 .data          0x0000000000000000        0x0 ..\..\..\..\Libraries\libs\libbtstack.a(btstack_adv0.o)
 .bss           0x0000000000000000        0x0 ..\..\..\..\Libraries\libs\libbtstack.a(btstack_adv0.o)
 .sbss          0x0000000000000000        0x1 ..\..\..\..\Libraries\libs\libbtstack.a(btstack_adv0.o)
 .data          0x0000000000000000        0x0 ..\..\..\..\Libraries\libs\libbtstack.a(sm.o)
 .data          0x0000000000000000        0x0 ..\..\..\..\Libraries\libs\libbtstack.a(le_device_db_memory.o)
 .bss           0x0000000000000000        0x0 ..\..\..\..\Libraries\libs\libbtstack.a(le_device_db_memory.o)
 .data          0x0000000000000000        0x0 ..\..\..\..\Libraries\libs\libbtstack.a(hci_transport_hcic.o)
 .bss           0x0000000000000000        0x0 ..\..\..\..\Libraries\libs\libbtstack.a(hci_transport_hcic.o)
 .data          0x0000000000000000        0x0 ..\..\..\..\Libraries\libs\libbtstack.a(btstack_chipset_inner.o)
 .bss           0x0000000000000000        0x0 ..\..\..\..\Libraries\libs\libbtstack.a(btstack_chipset_inner.o)
 .data          0x0000000000000000        0x0 ..\..\..\..\Libraries\libs\libbtstack.a(lm_hook.o)
 .bss           0x0000000000000000        0x0 ..\..\..\..\Libraries\libs\libbtstack.a(lm_hook.o)
 .data          0x0000000000000000        0x0 ..\..\..\..\Libraries\libs\libbtstack.a(lm_sp.o)
 .text.lm.sha256
                0x0000000000000000      0x13a ..\..\..\..\Libraries\libs\libbtstack.a(lm_sp.o)
 .data          0x0000000000000000        0x0 ..\..\..\..\Libraries\libs\libbtstack.a(lm_proc.o)
 .bss           0x0000000000000000        0x0 ..\..\..\..\Libraries\libs\libbtstack.a(lm_proc.o)
 .text.bb.lm.inq.start
                0x0000000000000000      0x104 ..\..\..\..\Libraries\libs\libbtstack.a(lm_proc.o)
 .text.bb.lm.inq.stop
                0x0000000000000000       0x32 ..\..\..\..\Libraries\libs\libbtstack.a(lm_proc.o)
 .text.bb.lm.inq.res
                0x0000000000000000      0x222 ..\..\..\..\Libraries\libs\libbtstack.a(lm_proc.o)
 .data          0x0000000000000000        0x0 ..\..\..\..\Libraries\libs\libbtstack.a(lm_key.o)
 .bss           0x0000000000000000        0x0 ..\..\..\..\Libraries\libs\libbtstack.a(lm_key.o)
 .data          0x0000000000000000        0x0 ..\..\..\..\Libraries\libs\libbtstack.a(lc.o)
 .bss           0x0000000000000000        0x0 ..\..\..\..\Libraries\libs\libbtstack.a(lc.o)
 .com_text.lc   0x0000000000000000       0x9c ..\..\..\..\Libraries\libs\libbtstack.a(lc.o)
 .data          0x0000000000000000        0x0 ..\..\..\..\Libraries\libs\libbtstack.a(mgr.o)
 .bss           0x0000000000000000        0x0 ..\..\..\..\Libraries\libs\libbtstack.a(mgr.o)
 .text          0x0000000000000000        0x0 ..\..\..\..\Libraries\libs\libbtstack.a(ll.o)
 .data          0x0000000000000000        0x0 ..\..\..\..\Libraries\libs\libbtstack.a(ll.o)
 .bss           0x0000000000000000        0x0 ..\..\..\..\Libraries\libs\libbtstack.a(ll.o)
 .data          0x0000000000000000        0x0 ..\..\..\..\Libraries\libs\libbtstack.a(ble_test.o)
 .bss           0x0000000000000000        0x0 ..\..\..\..\Libraries\libs\libbtstack.a(ble_test.o)
 .com_text.ble.isr.test
                0x0000000000000000      0x17a ..\..\..\..\Libraries\libs\libbtstack.a(ble_test.o)
 .com_text.ble.isr.test.ind
                0x0000000000000000       0x5a ..\..\..\..\Libraries\libs\libbtstack.a(ble_test.o)
 .text.bb.ble.test.start
                0x0000000000000000      0x4b0 ..\..\..\..\Libraries\libs\libbtstack.a(ble_test.o)
 .text.bb.ble.test.stop
                0x0000000000000000      0x200 ..\..\..\..\Libraries\libs\libbtstack.a(ble_test.o)
 .srodata       0x0000000000000000        0x7 ..\..\..\..\Libraries\libs\libbtstack.a(ble_test.o)
 .data          0x0000000000000000        0x0 ..\..\..\..\Libraries\libs\libbtstack.a(ble_scan.o)
 .bss           0x0000000000000000        0x0 ..\..\..\..\Libraries\libs\libbtstack.a(ble_scan.o)
 .com_rodata.bb.tbl
                0x0000000000000000       0x10 ..\..\..\..\Libraries\libs\libbtstack.a(ble_scan.o)
 .data          0x0000000000000000        0x0 ..\..\..\..\Libraries\libs\libbtstack.a(ble_per_adv.o)
 .bss           0x0000000000000000        0x0 ..\..\..\..\Libraries\libs\libbtstack.a(ble_per_adv.o)
 .data          0x0000000000000000        0x0 ..\..\..\..\Libraries\libs\libbtstack.a(ble_init.o)
 .bss           0x0000000000000000        0x0 ..\..\..\..\Libraries\libs\libbtstack.a(ble_init.o)
 .data          0x0000000000000000        0x0 ..\..\..\..\Libraries\libs\libbtstack.a(ble_buf.o)
 .text          0x0000000000000000        0x0 ..\..\..\..\Libraries\libs\libbtstack.a(ble_adv0.o)
 .data          0x0000000000000000        0x0 ..\..\..\..\Libraries\libs\libbtstack.a(ble_adv0.o)
 .bss           0x0000000000000000        0x0 ..\..\..\..\Libraries\libs\libbtstack.a(ble_adv0.o)
 .data          0x0000000000000000        0x0 ..\..\..\..\Libraries\libs\libbtstack.a(extern_hfhs.o)
 .bss           0x0000000000000000        0x0 ..\..\..\..\Libraries\libs\libbtstack.a(extern_hfhs.o)
 .sbss          0x0000000000000000        0x1 ..\..\..\..\Libraries\libs\libbtstack.a(extern_hfhs.o)
 .srodata       0x0000000000000000        0x1 ..\..\..\..\Libraries\libs\libbtstack.a(extern_hfhs.o)
 .text          0x0000000000000000       0x38 ..\..\..\..\Libraries\libs\libbtstack.a(l2cap_signaling.o)
 .data          0x0000000000000000        0x0 ..\..\..\..\Libraries\libs\libbtstack.a(l2cap_signaling.o)
 .bss           0x0000000000000000        0x0 ..\..\..\..\Libraries\libs\libbtstack.a(l2cap_signaling.o)
 .data          0x0000000000000000        0x0 ..\..\..\..\Libraries\libs\libbtstack.a(lc_hook.o)
 .bss           0x0000000000000000        0x0 ..\..\..\..\Libraries\libs\libbtstack.a(lc_hook.o)
 .data          0x0000000000000000        0x0 ..\..\..\..\Libraries\libs\libbtstack.a(lm_sco.o)
 .bss           0x0000000000000000        0x0 ..\..\..\..\Libraries\libs\libbtstack.a(lm_sco.o)
 .data          0x0000000000000000        0x0 ..\..\..\..\Libraries\libs\libbtstack.a(lc_util.o)
 .bss           0x0000000000000000        0x0 ..\..\..\..\Libraries\libs\libbtstack.a(lc_util.o)
 .data          0x0000000000000000        0x0 ..\..\..\..\Libraries\libs\libbtstack.a(lc_sniff.o)
 .bss           0x0000000000000000        0x0 ..\..\..\..\Libraries\libs\libbtstack.a(lc_sniff.o)
 .data          0x0000000000000000        0x0 ..\..\..\..\Libraries\libs\libbtstack.a(lc_sco.o)
 .bss           0x0000000000000000        0x0 ..\..\..\..\Libraries\libs\libbtstack.a(lc_sco.o)
 .data          0x0000000000000000        0x0 ..\..\..\..\Libraries\libs\libbtstack.a(lc_proc.o)
 .bss           0x0000000000000000        0x0 ..\..\..\..\Libraries\libs\libbtstack.a(lc_proc.o)
 .data          0x0000000000000000        0x0 ..\..\..\..\Libraries\libs\libbtstack.a(lc_lmppdu.o)
 .bss           0x0000000000000000        0x0 ..\..\..\..\Libraries\libs\libbtstack.a(lc_lmppdu.o)
 .data          0x0000000000000000        0x0 ..\..\..\..\Libraries\libs\libbtstack.a(mgr_proc.o)
 .bss           0x0000000000000000        0x0 ..\..\..\..\Libraries\libs\libbtstack.a(mgr_proc.o)
 .data          0x0000000000000000        0x0 ..\..\..\..\Libraries\libs\libbtstack.a(mgr_init.o)
 .bss           0x0000000000000000        0x0 ..\..\..\..\Libraries\libs\libbtstack.a(mgr_init.o)
 .data          0x0000000000000000        0x0 ..\..\..\..\Libraries\libs\libbtstack.a(mgr_hci.o)
 .bss           0x0000000000000000        0x0 ..\..\..\..\Libraries\libs\libbtstack.a(mgr_hci.o)
 .data          0x0000000000000000        0x0 ..\..\..\..\Libraries\libs\libbtstack.a(ll_scan.o)
 .bss           0x0000000000000000        0x0 ..\..\..\..\Libraries\libs\libbtstack.a(ll_scan.o)
 .data          0x0000000000000000        0x0 ..\..\..\..\Libraries\libs\libbtstack.a(ll_adv.o)
 .bss           0x0000000000000000        0x0 ..\..\..\..\Libraries\libs\libbtstack.a(ll_adv.o)
 .data          0x0000000000000000        0x0 ..\..\..\..\Libraries\libs\libbtstack.a(ll_proc.o)
 .data          0x0000000000000000        0x0 ..\..\..\..\Libraries\libs\libbtstack.a(ll_ping.o)
 .bss           0x0000000000000000        0x0 ..\..\..\..\Libraries\libs\libbtstack.a(ll_ping.o)
 .data          0x0000000000000000        0x0 ..\..\..\..\Libraries\libs\libbtstack.a(ll_phy_upd.o)
 .bss           0x0000000000000000        0x0 ..\..\..\..\Libraries\libs\libbtstack.a(ll_phy_upd.o)
 .data          0x0000000000000000        0x0 ..\..\..\..\Libraries\libs\libbtstack.a(ll_past.o)
 .bss           0x0000000000000000        0x0 ..\..\..\..\Libraries\libs\libbtstack.a(ll_past.o)
 .data          0x0000000000000000        0x0 ..\..\..\..\Libraries\libs\libbtstack.a(ll_length.o)
 .bss           0x0000000000000000        0x0 ..\..\..\..\Libraries\libs\libbtstack.a(ll_length.o)
 .data          0x0000000000000000        0x0 ..\..\..\..\Libraries\libs\libbtstack.a(ll_feature.o)
 .bss           0x0000000000000000        0x0 ..\..\..\..\Libraries\libs\libbtstack.a(ll_feature.o)
 .data          0x0000000000000000        0x0 ..\..\..\..\Libraries\libs\libbtstack.a(ll_encrypt.o)
 .bss           0x0000000000000000        0x0 ..\..\..\..\Libraries\libs\libbtstack.a(ll_encrypt.o)
 .data          0x0000000000000000        0x0 ..\..\..\..\Libraries\libs\libbtstack.a(ll_disconnect.o)
 .bss           0x0000000000000000        0x0 ..\..\..\..\Libraries\libs\libbtstack.a(ll_disconnect.o)
 .data          0x0000000000000000        0x0 ..\..\..\..\Libraries\libs\libbtstack.a(ll_con_upd.o)
 .bss           0x0000000000000000        0x0 ..\..\..\..\Libraries\libs\libbtstack.a(ll_con_upd.o)
 .data          0x0000000000000000        0x0 ..\..\..\..\Libraries\libs\libbtstack.a(ll_cntl.o)
 .bss           0x0000000000000000        0x0 ..\..\..\..\Libraries\libs\libbtstack.a(ll_cntl.o)
 .data          0x0000000000000000        0x0 ..\..\..\..\Libraries\libs\libbtstack.a(ll_clk_acc.o)
 .bss           0x0000000000000000        0x0 ..\..\..\..\Libraries\libs\libbtstack.a(ll_clk_acc.o)
 .data          0x0000000000000000        0x0 ..\..\..\..\Libraries\libs\libbtstack.a(ll_chmap_upd.o)
 .bss           0x0000000000000000        0x0 ..\..\..\..\Libraries\libs\libbtstack.a(ll_chmap_upd.o)
 .data          0x0000000000000000        0x0 ..\..\..\..\Libraries\libs\libbtstack.a(aes_rpa.o)
 .bss           0x0000000000000000        0x0 ..\..\..\..\Libraries\libs\libbtstack.a(aes_rpa.o)
 .data          0x0000000000000000        0x0 ..\..\..\..\Libraries\libs\libbtstack.a(scan_hook.o)
 .bss           0x0000000000000000        0x0 ..\..\..\..\Libraries\libs\libbtstack.a(scan_hook.o)
 .data          0x0000000000000000        0x0 ..\..\..\..\Libraries\libs\libbtstack.a(adv_hook.o)
 .bss           0x0000000000000000        0x0 ..\..\..\..\Libraries\libs\libbtstack.a(adv_hook.o)
 .data          0x0000000000000000        0x0 ..\..\..\..\Libraries\libs\libbtstack.a(ll_version.o)
 .bss           0x0000000000000000        0x0 ..\..\..\..\Libraries\libs\libbtstack.a(ll_version.o)
 .data          0x0000000000000000        0x0 ..\..\..\..\Libraries\libs\libbtstack.a(ll_pwr.o)
 .bss           0x0000000000000000        0x0 ..\..\..\..\Libraries\libs\libbtstack.a(ll_pwr.o)
 .text          0x0000000000000000        0x0 ..\..\..\..\Libraries\libs\libdrivers.a(usb_device_hid.o)
 .data          0x0000000000000000        0x0 ..\..\..\..\Libraries\libs\libdrivers.a(usb_device_hid.o)
 .bss           0x0000000000000000        0x0 ..\..\..\..\Libraries\libs\libdrivers.a(usb_device_hid.o)
 .com_text.bulkep
                0x0000000000000000       0x80 ..\..\..\..\Libraries\libs\libdrivers.a(usb_device_hid.o)
 .text.usb_hid_ep_config
                0x0000000000000000        0xa ..\..\..\..\Libraries\libs\libdrivers.a(usb_device_hid.o)
 .text.usb_user_ep_config
                0x0000000000000000       0x2e ..\..\..\..\Libraries\libs\libdrivers.a(usb_device_hid.o)
 .text          0x0000000000000000        0x0 ..\..\..\..\Libraries\libs\libdrivers.a(usb_device_printer.o)
 .data          0x0000000000000000        0x0 ..\..\..\..\Libraries\libs\libdrivers.a(usb_device_printer.o)
 .bss           0x0000000000000000        0x0 ..\..\..\..\Libraries\libs\libdrivers.a(usb_device_printer.o)
 .com_text.bulkep
                0x0000000000000000       0xaa ..\..\..\..\Libraries\libs\libdrivers.a(usb_device_printer.o)
 .text.usb_printer_ep_config
                0x0000000000000000       0x12 ..\..\..\..\Libraries\libs\libdrivers.a(usb_device_printer.o)
 .text.udp_init
                0x0000000000000000       0xa2 ..\..\..\..\Libraries\libs\libdrivers.a(usb_device_printer.o)
 .sdata         0x0000000000000000        0x2 ..\..\..\..\Libraries\libs\libdrivers.a(usb_device_printer.o)
 .text          0x0000000000000000        0x0 ..\..\..\..\Libraries\libs\libdrivers.a(usb_device_run_loop.o)
 .data          0x0000000000000000        0x0 ..\..\..\..\Libraries\libs\libdrivers.a(usb_device_run_loop.o)
 .bss           0x0000000000000000        0x0 ..\..\..\..\Libraries\libs\libdrivers.a(usb_device_run_loop.o)
 .text.usb_device_exit
                0x0000000000000000       0x32 ..\..\..\..\Libraries\libs\libdrivers.a(usb_device_run_loop.o)
 .usbdev.com    0x0000000000000000       0xa8 ..\..\..\..\Libraries\libs\libdrivers.a(usb_device_run_loop.o)
 .text.usb_device_init
                0x0000000000000000       0xac ..\..\..\..\Libraries\libs\libdrivers.a(usb_device_run_loop.o)
 .text.usb_device_enter
                0x0000000000000000       0x74 ..\..\..\..\Libraries\libs\libdrivers.a(usb_device_run_loop.o)
 .com_text.usb.device
                0x0000000000000000       0x62 ..\..\..\..\Libraries\libs\libdrivers.a(usb_device_run_loop.o)
 .com_text.irq  0x0000000000000000       0x10 ..\..\..\..\Libraries\libs\libdrivers.a(usb_device_run_loop.o)
 .usb_buf.device.desc.buf
                0x0000000000000000      0x400 ..\..\..\..\Libraries\libs\libdrivers.a(usb_device_run_loop.o)
 .usb_buf.isoc  0x0000000000000000      0x140 ..\..\..\..\Libraries\libs\libdrivers.a(usb_device_run_loop.o)
 .usb_buf.printer
                0x0000000000000000       0x80 ..\..\..\..\Libraries\libs\libdrivers.a(usb_device_run_loop.o)
 .text          0x0000000000000000        0x0 ..\..\..\..\Libraries\libs\libdrivers.a(usb_host_manage.o)
 .data          0x0000000000000000        0x0 ..\..\..\..\Libraries\libs\libdrivers.a(usb_host_manage.o)
 .bss           0x0000000000000000        0x0 ..\..\..\..\Libraries\libs\libdrivers.a(usb_host_manage.o)
 .text.usb_host_var_init
                0x0000000000000000       0x3c ..\..\..\..\Libraries\libs\libdrivers.a(usb_host_manage.o)
 .text.uhs_is_iphone
                0x0000000000000000       0x12 ..\..\..\..\Libraries\libs\libdrivers.a(usb_host_manage.o)
 .text.usb.host.init
                0x0000000000000000       0x96 ..\..\..\..\Libraries\libs\libdrivers.a(usb_host_manage.o)
 .com_text.irq  0x0000000000000000       0x12 ..\..\..\..\Libraries\libs\libdrivers.a(usb_host_manage.o)
 .text.udisk_suspend
                0x0000000000000000       0x32 ..\..\..\..\Libraries\libs\libdrivers.a(usb_host_manage.o)
 .text.udisk_resume
                0x0000000000000000       0x4c ..\..\..\..\Libraries\libs\libdrivers.a(usb_host_manage.o)
 .com_text.usb.host
                0x0000000000000000       0x82 ..\..\..\..\Libraries\libs\libdrivers.a(usb_host_manage.o)
 .text.udisk_read
                0x0000000000000000       0x7c ..\..\..\..\Libraries\libs\libdrivers.a(usb_host_manage.o)
 .text.uhs_set_nluns
                0x0000000000000000        0xa ..\..\..\..\Libraries\libs\libdrivers.a(usb_host_manage.o)
 .text.udisk_write
                0x0000000000000000       0x54 ..\..\..\..\Libraries\libs\libdrivers.a(usb_host_manage.o)
 .buf.usb       0x0000000000000000       0x74 ..\..\..\..\Libraries\libs\libdrivers.a(usb_host_manage.o)
 .comment       0x0000000000000000       0x13 ..\..\..\..\Libraries\libs\libdrivers.a(usb_host_manage.o)
 .riscv.attributes
                0x0000000000000000       0x32 ..\..\..\..\Libraries\libs\libdrivers.a(usb_host_manage.o)
 .text          0x0000000000000000        0x0 ..\..\..\..\Libraries\libs\libdrivers.a(usb_host_storage.o)
 .data          0x0000000000000000        0x0 ..\..\..\..\Libraries\libs\libdrivers.a(usb_host_storage.o)
 .bss           0x0000000000000000        0x0 ..\..\..\..\Libraries\libs\libdrivers.a(usb_host_storage.o)
 .text.do_transfer
                0x0000000000000000       0xae ..\..\..\..\Libraries\libs\libdrivers.a(usb_host_storage.o)
 .text.do_receive
                0x0000000000000000       0xf6 ..\..\..\..\Libraries\libs\libdrivers.a(usb_host_storage.o)
 .text.do_request
                0x0000000000000000      0x20a ..\..\..\..\Libraries\libs\libdrivers.a(usb_host_storage.o)
 .text.do_scsi_request
                0x0000000000000000       0xf8 ..\..\..\..\Libraries\libs\libdrivers.a(usb_host_storage.o)
 .text.uhs_start
                0x0000000000000000      0x18c ..\..\..\..\Libraries\libs\libdrivers.a(usb_host_storage.o)
 .text.uhs_read
                0x0000000000000000       0x64 ..\..\..\..\Libraries\libs\libdrivers.a(usb_host_storage.o)
 .text.uhs_write
                0x0000000000000000       0x64 ..\..\..\..\Libraries\libs\libdrivers.a(usb_host_storage.o)
 .text.uhs_init
                0x0000000000000000       0x26 ..\..\..\..\Libraries\libs\libdrivers.a(usb_host_storage.o)
 .rodata        0x0000000000000000       0x57 ..\..\..\..\Libraries\libs\libdrivers.a(usb_host_storage.o)
 .comment       0x0000000000000000       0x13 ..\..\..\..\Libraries\libs\libdrivers.a(usb_host_storage.o)
 .riscv.attributes
                0x0000000000000000       0x32 ..\..\..\..\Libraries\libs\libdrivers.a(usb_host_storage.o)
 .text          0x0000000000000000        0x0 ..\..\..\..\Libraries\libs\libdrivers.a(usb_comm.o)
 .data          0x0000000000000000        0x0 ..\..\..\..\Libraries\libs\libdrivers.a(usb_comm.o)
 .bss           0x0000000000000000        0x0 ..\..\..\..\Libraries\libs\libdrivers.a(usb_comm.o)
 .text.usb_init
                0x0000000000000000       0x80 ..\..\..\..\Libraries\libs\libdrivers.a(usb_comm.o)
 .text.usb_host_enter
                0x0000000000000000       0x56 ..\..\..\..\Libraries\libs\libdrivers.a(usb_comm.o)
 .usbdev.com    0x0000000000000000       0x20 ..\..\..\..\Libraries\libs\libdrivers.a(usb_comm.o)
 .com_text.irq  0x0000000000000000       0x2a ..\..\..\..\Libraries\libs\libdrivers.a(usb_comm.o)
 .buf.usb.ctrl  0x0000000000000000       0x40 ..\..\..\..\Libraries\libs\libdrivers.a(usb_comm.o)
 .text          0x0000000000000000        0x0 ..\..\..\..\Libraries\libs\libdrivers.a(usb_detect.o)
 .data          0x0000000000000000        0x0 ..\..\..\..\Libraries\libs\libdrivers.a(usb_detect.o)
 .bss           0x0000000000000000        0x0 ..\..\..\..\Libraries\libs\libdrivers.a(usb_detect.o)
 .com_text.usb.dectect
                0x0000000000000000      0x108 ..\..\..\..\Libraries\libs\libdrivers.a(usb_detect.o)
 .buf.usbchk.cb
                0x0000000000000000        0x2 ..\..\..\..\Libraries\libs\libdrivers.a(usb_detect.o)
 .comment       0x0000000000000000       0x13 ..\..\..\..\Libraries\libs\libdrivers.a(usb_detect.o)
 .riscv.attributes
                0x0000000000000000       0x32 ..\..\..\..\Libraries\libs\libdrivers.a(usb_detect.o)
 .text          0x0000000000000000        0x0 ..\..\..\..\Libraries\libs\libdrivers.a(usb_device_desc.o)
 .data          0x0000000000000000        0x0 ..\..\..\..\Libraries\libs\libdrivers.a(usb_device_desc.o)
 .bss           0x0000000000000000        0x0 ..\..\..\..\Libraries\libs\libdrivers.a(usb_device_desc.o)
 .text.usb_get_device_descriptor
                0x0000000000000000        0x8 ..\..\..\..\Libraries\libs\libdrivers.a(usb_device_desc.o)
 .text.usb_get_config_descriptor
                0x0000000000000000        0x8 ..\..\..\..\Libraries\libs\libdrivers.a(usb_device_desc.o)
 .text.usb_get_lang_id_str_descriptor
                0x0000000000000000        0x8 ..\..\..\..\Libraries\libs\libdrivers.a(usb_device_desc.o)
 .text.usb_get_manufacturer_str_descriptor
                0x0000000000000000        0x8 ..\..\..\..\Libraries\libs\libdrivers.a(usb_device_desc.o)
 .text.usb_get_product_str_descriptor
                0x0000000000000000        0x8 ..\..\..\..\Libraries\libs\libdrivers.a(usb_device_desc.o)
 .text.usb_get_serial_str_descriptor
                0x0000000000000000        0x8 ..\..\..\..\Libraries\libs\libdrivers.a(usb_device_desc.o)
 .text.usb_get_hid_config_descriptor
                0x0000000000000000        0x8 ..\..\..\..\Libraries\libs\libdrivers.a(usb_device_desc.o)
 .text.usb_get_hid_report_descriptor
                0x0000000000000000        0x8 ..\..\..\..\Libraries\libs\libdrivers.a(usb_device_desc.o)
 .comment       0x0000000000000000       0x13 ..\..\..\..\Libraries\libs\libdrivers.a(usb_device_desc.o)
 .riscv.attributes
                0x0000000000000000       0x32 ..\..\..\..\Libraries\libs\libdrivers.a(usb_device_desc.o)
 .text          0x0000000000000000        0x0 ..\..\..\..\Libraries\libs\libdrivers.a(usb_device_enum.o)
 .data          0x0000000000000000        0x0 ..\..\..\..\Libraries\libs\libdrivers.a(usb_device_enum.o)
 .bss           0x0000000000000000        0xa ..\..\..\..\Libraries\libs\libdrivers.a(usb_device_enum.o)
 .usbdev.com    0x0000000000000000      0x9c2 ..\..\..\..\Libraries\libs\libdrivers.a(usb_device_enum.o)
 .text.usb_ep0_out_data_callback
                0x0000000000000000        0x4 ..\..\..\..\Libraries\libs\libdrivers.a(usb_device_enum.o)
 .text.usb_itf_in_req
                0x0000000000000000        0x4 ..\..\..\..\Libraries\libs\libdrivers.a(usb_device_enum.o)
 .comment       0x0000000000000000       0x13 ..\..\..\..\Libraries\libs\libdrivers.a(usb_device_enum.o)
 .riscv.attributes
                0x0000000000000000       0x32 ..\..\..\..\Libraries\libs\libdrivers.a(usb_device_enum.o)
 .text          0x0000000000000000        0x0 ..\..\..\..\Libraries\libs\libdrivers.a(usb_device_ep.o)
 .data          0x0000000000000000        0x0 ..\..\..\..\Libraries\libs\libdrivers.a(usb_device_ep.o)
 .text          0x0000000000000000        0x0 ..\..\..\..\Libraries\libs\libdrivers.a(usb_host_enum.o)
 .data          0x0000000000000000        0x0 ..\..\..\..\Libraries\libs\libdrivers.a(usb_host_enum.o)
 .bss           0x0000000000000000        0x0 ..\..\..\..\Libraries\libs\libdrivers.a(usb_host_enum.o)
 .text.wait_transfering
                0x0000000000000000       0x3c ..\..\..\..\Libraries\libs\libdrivers.a(usb_host_enum.o)
 .text.do_receive
                0x0000000000000000       0x90 ..\..\..\..\Libraries\libs\libdrivers.a(usb_host_enum.o)
 .text.do_skip_rxdata
                0x0000000000000000       0x4c ..\..\..\..\Libraries\libs\libdrivers.a(usb_host_enum.o)
 .text.do_request.isra.0
                0x0000000000000000      0x298 ..\..\..\..\Libraries\libs\libdrivers.a(usb_host_enum.o)
 .text.uhe_reset
                0x0000000000000000       0x34 ..\..\..\..\Libraries\libs\libdrivers.a(usb_host_enum.o)
 .rodata.str1.4
                0x0000000000000000        0xb ..\..\..\..\Libraries\libs\libdrivers.a(usb_host_enum.o)
 .text.uhe_start
                0x0000000000000000      0x22c ..\..\..\..\Libraries\libs\libdrivers.a(usb_host_enum.o)
 .text.uhe_clear_feature
                0x0000000000000000       0x44 ..\..\..\..\Libraries\libs\libdrivers.a(usb_host_enum.o)
 .text.uhe_init
                0x0000000000000000       0x24 ..\..\..\..\Libraries\libs\libdrivers.a(usb_host_enum.o)
 .rodata        0x0000000000000000       0x40 ..\..\..\..\Libraries\libs\libdrivers.a(usb_host_enum.o)
 .rodata.uhe    0x0000000000000000       0x40 ..\..\..\..\Libraries\libs\libdrivers.a(usb_host_enum.o)
 .comment       0x0000000000000000       0x13 ..\..\..\..\Libraries\libs\libdrivers.a(usb_host_enum.o)
 .riscv.attributes
                0x0000000000000000       0x32 ..\..\..\..\Libraries\libs\libdrivers.a(usb_host_enum.o)
 .text          0x0000000000000000        0x0 ..\..\..\..\Libraries\libs\libdrivers.a(weak_symbol.o)
 .data          0x0000000000000000        0x0 ..\..\..\..\Libraries\libs\libdrivers.a(weak_symbol.o)
 .bss           0x0000000000000000        0x0 ..\..\..\..\Libraries\libs\libdrivers.a(weak_symbol.o)
 .text.iphone_power_set
                0x0000000000000000       0x12 ..\..\..\..\Libraries\libs\libdrivers.a(weak_symbol.o)
 .comment       0x0000000000000000       0x13 ..\..\..\..\Libraries\libs\libdrivers.a(weak_symbol.o)
 .riscv.attributes
                0x0000000000000000       0x32 ..\..\..\..\Libraries\libs\libdrivers.a(weak_symbol.o)
 .text          0x0000000000000000        0x0 ..\..\..\..\Libraries\libs\libdrivers.a(usb_device_audio.o)
 .data          0x0000000000000000        0x0 ..\..\..\..\Libraries\libs\libdrivers.a(usb_device_audio.o)
 .bss           0x0000000000000000        0x0 ..\..\..\..\Libraries\libs\libdrivers.a(usb_device_audio.o)
 .usbdev.com    0x0000000000000000      0x36a ..\..\..\..\Libraries\libs\libdrivers.a(usb_device_audio.o)
 .ude.aubuf     0x0000000000000000      0x8d4 ..\..\..\..\Libraries\libs\libdrivers.a(usb_device_audio.o)
 .usbdev.com.table
                0x0000000000000000        0x3 ..\..\..\..\Libraries\libs\libdrivers.a(usb_device_audio.o)
 .comment       0x0000000000000000       0x13 ..\..\..\..\Libraries\libs\libdrivers.a(usb_device_audio.o)
 .riscv.attributes
                0x0000000000000000       0x32 ..\..\..\..\Libraries\libs\libdrivers.a(usb_device_audio.o)

Memory Configuration

Name             Origin             Length             Attributes
init             0x0000000010000000 0x0000000000000200
flash            0x0000000010000200 0x0000000000064000 xr
comm             0x0000000000017000 0x0000000000009000 xr
stack            0x0000000000010800 0x0000000000000400
heap             0x0000000000010c00 0x0000000000003000
data             0x0000000000013c00 0x0000000000003400
bram             0x0000000000020000 0x000000000000c000
cram             0x000000000002c000 0x0000000000014000
aram             0x0000000000050000 0x0000000000004000
dram             0x0000000000058000 0x0000000000004500
eram             0x0000000000054000 0x0000000000000a00
rram             0x0000000000055800 0x0000000000000260
*default*        0x0000000000000000 0xffffffffffffffff

Linker script and memory map

LOAD Output\obj\Libraries\bsp\bsp_cm.o
LOAD Output\obj\Libraries\bsp\bsp_fot.o
LOAD Output\obj\Libraries\bsp\bsp_param.o
LOAD Output\obj\Libraries\bsp\bsp_sys.o
LOAD Output\obj\Libraries\BT\ble\ab_link\app.o
LOAD Output\obj\Libraries\BT\ble\adv0.o
LOAD Output\obj\Libraries\BT\ble\ble.o
LOAD Output\obj\Libraries\BT\spp\bt.o
LOAD Output\obj\Libraries\BT\spp\hid.o
LOAD Output\obj\Libraries\BT\spp\profile.o
LOAD Output\obj\Libraries\BT\spp\spp.o
LOAD Output\obj\Libraries\Device\Source\gw3323_clk.o
LOAD Output\obj\Libraries\Device\Source\gw3323_gpio.o
LOAD Output\obj\Libraries\Device\Source\gw3323_tmr.o
LOAD Output\obj\Libraries\libs\strong_symbol.o
LOAD Output\obj\Examples\TIMER\TIM_Capture\Source\timer_capture.o
LOAD Output\obj\Examples\TIMER\TIM_Capture\Source\timer_pwm.o
LOAD Output\obj\Examples\TIMER\TIM_Capture\Project\config.o
LOAD Output\obj\Examples\TIMER\TIM_Capture\Project\main.o
                0x0000000000064000                __max_flash_size = 0x64000
                0x0000000010000000                __base = 0x10000000
                0x0000000000010600                __cache_stack_vma = 0x10600
                0x0000000000000200                __cache_stack_size = 0x200
                0x0000000000010800                __stack_vma = 0x10800
                0x0000000000000400                __stack_ram_size = 0x400
                0x0000000000010c00                __heap_vma = 0x10c00
                0x0000000000003000                __heap_ram_size = 0x3000
                0x0000000000013c00                __data_vma = 0x13c00
                0x0000000000003400                __data_ram_size = 0x3400
                0x0000000000017000                __comm_vma = 0x17000
                0x0000000000009000                __comm_ram_size = 0x9000
                0x0000000000020000                __bram_vma = 0x20000
                0x000000000000c000                __bram_ram_size = 0xc000
                0x000000000002c000                __cram_vma = 0x2c000
                0x0000000000014000                __cram_ram_size = 0x14000
                0x0000000000050000                __aram_vma = 0x50000
                0x0000000000054000                __eram_vma = 0x54000
                0x0000000000058000                __dram_vma = 0x58000
                0x0000000000055800                __rram_vma = 0x55800

.init           0x0000000010000000       0x4e
 *(.reset)
 .reset         0x0000000010000000       0x4e ..\..\..\..\Libraries\libs\libplatform.a(reset.o)
                0x0000000010000000                _start

.comm           0x0000000000017000     0x3800 load address 0x0000000010000200
 *(.vector)
 .vector        0x0000000000017000      0x1a2 ..\..\..\..\Libraries\libs\libplatform.a(reset.o)
                0x00000000000170a0                _exception_isr
                0x00000000000170a2                nop_isr
 *(.plt)
 .plt           0x00000000000171a2       0x10 ..\..\..\..\Libraries\libs\libplatform.a(main.o)
 *(.com_text*)
 .com_text.fot  0x00000000000171b2       0x4e Output\obj\Libraries\bsp\bsp_fot.o
                0x00000000000171b2                fot_app_connect_auth
                0x00000000000171f4                bsp_fot_is_connect
 .com_text.const
                0x0000000000017200        0x7 Output\obj\Libraries\bsp\bsp_fot.o
 *fill*         0x0000000000017207        0x1 
 .com_text.timer
                0x0000000000017208       0x98 Output\obj\Libraries\bsp\bsp_sys.o
                0x0000000000017208                usr_tmr1ms_isr
                0x000000000001720a                usr_tmr5ms_thread
                0x0000000000017288                timer1_isr
 .com_text.sys  0x00000000000172a0        0x4 Output\obj\Libraries\bsp\bsp_sys.o
                0x00000000000172a0                spiflash_speed_up_en
 .com_text.gpio
                0x00000000000172a4       0x36 Output\obj\Libraries\Device\Source\gw3323_gpio.o
                0x00000000000172a4                gpio_set_bits
                0x00000000000172a8                gpio_reset_bits
                0x00000000000172ac                gpio_writebit
                0x00000000000172b6                gpio_write_data
                0x00000000000172c0                gpio_toggle_bits
                0x00000000000172c8                gpio_read_data
                0x00000000000172d0                gpio_read_bit
 .com_text.tmr  0x00000000000172da      0x118 Output\obj\Libraries\Device\Source\gw3323_tmr.o
                0x00000000000172da                tmr_set_counter
                0x00000000000172de                tmr_set_period
                0x00000000000172e2                tmr_get_counter
                0x00000000000172e6                tmr_get_period
                0x00000000000172ea                tmr_cmd
                0x000000000001732e                tmr_set_pwm0_duty
                0x000000000001734e                tmr_set_pwm1_duty
                0x000000000001736e                tmr_set_pwm2_duty
                0x000000000001738e                tmr_capture_config
                0x00000000000173bc                tmr_get_capture
                0x00000000000173e0                tmr_get_flag
                0x00000000000173ea                tmr_clear_flag
 .com_text.stack.uart_isr
                0x00000000000173f2        0x4 Output\obj\Libraries\libs\strong_symbol.o
                0x00000000000173f2                bt_uart_isr
 .com_text.isr  0x00000000000173f6      0x124 Output\obj\Examples\TIMER\TIM_Capture\Source\timer_capture.o
                0x00000000000173f6                timer3_cap_handle
 .com_text.spiflash
                0x000000000001751a      0x13e ..\..\..\..\Libraries\libs\libplatform.a(os_flash.o)
                0x000000000001751a                os_spiflash_read
                0x0000000000017554                os_spiflash_program
                0x00000000000175da                os_spiflash_erase
 .com_text.sd.isr
                0x0000000000017658       0x20 ..\..\..\..\Libraries\libs\libplatform.a(device.o)
                0x0000000000017658                sdctl_isr
 .com_text.exception.hook
                0x0000000000017678       0x3a ..\..\..\..\Libraries\libs\libplatform.a(main.o)
                0x0000000000017678                sys_error_hook
 .com_text.exception
                0x00000000000176b2       0x5e ..\..\..\..\Libraries\libs\libplatform.a(main.o)
                0x00000000000176b2                exception_isr
 .com_text.delay
                0x0000000000017710       0x4e ..\..\..\..\Libraries\libs\libplatform.a(main.o)
                0x0000000000017710                delay_5ms
                0x000000000001772a                delay_ms
                0x0000000000017742                delay_us
 .com_text.irq  0x000000000001775e      0x178 ..\..\..\..\Libraries\libs\libplatform.a(interrupt.o)
                0x000000000001775e                bthw_isr
                0x0000000000017778                aubuf_isr
                0x00000000000177f4                timer0_isr
                0x000000000001785e                register_isr
                0x0000000000017898                tick_get
                0x00000000000178a0                watch_point_isr
                0x00000000000178c4                tick_check_expire
 .com_text.timer
                0x00000000000178d6       0x10 ..\..\..\..\Libraries\libs\libplatform.a(startup.o)
 .com_text.irq  0x00000000000178e6       0x5a ..\..\..\..\Libraries\libs\libplatform.a(reset.o)
                0x00000000000178e6                cpu_irq_comm
                0x0000000000017938                btmdm_isr
 .com_text.util.isr
                0x0000000000017940        0x6 ..\..\..\..\Libraries\libs\libplatform.a(reset.o)
                0x0000000000017940                kick_soft_isr
 .com_text.spiflash
                0x0000000000017946      0x154 ..\..\..\..\Libraries\libs\libplatform.a(spiflash.o)
                0x00000000000179d8                spiflash_program
                0x0000000000017a22                spiflash_erase
                0x0000000000017a4e                spiflash_get_id
 .com_text.debug
                0x0000000000017a9a      0x1aa ..\..\..\..\Libraries\libs\libplatform.a(debug.o)
                0x0000000000017b6c                debug_dump_err_cache_irq
 .com_text.sys  0x0000000000017c44       0x68 ..\..\..\..\Libraries\libs\libplatform.a(s_sys.o)
                0x0000000000017c44                s_ff1
                0x0000000000017c4a                s_fl1
                0x0000000000017c50                s_log2
                0x0000000000017c58                s_clb
                0x0000000000017c5e                s_bcnt
                0x0000000000017c64                s_ror
                0x0000000000017c6a                s_swapw
                0x0000000000017c70                s_bitrvti
                0x0000000000017c76                s_clip16
                0x0000000000017c7c                s_abs
                0x0000000000017c82                mul_r
                0x0000000000017c8e                dummy_func
                0x0000000000017c90                __ashrdi3
                0x0000000000017c9e                __ashldi3
 .com_text.thread.driver
                0x0000000000017cac       0x56 ..\..\..\..\Libraries\libs\libplatform.a(usb.o)
                0x0000000000017cac                os_mq_usb_post
                0x0000000000017cd2                thread_user_kick
                0x0000000000017d00                thread_user_func_do
 *fill*         0x0000000000017d02        0x2 
 .com_text.thread.usb
                0x0000000000017d04       0xaa ..\..\..\..\Libraries\libs\libplatform.a(usb.o)
                0x0000000000017d04                thread_usb_entry
 .com_text.bthw
                0x0000000000017dae       0x22 ..\..\..\..\Libraries\libs\libplatform.a(bt.o)
                0x0000000000017dae                btstack_status_lock
                0x0000000000017dc0                btstack_status_unlock
 .com_text.stack.thread
                0x0000000000017dd0       0x32 ..\..\..\..\Libraries\libs\libplatform.a(bt.o)
                0x0000000000017dd0                thread_btstack_pend
                0x0000000000017df2                thread_btstack_post
 .com_text.stack.run_loop
                0x0000000000017e02       0x48 ..\..\..\..\Libraries\libs\libplatform.a(bt.o)
                0x0000000000017e02                thread_btstack_entry
 .com_text.bb.bthw
                0x0000000000017e4a       0x3c ..\..\..\..\Libraries\libs\libplatform.a(bt.o)
                0x0000000000017e4a                thread_bthw_entry
 .com_text.bb.nanos
                0x0000000000017e86       0x16 ..\..\..\..\Libraries\libs\libbtstack.a(nanos.o)
                0x0000000000017e86                nanos_event_set
 .com_text.bb.patch
                0x0000000000017e9c       0x9a ..\..\..\..\Libraries\libs\libbtstack.a(patch.o)
                0x0000000000017e9c                bb_v1_patch0_do
                0x0000000000017eaa                bt_acl_cal_offset_fix
 .com_text.bb.ll.tx
                0x0000000000017f36        0x2 ..\..\..\..\Libraries\libs\libbtstack.a(platform.o)
                0x0000000000017f36                bb_ll_tx_cb
 .com_text.bb.ll.rx
                0x0000000000017f38        0x2 ..\..\..\..\Libraries\libs\libbtstack.a(platform.o)
                0x0000000000017f38                bb_ll_rx_cb
 .com_text.bb.lmp.rx
                0x0000000000017f3a        0x2 ..\..\..\..\Libraries\libs\libbtstack.a(platform.o)
                0x0000000000017f3a                bb_lmp_tx_cb
 .com_text.bb.lmp.tx
                0x0000000000017f3c        0x2 ..\..\..\..\Libraries\libs\libbtstack.a(platform.o)
                0x0000000000017f3c                bb_lmp_rx_cb
 .com_text.timer
                0x0000000000017f3e        0x6 ..\..\..\..\Libraries\libs\libbtstack.a(platform.o)
                0x0000000000017f3e                timer_get_tick
                0x0000000000017f42                timer_sync
 .com_text.bb.sco
                0x0000000000017f44       0x1e ..\..\..\..\Libraries\libs\libbtstack.a(bt_sco.o)
                0x0000000000017f44                bt_sco_is_transp
                0x0000000000017f54                bt_codec_isr
                0x0000000000017f56                lc_sco_codec_pkt
 .com_text.bt21.isr
                0x0000000000017f62      0x212 ..\..\..\..\Libraries\libs\libbtstack.a(bt_acl.o)
                0x0000000000017fe4                bt_acl_lmp_tx_isr
                0x000000000001804c                bt_acl_data_tx_isr
                0x0000000000018082                bt_sco_audio_isr
                0x0000000000018134                bt_acl_get_clkoff
 .com_text.ble.isr.con
                0x0000000000018174       0x82 ..\..\..\..\Libraries\libs\libbtstack.a(ble_con.o)
                0x0000000000018174                ble_con_rx_end
                0x00000000000181c6                ble_con_evt_prio_check
 .com_text.bb.utils
                0x00000000000181f6        0xa ..\..\..\..\Libraries\libs\libbtstack.a(bb_utils.o)
                0x00000000000181f6                bb_slot_to_duration
 .com_text.bb.isr
                0x0000000000018200      0x19c ..\..\..\..\Libraries\libs\libbtstack.a(bb_int.o)
                0x0000000000018234                bb_lpcycles_2_hus
                0x0000000000018276                bb_isr
                0x000000000001838a                bb_hal_isr
 .com_text.bb.btisr
                0x000000000001839c       0x2e ..\..\..\..\Libraries\libs\libbtstack.a(bb.o)
                0x000000000001839c                bb_acl_rx0_parse
                0x00000000000183a0                bb_free_acl_buf
                0x00000000000183ac                bb_alloc_acl_buf
 .com_text.bb.isr
                0x00000000000183ca       0x32 ..\..\..\..\Libraries\libs\libbtstack.a(bb.o)
                0x00000000000183ca                bb_notice_status
 .com_text.dummy
                0x00000000000183fc        0x6 ..\..\..\..\Libraries\libs\libbtstack.a(platform.o)
                0x00000000000183fc                dummy_void
                0x00000000000183fe                dummy_false
 .com_text.aubuf.isr
                0x0000000000018402        0x2 ..\..\..\..\Libraries\libs\libbtstack.a(extern.o)
                0x0000000000018402                ext_aubuf_isr
 .com_text.pp.send_pkt
                0x0000000000018404       0x58 ..\..\..\..\Libraries\libs\libbtstack.a(spp.o)
                0x0000000000018404                spp_send_packet
 .com_text.spp.tx
                0x000000000001845c       0xd4 ..\..\..\..\Libraries\libs\libbtstack.a(spp.o)
                0x000000000001845c                spp_is_connect
                0x0000000000018470                spp_default_connected
                0x0000000000018486                spp_custom1_connected
                0x000000000001849c                spp_custom2_connected
                0x00000000000184b2                bt_spp_tx
                0x00000000000184dc                bt_spp_custom1_tx
                0x0000000000018506                bt_spp_custom2_tx
 .com_text.spp.send_kick
                0x0000000000018530        0xe ..\..\..\..\Libraries\libs\libbtstack.a(spp.o)
                0x0000000000018530                spp_send_kick
 .com_text.spp.send_req
                0x000000000001853e       0x12 ..\..\..\..\Libraries\libs\libbtstack.a(spp.o)
                0x000000000001853e                btstack_spp_send_req
 .com_text.spp.event_send
                0x0000000000018550       0x32 ..\..\..\..\Libraries\libs\libbtstack.a(spp.o)
                0x0000000000018550                spp_event_send
 .com_text.spp.rx_set_new_credit
                0x0000000000018582       0x7e ..\..\..\..\Libraries\libs\libbtstack.a(spp.o)
                0x0000000000018582                spp_set_rx_new_credit
                0x0000000000018590                spp_notify_rx_buffer_len
                0x00000000000185e6                btstack_spp_rx_set_new_credit
 .com_text.txpkt.send
                0x0000000000018600      0x15e ..\..\..\..\Libraries\libs\libbtstack.a(btstack_txpkt.o)
                0x0000000000018600                txpkt_send
                0x00000000000186de                txpkt_event_send
 .com_text.stack.run_loop
                0x000000000001875e       0xe2 ..\..\..\..\Libraries\libs\libbtstack.a(btstack_run_loop.o)
                0x000000000001875e                btstack_cmp_abs_tick
                0x0000000000018764                btstack_runtime_check
                0x00000000000187aa                btstack_run_loop_execute_once
 .com_text.stack.thread
                0x0000000000018840        0xe ..\..\..\..\Libraries\libs\libbtstack.a(btstack_run_loop.o)
                0x0000000000018840                btstack_run_loop_embedded_trigger
 .com_text.stack.ticks
                0x000000000001884e       0x34 ..\..\..\..\Libraries\libs\libbtstack.a(btstack_run_loop.o)
 .com_text.stack.linked_list
                0x0000000000018882       0x50 ..\..\..\..\Libraries\libs\libbtstack.a(btstack_linked_list.o)
                0x0000000000018882                btstack_linked_list_empty
                0x000000000001888a                btstack_linked_list_iterator_init
                0x0000000000018896                btstack_linked_list_iterator_has_next
                0x00000000000188b4                btstack_linked_list_iterator_next
 .com_text.ble.send_pkt
                0x00000000000188d2       0xd6 ..\..\..\..\Libraries\libs\libbtstack.a(gatt_server.o)
                0x00000000000188d2                ble_send_notify_packet
                0x0000000000018964                att_event_server_send
 .com_text.stack.ble.mtu
                0x00000000000189a8       0x10 ..\..\..\..\Libraries\libs\libbtstack.a(gatt_server.o)
                0x00000000000189a8                ble_get_gatt_mtu
 .com_text.stack.ticks
                0x00000000000189b8        0xa ..\..\..\..\Libraries\libs\libbtstack.a(btstack_hal.o)
                0x00000000000189ba                sys_tick_handler
 .com_text.isr  0x00000000000189c2       0x1a ..\..\..\..\Libraries\libs\libbtstack.a(btstack_hal.o)
                0x00000000000189c2                bt_timer_isr
 .com_text.stack.api
                0x00000000000189dc      0x13a ..\..\..\..\Libraries\libs\libbtstack.a(btstack_api.o)
                0x00000000000189dc                bt_is_testmode
                0x00000000000189ea                bt_is_l2cap_disconnected
                0x0000000000018a04                bt_is_disconnecting
                0x0000000000018a1e                btstack_status_update
                0x0000000000018a2c                btstack_set_play_status
                0x0000000000018a58                btstack_get_play_status
                0x0000000000018a68                bt_get_status
                0x0000000000018ab0                bt_get_disp_status
                0x0000000000018ab2                bt_is_calling
                0x0000000000018ac8                bt_get_l2cap_status
                0x0000000000018af4                bt_tws_get_status
 .com_text.stack.run_loop
                0x0000000000018b16        0x2 ..\..\..\..\Libraries\libs\libbtstack.a(btstack_api.o)
                0x0000000000018b16                btstack_msg
 .com_text.stack.ble.api0
                0x0000000000018b18       0x10 ..\..\..\..\Libraries\libs\libbtstack.a(ble_api.o)
                0x0000000000018b18                ble_get_status
 .com_text.stack.ble.api1
                0x0000000000018b28       0x16 ..\..\..\..\Libraries\libs\libbtstack.a(ble_api.o)
                0x0000000000018b28                ble_is_connect
 .com_text.bb.frag
                0x0000000000018b3e       0x3a ..\..\..\..\Libraries\libs\libbtstack.a(bb_sche.o)
 .com_text.bb.prog
                0x0000000000018b78      0x1f0 ..\..\..\..\Libraries\libs\libbtstack.a(bb_sche.o)
 .com_text.bb.patch
                0x0000000000018d68       0x52 ..\..\..\..\Libraries\libs\libbtstack.a(patch_asm.o)
                0x0000000000018d68                bb_v1_patch0
                0x0000000000018d74                bb_v1_patch6
                0x0000000000018d7c                bb_v1_patch7
                0x0000000000018d96                bb_v1_patch8
 .com_text.bb.isr
                0x0000000000018dba       0x1a ..\..\..\..\Libraries\libs\libbtstack.a(aes.o)
                0x0000000000018dba                ble_ecpy_aes_res_cb
 .com_text.bb.isr
                0x0000000000018dd4       0x50 ..\..\..\..\Libraries\libs\libbtstack.a(rf.o)
                0x0000000000018dd4                rf_rssi_calc_dbm
                0x0000000000018dde                rf_txpwr_get_lv
                0x0000000000018e12                rf_txpwr_get_dbm
                0x0000000000018e22                rf_agc_enable
 .com_text.isr.txrx
                0x0000000000018e24       0x76 ..\..\..\..\Libraries\libs\libbtstack.a(rf.o)
                0x0000000000018e24                bb_rf_ext_ctl_cb
                0x0000000000018e26                bthw_txrx_isr
 *fill*         0x0000000000018e9a        0x2 
 .com_text.bt21.isr
                0x0000000000018e9c      0x5c8 ..\..\..\..\Libraries\libs\libbtstack.a(bt_hook.o)
                0x0000000000018e9c                bt_page_init_func
                0x0000000000018ea4                bt_acl_rx_header
                0x000000000001909c                bt_acl_test_rx_end
                0x00000000000190a0                bt_acl_rx_end
                0x0000000000019108                bt_acl_sniff_cacl_win_size
                0x0000000000019160                bt_isr_hook
 .com_text.ble.isr
                0x0000000000019464       0x7c ..\..\..\..\Libraries\libs\libbtstack.a(ble_hook.o)
                0x0000000000019464                ble_isr_hook
 .com_text.bb.hct
                0x00000000000194e0       0x18 ..\..\..\..\Libraries\libs\libbtstack.a(hct_fc.o)
                0x00000000000194e0                hci_fc_acl_packet_sent
 .com_text.bt21.sco
                0x00000000000194f8       0x1e ..\..\..\..\Libraries\libs\libbtstack.a(tws_sco.o)
                0x00000000000194f8                bt_sco_get_index
 .com_text.bb.tws.sw.chk
                0x0000000000019516        0x4 ..\..\..\..\Libraries\libs\libbtstack.a(tws_acl.o)
                0x0000000000019516                tws_switch_acl_is_pause
 .com_text.bt21.isr
                0x000000000001951a       0x3c ..\..\..\..\Libraries\libs\libbtstack.a(bt_hal.o)
                0x000000000001951a                bt_channel_assess
 .com_text.bt21.isr
                0x0000000000019556       0x52 ..\..\..\..\Libraries\libs\libbtstack.a(bt21.o)
                0x0000000000019556                bt_buf_acl_rx_free
                0x0000000000019564                bt21_isr
 .com_text.ble.isr
                0x00000000000195a8      0x102 ..\..\..\..\Libraries\libs\libbtstack.a(ble_hal.o)
 .com_text.ble.isr.con
                0x00000000000196aa       0x3c ..\..\..\..\Libraries\libs\libbtstack.a(ble_hal.o)
                0x00000000000196aa                ble_channel_assess
 .com_text.ble.isr.adv
                0x00000000000196e6       0x52 ..\..\..\..\Libraries\libs\libbtstack.a(ble_adv.o)
                0x00000000000196e6                ble_adv_duration_update
 .com_text.bb.isr
                0x0000000000019738       0x18 ..\..\..\..\Libraries\libs\libbtstack.a(ble.o)
                0x0000000000019738                ble_isr
 .com_text.l2cap_test.con
                0x0000000000019750       0x4c ..\..\..\..\Libraries\libs\libbtstack.a(l2cap_test.o)
                0x0000000000019750                l2cap_vd_acl_check
 .com_text.stack.handler.l2cap
                0x000000000001979c       0x38 ..\..\..\..\Libraries\libs\libbtstack.a(l2cap.o)
                0x000000000001979c                l2cap_get_channel_for_local_cid
                0x00000000000197b4                l2cap_get_channel_for_remote_cid
 .com_text.sco  0x00000000000197d4        0x4 ..\..\..\..\Libraries\libs\libbtstack.a(hci_sco.o)
                0x00000000000197d4                sco_init_var
                0x00000000000197d6                sco_buffer_reset
 .com_text.stack.hci
                0x00000000000197d8       0x5a ..\..\..\..\Libraries\libs\libbtstack.a(hci.o)
                0x00000000000197d8                hci_connection_for_handle
                0x0000000000019800                hci_can_send_command_packet_now
 .com_text.stack.hci_recv
                0x0000000000019832        0xe ..\..\..\..\Libraries\libs\libbtstack.a(hci.o)
                0x0000000000019832                hci_host_recv_packet
 .com_text.bb.btisr
                0x0000000000019840        0x8 ..\..\..\..\Libraries\libs\libbtstack.a(avdtp.o)
                0x0000000000019840                a2dp_get_play_index
                0x0000000000019844                avdtp_rx_media_parse
 .com_text.stack.hcic
                0x0000000000019848       0x10 ..\..\..\..\Libraries\libs\libbtstack.a(hci_transport_hcic.o)
                0x0000000000019848                hcic_can_send_packet_now
 .com_text.ble.isr.test.clr
                0x0000000000019858       0x22 ..\..\..\..\Libraries\libs\libbtstack.a(ble_test.o)
 .com_text.ble.init
                0x000000000001987a      0xba2 ..\..\..\..\Libraries\libs\libbtstack.a(ble_init.o)
 .com_text.usbdev
                0x000000000001a41c       0x20 ..\..\..\..\Libraries\libs\libdrivers.a(usb_device_hid.o)
                0x000000000001a41c                ude_tmr_isr
 *fill*         0x000000000001a43c        0x0 
 .com_text.epsize.table
                0x000000000001a43c        0x4 ..\..\..\..\Libraries\libs\libdrivers.a(usb_comm.o)
                0x000000000001a43c                epsize_tbl
 *(.com_text.stack.handler)
 *(.com_rodata*)
 .com_rodata.exception
                0x000000000001a440       0x29 ..\..\..\..\Libraries\libs\libplatform.a(main.o)
 *fill*         0x000000000001a469        0x3 
 .com_rodata.irq
                0x000000000001a46c       0x1b ..\..\..\..\Libraries\libs\libplatform.a(interrupt.o)
                0x000000000001a46c                watch_point_str
 *fill*         0x000000000001a487        0x1 
 .com_rodata.miss
                0x000000000001a488       0x29 ..\..\..\..\Libraries\libs\libplatform.a(debug.o)
 *fill*         0x000000000001a4b1        0x3 
 .com_rodata.bb.sco
                0x000000000001a4b4       0x3c ..\..\..\..\Libraries\libs\libbtstack.a(bt_sco.o)
                0x000000000001a4b4                tbl_msbc_mute
 .com_rodata.bb.tbl
                0x000000000001a4f0       0x32 ..\..\..\..\Libraries\libs\libbtstack.a(bt_acl.o)
 *fill*         0x000000000001a522        0x2 
 .com_rodata.bb.tbl
                0x000000000001a524       0x10 ..\..\..\..\Libraries\libs\libbtstack.a(ble_con.o)
                0x000000000001a524                byte_tx_time
                0x000000000001a52c                fixed_tx_time
 .com_rodata.bb.tbl
                0x000000000001a534       0x44 ..\..\..\..\Libraries\libs\libbtstack.a(bb_utils.o)
                0x000000000001a534                one_bits
                0x000000000001a544                bb_rate_to_byte_dur_us
                0x000000000001a54c                bb_rate_to_phy_mask
                0x000000000001a550                bb_phy_value_to_mask
                0x000000000001a554                bb_phy_mask_to_value
                0x000000000001a55c                bb_phy_to_rate
                0x000000000001a560                bb_rate_to_phy
                0x000000000001a568                bb_sca2ppm
 .com_rodata.bb.tws
                0x000000000001a578        0xd ..\..\..\..\Libraries\libs\libbtstack.a(bb_int.o)
                0x000000000001a578                str_bb_err
 *fill*         0x000000000001a585        0x3 
 .com_rodata.bb.tbl
                0x000000000001a588       0x3c ..\..\..\..\Libraries\libs\libbtstack.a(bb.o)
                0x000000000001a588                bb_priority
 .com_rodata.bb.tbl
                0x000000000001a5c4        0xc ..\..\..\..\Libraries\libs\libbtstack.a(vs_proc.o)
                0x000000000001a5c4                vs_msg_env
 .com_rodata.bb.tbl
                0x000000000001a5d0        0x8 ..\..\..\..\Libraries\libs\libbtstack.a(rf.o)
 .com_rodata.bb.tbl
                0x000000000001a5d8        0xb ..\..\..\..\Libraries\libs\libbtstack.a(bt_hook.o)
 *fill*         0x000000000001a5e3        0x1 
 .com_rodata.bb.tbl
                0x000000000001a5e4       0x12 ..\..\..\..\Libraries\libs\libbtstack.a(bt21.o)
 *fill*         0x000000000001a5f6        0x2 
 .com_rodata.btstakc.hci
                0x000000000001a5f8        0x8 ..\..\..\..\Libraries\libs\libbtstack.a(hci_cmd.o)
                0x000000000001a5f8                hci_num_of_packet_complete
 .com_rodata.hci.trans
                0x000000000001a600       0x20 ..\..\..\..\Libraries\libs\libbtstack.a(hci_transport_hcic.o)
 .com_rodata.bb.tbl
                0x000000000001a620        0xc ..\..\..\..\Libraries\libs\libbtstack.a(lm_proc.o)
                0x000000000001a620                lm_msg_env
 .com_rodata.bb.tbl
                0x000000000001a62c        0x8 ..\..\..\..\Libraries\libs\libbtstack.a(ble_init.o)
                0x000000000001a62c                ble_init_max_aux_dur_tab
 .com_rodata.bb.tbl
                0x000000000001a634       0x18 ..\..\..\..\Libraries\libs\libbtstack.a(ble_buf.o)
 .com_rodata.bb.tbl
                0x000000000001a64c        0xc ..\..\..\..\Libraries\libs\libbtstack.a(lc_proc.o)
                0x000000000001a64c                lc_msg_env
 .com_rodata.bb.tbl
                0x000000000001a658        0xc ..\..\..\..\Libraries\libs\libbtstack.a(mgr_proc.o)
                0x000000000001a658                mgr_msg_env
 .com_rodata.bb.tbl
                0x000000000001a664        0xc ..\..\..\..\Libraries\libs\libbtstack.a(ll_proc.o)
                0x000000000001a664                ll_msg_env
 *debug.o(.rodata*)
 .rodata.str1.4
                0x000000000001a670       0xd0 ..\..\..\..\Libraries\libs\libplatform.a(debug.o)
                                         0xce (size before relaxing)
 *(.data*)
 .data          0x000000000001a740        0xc Output\obj\Libraries\BT\spp\profile.o
                0x000000000001a740                spp_sdp_record_item
 .data          0x000000000001a74c       0x18 ..\..\..\..\Libraries\libs\libbtstack.a(btstack_link_key_db.o)
 .data          0x000000000001a764       0x31 ..\..\..\..\Libraries\libs\libbtstack.a(btstack_run_loop.o)
                0x000000000001a764                data_source_debug_info
 *(.sdata*)
 *fill*         0x000000000001a795        0x1 
 .sdata         0x000000000001a796        0x2 Output\obj\Libraries\bsp\bsp_fot.o
                0x000000000001a796                dev_version
 .sdata         0x000000000001a798        0x1 Output\obj\Libraries\BT\ble\adv0.o
                0x000000000001a798                cfg_ble_adv0_en
 .sdata         0x000000000001a799        0x2 Output\obj\Libraries\BT\ble\ble.o
                0x000000000001a799                cfg_ble_mtu_request_en
                0x000000000001a79a                cfg_ble_security_en
 *fill*         0x000000000001a79b        0x1 
 .sdata         0x000000000001a79c       0x10 Output\obj\Libraries\BT\spp\bt.o
                0x000000000001a79c                bt_local_addr
                0x000000000001a7a2                cfg_bt_link_info_items
                0x000000000001a7a4                cfg_bt_sup_to_connect_times
                0x000000000001a7a6                cfg_bt_pwrup_connect_times
                0x000000000001a7a7                cfg_bt_connect_times
                0x000000000001a7a8                cfg_bt_support_profile
                0x000000000001a7aa                cfg_bt_dual_mode
                0x000000000001a7ab                cfg_bt_max_acl_link
 .sdata         0x000000000001a7ac        0x1 Output\obj\Libraries\libs\strong_symbol.o
                0x000000000001a7ac                cfg_bt_sniff_mode_dis
 *fill*         0x000000000001a7ad        0x1 
 .sdata         0x000000000001a7ae       0x11 ..\..\..\..\Libraries\libs\libbtstack.a(extern_bt.o)
                0x000000000001a7ae                cfg_bt_music_low_latency
                0x000000000001a7b0                cfg_bt_music_normal_latency
                0x000000000001a7b2                cfg_bt_ble_adv
                0x000000000001a7be                cfg_bt_sniff_clk_sel
 *fill*         0x000000000001a7bf        0x1 
 .sdata         0x000000000001a7c0        0x4 ..\..\..\..\Libraries\libs\libbtstack.a(sdp_server.o)
 .sdata         0x000000000001a7c4        0x4 ..\..\..\..\Libraries\libs\libbtstack.a(att_server.o)
 .sdata         0x000000000001a7c8        0xc ..\..\..\..\Libraries\libs\libbtstack.a(btstack_hal.o)
 .sdata         0x000000000001a7d4        0x1 ..\..\..\..\Libraries\libs\libbtstack.a(btstack_adv0.o)
 *fill*         0x000000000001a7d5        0x1 
 .sdata         0x000000000001a7d6        0x3 ..\..\..\..\Libraries\libs\libbtstack.a(sm.o)
 *fill*         0x000000000001a7d9        0x3 
 .sdata         0x000000000001a7dc        0x5 ..\..\..\..\Libraries\libs\libbtstack.a(ble_adv0.o)
 .sdata         0x000000000001a7e1        0x1 ..\..\..\..\Libraries\libs\libbtstack.a(extern_hfhs.o)
                0x000000000001a7e1                cfg_bt_hfp_feature
 .sdata         0x000000000001a7e2        0x3 ..\..\..\..\Libraries\libs\libbtstack.a(l2cap_signaling.o)
 .sdata         0x000000000001a7e5        0x4 ..\..\..\..\Libraries\libs\libdrivers.a(usb_device_hid.o)
                0x000000000001a7e5                user_ep_type
                0x000000000001a7e6                user_ep_dir
                0x000000000001a7e7                user_ep_idx
                0x000000000001a7e8                hid_in_ep
 *(.load_text)
 *fill*         0x000000000001a7e9        0x1 
 .load_text     0x000000000001a7ea       0x10 ..\..\..\..\Libraries\libs\libplatform.a(main.o)
 *(.load_rodata)
                0x000000000001a800                . = ALIGN (0x200)
 *fill*         0x000000000001a7fa        0x6 

.flash          0x0000000010003a00    0x42a00
                0x0000000010003a00                __code_start_sniff = .
 *(.sniff*)
                0x0000000010003a00                . = ALIGN (0x200)
                0x0000000010003a00                __code_end_sniff = .
                0x0000000010003a00                __code_start_usbdev = .
 *(.usbdev*)
 .usbdev.com    0x0000000010003a00      0x1b2 ..\..\..\..\Libraries\libs\libdrivers.a(usb_device_hid.o)
                0x0000000010003a00                usb_user_ep_tx_handler
                0x0000000010003a02                usb_user_ep_rx_handler
                0x0000000010003a04                ude_hid_setvalid
                0x0000000010003a18                ude_hid_send
                0x0000000010003a72                usb_user_ep_rx_ack
                0x0000000010003a96                usb_user_ep_tx_process
                0x0000000010003ab2                usb_user_ep_rx_process
                0x0000000010003ae0                usb_int_ep_reset
                0x0000000010003af6                udh_init
                0x0000000010003b52                udu_init
 .usbdev.com    0x0000000010003bb2       0x7c ..\..\..\..\Libraries\libs\libdrivers.a(usb_device_printer.o)
                0x0000000010003bb2                usb_bulk_reset
                0x0000000010003bc8                ude_rx_ack
                0x0000000010003be0                bulk_tx_handler
                0x0000000010003be2                bulk_rx_handler
                0x0000000010003be4                ude_bulk_tx_process
                0x0000000010003c00                ude_bulk_rx_process
 .usbdev.com    0x0000000010003c2e      0x36c ..\..\..\..\Libraries\libs\libdrivers.a(usb_device_ep.o)
                0x0000000010003c2e                usb_set_cur_ep
                0x0000000010003c44                usb_ep_init
                0x0000000010003cd0                usb_ep_halt
                0x0000000010003d1c                usb_ep_clear
                0x0000000010003d5c                usb_ep_transfer
                0x0000000010003eea                usb_ep_reset
                0x0000000010003f5e                usb_ep_start_transfer
                0x0000000010003f78                usb_ep_do_transfer
                0x0000000010004000                . = ALIGN (0x200)
 *fill*         0x0000000010003f9a       0x66 
                0x0000000010004000                __code_end_usbdev = .
                0x0000000010004000                __code_start_sleep = .
 *(.saradc_text*)
 *(.sleep_text*)
 .sleep_text.sleep.rc
                0x0000000010004000       0xc2 ..\..\..\..\Libraries\libs\libplatform.a(rc.o)
                0x0000000010004000                rc_sleep_trim_init
                0x0000000010004002                rc_sleep_trim_clear
                0x0000000010004004                rc_sleep_get_freqcnt
                0x0000000010004072                rc_sleep_reset_sta
                0x0000000010004074                rc_sleep_get_trim_freqcnt
 .sleep_text.rf
                0x00000000100040c2      0x21a ..\..\..\..\Libraries\libs\libbtstack.a(rf_smart.o)
                0x00000000100041a2                rfphy_deep_sleep
                0x000000001000424a                rfphy_idle
                0x0000000010004400                . = ALIGN (0x200)
 *fill*         0x00000000100042dc      0x124 
                0x0000000010004400                __code_end_sleep = .
                0x0000000010004400                __code_start_charge = .
 *(.charge_text*)
 *(.text.bsp.charge)
 *(.text.bsp.tkey)
 *(.text.vhouse)
                0x0000000010004400                . = ALIGN (0x200)
                0x0000000010004400                __code_end_charge = .
                0x0000000010004400                __code_start_pwrsave = .
 *(.text.pwroff*)
                0x0000000010004400                . = ALIGN (0x200)
                0x0000000010004400                __code_end_pwrsave = .
                0x0000000010004400                __code_start_bb_test = .
 *(.bb_test*)
 *(.bb_test_rodata*)
                0x0000000010004400                . = ALIGN (0x200)
                0x0000000010004400                __code_end_bb_test = .
                0x0000000010004400                __code_start_update = .
 *(.text.update*)
 .text.update_sd0baud
                0x0000000010004400       0x3c ..\..\..\..\Libraries\libs\libplatform.a(sys_clk.o)
                0x0000000010004400                update_sd0baud
 .text.update_complete
                0x000000001000443c        0x2 ..\..\..\..\Libraries\libs\libplatform.a(weak_symbol.o)
                0x000000001000443c                update_complete
                0x0000000010004600                . = ALIGN (0x200)
 *fill*         0x000000001000443e      0x1c2 
                0x0000000010004600                __code_end_update = .
                0x0000000010004600                __code_start_huart = .
 *(.com_huart*)
                0x0000000010004600                . = ALIGN (0x200)
                0x0000000010004600                __code_end_huart = .
                0x0000000010004600                __code_start_fota = .
 *(.text.fot.cache*)
 .text.fot.cache
                0x0000000010004600      0x744 Output\obj\Libraries\bsp\bsp_fot.o
                0x000000001000466a                fot_recv_proc
                0x0000000010004b5c                bsp_fot_process
                0x0000000010004c44                bsp_usb_fot_process
 *fill*         0x0000000010004d44        0x0 
 .text.fot.cache
                0x0000000010004d44      0x204 ..\..\..\..\Libraries\libs\libplatform.a(fot_update.o)
                0x0000000010004d44                fot_pkt_process_do
                0x0000000010004eae                fot_write
                0x0000000010005000                . = ALIGN (0x200)
 *fill*         0x0000000010004f48       0xb8 
                0x0000000010005000                __code_end_fota = .
                0x0000000010005000                __code_start_bts = .
 *(.text.stk.tws.txreq*)
 *(.text.stk.l2cap.txreq*)
 .text.stk.l2cap.txreq
                0x0000000010005000      0x110 ..\..\..\..\Libraries\libs\libbtstack.a(l2cap.o)
                0x00000000100050d4                l2cap_request_can_send_now_event
                0x00000000100050ee                l2cap_request_can_send_fix_channel_now_event
 *fill*         0x0000000010005110        0x0 
 .text.stk.l2cap.txreq.rodata
                0x0000000010005110        0xa ..\..\..\..\Libraries\libs\libbtstack.a(l2cap.o)
                0x0000000010005200                . = ALIGN (0x200)
 *fill*         0x000000001000511a       0xe6 
 *(.text.stk.tws.send*)
                0x0000000010005200                . = ALIGN (0x200)
 *(.text.stk.tws.recv*)
                0x0000000010005200                . = ALIGN (0x200)
 *(.text.stk.hci.tx*)
                0x0000000010005200                . = ALIGN (0x200)
 *(.text.bts.hci.rx*)
                0x0000000010005200                . = ALIGN (0x200)
 *(.text.stk.bt.acl.tx*)
 .text.stk.bt.acl.tx.done
                0x0000000010005200       0x76 ..\..\..\..\Libraries\libs\libbtstack.a(lc_proc.o)
                0x0000000010005400                . = ALIGN (0x200)
 *fill*         0x0000000010005276      0x18a 
                0x0000000010005400                __code_end_bts = .
 *(.irq_init.aligned)
                0x0000000010005400                . = ALIGN (0x200)
 *(.text.ble.chmap*)
 .text.ble.chmap
                0x0000000010005400       0x50 ..\..\..\..\Libraries\libs\libbtstack.a(ble_con.o)
                0x0000000010005400                ble_con_ch_map_update
                0x0000000010005600                . = ALIGN (0x200)
 *fill*         0x0000000010005450      0x1b0 
 *(.text*)
 .text.cm_loadparam
                0x0000000010005600       0x12 Output\obj\Libraries\bsp\bsp_cm.o
                0x0000000010005600                cm_loadparam
 .text.cm_factory
                0x0000000010005612       0x20 Output\obj\Libraries\bsp\bsp_cm.o
                0x0000000010005612                cm_factory
 .text.fot.update
                0x0000000010005632       0x6c Output\obj\Libraries\bsp\bsp_fot.o
                0x0000000010005632                is_fot_start
                0x000000001000563e                fot_update_pause
                0x0000000010005658                bsp_fot_init
                0x0000000010005680                fot_update_continue
 .text.fot_ble_disconnect_callback
                0x000000001000569e       0x32 Output\obj\Libraries\bsp\bsp_fot.o
                0x000000001000569e                fot_ble_disconnect_callback
 .text.fot_ble_connect_callback
                0x00000000100056d0        0xc Output\obj\Libraries\bsp\bsp_fot.o
                0x00000000100056d0                fot_ble_connect_callback
 .text.fot_spp_connect_callback
                0x00000000100056dc        0xc Output\obj\Libraries\bsp\bsp_fot.o
                0x00000000100056dc                fot_spp_connect_callback
 .text.fot_spp_disconnect_callback
                0x00000000100056e8       0x32 Output\obj\Libraries\bsp\bsp_fot.o
                0x00000000100056e8                fot_spp_disconnect_callback
 .text.bsp.param
                0x000000001000571a       0xee Output\obj\Libraries\bsp\bsp_param.o
                0x000000001000571a                param_init
                0x0000000010005738                bsp_param_write
                0x000000001000573c                bsp_param_read
                0x0000000010005740                bsp_param_sync
                0x0000000010005744                param_sync
                0x0000000010005748                param_get_xosc_addr
                0x000000001000574c                param_fot_addr_write
                0x0000000010005762                param_fot_addr_read
                0x000000001000576c                param_fot_remote_ver_write
                0x0000000010005782                param_fot_remote_ver_read
                0x000000001000578c                param_fot_head_info_write
                0x00000000100057a2                param_fot_head_info_read
                0x00000000100057ac                param_fot_hash_write
                0x00000000100057c2                param_fot_hash_read
                0x00000000100057cc                param_qcheck_code_write
                0x00000000100057e2                param_qcheck_code_read
                0x00000000100057ec                param_sys_vol_write
                0x00000000100057fa                param_sys_vol_read
 .text.bsp.sys.init
                0x0000000010005808      0x232 Output\obj\Libraries\bsp\bsp_sys.o
                0x0000000010005880                rtc_init
                0x00000000100058f2                bsp_update_init
                0x0000000010005938                bsp_sys_init
 .text.uart0_mapping_sel
                0x0000000010005a3a       0x90 Output\obj\Libraries\bsp\bsp_sys.o
                0x0000000010005a3a                uart0_mapping_sel
 .text.bsp_get_xosc_xcfg
                0x0000000010005aca       0x20 Output\obj\Libraries\bsp\bsp_sys.o
                0x0000000010005aca                bsp_get_xosc_xcfg
 .text.ble_fot_send_packet
                0x0000000010005aea       0x1a Output\obj\Libraries\BT\ble\ab_link\app.o
                0x0000000010005aea                ble_fot_send_packet
 .text.ble_get_local_bd_addr
                0x0000000010005b04       0x28 Output\obj\Libraries\BT\ble\ble.o
                0x0000000010005b04                ble_get_local_bd_addr
 .text.ble_disconnect_callback
                0x0000000010005b2c       0x18 Output\obj\Libraries\BT\ble\ble.o
                0x0000000010005b2c                ble_disconnect_callback
 .text.ble_connect_callback
                0x0000000010005b44       0x18 Output\obj\Libraries\BT\ble\ble.o
                0x0000000010005b44                ble_connect_callback
 .text.bt_get_class_of_device
                0x0000000010005b5c       0x18 Output\obj\Libraries\BT\spp\bt.o
                0x0000000010005b5c                bt_get_class_of_device
 .text.bt_get_pin_code
                0x0000000010005b74        0xa Output\obj\Libraries\BT\spp\bt.o
                0x0000000010005b74                bt_get_pin_code
 .text.bt_get_local_name
                0x0000000010005b7e        0x8 Output\obj\Libraries\BT\spp\bt.o
                0x0000000010005b7e                bt_get_local_name
 .text.bt_get_local_bd_addr
                0x0000000010005b86       0x14 Output\obj\Libraries\BT\spp\bt.o
                0x0000000010005b86                bt_get_local_bd_addr
 .text.bt_get_link_info
                0x0000000010005b9a       0x24 Output\obj\Libraries\BT\spp\bt.o
                0x0000000010005b9a                bt_get_link_info
 .text.bt_put_link_info
                0x0000000010005bbe       0x24 Output\obj\Libraries\BT\spp\bt.o
                0x0000000010005bbe                bt_put_link_info
 .text.bt_get_ext_link_info
                0x0000000010005be2        0x8 Output\obj\Libraries\BT\spp\bt.o
                0x0000000010005be2                bt_get_ext_link_info
 .text.bt_put_ext_link_info
                0x0000000010005bea        0x8 Output\obj\Libraries\BT\spp\bt.o
                0x0000000010005bea                bt_put_ext_link_info
 .text.bt_sync_link_info
                0x0000000010005bf2        0x4 Output\obj\Libraries\BT\spp\bt.o
                0x0000000010005bf2                bt_sync_link_info
 .text.bt_init_lib
                0x0000000010005bf6       0x24 Output\obj\Libraries\BT\spp\profile.o
                0x0000000010005bf6                bt_init_lib
 .text.spp_txpkt_init
                0x0000000010005c1a       0x30 Output\obj\Libraries\BT\spp\spp.o
                0x0000000010005c1a                spp_txpkt_init
 .text.spp_rxpkt_init
                0x0000000010005c4a        0x8 Output\obj\Libraries\BT\spp\spp.o
                0x0000000010005c4a                spp_rxpkt_init
 .text.get_spp_mtu_size
                0x0000000010005c52        0x6 Output\obj\Libraries\BT\spp\spp.o
                0x0000000010005c52                get_spp_mtu_size
 .text.spp_connect_callback
                0x0000000010005c58       0x18 Output\obj\Libraries\BT\spp\spp.o
                0x0000000010005c58                spp_connect_callback
 .text.spp_disconnect_callback
                0x0000000010005c70       0x18 Output\obj\Libraries\BT\spp\spp.o
                0x0000000010005c70                spp_disconnect_callback
 .text.spp_rx_callback
                0x0000000010005c88       0x86 Output\obj\Libraries\BT\spp\spp.o
                0x0000000010005c88                spp_rx_callback
 .text.clock_gate1_cmd
                0x0000000010005d0e       0x16 Output\obj\Libraries\Device\Source\gw3323_clk.o
                0x0000000010005d0e                clock_gate1_cmd
 .text.gpio_init
                0x0000000010005d24       0xf6 Output\obj\Libraries\Device\Source\gw3323_gpio.o
                0x0000000010005d24                gpio_init
 .text.gpio_func_mapping
                0x0000000010005e1a       0x5a Output\obj\Libraries\Device\Source\gw3323_gpio.o
                0x0000000010005e1a                gpio_func_mapping
 .text.tmr_base_init
                0x0000000010005e74       0xb4 Output\obj\Libraries\Device\Source\gw3323_tmr.o
                0x0000000010005e74                tmr_base_init
 .text.tmr_pic_config
                0x0000000010005f28       0x76 Output\obj\Libraries\Device\Source\gw3323_tmr.o
                0x0000000010005f28                tmr_pic_config
 .text.vs_ble_test
                0x0000000010005f9e        0x4 Output\obj\Libraries\libs\strong_symbol.o
                0x0000000010005f9e                vs_ble_test
 .text.vs_fcc_test_cmd
                0x0000000010005fa2        0x4 Output\obj\Libraries\libs\strong_symbol.o
                0x0000000010005fa2                vs_fcc_test_cmd
 .text.is_fot_update_en
                0x0000000010005fa6        0x4 Output\obj\Libraries\libs\strong_symbol.o
                0x0000000010005fa6                is_fot_update_en
 .text.usb_init
                0x0000000010005faa        0x2 Output\obj\Libraries\libs\strong_symbol.o
                0x0000000010005faa                usb_init
 .text.usb_isr  0x0000000010005fac        0x2 Output\obj\Libraries\libs\strong_symbol.o
                0x0000000010005fac                usb_isr
 .text.ude_ep_reset
                0x0000000010005fae        0x2 Output\obj\Libraries\libs\strong_symbol.o
                0x0000000010005fae                ude_ep_reset
 .text.ude_control_flow
                0x0000000010005fb0        0x2 Output\obj\Libraries\libs\strong_symbol.o
                0x0000000010005fb0                ude_control_flow
 .text.timer3_cap_init
                0x0000000010005fb2       0x82 Output\obj\Examples\TIMER\TIM_Capture\Source\timer_capture.o
                0x0000000010005fb2                timer3_cap_init
 .text.timer3_capture_example
                0x0000000010006034       0xac Output\obj\Examples\TIMER\TIM_Capture\Source\timer_capture.o
                0x0000000010006034                timer3_capture_example
 .text.timer4_pwm_init
                0x00000000100060e0       0x76 Output\obj\Examples\TIMER\TIM_Capture\Source\timer_pwm.o
                0x00000000100060e0                timer4_pwm_init
 .text.getcfg_vddbt_sel
                0x0000000010006156       0x18 Output\obj\Examples\TIMER\TIM_Capture\Project\config.o
                0x0000000010006156                getcfg_vddbt_sel
 .text.getcfg_vddio_sel
                0x000000001000616e        0xc Output\obj\Examples\TIMER\TIM_Capture\Project\config.o
                0x000000001000616e                getcfg_vddio_sel
 .text.getcfg_vddbt_capless_en
                0x000000001000617a        0xa Output\obj\Examples\TIMER\TIM_Capture\Project\config.o
                0x000000001000617a                getcfg_vddbt_capless_en
 .text.startup.main
                0x0000000010006184       0x30 Output\obj\Examples\TIMER\TIM_Capture\Project\main.o
                0x0000000010006184                main
 .text.pll_vco_band_trimming
                0x00000000100061b4       0x9a ..\..\..\..\Libraries\libs\libplatform.a(audio.o)
 *fill*         0x000000001000624e       0xb2 
 .text.adpll_divider_update_do
                0x0000000010006300       0xfa ..\..\..\..\Libraries\libs\libplatform.a(audio.o)
                0x0000000010006300                adpll_divider_update_do
 .text.adpll_divider_update
                0x00000000100063fa       0x68 ..\..\..\..\Libraries\libs\libplatform.a(audio.o)
                0x00000000100063fa                adpll_divider_update
 .text.adpll_init
                0x0000000010006462      0x106 ..\..\..\..\Libraries\libs\libplatform.a(audio.o)
                0x0000000010006462                adpll_init
 .text.cm_loadpage
                0x0000000010006568       0xb4 ..\..\..\..\Libraries\libs\libplatform.a(cm.o)
 .text.cm_next_freepage
                0x000000001000661c       0x54 ..\..\..\..\Libraries\libs\libplatform.a(cm.o)
 .text.cm_movepage
                0x0000000010006670       0x5e ..\..\..\..\Libraries\libs\libplatform.a(cm.o)
 .text.cm_release
                0x00000000100066ce      0x112 ..\..\..\..\Libraries\libs\libplatform.a(cm.o)
 .text.cm_savepage
                0x00000000100067e0       0xc8 ..\..\..\..\Libraries\libs\libplatform.a(cm.o)
 .text.cm_check_loadpage
                0x00000000100068a8       0xb0 ..\..\..\..\Libraries\libs\libplatform.a(cm.o)
 .text.cm_sync  0x0000000010006958       0x3e ..\..\..\..\Libraries\libs\libplatform.a(cm.o)
                0x0000000010006958                cm_sync
 .text.cm_read  0x0000000010006996       0x44 ..\..\..\..\Libraries\libs\libplatform.a(cm.o)
                0x0000000010006996                cm_read
 .text.cm_write
                0x00000000100069da       0x5e ..\..\..\..\Libraries\libs\libplatform.a(cm.o)
                0x00000000100069da                cm_write
 .text.cm_init  0x0000000010006a38      0x1e8 ..\..\..\..\Libraries\libs\libplatform.a(cm.o)
                0x0000000010006a38                cm_init
 .text.xcfg_init
                0x0000000010006c20       0x66 ..\..\..\..\Libraries\libs\libplatform.a(xcfg.o)
                0x0000000010006c20                xcfg_init
 .text.usb_disable
                0x0000000010006c86       0x22 ..\..\..\..\Libraries\libs\libplatform.a(device.o)
                0x0000000010006c86                usb_disable
 .text.device.init
                0x0000000010006ca8       0xb2 ..\..\..\..\Libraries\libs\libplatform.a(device.o)
                0x0000000010006ca8                dev_init
                0x0000000010006d02                dev_delay_times
                0x0000000010006d14                dev_delay_online_times
                0x0000000010006d22                dev_delay_offline_times
                0x0000000010006d30                dev_clr_sta
 .text.platform_main
                0x0000000010006d5a      0x212 ..\..\..\..\Libraries\libs\libplatform.a(main.o)
                0x0000000010006d5a                platform_main
 .text.main_startup
                0x0000000010006f6c       0x3e ..\..\..\..\Libraries\libs\libplatform.a(main.o)
                0x0000000010006f6c                main_startup
 .text.sys_irq_init.part.0
                0x0000000010006faa       0x50 ..\..\..\..\Libraries\libs\libplatform.a(interrupt.o)
 .text.sys_irq_init
                0x0000000010006ffa       0x48 ..\..\..\..\Libraries\libs\libplatform.a(interrupt.o)
                0x0000000010006ffa                sys_irq_init
 .text.timer0_init
                0x0000000010007042       0x64 ..\..\..\..\Libraries\libs\libplatform.a(interrupt.o)
                0x0000000010007042                timer0_init
 .text.soft_irq_init
                0x00000000100070a6       0x3c ..\..\..\..\Libraries\libs\libplatform.a(interrupt.o)
                0x00000000100070a6                soft_irq_init
 .text.bthw_irq_init
                0x00000000100070e2       0x38 ..\..\..\..\Libraries\libs\libplatform.a(interrupt.o)
                0x00000000100070e2                bthw_irq_init
 .text.sd0_irq_init
                0x000000001000711a       0x32 ..\..\..\..\Libraries\libs\libplatform.a(interrupt.o)
                0x000000001000711a                sd0_irq_init
 .text.usb_irq_init
                0x000000001000714c       0x26 ..\..\..\..\Libraries\libs\libplatform.a(interrupt.o)
                0x000000001000714c                usb_irq_init
 .text.aubuf_irq_init
                0x0000000010007172       0x32 ..\..\..\..\Libraries\libs\libplatform.a(interrupt.o)
                0x0000000010007172                aubuf_irq_init
 .text.thread_main_entry
                0x00000000100071a4      0x17a ..\..\..\..\Libraries\libs\libplatform.a(startup.o)
 .text.bt_set_timer_enable
                0x000000001000731e        0xa ..\..\..\..\Libraries\libs\libplatform.a(startup.o)
                0x000000001000731e                bt_set_timer_enable
 .text.sys_set_tmr_enable
                0x0000000010007328        0xe ..\..\..\..\Libraries\libs\libplatform.a(startup.o)
                0x0000000010007328                sys_set_tmr_enable
 .text.thread_idle_create
                0x0000000010007336       0x30 ..\..\..\..\Libraries\libs\libplatform.a(startup.o)
                0x0000000010007336                thread_idle_create
 .text.startup.init
                0x0000000010007366      0x116 ..\..\..\..\Libraries\libs\libplatform.a(startup.o)
                0x0000000010007366                platform_init
                0x0000000010007368                sys_startup
 .text.sys_hook_init
                0x000000001000747c        0x2 ..\..\..\..\Libraries\libs\libplatform.a(sys_hook.o)
                0x000000001000747c                sys_hook_init
 .text.debug_set
                0x000000001000747e       0x1a ..\..\..\..\Libraries\libs\libplatform.a(debug.o)
                0x000000001000747e                debug_set
 .text.fot.update
                0x0000000010007498      0x88e ..\..\..\..\Libraries\libs\libplatform.a(fot_update.o)
                0x0000000010007694                get_keep_mac
                0x00000000100076d8                calc_mac
                0x0000000010007712                mac_init
                0x00000000100077e0                set_macbuf
                0x0000000010007834                clear_macbuf
                0x000000001000787c                fot_head_info_analize
                0x0000000010007890                fot_set_keep
                0x0000000010007908                fot_clear_keep
                0x0000000010007938                fot_down_first4k
                0x0000000010007c04                fot_tws_done_try
                0x0000000010007c06                fot_tws_done
                0x0000000010007c44                fot_tws_done_sync_err_deal
                0x0000000010007c6a                fot_head_info_save
                0x0000000010007c76                fot_breakpoint_info_read
                0x0000000010007cf8                fot_get_err
                0x0000000010007d02                is_fot_update_success
                0x0000000010007d12                fot_get_curaddr
 .text.fot.init
                0x0000000010007d26       0xa2 ..\..\..\..\Libraries\libs\libplatform.a(fot_update.o)
 .text.is_fot_tws_support
                0x0000000010007dc8        0x4 ..\..\..\..\Libraries\libs\libplatform.a(fot_update.o)
                0x0000000010007dc8                is_fot_tws_support
 .text.get_spiloader_offset
                0x0000000010007dcc        0xc ..\..\..\..\Libraries\libs\libplatform.a(fot_update.o)
                0x0000000010007dcc                get_spiloader_offset
 .text.fot_checksum_cal
                0x0000000010007dd8       0xde ..\..\..\..\Libraries\libs\libplatform.a(fot_update.o)
                0x0000000010007dd8                fot_checksum_cal
 .text.fot_down_first4k_checksum_cal
                0x0000000010007eb6       0x98 ..\..\..\..\Libraries\libs\libplatform.a(fot_update.o)
                0x0000000010007eb6                fot_down_first4k_checksum_cal
 .text.fot_init
                0x0000000010007f4e       0x2e ..\..\..\..\Libraries\libs\libplatform.a(fot_update.o)
                0x0000000010007f4e                fot_init
 .text.fot_set_base_offset
                0x0000000010007f7c       0x28 ..\..\..\..\Libraries\libs\libplatform.a(fot_update.o)
                0x0000000010007f7c                fot_set_base_offset
 .text.lock_init
                0x0000000010007fa4       0x10 ..\..\..\..\Libraries\libs\libplatform.a(lock.o)
                0x0000000010007fa4                lock_init
 .text.load_code_fota
                0x0000000010007fb4       0x42 ..\..\..\..\Libraries\libs\libplatform.a(lock.o)
                0x0000000010007fb4                load_code_fota
 .text.patch_init
                0x0000000010007ff6       0x1e ..\..\..\..\Libraries\libs\libplatform.a(patch.o)
                0x0000000010007ff6                patch_init
 .text.set_buck_mode
                0x0000000010008014       0x46 ..\..\..\..\Libraries\libs\libplatform.a(power.o)
                0x0000000010008014                set_buck_mode
 .text.vddio_voltage_configure
                0x000000001000805a       0x54 ..\..\..\..\Libraries\libs\libplatform.a(power.o)
                0x000000001000805a                vddio_voltage_configure
 .text.vddbt_voltage_configure
                0x00000000100080ae       0x4e ..\..\..\..\Libraries\libs\libplatform.a(power.o)
                0x00000000100080ae                vddbt_voltage_configure
 .text.pmu_voltage_configure
                0x00000000100080fc       0x64 ..\..\..\..\Libraries\libs\libplatform.a(power.o)
                0x00000000100080fc                pmu_voltage_configure
 .text.pmu_init
                0x0000000010008160      0x15e ..\..\..\..\Libraries\libs\libplatform.a(power.o)
                0x0000000010008160                pmu_init
 .text.udivmoddi4
                0x00000000100082be       0x96 ..\..\..\..\Libraries\libs\libplatform.a(sys.o)
 .text.sys_get_rc2m_clkhz
                0x0000000010008354      0x178 ..\..\..\..\Libraries\libs\libplatform.a(sys.o)
                0x0000000010008354                sys_get_rc2m_clkhz
 .text.sys_get_rand_key_init
                0x00000000100084cc       0x76 ..\..\..\..\Libraries\libs\libplatform.a(sys.o)
                0x00000000100084cc                sys_get_rand_key_init
 .text.sys_get_rand_key
                0x0000000010008542       0x5a ..\..\..\..\Libraries\libs\libplatform.a(sys.o)
                0x0000000010008542                sys_get_rand_key
 .text.bsp.param
                0x000000001000859c       0x66 ..\..\..\..\Libraries\libs\libplatform.a(sys.o)
                0x000000001000859c                param_bt_xosc_read
                0x00000000100085d0                bt_save_xosc_cap
 .text.xosc_init
                0x0000000010008602       0xa2 ..\..\..\..\Libraries\libs\libplatform.a(sys.o)
                0x0000000010008602                xosc_init
 .text.bt_restore_xosc_cap
                0x00000000100086a4        0x4 ..\..\..\..\Libraries\libs\libplatform.a(sys.o)
                0x00000000100086a4                bt_restore_xosc_cap
 .text.bt_get_xosc_cap
                0x00000000100086a8       0x18 ..\..\..\..\Libraries\libs\libplatform.a(sys.o)
                0x00000000100086a8                bt_get_xosc_cap
 .text.bt_set_xosc_cap
                0x00000000100086c0       0x26 ..\..\..\..\Libraries\libs\libplatform.a(sys.o)
                0x00000000100086c0                bt_set_xosc_cap
 .text.bt_adj_xosc_cap
                0x00000000100086e6       0x8a ..\..\..\..\Libraries\libs\libplatform.a(sys.o)
                0x00000000100086e6                bt_adj_xosc_cap
 .text.__udivdi3
                0x0000000010008770        0x6 ..\..\..\..\Libraries\libs\libplatform.a(sys.o)
                0x0000000010008770                __udivdi3
 .text.sys_clk_cacl_curr
                0x0000000010008776       0x24 ..\..\..\..\Libraries\libs\libplatform.a(sys_clk.o)
 *fill*         0x000000001000879a        0x2 
 .text.sys_clk  0x000000001000879c      0x1f8 ..\..\..\..\Libraries\libs\libplatform.a(sys_clk.o)
                0x000000001000879c                get_clksel_val
                0x00000000100087ae                get_cur_sysclk
                0x00000000100087b6                set_audec_clkdiv
                0x00000000100087d4                set_sbcec_clkdiv
                0x00000000100087d6                sysclk_update_baud
                0x000000001000880e                update_uart1baud_in_sysclk_set
                0x0000000010008832                sys_clk_set_do
 *fill*         0x0000000010008994       0x6c 
 .text.set_sys_clk_do
                0x0000000010008a00      0x1f0 ..\..\..\..\Libraries\libs\libplatform.a(sys_clk.o)
                0x0000000010008a00                set_sys_clk_do
 .text.set_peripherals_clkdiv
                0x0000000010008bf0      0x11c ..\..\..\..\Libraries\libs\libplatform.a(sys_clk.o)
                0x0000000010008bf0                set_peripherals_clkdiv
 .text.get_sysclk_nhz
                0x0000000010008d0c       0x7e ..\..\..\..\Libraries\libs\libplatform.a(sys_clk.o)
                0x0000000010008d0c                get_sysclk_nhz
 .text.set_sys_clk
                0x0000000010008d8a       0x34 ..\..\..\..\Libraries\libs\libplatform.a(sys_clk.o)
                0x0000000010008d8a                set_sys_clk
 *fill*         0x0000000010008dbe        0x2 
 .text.sys_clk.table
                0x0000000010008dc0        0xa ..\..\..\..\Libraries\libs\libplatform.a(sys_clk.o)
                0x0000000010008dc0                sysclk_sel_tbl
 .text.voltage.trim
                0x0000000010008dca      0x188 ..\..\..\..\Libraries\libs\libplatform.a(voltage_trim.o)
                0x0000000010008dca                bt_get_ft_trim_value
                0x0000000010008e00                dac_get_ft_trim_value
                0x0000000010008e1e                voltage_trim_value_init
 .text.stack.api
                0x0000000010008f52       0x2a ..\..\..\..\Libraries\libs\libplatform.a(bt.o)
                0x0000000010008f52                bt_send_msg_do
 .text          0x0000000010008f7c       0x70 ..\..\..\..\Libraries\libs\libbtstack.a(nanos.o)
                0x0000000010008f7c                nanos_init
                0x0000000010008fb0                nanos_var_init
 .text          0x0000000010008fec       0x68 ..\..\..\..\Libraries\libs\libbtstack.a(patch.o)
                0x0000000010008fec                bb_patch_init
 .text          0x0000000010009054        0x2 ..\..\..\..\Libraries\libs\libbtstack.a(platform.o)
                0x0000000010009054                timer_sync_init
 .text          0x0000000010009056       0x1c ..\..\..\..\Libraries\libs\libbtstack.a(bt_sco.o)
                0x0000000010009056                lc_sco_pkt_init
                0x0000000010009058                lc_sco_codec_init
                0x000000001000905c                lc_sco_codec_exit
                0x0000000010009060                lc_sco_codec_setup
                0x0000000010009070                lc_sco_codec_kill
 *fill*         0x0000000010009072      0x18e 
 .text          0x0000000010009200     0x216e ..\..\..\..\Libraries\libs\libbtstack.a(bt_acl.o)
                0x00000000100093d2                bt_acl_init
                0x000000001000940e                bt_acl_reset
                0x0000000010009478                bt_acl_start
                0x000000001000971e                bt_acl_init_param
                0x0000000010009800                bt_acl_stop
                0x00000000100098c0                bt_acl_flow_off
                0x0000000010009900                bt_acl_flow_on
                0x0000000010009980                bt_acl_flush_to_get
                0x00000000100099c0                bt_acl_flush_to_set
                0x0000000010009a00                bt_acl_poll_int_get
                0x0000000010009a40                bt_acl_poll_int_set
                0x0000000010009b00                bt_acl_sniff_trans
                0x0000000010009c00                bt_acl_sniff
                0x0000000010009d00                bt_acl_unsniff
                0x0000000010009db2                bt_acl_tx_enc
                0x0000000010009dd4                bt_acl_rx_enc
                0x0000000010009dfa                bt_acl_bcst_rx_enc
                0x0000000010009e24                bt_acl_enc_key_set
                0x0000000010009f00                bt_acl_master_clock_get
                0x0000000010009f80                bt_acl_clock_offset_get
                0x000000001000a000                bt_acl_rsw_slot_offset_get
                0x000000001000a080                bt_acl_rsw_slot_offset_set
                0x000000001000a100                bt_acl_sup_to_get
                0x000000001000a140                bt_acl_sup_to_set
                0x000000001000a180                bt_acl_tim_acc_set
                0x000000001000a200                bt_acl_edr_set
                0x000000001000a300                bt_acl_tx_pkt_types_set
                0x000000001000a400                bt_acl_dm1_pkt_type_dis
                0x000000001000a480                bt_acl_curr_txpwr_get
                0x000000001000a600                bt_acl_afh_set
                0x000000001000a800                bt_acl_afh_new
                0x000000001000a900                bt_acl_afh_cfm
                0x000000001000a980                bt_acl_rx_max_slot_get
                0x000000001000a9c0                bt_acl_rx_max_slot_set
                0x000000001000aa00                bt_acl_test_mode_set
                0x000000001000aac0                bt_acl_rssi_thr_get
                0x000000001000aaf0                bt_sco_start
                0x000000001000af00                bt_sco_stop
                0x000000001000af80                bt_acl_sniff_clock_set
                0x000000001000b000                bt_acl_sniff_clock_diff
                0x000000001000b100                bt_acl_resche
 *fill*         0x000000001000b36e       0x92 
 .text          0x000000001000b400      0xca6 ..\..\..\..\Libraries\libs\libbtstack.a(ble_con.o)
                0x000000001000b400                ble_con_evt_time_update_fix
                0x000000001000b500                ble_con_start_do
                0x000000001000b528                ble_con_start
                0x000000001000ba00                ble_con_stop
                0x000000001000ba80                ble_con_param_update
                0x000000001000bb00                ble_con_phys_update
                0x000000001000bb80                ble_con_tx_len_update_for_intv
                0x000000001000bc00                ble_con_tx_len_update_for_rate
                0x000000001000bc80                ble_con_event_counter_get
                0x000000001000bcb0                ble_con_tx_enc
                0x000000001000bcfc                ble_con_rx_enc
                0x000000001000bd48                ble_con_enc_key_load
                0x000000001000be00                ble_con_current_tx_power_get
                0x000000001000be80                ble_con_rssi_get
                0x000000001000beb0                ble_con_offset_get
                0x000000001000beec                ble_con_pref_slave_latency_set
                0x000000001000bf2c                ble_con_pref_slave_evt_dur_set
                0x000000001000bf80                ble_con_peer_sca_set
                0x000000001000bfaa                ble_con_duration_min_set
 *fill*         0x000000001000c0a6       0x5a 
 .text.bb.ble.con.flow
                0x000000001000c100       0xfa ..\..\..\..\Libraries\libs\libbtstack.a(ble_con.o)
                0x000000001000c100                ble_con_data_flow_set
 *fill*         0x000000001000c1fa        0x6 
 .text.bb.ble.con.data_len
                0x000000001000c200       0xfa ..\..\..\..\Libraries\libs\libbtstack.a(ble_con.o)
                0x000000001000c200                ble_con_data_len_update
 .text.le.con   0x000000001000c2fa       0x8c ..\..\..\..\Libraries\libs\libbtstack.a(ble_con.o)
                0x000000001000c2fa                ble_get_con_var
                0x000000001000c304                ble_con_init
 *fill*         0x000000001000c386        0x2 
 .text          0x000000001000c388      0x5d2 ..\..\..\..\Libraries\libs\libbtstack.a(bb_utils.o)
                0x000000001000c3d4                bb_bytes_to_string
                0x000000001000c412                bb_nb_good_channels
                0x000000001000c446                bb_util_pack
                0x000000001000c6c8                bb_util_unpack
 .text          0x000000001000c95a      0x1ba ..\..\..\..\Libraries\libs\libbtstack.a(bb_int.o)
                0x000000001000c95a                bb_time_set
                0x000000001000c978                bb_sleep_init
                0x000000001000c9d0                bb_driver_init
 *fill*         0x000000001000cb14       0xec 
 .text.bb.aes   0x000000001000cc00      0x1f6 ..\..\..\..\Libraries\libs\libbtstack.a(bb_int.o)
                0x000000001000cc00                bb_aes_encrypt
 .text          0x000000001000cdf6      0x2b6 ..\..\..\..\Libraries\libs\libbtstack.a(bb.o)
                0x000000001000cdf6                bb_rand_init
                0x000000001000ce00                bb_get_heap_info
                0x000000001000ce14                bb_var_init
                0x000000001000ce1c                bb_reset
                0x000000001000ceac                bb_init
                0x000000001000d02e                bb_off
                0x000000001000d080                bb_run_loop
 .text          0x000000001000d0ac       0x1a ..\..\..\..\Libraries\libs\libbtstack.a(platform.o)
                0x000000001000d0ac                lm_inq_start_do
                0x000000001000d0b0                lm_inq_stop_do
                0x000000001000d0b4                lm_inq_res_ind_do
                0x000000001000d0b6                bt_pf_init
                0x000000001000d0b8                bt_pf_exit
                0x000000001000d0ba                bt_pf_post
                0x000000001000d0bc                bt_pf_get_info
                0x000000001000d0be                bt_is_ota_enable
 .text          0x000000001000d0c6       0x50 ..\..\..\..\Libraries\libs\libbtstack.a(extern_tws.o)
                0x000000001000d0c6                bt_tws_get_force_role
                0x000000001000d0ca                tws_get_spp_eq_info
                0x000000001000d0ce                tws_set_spp_eq_info
                0x000000001000d0d0                bt_get_right_ear_sta
                0x000000001000d0d4                bt_get_left_ear_sta
                0x000000001000d0d8                bt_change_nr_sta
                0x000000001000d0dc                bt_get_loc_nr_sta
                0x000000001000d0e0                bt_get_auto_anwer_sta
                0x000000001000d0e4                bt_set_menu_ctrl_sta
                0x000000001000d0e6                tws_get_new_bt_name
                0x000000001000d0ea                bt_get_serial_number
                0x000000001000d0ee                bt_get_ch_serial_number
                0x000000001000d0f2                bt_inear_test
                0x000000001000d10e                bt_get_model_number
                0x000000001000d112                bt_get_fw_version
 .text          0x000000001000d116       0x9a ..\..\..\..\Libraries\libs\libbtstack.a(extern_bt.o)
                0x000000001000d116                bt_rf_get_inq_param
                0x000000001000d11a                bt_rf_get_param
                0x000000001000d11e                bt_rf_get_sco_param
                0x000000001000d122                bt_rf_get_fcc_param
                0x000000001000d13a                bt_get_new_local_name
                0x000000001000d13e                bt_set_new_local_name
                0x000000001000d14e                bt_is_always_reconn
                0x000000001000d152                bt_get_conn_fail_delay
                0x000000001000d158                bt_get_connect_addr
                0x000000001000d170                bt_emit_notice
                0x000000001000d180                tws_set_fot_data
                0x000000001000d184                tws_get_fot_data
                0x000000001000d188                tws_get_dueros_dma_data
                0x000000001000d18c                tws_set_dueros_dma_data
                0x000000001000d190                tws_send_dueros_dma_data_cfm
                0x000000001000d192                tws_set_switch_fix_acl
                0x000000001000d196                is_bt_nor_linkkey_prohibit_del
                0x000000001000d19a                bt_voice_callback
                0x000000001000d19c                spp_custom1_rx_callback
                0x000000001000d19e                spp_custom2_rx_callback
                0x000000001000d1a2                spp_client_cfg_callback
                0x000000001000d1a8                spp_custom1_connect_callback
                0x000000001000d1aa                spp_custom1_disconnect_callback
                0x000000001000d1ac                spp_custom2_connect_callback
                0x000000001000d1ae                spp_custom2_disconnect_callback
 .text          0x000000001000d1b0      0x398 ..\..\..\..\Libraries\libs\libbtstack.a(spp.o)
                0x000000001000d214                spp_disconnect
                0x000000001000d2cc                spp_service_flush
                0x000000001000d2d8                get_spp_connection_context_for_rfcomm_cid
                0x000000001000d308                get_spp_connection_context_for_bd_addr
                0x000000001000d3e4                provide_spp_connection_context_for_bd_addr
                0x000000001000d44c                spp_establish_service_level_connection
                0x000000001000d4c6                spp_release_service_level_connection
                0x000000001000d510                spp_init
                0x000000001000d530                spp_init_var
                0x000000001000d540                spp_support_mul_server
 .text.stack.spp.handler
                0x000000001000d548      0x23c ..\..\..\..\Libraries\libs\libbtstack.a(spp.o)
                0x000000001000d548                spp_packet_handler
 .text.stack.sdp.util
                0x000000001000d784      0x60e ..\..\..\..\Libraries\libs\libbtstack.a(sdp_util.o)
                0x000000001000d836                de_get_size_type
                0x000000001000d83e                de_get_element_type
                0x000000001000d846                de_get_header_size
                0x000000001000d864                de_get_data_size
                0x000000001000d8a8                de_get_len
                0x000000001000d980                de_element_get_uint16
                0x000000001000d9ac                de_get_normalized_uuid
                0x000000001000da06                de_get_uuid32
                0x000000001000da2e                de_store_descriptor_with_len
                0x000000001000da6c                des_iterator_init
                0x000000001000da9c                des_iterator_get_type
                0x000000001000daac                des_iterator_get_size
                0x000000001000dad4                des_iterator_has_more
                0x000000001000dae2                des_iterator_get_element
                0x000000001000daf8                des_iterator_next
                0x000000001000db16                sdp_attribute_list_constains_id
                0x000000001000dc42                sdp_filter_attributes_in_attributeIDList
                0x000000001000dc7a                spd_get_filtered_size
                0x000000001000dc9c                sdp_get_attribute_value_for_attribute_id
                0x000000001000dcbc                sdp_set_attribute_value_for_attribute_id
                0x000000001000dce2                sdp_record_contains_UUID128
                0x000000001000dd40                sdp_traversal_match_pattern
                0x000000001000dd6c                sdp_record_matches_service_search_pattern
                0x000000001000dd90                de_dump_data_element
 .text          0x000000001000dd92       0x42 ..\..\..\..\Libraries\libs\libbtstack.a(sdp_server.o)
                0x000000001000ddca                remove_sdp_server_context
 .text.stack.sdp.server
                0x000000001000ddd4      0x750 ..\..\..\..\Libraries\libs\libbtstack.a(sdp_server.o)
                0x000000001000de22                sdp_get_service_record_handle
                0x000000001000de56                sdp_get_record_for_handle
                0x000000001000de64                sdp_create_service_record_handle
                0x000000001000de84                sdp_handle_service_search_request
                0x000000001000e024                sdp_handle_service_attribute_request
                0x000000001000e1a0                sdp_handle_service_search_attribute_request
 .text.stack.setup
                0x000000001000e524       0x3a ..\..\..\..\Libraries\libs\libbtstack.a(sdp_server.o)
                0x000000001000e524                sdp_init
 .text.stack.sdp.server_add
                0x000000001000e55e       0x46 ..\..\..\..\Libraries\libs\libbtstack.a(sdp_server.o)
                0x000000001000e55e                sdp_add_service
 *fill*         0x000000001000e5a4        0x0 
 .text          0x000000001000e5a4      0x79c ..\..\..\..\Libraries\libs\libbtstack.a(sdp_client.o)
                0x000000001000e5a4                remove_sdp_client_context
                0x000000001000e5ae                de_state_init
                0x000000001000e5be                de_state_size
                0x000000001000e61c                sdp_parser_init
                0x000000001000e642                sdp_parser_handle_chunk
                0x000000001000e886                sdp_parser_handle_done
                0x000000001000e8e2                sdp_client_packet_handler
                0x000000001000ec26                sdp_client_init
                0x000000001000ec42                sdp_client_free
                0x000000001000ec56                sdp_client_query
 .text          0x000000001000ed40     0x195a ..\..\..\..\Libraries\libs\libbtstack.a(rfcomm.o)
                0x000000001000f308                rfcomm_multiplexer_finalize
                0x000000001000f3a2                rfcomm_set_required_security_level
                0x000000001000f3aa                rfcomm_can_send_packet_now
                0x000000001000f3bc                rfcomm_request_can_send_now_event
                0x000000001000f3d8                rfcomm_reserve_packet_buffer
                0x000000001000f3dc                rfcomm_release_packet_buffer
                0x000000001000f3e0                rfcomm_get_outgoing_buffer
                0x000000001000f3ee                rfcomm_get_max_frame_size
                0x000000001000f402                rfcomm_create_channel_with_initial_credits
                0x000000001000f40a                rfcomm_create_channel
                0x000000001000f412                rfcomm_disconnect
                0x000000001000f442                rfcomm_register_service_with_initial_credits
                0x000000001000f44a                rfcomm_unregister_service
                0x000000001000f480                rfcomm_accept_connection
                0x000000001000f4d0                crc8_calc
                0x000000001000f506                rfcomm_send_prepared
                0x000000001000f5c2                rfcomm_send
                0x00000000100105c6                provide_rfcomm_multiplexer
                0x00000000100105e2                provide_rfcomm_channel
                0x000000001001063a                rfcomm_set_packet_handler_for_channels
                0x000000001001064e                rfcomm_get_now_incoming_credit
                0x0000000010010664                rfcomm_set_to_send_new_incoming_credit
 .text.stack.rfcomm
                0x000000001001069a       0x90 ..\..\..\..\Libraries\libs\libbtstack.a(rfcomm.o)
                0x0000000010010724                rfcomm_register_service
 .text.stack.setup
                0x000000001001072a       0x22 ..\..\..\..\Libraries\libs\libbtstack.a(rfcomm.o)
                0x000000001001072a                rfcomm_init
 .text.stack.link_key
                0x000000001001074c      0x60c ..\..\..\..\Libraries\libs\libbtstack.a(btstack_link_key_db.o)
                0x00000000100108be                btstack_get_link_addr
                0x0000000010010972                btstack_get_link_key
                0x0000000010010a06                btstack_get_link_feature
                0x0000000010010a3a                btstack_delete_link_key
                0x0000000010010ad4                btstack_delete_all_link_key
                0x0000000010010b42                btstack_put_link_key
                0x0000000010010c40                btstack_put_link_offset
                0x0000000010010c8c                btstack_delete_all_link_offset
                0x0000000010010cf8                btstack_put_link_feature
 .text.stack.setup
                0x0000000010010d58      0x184 ..\..\..\..\Libraries\libs\libbtstack.a(btstack_link_key_db.o)
                0x0000000010010d58                btstack_open_link_info
 .text.stack.link_key.get.name
                0x0000000010010edc       0x62 ..\..\..\..\Libraries\libs\libbtstack.a(btstack_link_key_db.o)
                0x0000000010010edc                btstack_get_link_name
 .text.stack.link_key.put.name
                0x0000000010010f3e       0x94 ..\..\..\..\Libraries\libs\libbtstack.a(btstack_link_key_db.o)
                0x0000000010010f3e                btstack_put_link_name
 .text          0x0000000010010fd2       0xac ..\..\..\..\Libraries\libs\libbtstack.a(btstack_util.o)
                0x0000000010010fd2                log_info_hexdump
                0x0000000010010fd4                log_info_key
                0x0000000010010fd6                uuid_add_bluetooth_prefix
                0x0000000010010ff8                uuid_has_bluetooth_prefix
                0x0000000010011014                sscanf_bd_addr
 .text.stack.util
                0x000000001001107e      0x126 ..\..\..\..\Libraries\libs\libbtstack.a(btstack_util.o)
                0x000000001001107e                bd_addr_cmp
                0x0000000010011084                bd_addr_copy
                0x000000001001108a                big_endian_read_16
                0x000000001001109a                big_endian_read_32
                0x00000000100110ba                big_endian_store_16
                0x00000000100110ce                big_endian_store_32
                0x0000000010011102                reverse_bytes
                0x000000001001111e                reverse_24
                0x0000000010011122                reverse_48
                0x0000000010011126                reverse_56
                0x000000001001112a                reverse_64
                0x000000001001112e                reverse_128
                0x0000000010011132                reverse_256
                0x0000000010011138                reverse_bd_addr
                0x000000001001113a                btstack_min
                0x0000000010011140                btstack_max
                0x0000000010011146                char_for_nibble
                0x000000001001116c                nibble_for_char
 .text.stack.hci_dump
                0x00000000100111a4       0x52 ..\..\..\..\Libraries\libs\libbtstack.a(btstack_util.o)
                0x00000000100111a4                bd_addr_to_str
 .text          0x00000000100111f6       0x7c ..\..\..\..\Libraries\libs\libbtstack.a(btstack_txpkt.o)
                0x00000000100111f6                txpkt_init
 *fill*         0x0000000010011272        0xe 
 .text.stk.txpkt.flush
                0x0000000010011280       0x82 ..\..\..\..\Libraries\libs\libbtstack.a(btstack_txpkt.o)
                0x0000000010011280                txpkt_flush
 *fill*         0x0000000010011302       0x7e 
 .text.stack.run_loop
                0x0000000010011380      0x174 ..\..\..\..\Libraries\libs\libbtstack.a(btstack_run_loop.o)
                0x0000000010011380                btstack_run_loop_set_timer_handler
                0x0000000010011384                btstack_run_loop_set_data_source_handler
                0x0000000010011388                btstack_run_loop_set_data_source_fd
                0x000000001001138c                btstack_run_loop_get_data_source_fd
                0x0000000010011390                btstack_run_loop_enable_data_source_callbacks
                0x000000001001139c                btstack_run_loop_disable_data_source_callbacks
                0x00000000100113ac                btstack_run_loop_add_data_source
                0x00000000100113b8                btstack_run_loop_remove_data_source
                0x00000000100113c4                btstack_run_loop_set_timer
                0x00000000100113e0                btstack_run_loop_set_timer_context
                0x00000000100113e4                btstack_run_loop_get_timer_context
                0x0000000010011400                btstack_run_loop_set_trig_ticks
                0x000000001001143c                btstack_run_loop_add_timer
                0x000000001001146c                btstack_run_loop_remove_timer
                0x000000001001149a                btstack_run_loop_get_ticks
                0x00000000100114a6                btstack_run_loop_ticks_for_ms
                0x00000000100114ac                btstack_run_loop_get_time_ms
                0x00000000100114ba                btstack_run_loop_timer_dump
 .text.stack.setup
                0x00000000100114f4       0x34 ..\..\..\..\Libraries\libs\libbtstack.a(btstack_run_loop.o)
                0x00000000100114f4                btstack_run_loop_init
 .text.stack.memory
                0x0000000010011528       0x9a ..\..\..\..\Libraries\libs\libbtstack.a(btstack_memory.o)
                0x0000000010011528                btstack_memory_l2cap_service_get
                0x0000000010011532                btstack_memory_l2cap_service_free
                0x000000001001153e                btstack_memory_l2cap_channel_get
                0x0000000010011548                btstack_memory_l2cap_channel_free
                0x0000000010011554                btstack_memory_rfcomm_multiplexer_get
                0x000000001001155e                btstack_memory_rfcomm_multiplexer_free
                0x000000001001156a                btstack_memory_rfcomm_service_get
                0x0000000010011574                btstack_memory_rfcomm_service_free
                0x0000000010011580                btstack_memory_rfcomm_channel_get
                0x000000001001158a                btstack_memory_rfcomm_channel_free
                0x0000000010011596                btstack_memory_whitelist_entry_get
                0x00000000100115a0                btstack_memory_whitelist_entry_free
                0x00000000100115ac                btstack_memory_sm_lookup_entry_get
                0x00000000100115b6                btstack_memory_sm_lookup_entry_free
 .text.stack.setup
                0x00000000100115c2       0xa6 ..\..\..\..\Libraries\libs\libbtstack.a(btstack_memory.o)
                0x00000000100115c2                btstack_memory_init
 .text.stack.linked_list
                0x0000000010011668       0x6c ..\..\..\..\Libraries\libs\libbtstack.a(btstack_linked_list.o)
                0x0000000010011668                btstack_linked_list_get_last_item
                0x0000000010011676                btstack_linked_list_add
                0x000000001001168a                btstack_linked_list_add_tail
                0x000000001001169e                btstack_linked_list_remove
                0x00000000100116b6                btstack_linked_list_count
                0x00000000100116c4                btstack_linked_list_iterator_remove
 .text          0x00000000100116d4      0x270 ..\..\..\..\Libraries\libs\libbtstack.a(btstack_link_ctrl.o)
                0x00000000100116d4                alloc_link_ctrl_context_for_bd_addr
                0x0000000010011758                btstack_link_ctrl_stop_timer
                0x0000000010011774                btstack_link_ctrl_set_timer
                0x00000000100117aa                link_ctrl_timer_handler
                0x0000000010011836                btstack_link_ctrl_get_num
                0x0000000010011854                btstack_link_ctrl_get_recon_sta
                0x000000001001187e                btstack_link_ctrl_get_links
                0x0000000010011892                btstack_link_ctrl_is_exist
                0x00000000100118ca                btstack_link_ctrl_abort_reconnect
 .text.stack.linkctrl
                0x0000000010011944      0x17a ..\..\..\..\Libraries\libs\libbtstack.a(btstack_link_ctrl.o)
                0x0000000010011944                chk_link_ctrl_context_use_up
                0x000000001001195e                get_link_ctrl_context_for_bd_addr
                0x00000000100119a8                provide_link_ctrl_context_for_bd_addr
                0x00000000100119c0                remove_link_ctrl_context
                0x0000000010011a2a                remove_pending_link_ctrl_context
                0x0000000010011a6c                remove_waiting_link_ctrl_context_for_bd_addr
 .text.stack.setup
                0x0000000010011abe       0x16 ..\..\..\..\Libraries\libs\libbtstack.a(btstack_link_ctrl.o)
                0x0000000010011abe                btstack_link_ctrl_init
 .text          0x0000000010011ad4      0x1cc ..\..\..\..\Libraries\libs\libbtstack.a(gatt_server.o)
                0x0000000010011af8                ble_init_att_do
                0x0000000010011b3a                ble_init_att_for_handle
                0x0000000010011b78                ble_register_att_buf_for_handle
                0x0000000010011bc2                ble_tx_notify
                0x0000000010011c1c                ble_tx_indication
                0x0000000010011c1e                ble_update_conn_param
                0x0000000010011c40                ble_set_adv_interval
                0x0000000010011c6c                btstack_ble_disconnect
                0x0000000010011c78                btstack_ble_set_adv_data
                0x0000000010011c8c                btstack_ble_set_scan_rsp_data
 .text.att.r_cb
                0x0000000010011ca0       0xb6 ..\..\..\..\Libraries\libs\libbtstack.a(gatt_server.o)
                0x0000000010011ca0                att_read_callback
 .text.att.w_cb
                0x0000000010011d56      0x1c8 ..\..\..\..\Libraries\libs\libbtstack.a(gatt_server.o)
                0x0000000010011d56                att_write_callback
 .text.ble.att  0x0000000010011f1e       0x76 ..\..\..\..\Libraries\libs\libbtstack.a(gatt_server.o)
                0x0000000010011f1e                btstack_gatt_init
                0x0000000010011f88                btstack_ble_send_req
 .text.ble.hci  0x0000000010011f94       0x6a ..\..\..\..\Libraries\libs\libbtstack.a(gatt_server.o)
                0x0000000010011f94                btstack_ble_update_conn_param
                0x0000000010011fd2                btstack_ble_set_adv_interval
 .text          0x0000000010011ffe      0x5b4 ..\..\..\..\Libraries\libs\libbtstack.a(gatt_profile.o)
                0x0000000010011ffe                ble_gatts_service_add
                0x00000000100120bc                ble_gatts_characteristic_add
                0x00000000100122ac                ble_gatts_add_server_characteristic_descriptor
                0x0000000010012500                ble_gatts_init
                0x000000001001252c                ble_att_write_callback
                0x000000001001256a                ble_att_read_callback
                0x00000000100125a8                ble_get_profile_data
 .text          0x00000000100125b2      0x726 ..\..\..\..\Libraries\libs\libbtstack.a(att_server.o)
                0x00000000100127de                ble_get_max_mtu
                0x00000000100127e4                att_server_register_service_handler
                0x000000001001280c                att_server_init
                0x000000001001288a                att_server_register_packet_handler
                0x0000000010012892                att_server_can_send_packet_now
                0x00000000100128a4                att_server_request_can_send_now_event
                0x0000000010012c08                att_server_notify
                0x0000000010012c54                att_server_indicate
 .text          0x0000000010012cd8       0xe6 ..\..\..\..\Libraries\libs\libbtstack.a(att_dispatch.o)
                0x0000000010012d72                att_dispatch_register_client
                0x0000000010012d86                att_dispatch_register_server
                0x0000000010012d9a                att_dispatch_client_can_send_now
                0x0000000010012da0                att_dispatch_server_can_send_now
                0x0000000010012da2                att_dispatch_client_request_can_send_now_event
                0x0000000010012db0                att_dispatch_server_request_can_send_now_event
 *fill*         0x0000000010012dbe        0x2 
 .text          0x0000000010012dc0      0xf8c ..\..\..\..\Libraries\libs\libbtstack.a(att_db.o)
                0x0000000010012fba                att_uuid_for_handle
                0x0000000010012fe4                att_set_db
                0x0000000010012fec                att_set_read_callback
                0x0000000010012ff4                att_set_write_callback
                0x0000000010012ffc                att_dump_attributes
                0x0000000010013040                att_clear_transaction_queue
                0x000000001001305c                att_prepare_handle_value_notification
                0x000000001001309a                att_prepare_handle_value_indication
                0x00000000100130d8                att_handle_request
                0x0000000010013b12                gatt_server_get_get_handle_range_for_service_with_uuid16
                0x0000000010013b98                gatt_server_get_value_handle_for_characteristic_with_uuid16
                0x0000000010013bda                gatt_server_get_client_configuration_handle_for_characteristic_with_uuid16
                0x0000000010013c66                gatt_server_get_value_handle_for_characteristic_with_uuid128
                0x0000000010013cb4                gatt_server_get_client_configuration_handle_for_characteristic_with_uuid128
 .text          0x0000000010013d4c       0x8c ..\..\..\..\Libraries\libs\libbtstack.a(btstack_main.o)
                0x0000000010013dce                btstack_test_func
                0x0000000010013dd0                btstack_ble_set_init_callback
 .text.stack.handler
                0x0000000010013dd8      0x1b6 ..\..\..\..\Libraries\libs\libbtstack.a(btstack_main.o)
 .text.stack.ble.setup
                0x0000000010013f8e       0x1c ..\..\..\..\Libraries\libs\libbtstack.a(btstack_main.o)
                0x0000000010013f8e                btstack_ble_init
 .text.stack.setup
                0x0000000010013faa       0x8c ..\..\..\..\Libraries\libs\libbtstack.a(btstack_main.o)
                0x0000000010013faa                btstack_main
 .text          0x0000000010014036       0x18 ..\..\..\..\Libraries\libs\libbtstack.a(btstack_hal.o)
                0x0000000010014036                hal_tick_init
                0x000000001001403c                hal_tick_set_handler
 .text          0x000000001001404e      0x760 ..\..\..\..\Libraries\libs\libbtstack.a(btstack_api.o)
                0x000000001001404e                dma_start_speech_to_ai
                0x0000000010014050                btstack_ctl0_api
                0x0000000010014060                btstack_comm_api
                0x000000001001407a                btstack_hid_api
                0x0000000010014094                btstack_fcc_test_func
                0x0000000010014098                btstack_spp_api
                0x00000000100140a4                btstack_audio_bypass
                0x00000000100140f6                btstack_audio_enable
                0x0000000010014134                btstack_ctl_api
                0x00000000100141c0                btstack_tws_api
                0x00000000100141c2                btstack_a2dp_msg
                0x00000000100141c4                dma_stop_speech_to_ai
                0x00000000100141c6                btstack_reset_bt_name
                0x00000000100141c8                btstack_tws_switch_role
                0x00000000100141ca                btstack_tws_connect
                0x00000000100141cc                btstack_low_latency_en
                0x00000000100141ce                btstack_low_latency_dis
                0x00000000100141d0                btstack_ble_conn_by_addr
                0x00000000100141d2                btstack_ble_enable_scan
                0x00000000100141d4                btstack_ble_set_scan_param
                0x00000000100141d6                btstack_nor_connect
                0x00000000100141d8                btstack_ble_set_adv_param
                0x00000000100141da                btstack_ble_disable_scan
                0x00000000100141dc                bt_decode_init
                0x00000000100141de                btstack_var_init
                0x000000001001420e                btstack_establish_service_connection_do
                0x000000001001422e                btstack_establish_service_connection
                0x0000000010014236                btstack_continue_establish_service_connection
                0x000000001001425e                btstack_tws_search_slave
                0x0000000010014260                btstack_emit_notice_status
                0x0000000010014298                btstack_connect_address
                0x0000000010014328                btstack_emit_notice
                0x000000001001433c                btstack_tws_disc_continue
                0x000000001001433e                bt_emit_player_notice
                0x000000001001438c                btstack_tws_set_status
                0x000000001001438e                btstack_clr_dis_flag
                0x00000000100143a6                btstack_get_ext_feature
                0x00000000100143d0                btstack_set_hfp_status_ptr
                0x0000000010014402                btstack_set_hsp_status_ptr
                0x0000000010014418                btstack_clr_hfp_status_ptr
                0x000000001001445e                btstack_clr_hsp_status_ptr
                0x000000001001447a                bt_get_siri_status
                0x000000001001447e                btstack_get_tws_key
                0x00000000100144aa                btstack_get_tws_msg
                0x00000000100144d8                btstack_get_tws_hid_key
                0x00000000100144fe                btstack_get_tws_hid_msg
                0x000000001001453c                bt_tws_is_playing
                0x0000000010014552                bt_tws_is_calling
                0x0000000010014556                btstack_clr_l2cap_status
                0x000000001001461a                btstack_sco_setup
                0x0000000010014668                btstack_sco_kill
                0x00000000100146d0                btstack_msg_is_busy
                0x00000000100146e4                btstack_msg_set_busy
                0x00000000100146fa                btstack_audio_is_busy
                0x000000001001470e                btstack_audio_set_busy
                0x000000001001471c                audio_bypass_get_cnt
                0x000000001001472c                btstack_set_lmp_test
                0x0000000010014744                btstack_set_clk_offset
                0x000000001001475c                tws_remote_is_busy
                0x0000000010014760                btstack_tws_is_nego_ring
                0x0000000010014764                btstack_tws_is_connected_for_handle
                0x0000000010014768                btstack_tws_user_key
                0x000000001001476a                btstack_sync_info
                0x000000001001476c                btstack_tws_set_ring
                0x000000001001476e                btstack_tws_remote_switch_role
                0x0000000010014770                btstack_get_connect_delay
 .text.stack.api
                0x00000000100147ae      0x5c8 ..\..\..\..\Libraries\libs\libbtstack.a(btstack_api.o)
                0x00000000100147ae                btstack_tws_disconnect
                0x00000000100147ce                btstack_nor_disconnect
                0x00000000100147d0                btstack_dma_stat_change
                0x00000000100147d2                btstack_off
                0x0000000010014800                btstack_start_work
                0x0000000010014818                btstack_set_scan
                0x0000000010014840                btstack_set_scan_param
                0x0000000010014856                btstack_hid_connect
                0x0000000010014886                btstack_spp_disconnect
                0x00000000100148c2                btstack_hid_disconnect
                0x00000000100148fe                btstack_fot_resp
                0x0000000010014900                bt_init
                0x0000000010014918                btstack_tws_set_scan
                0x000000001001491a                btstack_connect_for_bd_addr_do
                0x00000000100149b0                btstack_tws_disconnect_do
                0x00000000100149b2                btstack_connect_for_bd_addr
                0x00000000100149d2                btstack_connect
                0x0000000010014a2a                btstack_disconnect_do
                0x0000000010014aa4                btstack_disconnect
                0x0000000010014acc                bt_hid_is_ready_to_discon
                0x0000000010014b0c                btstack_set_l2cap_status
                0x0000000010014c70                bt_get_call_indicate
                0x0000000010014cec                bt_is_playing
                0x0000000010014d0a                bt_is_ios_device
                0x0000000010014d0e                bt_is_support_vol_ctrl
                0x0000000010014d12                bt_is_connected
                0x0000000010014d2a                dma_get_change_key
                0x0000000010014d2e                dma_get_change_value
                0x0000000010014d32                btstack_message
 .text.stack.sleep
                0x0000000010014d76       0x32 ..\..\..\..\Libraries\libs\libbtstack.a(btstack_api.o)
                0x0000000010014d76                btstack_enter_sleep
                0x0000000010014d8e                btstack_exit_sleep
 .text.stack.setup
                0x0000000010014da8       0xc4 ..\..\..\..\Libraries\libs\libbtstack.a(btstack_api.o)
                0x0000000010014da8                btstack_setup
 *fill*         0x0000000010014e6c      0x194 
 .text.stack.status
                0x0000000010015000      0x1ec ..\..\..\..\Libraries\libs\libbtstack.a(btstack_api.o)
                0x0000000010015000                bt_get_status_do
 .text          0x00000000100151ec      0x158 ..\..\..\..\Libraries\libs\libbtstack.a(bt_api.o)
                0x000000001001520c                bt_wait_disconnect
                0x0000000010015250                bt_sync_info
                0x000000001001525e                bt_start_work
                0x000000001001526c                bt_updata_local_name
                0x0000000010015276                bt_nor_connect
                0x0000000010015278                bt_nor_disconnect
                0x000000001001527a                bt_tws_get_scan
                0x000000001001527e                bt_tws_set_scan
                0x0000000010015280                bt_tws_get_link_info
                0x0000000010015284                bt_tws_delete_link_info
                0x0000000010015286                bt_tws_user_key
                0x000000001001528a                bt_tws_switch
                0x000000001001528c                bt_sync_init
                0x000000001001528e                bt_tws_get_first_role
                0x0000000010015292                bt_tws_is_en
                0x0000000010015296                bt_nor_delete_link_info
                0x000000001001529c                bt_nor_get_link_info_addr
                0x00000000100152cc                bt_nor_get_link_info
                0x00000000100152d0                bt_get_link_btname
                0x0000000010015328                bt_is_low_latency
                0x0000000010015336                bt_connect_address
                0x0000000010015340                bt_map_start
                0x0000000010015342                bt_map_abort
 .text          0x0000000010015344       0x9e ..\..\..\..\Libraries\libs\libbtstack.a(ble_api.o)
                0x0000000010015344                ble_disconnect
                0x000000001001534e                ble_set_adv_data
                0x0000000010015386                ble_set_scan_rsp_data
                0x00000000100153be                ble_enable_adv
                0x00000000100153c4                ble_disable_adv
                0x00000000100153ca                ble_set_scan_param
                0x00000000100153ce                ble_scan_en
                0x00000000100153d0                ble_scan_dis
                0x00000000100153d2                ble_adv0_set_ctrl
                0x00000000100153da                ble_connect_by_addr
                0x00000000100153de                ble_init_callback_register
 .text          0x00000000100153e2       0x44 ..\..\..\..\Libraries\libs\libbtstack.a(bb_sche.o)
                0x00000000100153e2                bb_sche_frag_ble_dur_set
                0x00000000100153f4                bb_sche_init
 .text          0x0000000010015426       0x68 ..\..\..\..\Libraries\libs\libbtstack.a(bb_dbg.o)
                0x0000000010015426                my_spi_init
                0x000000001001548c                bb_dbg_init
 .text          0x000000001001548e       0xf6 ..\..\..\..\Libraries\libs\libbtstack.a(bb_clk.o)
                0x000000001001548e                bb_clk_init
                0x0000000010015582                bb_clk_off
 .text.bb.aes   0x0000000010015584      0x2a6 ..\..\..\..\Libraries\libs\libbtstack.a(aes.o)
                0x0000000010015584                aes_init
                0x00000000100155ce                aes_alloc
                0x00000000100155f0                aes_start
                0x000000001001562e                aes_encrypt
                0x000000001001567a                aes_rand
                0x00000000100156b6                aes_result_handler
                0x000000001001571e                aes_xor_128
                0x0000000010015740                aes_shift_left_128
                0x000000001001576a                ble_ecpy
 .text          0x000000001001582a      0x102 ..\..\..\..\Libraries\libs\libbtstack.a(vs_proc.o)
                0x000000001001591c                bt_fcc_test_ctrl
 .text          0x000000001001592c       0xd4 ..\..\..\..\Libraries\libs\libbtstack.a(vs_fcc.o)
                0x000000001001597e                vs_con_start
                0x00000000100159aa                vs_con_end
                0x00000000100159c6                vs_fcc_3m_packet_filter
 .text.bb.vs.fcc
                0x0000000010015a00      0x1b8 ..\..\..\..\Libraries\libs\libbtstack.a(vs_fcc.o)
                0x0000000010015a04                vs_fcc_test_cmd_do
 .text          0x0000000010015bb8       0x9e ..\..\..\..\Libraries\libs\libbtstack.a(vs.o)
                0x0000000010015bb8                vs_init
                0x0000000010015bf6                vs_reset_complete_evt
 .text          0x0000000010015c56      0xb48 ..\..\..\..\Libraries\libs\libbtstack.a(rf_smart.o)
                0x0000000010015e30                rfphy_pll_afc
                0x0000000010015e8c                rfphy_pll_idle
                0x0000000010015ea2                rfphy_rx_dcoc
                0x0000000010015eb6                rfphy_rx_rccal
                0x0000000010015f40                rfphy_t2r
                0x0000000010015fd4                rfphy_tx_dcoc
                0x0000000010016030                rfphy_rx
                0x00000000100160da                rfphy_tx
                0x0000000010016170                rfphy_tx_tone
                0x00000000100161b4                rfphy_sw_ctrl
                0x00000000100161e2                rfphy_test
                0x00000000100161e4                rfphy_txrx_init
                0x000000001001622c                rfphy_init
 .text.bb.rf    0x000000001001679e       0x48 ..\..\..\..\Libraries\libs\libbtstack.a(rf_smart.o)
                0x000000001001679e                rfphy_tx_pwr
 .text          0x00000000100167e6      0x3f6 ..\..\..\..\Libraries\libs\libbtstack.a(rf.o)
                0x00000000100167e6                rf_txpwr_dec
                0x0000000010016822                rf_txpwr_inc
                0x000000001001685e                rf_txpwr_max
                0x0000000010016884                rf_txpwr_epc_inc
                0x00000000100168c4                rf_txpwr_epc_dec
                0x0000000010016906                rf_off
                0x0000000010016916                rf_reset
                0x0000000010016918                rf_init
 *fill*         0x0000000010016bdc       0x24 
 .text          0x0000000010016c00       0x82 ..\..\..\..\Libraries\libs\libbtstack.a(bt_hook.o)
                0x0000000010016c00                bt_scan_update_param
                0x0000000010016c58                bt_inq_scan_hook
 .text          0x0000000010016c82       0x1c ..\..\..\..\Libraries\libs\libbtstack.a(ble_hook.o)
                0x0000000010016c82                ble_hal_init_hook
 *fill*         0x0000000010016c9e      0x162 
 .text          0x0000000010016e00      0xdcc ..\..\..\..\Libraries\libs\libbtstack.a(hct_tl.o)
                0x0000000010017200                hct_flush_acl_rx_pend
                0x0000000010017400                hci_tx_done_do
                0x00000000100174f4                hci_tx_done
                0x0000000010017600                hci_tl_send
                0x0000000010017754                hci_tl_init
                0x0000000010017792                hci_cmd_get_max_param_size
                0x00000000100177aa                hci_cmd_received
                0x00000000100179fe                hci_acl_tx_data_alloc
                0x0000000010017af4                hci_acl_tx_data_received
 .text          0x0000000010017bcc      0x6da ..\..\..\..\Libraries\libs\libbtstack.a(hct_msg.o)
                0x0000000010018182                hci_check_desc_tabs_order
                0x0000000010018184                hci_look_for_cmd_desc
                0x0000000010018206                hci_look_for_evt_desc
                0x000000001001824a                hci_look_for_dbg_evt_desc
                0x0000000010018264                hci_look_for_le_evt_desc
 .text          0x00000000100182a6       0xb8 ..\..\..\..\Libraries\libs\libbtstack.a(hct_fc.o)
                0x00000000100182a6                hci_fc_init
                0x00000000100182b6                hci_fc_acl_buf_size_set
                0x00000000100182cc                hci_fc_acl_en
                0x0000000010018312                hci_fc_host_nb_acl_pkts_complete
                0x0000000010018334                hci_fc_check_host_available_nb_acl_packets
 .text          0x000000001001835e      0x710 ..\..\..\..\Libraries\libs\libbtstack.a(hct.o)
                0x00000000100183d0                hci_send_2_host
                0x000000001001878e                hci_ble_conhdl_register
                0x00000000100187a0                hci_ble_conhdl_unregister
                0x00000000100187b0                hci_bt_acl_bdaddr_register
                0x00000000100187da                hci_bt_acl_conhdl_register
                0x00000000100187f2                hci_bt_acl_bdaddr_unregister
                0x0000000010018808                hci_evt_mask_set
                0x0000000010018846                hct_init
                0x0000000010018890                hci_evt_filter_add
                0x0000000010018a58                hci_voice_settings_get
                0x0000000010018a62                hci_voice_settings_set
 .text          0x0000000010018a6e      0x81a ..\..\..\..\Libraries\libs\libbtstack.a(lm.o)
                0x0000000010018ac2                lm_init
                0x0000000010018c54                lm_set_scan_int
                0x0000000010018c68                lm_new_link_alloc
                0x0000000010018c82                lm_stop_link_alloc
                0x0000000010018ca8                lm_lt_addr_alloc
                0x0000000010018ce0                lm_lt_addr_free
                0x0000000010018d0c                lm_get_nb_acl
                0x0000000010018d70                lm_role_switch_start
                0x0000000010018dba                lm_role_switch_finished
                0x0000000010018e42                lm_get_features
                0x0000000010018ec4                lm_pscan_start
                0x0000000010018f14                lm_pscan_restart
                0x0000000010018f24                lm_acl_disc
                0x0000000010018f58                lm_get_auth_en
                0x0000000010018f68                lm_get_sp_en
                0x0000000010018f78                lm_get_sec_con_host_supp
                0x0000000010018f86                lm_get_pin_type
                0x0000000010018f90                lm_get_con_accept_timeout
                0x0000000010018f9a                lm_set_loc_name
                0x0000000010019004                lm_get_loc_name
                0x000000001001900e                lm_get_loc_name_seg
                0x0000000010019068                lm_get_loopback_mode
                0x0000000010019072                lm_get_pub_key_192
                0x0000000010019094                lm_get_priv_key_192
                0x00000000100190b4                lm_get_oob_local_commit
                0x00000000100190de                lm_get_sp_debug_mode
                0x00000000100190e8                lm_debug_key_compare_192
                0x000000001001911a                lm_get_dut_mode_en
                0x0000000010019124                lm_afh_get_ch_ass_en
                0x000000001001912e                lm_afh_get_host_ch_class
                0x0000000010019138                lm_afh_set_peer_ch_class
                0x0000000010019152                lm_afh_get_master_ch_map
                0x000000001001915c                lm_afh_init_timer
                0x0000000010019188                lm_is_acl_con
                0x00000000100191a4                lm_is_acl_con_role
                0x00000000100191ce                lm_page_scan_rep_mode_get
                0x00000000100191d8                lm_sco_move_en
                0x00000000100191e2                lm_extract_max_enc_key_size
                0x00000000100191fc                lm_create_master_key
                0x0000000010019248                lm_create_master_key_rand
                0x0000000010019254                lm_get_master_key
                0x0000000010019262                lm_get_master_key_rand
                0x0000000010019270                lm_get_master_enc_rand
                0x000000001001927e                lm_get_master_enc_key_size
 .text          0x0000000010019288      0x382 ..\..\..\..\Libraries\libs\libbtstack.a(bt_hal.o)
                0x0000000010019288                bt_hal_init
                0x000000001001940a                bt_hal_reset
                0x000000001001958e                bt_bd_addr_get
                0x000000001001959c                bt_bd_addr_set
                0x00000000100195c8                bt_class_of_dev_get
                0x00000000100195d6                bt_class_of_dev_set
                0x00000000100195e6                bt_tim_acc_get
                0x0000000010019600                bt_afh_ch_assess_get
 .text          0x000000001001960a      0x14e ..\..\..\..\Libraries\libs\libbtstack.a(bt21.o)
                0x000000001001960a                bt_buf_init
                0x00000000100196f4                bt21_init
                0x000000001001972e                bt21_reset
 .text          0x0000000010019758       0x62 ..\..\..\..\Libraries\libs\libbtstack.a(bc.o)
                0x0000000010019758                bc_init
                0x000000001001977a                bc_reset
                0x00000000100197aa                bc_get_nb_broadcast
                0x00000000100197b2                bc_set_nb_broadcast
 *fill*         0x00000000100197ba        0x6 
 .text          0x00000000100197c0      0x430 ..\..\..\..\Libraries\libs\libbtstack.a(ble_hal.o)
                0x00000000100197e6                ble_ral_search
                0x0000000010019838                ble_hal_init
                0x0000000010019aa4                ble_ch_assess_data_get
                0x0000000010019aae                ble_rpa_renew
                0x0000000010019b2c                ble_aa_gen
 *fill*         0x0000000010019bf0       0x10 
 .text          0x0000000010019c00      0xb76 ..\..\..\..\Libraries\libs\libbtstack.a(ble_adv.o)
                0x0000000010019c00                ble_get_adv_var
                0x0000000010019c0a                ble_adv_init
                0x0000000010019d00                ble_adv_stop
                0x0000000010019d80                ble_adv_adv_data_update
                0x0000000010019e00                ble_adv_scan_rsp_data_update
                0x0000000010019f00                ble_adv_start_do
                0x0000000010019fac                ble_adv_start
                0x000000001001a680                ble_adv_rand_addr_update
                0x000000001001a700                ble_adv_restart
 .text          0x000000001001a776       0x48 ..\..\..\..\Libraries\libs\libbtstack.a(ble.o)
                0x000000001001a776                ble_init
 .text.ble.var.init
                0x000000001001a7be       0x38 ..\..\..\..\Libraries\libs\libbtstack.a(ble.o)
                0x000000001001a7be                ble_var_init
 .text          0x000000001001a7f6       0x4c ..\..\..\..\Libraries\libs\libbtstack.a(extern_ble.o)
                0x000000001001a810                ble_get_aap_addr
                0x000000001001a81c                ble_client_cfg_callback
                0x000000001001a81e                ble_adv0_get_adv_data_cb
                0x000000001001a822                ble_adv0_get_tws_role
                0x000000001001a836                ble_adv0_get_tws_loc_var
                0x000000001001a83a                ble_adv0_set_tws_rem_var
                0x000000001001a840                ble_tx_test
 .text.bb.ble.adv0
                0x000000001001a842       0x28 ..\..\..\..\Libraries\libs\libbtstack.a(extern_ble.o)
                0x000000001001a842                ble_adv0_get_addr_cb
 .text          0x000000001001a86a      0x30c ..\..\..\..\Libraries\libs\libbtstack.a(l2cap_test.o)
                0x000000001001a964                l2cap_end_of_test
                0x000000001001a97a                l2cap_test_support_ext_feature
                0x000000001001a996                l2cap_test_cmd
                0x000000001001aa9e                l2cap_test_rsp
                0x000000001001aaa0                l2cap_vd_acl_init
                0x000000001001aac2                l2cap_vd_enter_updateota
                0x000000001001aad0                l2cap_vd_exit_updateota
                0x000000001001aadc                l2cap_vd_acl_tx_request
 .text          0x000000001001ab76      0x34e ..\..\..\..\Libraries\libs\libbtstack.a(l2cap.o)
                0x000000001001abc6                l2cap_register_packet_handler
                0x000000001001abce                l2cap_send_test_cmd
                0x000000001001ac20                l2cap_send_test_key
                0x000000001001ac4e                gap_request_connection_parameter_update
                0x000000001001ac86                l2cap_get_outgoing_buffer
                0x000000001001ac94                l2cap_reserve_packet_buffer
                0x000000001001ac98                l2cap_release_packet_buffer
                0x000000001001ac9c                l2cap_send_prepared_connectionless
                0x000000001001acee                l2cap_send_connectionless
                0x000000001001ad24                l2cap_send_echo_request
                0x000000001001ad30                l2cap_max_mtu
                0x000000001001ad36                l2cap_max_le_mtu
                0x000000001001ad3c                l2cap_create_channel
                0x000000001001ae1c                l2cap_disconnect
                0x000000001001ae38                provide_l2cap_channel
                0x000000001001ae9a                l2cap_unregister_service
 *fill*         0x000000001001aec4        0x0 
 .text.stack.handler.l2cap
                0x000000001001aec4      0x94c ..\..\..\..\Libraries\libs\libbtstack.a(l2cap.o)
                0x000000001001b160                l2cap_emit_channel_closed
                0x000000001001b7ae                l2cap_can_send_packet_now
                0x000000001001b7cc                l2cap_can_send_prepared_packet_now
                0x000000001001b7ea                l2cap_can_send_fixed_channel_packet_now
                0x000000001001b7ee                l2cap_get_remote_mtu_for_local_cid
                0x000000001001b808                l2cap_stop_rtx
 .text.stack.l2cap
                0x000000001001b810      0x860 ..\..\..\..\Libraries\libs\libbtstack.a(l2cap.o)
                0x000000001001b828                l2cap_clear_pending_tx
                0x000000001001bf38                l2cap_send_prepared
                0x000000001001bfa0                l2cap_send
                0x000000001001bff2                l2cap_accept_connection
                0x000000001001c00c                l2cap_decline_connection
                0x000000001001c02c                l2cap_register_service
 .text.stack.setup
                0x000000001001c070       0x72 ..\..\..\..\Libraries\libs\libbtstack.a(l2cap.o)
                0x000000001001c070                l2cap_init
                0x000000001001c0c0                l2cap_register_fixed_channel
 .text.stack.setup
                0x000000001001c0e2        0x2 ..\..\..\..\Libraries\libs\libbtstack.a(hci_dump.o)
                0x000000001001c0e2                hci_dump_open
 .text.stack.hci_send
                0x000000001001c0e4      0x26c ..\..\..\..\Libraries\libs\libbtstack.a(hci_cmd.o)
                0x000000001001c0e4                hci_cmd_create_from_template
 .text          0x000000001001c350      0x562 ..\..\..\..\Libraries\libs\libbtstack.a(hci.o)
                0x000000001001c4fc                hci_alloc_num_packets_sent
                0x000000001001c53c                hci_shutdown_connection
                0x000000001001c578                gap_advertisements_get_address
                0x000000001001c5a4                hci_free_connect_waiting
                0x000000001001c602                gap_local_bd_addr
                0x000000001001c612                hci_emit_start_action
                0x000000001001c648                hci_emit_service_establish
                0x000000001001c676                gap_get_connection_type
                0x000000001001c6ac                hci_set_sco_voice_setting_for_addr
                0x000000001001c6c4                hci_get_sco_voice_setting_for_addr
                0x000000001001c72e                gap_advertisements_set_data
                0x000000001001c74a                gap_scan_response_set_data
                0x000000001001c766                hci_le_advertisements_set_params
                0x000000001001c7aa                gap_advertisements_enable
                0x000000001001c7e0                gap_inquiry
                0x000000001001c7f6                gap_inquiry_cancel
                0x000000001001c80c                gap_disconnect
                0x000000001001c85e                hci_set_sco_voice_setting
                0x000000001001c86a                hci_setup_sync
                0x000000001001c8ae                hci_rx_flush
 .text.stack.hci
                0x000000001001c8b2      0x934 ..\..\..\..\Libraries\libs\libbtstack.a(hci.o)
                0x000000001001c9a2                hci_authentication_active_for_handle
                0x000000001001c9c2                gap_drop_link_key_for_bd_addr
                0x000000001001c9e4                gap_store_link_key_for_bd_addr
                0x000000001001ca08                gap_get_link_feature_for_bd_addr
                0x000000001001ca26                gap_store_link_feature_for_bd_addr
                0x000000001001ca44                gap_get_link_addr_by_order
                0x000000001001ca48                hci_number_free_acl_slots_for_handle
                0x000000001001ca62                hci_can_send_acl_classic_packet_now
                0x000000001001ca78                hci_can_send_acl_le_packet_now
                0x000000001001ca8a                hci_can_send_prepared_acl_packet_now
                0x000000001001caaa                hci_can_send_acl_packet_now
                0x000000001001cabc                hci_is_packet_buffer_reserved
                0x000000001001cac8                hci_reserve_packet_buffer
                0x000000001001cae0                hci_release_packet_buffer
                0x000000001001cbb0                hci_send_acl_packet_buffer
                0x000000001001cc00                hci_usable_acl_packet_types
                0x000000001001cc0c                hci_get_outgoing_packet_buffer
                0x000000001001cc16                hci_max_acl_data_packet_length
                0x000000001001cc22                hci_non_flushable_packet_boundary_flag_supported
                0x000000001001cc32                hci_disconnect_security_block
                0x000000001001cc4c                gap_ssp_set_enable
                0x000000001001cc58                update_extend_inquiry_response
                0x000000001001cc80                hci_run_le_connection
                0x000000001001cd64                hci_remote_esco_supported
                0x000000001001cd7e                gap_ssp_supported_on_both_sides
                0x000000001001cdb0                hci_local_had_auth_request
                0x000000001001cdda                gap_security_level_for_link_key_type
                0x000000001001ce0c                hci_run_pend_connection
                0x000000001001d0a4                gap_mitm_protection_required_for_security_level
                0x000000001001d0ae                gap_security_level
                0x000000001001d0c6                hci_run_w2_connection
                0x000000001001d186                gap_w_scan_control
                0x000000001001d1a0                gap_request_security_level
 *fill*         0x000000001001d1e6        0x2 
 .text.stack.hci_init
                0x000000001001d1e8      0x3c6 ..\..\..\..\Libraries\libs\libbtstack.a(hci.o)
                0x000000001001d220                gap_set_local_name
                0x000000001001d57c                hci_power_control
 .text.stack.handler.acl
                0x000000001001d5ae       0x16 ..\..\..\..\Libraries\libs\libbtstack.a(hci.o)
 .text.stack.setup
                0x000000001001d5c4      0x166 ..\..\..\..\Libraries\libs\libbtstack.a(hci.o)
                0x000000001001d614                hci_add_event_handler
                0x000000001001d622                hci_register_acl_packet_handler
                0x000000001001d62c                hci_init
                0x000000001001d6c8                hci_set_chipset
                0x000000001001d6dc                gap_set_class_of_device
                0x000000001001d6e6                hci_set_bd_addr
                0x000000001001d706                gap_ssp_set_io_capability
                0x000000001001d712                gap_ssp_set_authentication_requirement
                0x000000001001d71e                gap_ssp_set_auto_accept
 .text.stack.hci_emit
                0x000000001001d72a      0x148 ..\..\..\..\Libraries\libs\libbtstack.a(hci.o)
                0x000000001001d7d8                hci_emit_state
                0x000000001001d806                hci_emit_scan_ctrl
                0x000000001001d82c                hci_emit_inquiry_ctrl
                0x000000001001d852                hci_emit_test_active
 .text.stack.hci.conn
                0x000000001001d872      0x1e2 ..\..\..\..\Libraries\libs\libbtstack.a(hci.o)
                0x000000001001d872                create_connection_for_bd_addr_and_type
                0x000000001001d97c                gap_get_connection_parameter_range
                0x000000001001d98c                gap_set_connection_parameter_range
                0x000000001001d99e                hci_get_connections
                0x000000001001d9a8                hci_connection_for_bd_addr_and_type
                0x000000001001d9e6                hci_connection_get_other_for_bd_addr_and_type
                0x000000001001da24                hci_connection_for_index
 .text.ble.hci  0x000000001001da54      0x132 ..\..\..\..\Libraries\libs\libbtstack.a(hci.o)
                0x000000001001da54                ble_event_cmd_complete
                0x000000001001daf2                ble_event_meta
 .text.stack.hci_send
                0x000000001001db86      0x2bc ..\..\..\..\Libraries\libs\libbtstack.a(hci.o)
                0x000000001001db86                hci_send_cmd_packet
                0x000000001001dd46                hci_send_cmd
                0x000000001001dd9c                hci_send_create_connection_cmd
 *fill*         0x000000001001de42      0x1be 
 .text.stack.hci.run
                0x000000001001e000      0x1c8 ..\..\..\..\Libraries\libs\libbtstack.a(hci.o)
 .text.stack.hci_rx
                0x000000001001e1c8      0x106 ..\..\..\..\Libraries\libs\libbtstack.a(hci.o)
                0x000000001001e1c8                acl_handler
 *fill*         0x000000001001e2ce        0x2 
 .text.stack.handler.event
                0x000000001001e2d0      0xd3c ..\..\..\..\Libraries\libs\libbtstack.a(hci.o)
 .text          0x000000001001f00c      0x1d4 ..\..\..\..\Libraries\libs\libbtstack.a(hid_usage.o)
                0x000000001001f00c                hid_report_init
                0x000000001001f01e                hid_report_set
                0x000000001001f03e                hid_send_report_callback
                0x000000001001f08c                btstack_hid_send
                0x000000001001f0b2                btstack_hid_key
                0x000000001001f10c                btstack_hid_consumer
                0x000000001001f140                btstack_hid_touch_screen
                0x000000001001f1ce                bt_hid_is_send_complete
 .text          0x000000001001f1e0      0x55e ..\..\..\..\Libraries\libs\libbtstack.a(hid_device.o)
                0x000000001001f5fe                bt_hid_is_connected
                0x000000001001f626                hid_device_init
                0x000000001001f666                hid_device_request_can_send_now_event
                0x000000001001f66a                hid_device_send_interrupt_message
                0x000000001001f66e                hid_device_send_contro_message
                0x000000001001f672                hid_establish_service_level_connection
                0x000000001001f6e8                hid_release_service_level_connection
                0x000000001001f70e                bt_hid_index_set
                0x000000001001f710                hid_get_interrupt_cid
 *fill*         0x000000001001f73e        0x2 
 .text          0x000000001001f740      0xbd8 ..\..\..\..\Libraries\libs\libbtstack.a(hfp_hf.o)
                0x0000000010020168                hfp_hf_packet_handler
                0x00000000100201da                hfp_hf_init_codecs
                0x0000000010020204                hfp_hf_init_supported_features
                0x000000001002020c                hfp_hf_init_hf_indicators
                0x000000001002020e                hfp_hf_establish_service_level_connection
                0x0000000010020218                hfp_hf_release_service_level_connection
                0x0000000010020232                hfp_hf_get_siri_status
                0x0000000010020266                hfp_hf_set_call_switch_flag
                0x000000001002027a                hfp_hf_call_switch_for_index
                0x00000000100202d8                hfp_hf_call_for_index
                0x0000000010020316                hfp_hf_init
 .text.stack.api
                0x0000000010020318      0x316 ..\..\..\..\Libraries\libs\libbtstack.a(hfp_hf.o)
                0x0000000010020318                hfp_hf_switch_siri
                0x0000000010020350                hfp_hf_is_calling
                0x000000001002036c                hfp_hf_answer_incoming_call
                0x00000000100203e2                hfp_hf_terminate_call
                0x0000000010020436                hfp_hf_reject_incoming_call
                0x0000000010020438                hfp_hf_swap_calls
                0x0000000010020468                hfp_hf_dial_number
                0x00000000100204a6                hfp_hf_at_cmd
                0x00000000100204dc                hfp_hf_custom_at_cmd
                0x000000001002050a                hfp_hf_redial_last_number_do
                0x000000001002054a                hfp_hf_redial_last_number
                0x000000001002055e                hfp_hf_set_speaker_gain
                0x0000000010020598                hfp_hf_set_microphone_gain
                0x00000000100205d2                hfp_hf_report_bat_state
                0x0000000010020610                hfp_hf_start_codec
 .text.stack.hfp.api1
                0x000000001002062e       0x28 ..\..\..\..\Libraries\libs\libbtstack.a(hfp_hf.o)
                0x000000001002062e                hfp_is_connect
 *fill*         0x0000000010020656        0x2 
 .text          0x0000000010020658      0xbcc ..\..\..\..\Libraries\libs\libbtstack.a(hfp.o)
                0x0000000010020658                hfp_init
                0x000000001002066a                hfp_var_init
                0x000000001002066c                send_str_over_rfcomm
                0x0000000010020694                join
                0x0000000010020708                join_bitmap
                0x0000000010020786                hfp_emit_call_indicate
                0x0000000010020788                hfp_get_connections
                0x0000000010020792                hfp_get_connection_for_index
                0x0000000010020796                get_hfp_connection_context_for_rfcomm_cid
                0x000000001002079a                get_hfp_connection_context_for_bd_addr
                0x000000001002079e                get_hfp_connection_context_for_sco_handle
                0x00000000100207a2                hfp_reset_context_flags
                0x00000000100207ca                hfp_reset_voice_recognition_flags
                0x00000000100207e4                provide_hfp_connection_context_for_bd_addr
                0x00000000100207fc                hfp_handle_hci_event
                0x00000000100208b0                hfp_parse
                0x0000000010021114                hfp_establish_service_level_connection
                0x0000000010021156                hfp_rfcomm_service_supported
                0x000000001002115a                hfp_release_audio_connection
                0x0000000010021172                hfp_release_service_level_connection
                0x00000000100211cc                hfp_setup_synchronous_connection
                0x0000000010021222                hfp_set_packet_handler_for_rfcomm_connections
 .text          0x0000000010021224        0x8 ..\..\..\..\Libraries\libs\libbtstack.a(a2dp.o)
                0x0000000010021224                a2dp_is_playing
                0x0000000010021228                a2dp_is_playing_fast
 .text.stack.memory
                0x000000001002122c       0x46 ..\..\..\..\Libraries\libs\libbtstack.a(btstack_memory_pool.o)
                0x000000001002122c                btstack_memory_pool_get
                0x0000000010021238                btstack_memory_pool_free
                0x000000001002124c                btstack_memory_pool_create
 .text          0x0000000010021272       0x92 ..\..\..\..\Libraries\libs\libbtstack.a(btstack_adv0.o)
                0x0000000010021272                btstack_adv0_ctrl
                0x00000000100212d6                ble_adv0_set_intv
                0x00000000100212f2                ble_adv0_get_adv_en
                0x0000000010021302                ble_adv0_idx_update
 .text          0x0000000010021304     0x245e ..\..\..\..\Libraries\libs\libbtstack.a(sm.o)
                0x000000001002314a                sm_address_resolution_lookup
                0x00000000100231cc                sm_cmac_ready
                0x00000000100231da                sm_cmac_general_start
                0x0000000010023240                sm_cmac_signed_write_start
                0x0000000010023272                get_rand_addr
                0x0000000010023280                sm_register_oob_data_callback
                0x0000000010023288                sm_add_event_handler
                0x0000000010023296                sm_set_accepted_stk_generation_methods
                0x00000000100232a0                sm_set_encryption_key_size_range
                0x00000000100232b2                sm_set_authentication_requirements
                0x00000000100232ba                sm_set_io_capabilities
                0x00000000100232c2                sm_set_request_security
                0x00000000100232cc                sm_set_er
                0x00000000100232dc                sm_set_ir
                0x00000000100232ec                sm_test_set_irk
                0x000000001002330c                sm_test_use_fixed_local_csrk
                0x0000000010023318                sm_init
                0x00000000100233fa                sm_use_fixed_ec_keypair
                0x00000000100233fc                sm_test_use_fixed_ec_keypair
                0x00000000100233fe                sm_encryption_key_size
                0x000000001002341e                sm_authenticated
                0x000000001002343e                sm_authorization_state
                0x0000000010023462                sm_send_security_request
                0x0000000010023486                sm_request_pairing
                0x000000001002350a                sm_authorization_decline
                0x0000000010023554                sm_authorization_grant
                0x00000000100235a0                sm_bonding_decline
                0x00000000100235fa                sm_just_works_confirm
                0x0000000010023632                sm_numeric_comparison_confirm
                0x0000000010023634                sm_passkey_input
                0x0000000010023672                sm_keypress_notification
                0x0000000010023694                sm_le_device_index
                0x00000000100236a8                gap_random_address_set_mode
                0x00000000100236e4                gap_random_address_get_mode
                0x00000000100236ec                gap_random_address_set_update_period
                0x0000000010023712                gap_random_address_set
                0x000000001002374e                gap_advertisements_set_params
 .text          0x0000000010023762      0x3bc ..\..\..\..\Libraries\libs\libbtstack.a(le_device_db_memory.o)
                0x0000000010023762                le_device_db_init
                0x000000001002377c                le_device_db_set_local_bd_addr
                0x000000001002377e                le_device_db_count
                0x00000000100237aa                le_device_db_remove
                0x00000000100237c4                le_device_db_add
                0x000000001002383a                le_device_db_info
                0x000000001002389a                le_device_db_encryption_set
                0x0000000010023904                le_device_db_encryption_get
                0x00000000100239c8                le_device_db_remote_csrk_get
                0x00000000100239f2                le_device_db_remote_csrk_set
                0x0000000010023a18                le_device_db_local_csrk_get
                0x0000000010023a42                le_device_db_local_csrk_set
                0x0000000010023a68                le_device_db_remote_counter_get
                0x0000000010023a7e                le_device_db_remote_counter_set
                0x0000000010023a94                le_device_db_local_counter_get
                0x0000000010023aaa                le_device_db_local_counter_set
                0x0000000010023ac0                le_device_db_dump
 .text          0x0000000010023b1e       0x7c ..\..\..\..\Libraries\libs\libbtstack.a(hci_transport_hcic.o)
                0x0000000010023b1e                hcic_recv_packet
                0x0000000010023b3a                hcic_send_acl_segment
                0x0000000010023b6e                hcic_rx_flush
                0x0000000010023b8c                hci_init_var
 .text.stack.hcic
                0x0000000010023b9a      0x128 ..\..\..\..\Libraries\libs\libbtstack.a(hci_transport_hcic.o)
                0x0000000010023b9c                hcic_register_packet_handler
                0x0000000010023c04                hcic_close
                0x0000000010023c1a                hcic_open
                0x0000000010023c5c                hcic_send_packet
 .text          0x0000000010023cc2       0x24 ..\..\..\..\Libraries\libs\libbtstack.a(btstack_chipset_inner.o)
                0x0000000010023cdc                btstack_chipset_inner_instance
 .text          0x0000000010023ce6       0x1e ..\..\..\..\Libraries\libs\libbtstack.a(lm_hook.o)
                0x0000000010023ce6                lm_init_hook
                0x0000000010023d00                lm_set_iac_en
                0x0000000010023d02                lm_page_scan_end_hook
 .text          0x0000000010023d04     0x1d9a ..\..\..\..\Libraries\libs\libbtstack.a(lm_sp.o)
                0x000000001002441c                lm_n_is_zero
                0x0000000010024846                lm_sp_sha256_calculate
                0x00000000100248ce                lm_sp_n_one
                0x0000000010024a8a                lm_sp_n192_convert_wnaf
                0x0000000010024b2e                lm_sp_p192_point_to_inf
                0x0000000010024b42                lm_sp_p192_point_jacobian_to_affine
                0x0000000010024bb8                lm_sp_p192_points_jacobian_to_affine
                0x0000000010024cc8                lm_sp_p192_dbl
                0x0000000010024e40                lm_sp_p192_add
                0x00000000100250d8                lm_sp_pre_compute_points
                0x0000000010025120                lm_sp_p192_invert
                0x0000000010025166                lm_f1
                0x00000000100252d8                lm_f2
                0x0000000010025456                lm_oob_f1
                0x00000000100255c8                lm_g
                0x000000001002568a                lm_f3
                0x0000000010025834                lm_generate_rand_16bytes
                0x0000000010025892                lm_dhkey_calc_init
                0x00000000100259ca                lm_dhkey_compare
 .text          0x0000000010025a9e     0x1cca ..\..\..\..\Libraries\libs\libbtstack.a(lm_proc.o)
                0x0000000010027724                lm_inq_start
                0x000000001002773e                lm_inq_stop
 .text          0x0000000010027768      0xd3c ..\..\..\..\Libraries\libs\libbtstack.a(lm_key.o)
                0x0000000010027bba                lm_e1
                0x0000000010027c16                lm_e21
                0x0000000010027c52                lm_e22
                0x0000000010027cd2                lm_e3
                0x0000000010027d30                lm_kc_key
                0x0000000010028480                lm_xor_key
                0x0000000010028484                lm_get_rand_vec
 *fill*         0x00000000100284a4        0x0 
 .text          0x00000000100284a4     0x2e60 ..\..\..\..\Libraries\libs\libbtstack.a(lc.o)
                0x0000000010028516                lc_util_set_loc_trans_coll
                0x0000000010028532                lc_cmd_stat_send
                0x000000001002855a                lc_mode_chg_evt_send
                0x0000000010028596                lc_init
                0x00000000100285dc                lc_reset
                0x000000001002862c                lc_afh_set
                0x00000000100286fa                lc_chg_pkt_type_cmp
                0x0000000010028760                lc_chg_pkt_type_cont
                0x00000000100287ce                lc_afh_start
                0x0000000010028838                lc_con_cmp_evt_send
                0x00000000100288a0                lc_max_slot_mgt
                0x0000000010028952                lc_mst_qos_done
                0x00000000100289c6                lc_ptt
                0x0000000010028a6c                lc_ptt_cmp
                0x0000000010028ad2                lc_resp_auth
                0x0000000010028b8c                lc_release
                0x0000000010028bac                lc_restore_to
                0x0000000010028bf8                lc_start_lmp_to
                0x0000000010028c62                lc_start
                0x0000000010028e86                lc_comb_key_svr
                0x0000000010028f88                lc_locepr_rsw
                0x0000000010028fdc                lc_locepr_lkref
                0x0000000010029034                lc_enc_key_refresh
                0x0000000010029116                lc_initiator_epr
                0x0000000010029160                lc_init_calc_f3
                0x00000000100291e2                lc_dhkey
                0x0000000010029228                lc_init_start_mutual_auth
                0x0000000010029276                lc_mst_send_mst_key
                0x0000000010029366                lc_init_passkey_loop
                0x00000000100293d4                lc_pairing_cont
                0x0000000010029506                lc_legacy_pair
                0x000000001002956a                lc_passkey_comm
                0x0000000010029602                lc_qos_setup
                0x000000001002967a                lc_rd_rem_name
                0x00000000100296ca                lc_resp_oob_wait_nonce
                0x00000000100296e8                lc_start_enc
                0x00000000100297ea                lc_epr_rsw_cmp
                0x0000000010029852                lc_start_enc_key_size
                0x00000000100298be                lc_start_key_exch
                0x000000001002992e                lc_resp_num_comp
                0x0000000010029992                lc_stop_enc
                0x00000000100299fa                lc_epr_resp
                0x0000000010029a74                lc_rem_enc
                0x0000000010029aee                lc_stop_afh_reporting
                0x0000000010029b1c                lc_local_switch
                0x0000000010029bf6                lc_restore_afh_reporting
                0x0000000010029c4a                lc_skip_hl_oob_req
                0x0000000010029ca4                lc_start_oob
                0x0000000010029cd0                lc_send_enc_mode
                0x0000000010029d3a                lc_restart_enc
                0x0000000010029d80                lc_restart_enc_cont
                0x0000000010029e38                lc_detach
                0x0000000010029ee8                lc_chg_pkt_type_retry
                0x0000000010029fca                lc_rem_name_cont
                0x000000001002a040                lc_semi_key_cmp
                0x000000001002a10a                lc_mst_key
                0x000000001002a1f0                lc_feat
                0x000000001002a248                lc_hl_connect
                0x000000001002a294                lc_version
                0x000000001002a2d0                lc_ext_feat
                0x000000001002a30e                lc_loc_auth
                0x000000001002a3bc                lc_packet_type
                0x000000001002a446                lc_conn_seq_done
                0x000000001002a468                lc_rsw_done
                0x000000001002a58e                lc_switch_cmp
                0x000000001002a5aa                lc_rem_switch
                0x000000001002a696                lc_send_enc_chg_evt
                0x000000001002a6ec                lc_auth_cmp
                0x000000001002a7ca                lc_con_cmp
                0x000000001002a8a2                lc_end_chk_colli
                0x000000001002a8f6                lc_enc_cmp
                0x000000001002a9ac                lc_mutual_auth_end2
                0x000000001002aaec                lc_epr_change_lk
                0x000000001002ab42                lc_epr_cmp
                0x000000001002abce                lc_mutual_auth_end
                0x000000001002ad00                lc_key_exch_end
                0x000000001002ad72                lc_sp_end
                0x000000001002adc8                lc_calc_link_key
                0x000000001002ae64                lc_sp_fail
                0x000000001002ae9c                lc_resp_oob_nonce
                0x000000001002af22                lc_resp_calc_f3
                0x000000001002afee                lc_start_passkey_loop
                0x000000001002b05a                lc_start_passkey
                0x000000001002b128                lc_resp_pair
                0x000000001002b1e4                lc_pair
                0x000000001002b29a                lc_check_all_slaves_support_sec_con
                0x000000001002b2d0                lc_get_curr_mode
 .text          0x000000001002b304      0x52c ..\..\..\..\Libraries\libs\libbtstack.a(mgr.o)
                0x000000001002b304                mgr_cmd_cmp_send
                0x000000001002b32c                mgr_cmd_stat_send
                0x000000001002b354                mgr_is_dev_connected
                0x000000001002b3a8                mgr_is_dev_synced
                0x000000001002b414                mgr_ral_search
                0x000000001002b45a                mgr_ral_is_empty
                0x000000001002b46c                mgr_ch_map_update
                0x000000001002b5da                mgr_init
                0x000000001002b6dc                mgr_clk_acc_set
                0x000000001002b71c                mgr_link_disc
                0x000000001002b754                mgr_master_ch_map_get
                0x000000001002b75e                mgr_le_evt_mask_check
                0x000000001002b77a                mgr_le_get_features
                0x000000001002b79e                mgr_ral_get
                0x000000001002b7a8                mgr_plan_elt_get
                0x000000001002b7ba                mgr_act_get_free
                0x000000001002b80a                mgr_act_set_free
 .text.le.ll_cntl
                0x000000001002b830      0x2f4 ..\..\..\..\Libraries\libs\libbtstack.a(ll.o)
                0x000000001002b898                ll_cleanup
                0x000000001002b924                ll_init
                0x000000001002b990                ll_role_get
                0x000000001002b9c6                ll_proc_reg
                0x000000001002ba12                ll_proc_id_get
                0x000000001002ba32                ll_proc_state_get
                0x000000001002ba38                ll_proc_state_set
                0x000000001002ba3e                ll_proc_get
                0x000000001002ba56                ll_proc_err_ind
                0x000000001002ba7e                ll_proc_unreg
                0x000000001002baee                ll_proc_collision_check
 .text.le.ll_cntl.start
                0x000000001002bb24      0x20e ..\..\..\..\Libraries\libs\libbtstack.a(ll.o)
                0x000000001002bb24                ll_start
 .text.le.ll_cntl.state
                0x000000001002bd32       0x60 ..\..\..\..\Libraries\libs\libbtstack.a(ll.o)
                0x000000001002bd32                ll_cntl_state_set
 .text.le.ll_cntl.stop
                0x000000001002bd92       0x48 ..\..\..\..\Libraries\libs\libbtstack.a(ll.o)
                0x000000001002bd92                ll_stop
 .text.le.ll_cntl.timer
                0x000000001002bdda       0xd8 ..\..\..\..\Libraries\libs\libbtstack.a(ll.o)
                0x000000001002bdda                ll_proc_timer_set
                0x000000001002be4a                ll_proc_timer_set_state
 .text          0x000000001002beb2       0x20 ..\..\..\..\Libraries\libs\libbtstack.a(ble_test.o)
                0x000000001002beb2                ble_test_init
 *fill*         0x000000001002bed2       0x2e 
 .text          0x000000001002bf00      0x702 ..\..\..\..\Libraries\libs\libbtstack.a(ble_scan.o)
                0x000000001002bf66                ble_get_scan_var
                0x000000001002bf70                ble_get_sync_var
                0x000000001002bf7a                ble_scan_init
                0x000000001002bff2                ble_scan_start
                0x000000001002c500                ble_scan_stop
                0x000000001002c538                ble_scan_params_update
 .text          0x000000001002c602        0x4 ..\..\..\..\Libraries\libs\libbtstack.a(ble_per_adv.o)
                0x000000001002c602                ble_get_per_adv_var
 *fill*         0x000000001002c606       0x3a 
 .text          0x000000001002c640      0x86e ..\..\..\..\Libraries\libs\libbtstack.a(ble_init.o)
                0x000000001002c640                ble_init_connect_req_pack
                0x000000001002c6ea                ble_init_init
                0x000000001002c758                ble_init_start
                0x000000001002ce40                ble_init_stop
 .text          0x000000001002ceae      0x158 ..\..\..\..\Libraries\libs\libbtstack.a(ble_buf.o)
                0x000000001002ceae                ble_buf_init_do
                0x000000001002cfbc                ble_buf_init
 .text.bb.ble.adv0
                0x000000001002d006      0x20a ..\..\..\..\Libraries\libs\libbtstack.a(ble_adv0.o)
                0x000000001002d0be                ble_adv0_init
                0x000000001002d110                ble_adv0_end_ind
                0x000000001002d14a                ble_adv0_set_en
                0x000000001002d1a2                ble_adv0_update_adv_data
                0x000000001002d206                ble_adv0_set_interval
                0x000000001002d20e                ble_adv0_copy
 .text          0x000000001002d210       0x2a ..\..\..\..\Libraries\libs\libbtstack.a(extern_hfhs.o)
                0x000000001002d210                hfp_notice_network_time
                0x000000001002d212                hfp_notice_ring_number
                0x000000001002d218                hfp_get_last_call_number
                0x000000001002d21c                msbc_exit
                0x000000001002d21e                bt_pbap_data_callback
                0x000000001002d220                hfp_get_mic_gain
                0x000000001002d224                hfp_get_spk_gain
                0x000000001002d228                hfp_get_bat_level
                0x000000001002d22c                hfp_hf_established_hook
                0x000000001002d230                hfp_hf_send_custom_at_cmd_hook
                0x000000001002d234                hfp_hf_recv_custom_at_cmd_hook
                0x000000001002d238                hfp_hf_release_hook
 .text.func.outgoing
                0x000000001002d23a       0x14 ..\..\..\..\Libraries\libs\libbtstack.a(extern_hfhs.o)
                0x000000001002d23a                hfp_get_outgoing_number
                0x000000001002d244                hfp_get_at_cmd
 .text.func.btring
                0x000000001002d24e        0x6 ..\..\..\..\Libraries\libs\libbtstack.a(extern_hfhs.o)
                0x000000001002d24e                hfp_is_list_curr_calls
                0x000000001002d252                hfp_hf_emit_curr_calls
 .text.stack.l2cap_sig
                0x000000001002d254      0x134 ..\..\..\..\Libraries\libs\libbtstack.a(l2cap_signaling.o)
                0x000000001002d334                l2cap_next_sig_id
                0x000000001002d350                l2cap_next_local_cid
                0x000000001002d374                l2cap_create_signaling_classic
                0x000000001002d37e                l2cap_create_signaling_le
 .text          0x000000001002d388       0xdc ..\..\..\..\Libraries\libs\libbtstack.a(lc_hook.o)
                0x000000001002d388                lc_lmp_ver_req_hook
                0x000000001002d3ae                lc_lmp_ver_res_hook
                0x000000001002d3b0                lc_loc_sniff_req_hook
                0x000000001002d3ec                lmp_sniff_req_hook
                0x000000001002d40e                lc_auto_sniff_step_set
 *fill*         0x000000001002d464        0x0 
 .text          0x000000001002d464     0x17ca ..\..\..\..\Libraries\libs\libbtstack.a(lm_sco.o)
                0x000000001002dee8                lm_get_sync_param
                0x000000001002e862                lm_init_sync
                0x000000001002e884                lm_reset_sync
                0x000000001002e8b4                lm_check_active_sync
                0x000000001002e8c2                lm_add_sync
                0x000000001002ea4c                lm_check_sync_hl_rsp
                0x000000001002eb20                lm_get_synchdl
                0x000000001002eb3e                lm_look_for_sync
                0x000000001002eb88                lm_get_nb_sync_link
                0x000000001002eb92                lm_get_min_sync_intv
                0x000000001002ebb6                lm_remove_sync
                0x000000001002ec24                lm_sco_nego_end
 .text          0x000000001002ec2e      0x498 ..\..\..\..\Libraries\libs\libbtstack.a(lc_util.o)
                0x000000001002ec2e                lc_get_max_pkt_size
                0x000000001002ec9a                lc_compute_pkt_types
                0x000000001002ecc0                lc_update_acl_pkt_types
                0x000000001002ed12                lc_update_acl_edr_pkt_types
                0x000000001002ed8a                lc_reduce_acl_pkt_types
                0x000000001002edc0                lc_pkt_types_to_max_slot
                0x000000001002ee06                lc_get_qos_param
                0x000000001002ef34                lc_gen_cof_for_addr
                0x000000001002ef5a                lc_check_edr_feature_for_pkt_types
                0x000000001002ef6a                lc_check_feature
                0x000000001002ef98                lc_pref_rate_to_pkt_types
                0x000000001002f028                lc_max_slot_to_pkt_types
                0x000000001002f048                lc_get_common_pkt_types
 .text          0x000000001002f0c6      0x9b2 ..\..\..\..\Libraries\libs\libbtstack.a(lc_sniff.o)
                0x000000001002f302                lc_sniff_init
                0x000000001002f314                lc_sniff_clear
                0x000000001002f34a                lc_sniff_interval_get
                0x000000001002f36a                lc_sniff_offset_update
                0x000000001002f39a                lc_sniff_host_request
                0x000000001002f530                lc_sniff_peer_request
                0x000000001002f800                lc_sniff_peer_accept
                0x000000001002f8d0                lc_sniff_peer_reject
                0x000000001002f8fa                lc_sniff_acc_tx_cfm
                0x000000001002f8fc                lc_sniff_timeout
                0x000000001002f902                lc_sniff_unsniff
                0x000000001002f966                lc_sniff_unsniff_peer_request
                0x000000001002fa12                lc_sniff_unsniff_peer_accept
                0x000000001002fa32                lc_sniff_unsniff_peer_reject
 .text          0x000000001002fa78     0x164c ..\..\..\..\Libraries\libs\libbtstack.a(lc_sco.o)
                0x0000000010030246                lc_sco_alloc_link
                0x000000001003028e                lc_sco_free_link
                0x00000000100302c6                lc_sco_get_conhdl
                0x0000000010030302                lc_sco_get_snoop_service
                0x0000000010030346                lc_sco_set_snoop_service
                0x0000000010030376                lc_sco_start_snoop
                0x0000000010030468                lc_sco_init
                0x0000000010030496                lc_sco_reset
                0x00000000100304e2                lc_sco_detach
                0x000000001003057a                lc_sco_release
                0x00000000100305f4                lc_sco_host_request
                0x00000000100306f2                lc_sco_host_accept
                0x0000000010030880                lc_sco_host_reject
                0x000000001003091a                lc_sco_host_request_disc
                0x00000000100309a4                lc_sco_peer_request
                0x0000000010030c0c                lc_sco_peer_accept
                0x0000000010030c7c                lc_sco_peer_reject
                0x0000000010030cfe                lc_sco_peer_request_disc
                0x0000000010030dee                lc_sco_peer_accept_disc
                0x0000000010030e94                lc_sco_peer_reject_disc
                0x0000000010030f14                lc_sco_baseband_ack
                0x0000000010030fe4                lc_sco_timeout
                0x0000000010031090                lc_sco_offset_update
 *fill*         0x00000000100310c4        0x0 
 .text          0x00000000100310c4     0x9234 ..\..\..\..\Libraries\libs\libbtstack.a(lc_proc.o)
                0x000000001003129e                hci_acl_data_lc_func
                0x0000000010031850                lmp_detach_func
                0x0000000010031946                lc_acl_rx_ind_func
                0x000000001003a2ae                lc_flush_acl_tx_pend
 .text          0x000000001003a2f8      0x6dc ..\..\..\..\Libraries\libs\libbtstack.a(lc_lmppdu.o)
                0x000000001003a2f8                lmp_find_desc
                0x000000001003a346                lmp_estab_allowed
                0x000000001003a37e                lmp_msg_pk
                0x000000001003a3e2                lmp_msg_unpk
                0x000000001003a454                lc_send_lmp
                0x000000001003a4be                lc_send_pdu_acc
                0x000000001003a4dc                lc_send_pdu_acc_ext4
                0x000000001003a506                lc_send_pdu_not_acc
                0x000000001003a528                lc_send_pdu_not_acc_ext4
                0x000000001003a556                lc_send_pdu_set_afh
                0x000000001003a598                lc_send_pdu_au_rand
                0x000000001003a5c2                lc_send_pdu_in_rand
                0x000000001003a5ec                lc_send_pdu_comb_key
                0x000000001003a616                lc_send_pdu_max_slot
                0x000000001003a634                lc_send_pdu_max_slot_req
                0x000000001003a652                lc_send_pdu_encaps_payl
                0x000000001003a67c                lc_send_pdu_encaps_head
                0x000000001003a6a2                lc_send_pdu_ptt_req
                0x000000001003a6c4                lc_send_pdu_sp_nb
                0x000000001003a6ee                lc_send_pdu_sp_cfm
                0x000000001003a718                lc_send_pdu_sres
                0x000000001003a742                lc_send_pdu_sco_lk_rem_req
                0x000000001003a764                lc_send_pdu_esco_lk_rem_req
                0x000000001003a78a                lc_send_pdu_auto_rate
                0x000000001003a7a4                lc_send_pdu_sup_to
                0x000000001003a7c2                lc_send_pdu_enc_key_sz_req
                0x000000001003a7e0                lc_send_pdu_feats_res
                0x000000001003a80c                lc_send_pdu_tim_acc
                0x000000001003a826                lc_send_pdu_feats_ext_req
                0x000000001003a85c                lc_send_pdu_io_cap_res
                0x000000001003a8a6                lc_send_pdu_num_comp_fail
                0x000000001003a8c4                lc_send_pdu_paus_enc_req
                0x000000001003a8e2                lc_send_pdu_resu_enc_req
                0x000000001003a900                lc_send_pdu_setup_cmp
                0x000000001003a91a                lc_send_pdu_qos_req
                0x000000001003a93c                lc_send_pdu_slot_off
                0x000000001003a97e                lc_send_pdu_vers_req
                0x000000001003a9ac                lc_send_pdu_dhkey_chk
 .text          0x000000001003a9d4      0x11a ..\..\..\..\Libraries\libs\libbtstack.a(mgr_proc.o)
 .text          0x000000001003aaee      0xa60 ..\..\..\..\Libraries\libs\libbtstack.a(mgr_init.o)
                0x000000001003aaee                hci_le_create_con_cmd_func
                0x000000001003ae06                hci_le_ext_create_con_cmd_func
                0x000000001003b164                hci_le_create_con_cancel_cmd_func
                0x000000001003b1da                ble_init_end_ind_func
 .text          0x000000001003b54e      0x6da ..\..\..\..\Libraries\libs\libbtstack.a(mgr_hci.o)
 .text.le.mgr   0x000000001003bc28       0x38 ..\..\..\..\Libraries\libs\libbtstack.a(mgr_hci.o)
                0x000000001003bc28                hci_command_mgr_func
 .text          0x000000001003bc60      0x40a ..\..\..\..\Libraries\libs\libbtstack.a(ll_scan.o)
                0x000000001003bc60                hci_le_set_scan_param_cmd_func
                0x000000001003bdae                hci_le_set_scan_en_cmd_func
 .text.le.ll_scan
                0x000000001003c06a      0x628 ..\..\..\..\Libraries\libs\libbtstack.a(ll_scan.o)
                0x000000001003c06a                ble_adv_rep_ind_func
                0x000000001003c600                ble_scan_end_ind_func
 .text          0x000000001003c692      0x826 ..\..\..\..\Libraries\libs\libbtstack.a(ll_adv.o)
                0x000000001003c74a                ll_adv_hdl_to_idx
                0x000000001003c78e                hci_le_rd_adv_ch_tx_pw_cmd_func
                0x000000001003c7ee                hci_le_set_adv_param_cmd_func
                0x000000001003c998                hci_le_set_adv_data_cmd_func
                0x000000001003ca6c                hci_le_set_scan_rsp_data_cmd_func
                0x000000001003cb40                hci_le_set_adv_en_cmd_func
                0x000000001003cdc2                ll_adv_get_act_idx
                0x000000001003ce2c                ll_adv_get_set_id
 .text.le.ll_adv
                0x000000001003ceb8      0x30a ..\..\..\..\Libraries\libs\libbtstack.a(ll_adv.o)
                0x000000001003ceb8                ble_scan_req_ind_func
                0x000000001003cf20                ble_adv_end_ind_func
 .text.le.ll_adv.con
                0x000000001003d1c2      0x250 ..\..\..\..\Libraries\libs\libbtstack.a(ll_adv.o)
                0x000000001003d1c2                ble_adv_end_con_ind
 .text          0x000000001003d412      0x3ae ..\..\..\..\Libraries\libs\libbtstack.a(ll_proc.o)
                0x000000001003d412                hci_command_ll_func
                0x000000001003d462                ble_acl_rx_ind_func
                0x000000001003d5f8                ble_acl_tx_cfm_func
                0x000000001003d608                hci_acl_data_func
                0x000000001003d6da                ll_cmd_cmp_send
                0x000000001003d708                hci_vs_set_pref_slave_latency_cmd_func
                0x000000001003d74c                hci_vs_set_pref_slave_evt_dur_cmd_func
                0x000000001003d798                ll_cmd_stat_send
 .text          0x000000001003d7c0      0x32e ..\..\..\..\Libraries\libs\libbtstack.a(ll_ping.o)
                0x000000001003d840                hci_rd_auth_payl_to_cmd_func
                0x000000001003d8a4                ll_op_ping_ind_func
                0x000000001003d8fa                ll_auth_payl_nearly_to_func
                0x000000001003d968                ll_ping_restart
                0x000000001003d9c0                ll_auth_payl_real_to_func
                0x000000001003da1e                ll_ping_set
                0x000000001003da86                hci_wr_auth_payl_to_cmd_func
 .text.le.ll_cntl.pdu
                0x000000001003daee       0x3c ..\..\..\..\Libraries\libs\libbtstack.a(ll_ping.o)
                0x000000001003daee                ll_ping_req_func
                0x000000001003db0a                ll_ping_rsp_func
 *fill*         0x000000001003db2a        0x2 
 .text          0x000000001003db2c      0xad0 ..\..\..\..\Libraries\libs\libbtstack.a(ll_phy_upd.o)
                0x000000001003e320                hci_le_rd_phy_cmd_func
                0x000000001003e388                hci_le_set_phy_cmd_func
                0x000000001003e4ca                ll_op_phy_upd_ind_func
                0x000000001003e554                ble_phy_upd_cfm_func
                0x000000001003e590                ll_phy_upd_proc_start
 .text.le.ll_cntl.pdu
                0x000000001003e5fc      0x212 ..\..\..\..\Libraries\libs\libbtstack.a(ll_phy_upd.o)
                0x000000001003e5fc                ll_phy_req_func
                0x000000001003e6c0                ll_phy_rsp_func
                0x000000001003e754                ll_phy_update_ind_func
 .text          0x000000001003e80e      0x136 ..\..\..\..\Libraries\libs\libbtstack.a(ll_past.o)
                0x000000001003e80e                hci_le_per_adv_set_info_transf_cmd_func
                0x000000001003e8c2                hci_le_set_per_adv_sync_transf_param_cmd_func
 .text          0x000000001003e944      0x57c ..\..\..\..\Libraries\libs\libbtstack.a(ll_length.o)
                0x000000001003ebac                hci_le_set_data_len_cmd_func
                0x000000001003ecba                hci_vs_set_max_rx_size_and_time_cmd_func
                0x000000001003edce                ll_op_length_upd_ind_func
                0x000000001003ee34                ll_length_proc_start
 .text.le.ll_cntl.pdu
                0x000000001003eec0      0x204 ..\..\..\..\Libraries\libs\libbtstack.a(ll_length.o)
                0x000000001003eec0                ll_length_req_func
                0x000000001003f02a                ll_length_rsp_func
 .text          0x000000001003f0c4      0x2d6 ..\..\..\..\Libraries\libs\libbtstack.a(ll_feature.o)
                0x000000001003f274                hci_le_rd_rem_feats_cmd_func
                0x000000001003f324                ll_op_feats_exch_ind_func
 .text.le.ll_cntl.pdu
                0x000000001003f39a      0x168 ..\..\..\..\Libraries\libs\libbtstack.a(ll_feature.o)
                0x000000001003f39a                ll_feature_req_func
                0x000000001003f410                ll_slave_feature_req_func
                0x000000001003f486                ll_feature_rsp_func
 *fill*         0x000000001003f502        0x2 
 .text          0x000000001003f504      0xaa0 ..\..\..\..\Libraries\libs\libbtstack.a(ll_encrypt.o)
                0x000000001003fc5c                hci_le_en_enc_cmd_func
                0x000000001003fd32                hci_le_ltk_req_reply_cmd_func
                0x000000001003fda6                hci_le_ltk_req_neg_reply_cmd_func
                0x000000001003fe32                ll_encrypt_ind_func
                0x000000001003ff3c                ll_op_encrypt_ind_func
 .text.le.ll_cntl.pdu
                0x000000001003ffa4      0x2fa ..\..\..\..\Libraries\libs\libbtstack.a(ll_encrypt.o)
                0x000000001003ffa4                ll_pause_enc_req_func
                0x0000000010040022                ll_pause_enc_rsp_func
                0x0000000010040084                ll_enc_req_func
                0x000000001004016a                ll_enc_rsp_func
                0x00000000100401ec                ll_start_enc_req_func
                0x0000000010040246                ll_start_enc_rsp_func
 .text          0x000000001004029e      0x30a ..\..\..\..\Libraries\libs\libbtstack.a(ll_disconnect.o)
                0x000000001004029e                ble_disc_ind_func
                0x00000000100402f6                ll_stopped_ind_func
                0x000000001004034e                hci_disconnect_cmd_func
                0x00000000100403fc                ll_disconnect
                0x00000000100404de                ll_op_disconnect_ind_func
                0x0000000010040558                ll_init_term_proc
 .text.le.ll_cntl.pdu
                0x00000000100405a8       0x44 ..\..\..\..\Libraries\libs\libbtstack.a(ll_disconnect.o)
                0x00000000100405a8                ll_terminate_ind_func
 .text          0x00000000100405ec      0xce4 ..\..\..\..\Libraries\libs\libbtstack.a(ll_con_upd.o)
                0x0000000010040e62                hci_le_con_upd_cmd_func
                0x0000000010040f8e                hci_le_rem_con_param_req_reply_cmd_func
                0x0000000010041028                hci_le_rem_con_param_req_neg_reply_cmd_func
                0x000000001004108a                ll_op_con_upd_ind_func
                0x000000001004111c                ble_con_param_upd_cfm_func
                0x0000000010041188                ble_con_offset_upd_ind_func
                0x00000000100411da                ll_con_move_cb
 .text.le.ll_cntl.pdu
                0x00000000100412d0      0x30c ..\..\..\..\Libraries\libs\libbtstack.a(ll_con_upd.o)
                0x00000000100412d0                ll_con_update_ind_func
                0x0000000010041430                ll_con_param_req_func
                0x0000000010041546                ll_con_param_rsp_func
 .text          0x00000000100415dc      0x2cc ..\..\..\..\Libraries\libs\libbtstack.a(ll_cntl.o)
                0x00000000100415dc                ll_pdu_send_reject_ind
                0x0000000010041630                ble_cntl_rx_ind_func
                0x0000000010041798                ble_cntl_tx_cfm_func
                0x00000000100417f0                hci_vs_send_cntl_cmd_func
                0x0000000010041854                hci_vs_cntl_discard_cmd_func
 .text.le.ll_cntl.pdu
                0x00000000100418a8       0x64 ..\..\..\..\Libraries\libs\libbtstack.a(ll_cntl.o)
 .text.le.ll_cntl.send
                0x000000001004190c      0x18a ..\..\..\..\Libraries\libs\libbtstack.a(ll_cntl.o)
                0x000000001004190c                ll_cntl_tx_check
                0x00000000100419fc                ll_cntl_send
 .text          0x0000000010041a96      0x2d6 ..\..\..\..\Libraries\libs\libbtstack.a(ll_clk_acc.o)
                0x0000000010041bf6                ll_op_clk_acc_ind_func
                0x0000000010041c4c                ll_clk_acc_modify
                0x0000000010041cca                hci_le_req_peer_sca_cmd_func
 .text.le.ll_cntl.pdu
                0x0000000010041d6c       0xb4 ..\..\..\..\Libraries\libs\libbtstack.a(ll_clk_acc.o)
                0x0000000010041d6c                ll_clk_acc_req_func
                0x0000000010041dca                ll_clk_acc_rsp_func
 .text          0x0000000010041e20      0x37a ..\..\..\..\Libraries\libs\libbtstack.a(ll_chmap_upd.o)
                0x0000000010042022                hci_le_rd_chnl_map_cmd_func
                0x000000001004208c                ll_op_ch_map_upd_ind_func
                0x00000000100420ec                mgr_ch_map_update_ind_func
                0x0000000010042166                ble_ch_map_upd_cfm_func
 .text.le.ll_cntl.pdu
                0x000000001004219a      0x172 ..\..\..\..\Libraries\libs\libbtstack.a(ll_chmap_upd.o)
                0x000000001004219a                ll_channel_map_ind_func
                0x0000000010042262                ll_min_used_channels_ind_func
 .text          0x000000001004230c      0x176 ..\..\..\..\Libraries\libs\libbtstack.a(aes_rpa.o)
                0x00000000100423ce                aes_rpa_gen
                0x0000000010042420                aes_rpa_resolve
 .text          0x0000000010042482        0x4 ..\..\..\..\Libraries\libs\libbtstack.a(scan_hook.o)
                0x0000000010042482                ble_scan_end_ind_hook
 .text          0x0000000010042486        0x8 ..\..\..\..\Libraries\libs\libbtstack.a(adv_hook.o)
                0x0000000010042486                ble_adv_end_ind_hook
 .text          0x000000001004248e      0x21e ..\..\..\..\Libraries\libs\libbtstack.a(ll_version.o)
                0x000000001004259c                ll_op_ver_exch_ind_func
                0x0000000010042612                hci_rd_rem_ver_info_cmd_func
 .text.le.ll_cntl.pdu
                0x00000000100426ac       0x6e ..\..\..\..\Libraries\libs\libbtstack.a(ll_version.o)
                0x00000000100426ac                ll_version_ind_func
 .text          0x000000001004271a      0x11a ..\..\..\..\Libraries\libs\libbtstack.a(ll_pwr.o)
                0x000000001004271a                hci_rd_tx_pwr_lvl_cmd_func
                0x00000000100427b0                hci_rd_rssi_cmd_func
 *(.rodata*)
 *fill*         0x0000000010042834        0x0 
 .rodata.str1.4
                0x0000000010042834      0x11d Output\obj\Libraries\bsp\bsp_fot.o
 *fill*         0x0000000010042951        0x3 
 .rodata.str1.4
                0x0000000010042954       0x76 Output\obj\Libraries\bsp\bsp_sys.o
 *fill*         0x00000000100429ca        0x2 
 .rodata.str1.4
                0x00000000100429cc       0x3a Output\obj\Libraries\BT\ble\ble.o
 *fill*         0x0000000010042a06        0x2 
 .rodata.str1.4
                0x0000000010042a08        0x5 Output\obj\Libraries\BT\spp\bt.o
 *fill*         0x0000000010042a0d        0x3 
 .rodata.str1.4
                0x0000000010042a10       0x58 Output\obj\Libraries\BT\spp\spp.o
 .rodata.str1.4
                0x0000000010042a68       0x48 Output\obj\Examples\TIMER\TIM_Capture\Source\timer_capture.o
 .rodata.str1.4
                0x0000000010042ab0       0x1d Output\obj\Examples\TIMER\TIM_Capture\Project\main.o
 *fill*         0x0000000010042acd        0x3 
 .rodata.str1.4
                0x0000000010042ad0       0xfc ..\..\..\..\Libraries\libs\libplatform.a(cm.o)
 .rodata.str1.4
                0x0000000010042bcc       0x10 ..\..\..\..\Libraries\libs\libplatform.a(main.o)
 .rodata.str1.4
                0x0000000010042bdc       0x57 ..\..\..\..\Libraries\libs\libplatform.a(startup.o)
 *fill*         0x0000000010042c33        0x1 
 .rodata.str1.4
                0x0000000010042c34      0x104 ..\..\..\..\Libraries\libs\libplatform.a(lock.o)
 .rodata.str1.4
                0x0000000010042d38       0x1d ..\..\..\..\Libraries\libs\libplatform.a(sys.o)
 *fill*         0x0000000010042d55        0x3 
 .rodata.volt_trim
                0x0000000010042d58       0xbc ..\..\..\..\Libraries\libs\libplatform.a(voltage_trim.o)
                0x0000000010042d58                charge_trim_step
                0x0000000010042d6c                vddcore_trim_step
                0x0000000010042d8c                vddio_trim_step
                0x0000000010042dac                vddbko_trim_step
 .rodata.bb.tbl
                0x0000000010042e14        0x8 ..\..\..\..\Libraries\libs\libbtstack.a(ble_con.o)
                0x0000000010042e14                connect_req_dur_tab
 .rodata.bb.tbl
                0x0000000010042e1c       0x16 ..\..\..\..\Libraries\libs\libbtstack.a(bb_utils.o)
                0x0000000010042e1c                null_array
                0x0000000010042e2c                dft_addr
 *fill*         0x0000000010042e32        0x2 
 .rodata        0x0000000010042e34       0x20 ..\..\..\..\Libraries\libs\libbtstack.a(bb.o)
                0x0000000010042e34                bb_hook
 .rodata.str1.4
                0x0000000010042e54        0x5 ..\..\..\..\Libraries\libs\libbtstack.a(extern_bt.o)
                                          0xd (size before relaxing)
 *fill*         0x0000000010042e59        0x3 
 .rodata        0x0000000010042e5c       0x18 ..\..\..\..\Libraries\libs\libbtstack.a(spp.o)
 .rodata.stack.spp
                0x0000000010042e74        0x2 ..\..\..\..\Libraries\libs\libbtstack.a(spp.o)
 *fill*         0x0000000010042e76        0x2 
 .rodata        0x0000000010042e78       0x10 ..\..\..\..\Libraries\libs\libbtstack.a(sdp_util.o)
                0x0000000010042e78                mfi_search_uuid128
 .rodata.sdp.tbl.spp
                0x0000000010042e88      0x11f ..\..\..\..\Libraries\libs\libbtstack.a(sdp_tbl.o)
                0x0000000010042e88                sdp_spp_dueros_ota_service_record
                0x0000000010042eec                sdp_spp_proc_test_service_record
                0x0000000010042f50                sdp_spp_service_record
 *fill*         0x0000000010042fa7        0x1 
 .rodata.str1.4
                0x0000000010042fa8        0x8 ..\..\..\..\Libraries\libs\libbtstack.a(sdp_client.o)
 .rodata        0x0000000010042fb0       0x17 ..\..\..\..\Libraries\libs\libbtstack.a(sdp_client.o)
 *fill*         0x0000000010042fc7        0x1 
 .rodata        0x0000000010042fc8      0x100 ..\..\..\..\Libraries\libs\libbtstack.a(rfcomm.o)
 .rodata        0x00000000100430c8       0x20 ..\..\..\..\Libraries\libs\libbtstack.a(btstack_util.o)
                0x00000000100430d8                bluetooth_base_uuid
 .rodata.str1.4
                0x00000000100430e8       0x1a ..\..\..\..\Libraries\libs\libbtstack.a(btstack_link_ctrl.o)
 *fill*         0x0000000010043102        0x2 
 .rodata        0x0000000010043104       0x11 ..\..\..\..\Libraries\libs\libbtstack.a(gatt_server.o)
 *fill*         0x0000000010043115        0x3 
 .rodata        0x0000000010043118       0x38 ..\..\..\..\Libraries\libs\libbtstack.a(gatt_profile.o)
 .rodata        0x0000000010043150       0x10 ..\..\..\..\Libraries\libs\libbtstack.a(att_db.o)
 .rodata.str1.4
                0x0000000010043160       0x2e ..\..\..\..\Libraries\libs\libbtstack.a(btstack_api.o)
 *fill*         0x000000001004318e        0x2 
 .rodata        0x0000000010043190       0xe0 ..\..\..\..\Libraries\libs\libbtstack.a(btstack_api.o)
                0x0000000010043190                tws_key_tbl
                0x0000000010043258                tws_hid_key_tbl
 .rodata.stack.api
                0x0000000010043270      0x184 ..\..\..\..\Libraries\libs\libbtstack.a(btstack_api.o)
                0x0000000010043270                btstack_ctl0_tbl
                0x00000000100432c8                btstack_comm_tbl
                0x00000000100432e8                btstack_hid_tbl
                0x00000000100432f4                btstack_ctl_tbl
                0x00000000100433c0                btstack_api_tbl
                0x00000000100433f0                btstack_spp_tbl
 .rodata.stack.setup
                0x00000000100433f4       0x14 ..\..\..\..\Libraries\libs\libbtstack.a(btstack_api.o)
 .rodata        0x0000000010043408       0x2c ..\..\..\..\Libraries\libs\libbtstack.a(bb_sche.o)
 .rodata        0x0000000010043434       0x18 ..\..\..\..\Libraries\libs\libbtstack.a(vs_proc.o)
 .rodata.bb.tbl
                0x000000001004344c        0x6 ..\..\..\..\Libraries\libs\libbtstack.a(rf_smart.o)
 *fill*         0x0000000010043452        0x2 
 .rodata.str1.4
                0x0000000010043454       0x20 ..\..\..\..\Libraries\libs\libbtstack.a(hct_tl.o)
 .rodata.str1.4
                0x0000000010043474      0x312 ..\..\..\..\Libraries\libs\libbtstack.a(hct_msg.o)
                                        0x362 (size before relaxing)
 *fill*         0x0000000010043786        0x2 
 .rodata        0x0000000010043788      0xc20 ..\..\..\..\Libraries\libs\libbtstack.a(hct_msg.o)
                0x0000000010043788                hci_cmd_desc_root_tab
                0x00000000100437c8                hci_evt_desc_tab
                0x0000000010043948                hci_evt_le_desc_tab
                0x00000000100439b8                hci_cmd_desc_tab_vs
                0x0000000010043a84                hci_cmd_desc_tab_le
                0x0000000010043ce8                hci_cmd_desc_tab_testing
                0x0000000010043d24                hci_cmd_desc_tab_stat_par
                0x0000000010043d78                hci_cmd_desc_tab_info_par
                0x0000000010043dfc                hci_cmd_desc_tab_ctrl_bb
                0x0000000010044174                hci_cmd_desc_tab_lk_pol
                0x00000000100441f8                hci_cmd_desc_tab_lk_ctrl
 .rodata        0x00000000100443a8       0x9c ..\..\..\..\Libraries\libs\libbtstack.a(lm.o)
 .rodata.bb.tbl
                0x0000000010044444       0x14 ..\..\..\..\Libraries\libs\libbtstack.a(bt21.o)
                0x0000000010044444                bt_ctl
 .rodata.bb.tbl
                0x0000000010044458        0x7 ..\..\..\..\Libraries\libs\libbtstack.a(ble_hal.o)
 *fill*         0x000000001004445f        0x1 
 .rodata.bb.tbl
                0x0000000010044460       0x14 ..\..\..\..\Libraries\libs\libbtstack.a(ble.o)
                0x0000000010044460                ble_ctl
 .rodata.l2cap  0x0000000010044474        0x9 ..\..\..\..\Libraries\libs\libbtstack.a(l2cap_test.o)
                0x0000000010044474                vs_test_actived_cmd
 *fill*         0x000000001004447d        0x3 
 .rodata.stack.l2cap
                0x0000000010044480        0x5 ..\..\..\..\Libraries\libs\libbtstack.a(l2cap.o)
 *fill*         0x0000000010044485        0x3 
 .rodata.str1.4
                0x0000000010044488       0xb8 ..\..\..\..\Libraries\libs\libbtstack.a(hci_cmd.o)
                                         0xd0 (size before relaxing)
 .rodata.stack.hci_send
                0x0000000010044540      0x2a0 ..\..\..\..\Libraries\libs\libbtstack.a(hci_cmd.o)
                0x0000000010044540                hci_le_set_default_phy
                0x0000000010044548                hci_le_write_suggested_default_data_len
                0x0000000010044550                hci_le_test_end
                0x0000000010044558                hci_le_transmitter_test
                0x0000000010044560                hci_le_receiver_test
                0x0000000010044568                hci_le_read_supported_states
                0x0000000010044570                hci_le_long_term_key_negative_reply
                0x0000000010044578                hci_le_long_term_key_request_reply
                0x0000000010044580                hci_le_start_encryption
                0x0000000010044588                hci_le_rand
                0x0000000010044590                hci_le_encrypt
                0x0000000010044598                hci_le_read_remote_used_features
                0x00000000100445a0                hci_le_read_channel_map
                0x00000000100445a8                hci_le_set_host_channel_classification
                0x00000000100445b0                hci_le_connection_update
                0x00000000100445b8                hci_le_remove_device_from_white_list
                0x00000000100445c0                hci_le_add_device_to_white_list
                0x00000000100445c8                hci_le_clear_white_list
                0x00000000100445d0                hci_le_read_white_list_size
                0x00000000100445d8                hci_le_create_connection_cancel
                0x00000000100445e0                hci_le_create_connection
                0x00000000100445e8                hci_le_set_scan_enable
                0x00000000100445f0                hci_le_set_scan_parameters
                0x00000000100445f8                hci_le_set_advertise_enable
                0x0000000010044600                hci_le_set_scan_response_data
                0x0000000010044608                hci_le_set_advertising_data
                0x0000000010044610                hci_le_read_advertising_channel_tx_power
                0x0000000010044618                hci_le_set_advertising_parameters
                0x0000000010044620                hci_le_set_random_address
                0x0000000010044628                hci_le_read_supported_features
                0x0000000010044630                hci_le_read_buffer_size
                0x0000000010044638                hci_le_set_event_mask
                0x0000000010044640                hci_test_mode_emul
                0x0000000010044648                hci_read_rssi
                0x0000000010044650                hci_read_bd_addr
                0x0000000010044658                hci_read_buffer_size
                0x0000000010044660                hci_read_local_supported_features
                0x0000000010044668                hci_read_local_supported_commands
                0x0000000010044670                hci_write_loopback_mode
                0x0000000010044678                hci_read_loopback_mode
                0x0000000010044680                hci_write_le_host_supported
                0x0000000010044688                hci_read_le_host_supported
                0x0000000010044690                hci_write_simple_pairing_mode
                0x0000000010044698                hci_write_extended_inquiry_response
                0x00000000100446a0                hci_write_inquiry_scan_type
                0x00000000100446a8                hci_write_inquiry_mode
                0x00000000100446b0                hci_write_link_supervision_timeout
                0x00000000100446b8                hci_host_buffer_size
                0x00000000100446c0                hci_write_class_of_device
                0x00000000100446c8                hci_write_scan_enable
                0x00000000100446d0                hci_write_page_timeout
                0x00000000100446d8                hci_write_local_name
                0x00000000100446e0                hci_reset
                0x00000000100446e8                hci_set_event_mask
                0x00000000100446f0                hci_switch_role_command
                0x00000000100446f8                hci_role_discovery
                0x0000000010044700                hci_io_capability_request_negative_reply
                0x0000000010044708                hci_remote_oob_data_request_negative_reply
                0x0000000010044710                hci_user_passkey_request_negative_reply
                0x0000000010044718                hci_user_passkey_request_reply
                0x0000000010044720                hci_user_confirmation_request_negative_reply
                0x0000000010044728                hci_user_confirmation_request_reply
                0x0000000010044730                hci_io_capability_request_reply
                0x0000000010044738                hci_accept_synchronous_connection
                0x0000000010044740                hci_setup_synchronous_connection
                0x0000000010044748                hci_read_clock_offset_command
                0x0000000010044750                hci_read_remote_version_info_command
                0x0000000010044758                hci_read_remote_supported_features_command
                0x0000000010044760                hci_remote_name_request_cancel
                0x0000000010044768                hci_remote_name_request
                0x0000000010044770                hci_change_connection_link_key
                0x0000000010044778                hci_set_connection_encryption
                0x0000000010044780                hci_authentication_requested
                0x0000000010044788                hci_pin_code_request_negative_reply
                0x0000000010044790                hci_pin_code_request_reply
                0x0000000010044798                hci_link_key_request_negative_reply
                0x00000000100447a0                hci_link_key_request_reply
                0x00000000100447a8                hci_reject_connection_request
                0x00000000100447b0                hci_accept_connection_request
                0x00000000100447b8                hci_create_connection_cancel
                0x00000000100447c0                hci_disconnect
                0x00000000100447c8                hci_create_connection
                0x00000000100447d0                hci_inquiry_cancel
                0x00000000100447d8                hci_inquiry
 .rodata        0x00000000100447e0        0xc ..\..\..\..\Libraries\libs\libbtstack.a(hci.o)
 .rodata        0x00000000100447ec       0x2d ..\..\..\..\Libraries\libs\libbtstack.a(hid_usage.o)
                0x0000000010044804                ts_release
                0x0000000010044810                ts_press
 *fill*         0x0000000010044819        0x3 
 .rodata.str1.4
                0x000000001004481c      0x116 ..\..\..\..\Libraries\libs\libbtstack.a(hfp_hf.o)
                                        0x11a (size before relaxing)
 *fill*         0x0000000010044932        0x2 
 .rodata.str1.4
                0x0000000010044934       0x6d ..\..\..\..\Libraries\libs\libbtstack.a(hfp.o)
                                         0xd5 (size before relaxing)
 *fill*         0x00000000100449a1        0x3 
 .rodata        0x00000000100449a4       0x12 ..\..\..\..\Libraries\libs\libbtstack.a(hfp.o)
 *fill*         0x00000000100449b6        0x2 
 .rodata.str1.4
                0x00000000100449b8       0x51 ..\..\..\..\Libraries\libs\libbtstack.a(sm.o)
                                         0x55 (size before relaxing)
 *fill*         0x0000000010044a09        0x3 
 .rodata        0x0000000010044a0c       0x64 ..\..\..\..\Libraries\libs\libbtstack.a(sm.o)
 .rodata.str1.4
                0x0000000010044a70       0x18 ..\..\..\..\Libraries\libs\libbtstack.a(le_device_db_memory.o)
                                         0x1c (size before relaxing)
 .rodata.str1.4
                0x0000000010044a88        0x6 ..\..\..\..\Libraries\libs\libbtstack.a(btstack_chipset_inner.o)
 *fill*         0x0000000010044a8e        0x2 
 .rodata        0x0000000010044a90       0x14 ..\..\..\..\Libraries\libs\libbtstack.a(btstack_chipset_inner.o)
 .rodata        0x0000000010044aa4      0x1c8 ..\..\..\..\Libraries\libs\libbtstack.a(lm_sp.o)
 .rodata        0x0000000010044c6c      0x2f4 ..\..\..\..\Libraries\libs\libbtstack.a(lm_proc.o)
 .rodata.bb.tbl
                0x0000000010044f60       0x1e ..\..\..\..\Libraries\libs\libbtstack.a(lm_proc.o)
                0x0000000010044f60                lm_local_supp_feats
 *fill*         0x0000000010044f7e        0x2 
 .rodata        0x0000000010044f80      0x420 ..\..\..\..\Libraries\libs\libbtstack.a(lm_key.o)
 .rodata        0x00000000100453a0       0x10 ..\..\..\..\Libraries\libs\libbtstack.a(lc.o)
 .rodata.str1.4
                0x00000000100453b0        0x2 ..\..\..\..\Libraries\libs\libbtstack.a(extern_hfhs.o)
                                          0x6 (size before relaxing)
 *fill*         0x00000000100453b2        0x2 
 .rodata.str1.4
                0x00000000100453b4       0x16 ..\..\..\..\Libraries\libs\libbtstack.a(l2cap_signaling.o)
                                         0x2a (size before relaxing)
 *fill*         0x00000000100453ca        0x2 
 .rodata        0x00000000100453cc       0x58 ..\..\..\..\Libraries\libs\libbtstack.a(l2cap_signaling.o)
 .rodata        0x0000000010045424       0x7c ..\..\..\..\Libraries\libs\libbtstack.a(lm_sco.o)
 .rodata        0x00000000100454a0       0x40 ..\..\..\..\Libraries\libs\libbtstack.a(lc_util.o)
 .rodata        0x00000000100454e0      0x5dc ..\..\..\..\Libraries\libs\libbtstack.a(lc_proc.o)
 .rodata.str1.4
                0x0000000010045abc       0x6b ..\..\..\..\Libraries\libs\libbtstack.a(lc_lmppdu.o)
                                         0x9b (size before relaxing)
 *fill*         0x0000000010045b27        0x1 
 .rodata        0x0000000010045b28      0x280 ..\..\..\..\Libraries\libs\libbtstack.a(lc_lmppdu.o)
 .rodata        0x0000000010045da8       0x60 ..\..\..\..\Libraries\libs\libbtstack.a(mgr_proc.o)
 .rodata.le.mgr_cntl.tbl
                0x0000000010045e08       0xf0 ..\..\..\..\Libraries\libs\libbtstack.a(mgr_hci.o)
                0x0000000010045e08                mgr_hci_cmd_tbl
 .rodata        0x0000000010045ef8       0x1c ..\..\..\..\Libraries\libs\libbtstack.a(ll_scan.o)
 .rodata.le.ll_cntl.tbl
                0x0000000010045f14      0x1a8 ..\..\..\..\Libraries\libs\libbtstack.a(ll_proc.o)
                0x0000000010045f14                ll_msg_tbl
                0x0000000010045ff4                ll_hci_cmd_tbl
 .rodata.str1.4
                0x00000000100460bc       0x3c ..\..\..\..\Libraries\libs\libbtstack.a(ll_cntl.o)
                                         0x59 (size before relaxing)
 .rodata.le.ll_cntl.tbl
                0x00000000100460f8      0x1c8 ..\..\..\..\Libraries\libs\libbtstack.a(ll_cntl.o)
                0x00000000100460f8                ll_cntl_pdu_tbl
 *(.srodata*)
 .srodata       0x00000000100462c0        0x4 ..\..\..\..\Libraries\libs\libbtstack.a(bt_acl.o)
 .srodata       0x00000000100462c4        0x3 ..\..\..\..\Libraries\libs\libbtstack.a(extern_bt.o)
                0x00000000100462c5                cfg_bb_rf_ctl
 *fill*         0x00000000100462c7        0x1 
 .srodata       0x00000000100462c8        0x2 ..\..\..\..\Libraries\libs\libbtstack.a(btstack_link_key_db.o)
                0x00000000100462c8                link_info_page_size
 *fill*         0x00000000100462ca        0x2 
 .srodata       0x00000000100462cc        0x8 ..\..\..\..\Libraries\libs\libbtstack.a(vs_proc.o)
 .srodata       0x00000000100462d4        0x8 ..\..\..\..\Libraries\libs\libbtstack.a(hct_msg.o)
                0x00000000100462d4                hci_evt_dbg_desc_tab
 .srodata       0x00000000100462dc       0x1c ..\..\..\..\Libraries\libs\libbtstack.a(hct.o)
 .srodata       0x00000000100462f8        0x6 ..\..\..\..\Libraries\libs\libbtstack.a(hci.o)
 *fill*         0x00000000100462fe        0x2 
 .srodata       0x0000000010046300       0x10 ..\..\..\..\Libraries\libs\libbtstack.a(mgr.o)
 .srodata       0x0000000010046310        0x3 ..\..\..\..\Libraries\libs\libbtstack.a(lc_proc.o)
 *fill*         0x0000000010046313        0x1 
 .srodata       0x0000000010046314        0x8 ..\..\..\..\Libraries\libs\libbtstack.a(mgr_hci.o)
 .srodata       0x000000001004631c        0x5 ..\..\..\..\Libraries\libs\libbtstack.a(ll_adv.o)
 *(.rela*)
 .rela.text.cm_factory
                0x0000000010046321        0x0 Output\obj\Libraries\bsp\bsp_cm.o
 .rela.text.fot.cache
                0x0000000010046321        0x0 Output\obj\Libraries\bsp\bsp_cm.o
 .rela.text.fot.update
                0x0000000010046321        0x0 Output\obj\Libraries\bsp\bsp_cm.o
 .rela.text.fot_ble_disconnect_callback
                0x0000000010046321        0x0 Output\obj\Libraries\bsp\bsp_cm.o
 .rela.text.fot_ble_connect_callback
                0x0000000010046321        0x0 Output\obj\Libraries\bsp\bsp_cm.o
 .rela.text.fot_spp_connect_callback
                0x0000000010046321        0x0 Output\obj\Libraries\bsp\bsp_cm.o
 .rela.text.fot_spp_disconnect_callback
                0x0000000010046321        0x0 Output\obj\Libraries\bsp\bsp_cm.o
 .rela.com_text.fot
                0x0000000010046321        0x0 Output\obj\Libraries\bsp\bsp_cm.o
 .rela.text.bsp.param
                0x0000000010046321        0x0 Output\obj\Libraries\bsp\bsp_cm.o
 .rela.text.bsp.sys.init
                0x0000000010046321        0x0 Output\obj\Libraries\bsp\bsp_cm.o
 .rela.com_text.timer
                0x0000000010046321        0x0 Output\obj\Libraries\bsp\bsp_cm.o
 .rela.text.bsp_get_xosc_xcfg
                0x0000000010046321        0x0 Output\obj\Libraries\bsp\bsp_cm.o
 .rela.text.gatt_callback_fota
                0x0000000010046321        0x0 Output\obj\Libraries\bsp\bsp_cm.o
 .rela.text.gatt_callback_app
                0x0000000010046321        0x0 Output\obj\Libraries\bsp\bsp_cm.o
 .rela.text.ble_get_scan_data
                0x0000000010046321        0x0 Output\obj\Libraries\bsp\bsp_cm.o
 .rela.text.ble_get_adv_data
                0x0000000010046321        0x0 Output\obj\Libraries\bsp\bsp_cm.o
 .rela.text.ble_txpkt_init
                0x0000000010046321        0x0 Output\obj\Libraries\bsp\bsp_cm.o
 .rela.text.ble_send_packet1
                0x0000000010046321        0x0 Output\obj\Libraries\bsp\bsp_cm.o
 .rela.text.ble_send_packet2
                0x0000000010046321        0x0 Output\obj\Libraries\bsp\bsp_cm.o
 .rela.text.ble_read_value
                0x0000000010046321        0x0 Output\obj\Libraries\bsp\bsp_cm.o
 .rela.text.ble_fot_send_packet
                0x0000000010046321        0x0 Output\obj\Libraries\bsp\bsp_cm.o
 .rela.text.ble_app_gatts_service_init
                0x0000000010046321        0x0 Output\obj\Libraries\bsp\bsp_cm.o
 .rela.text.ble_get_local_bd_addr
                0x0000000010046321        0x0 Output\obj\Libraries\bsp\bsp_cm.o
 .rela.text.ble_enter_transmit
                0x0000000010046321        0x0 Output\obj\Libraries\bsp\bsp_cm.o
 .rela.text.ble_exit_transmit
                0x0000000010046321        0x0 Output\obj\Libraries\bsp\bsp_cm.o
 .rela.text.ble_disconnect_callback
                0x0000000010046321        0x0 Output\obj\Libraries\bsp\bsp_cm.o
 .rela.text.ble_connect_callback
                0x0000000010046321        0x0 Output\obj\Libraries\bsp\bsp_cm.o
 .rela.text.bt_get_local_name
                0x0000000010046321        0x0 Output\obj\Libraries\bsp\bsp_cm.o
 .rela.text.bt_clr_all_link_info
                0x0000000010046321        0x0 Output\obj\Libraries\bsp\bsp_cm.o
 .rela.text.bt_get_local_bd_addr
                0x0000000010046321        0x0 Output\obj\Libraries\bsp\bsp_cm.o
 .rela.text.bt_get_link_info
                0x0000000010046321        0x0 Output\obj\Libraries\bsp\bsp_cm.o
 .rela.text.bt_put_link_info
                0x0000000010046321        0x0 Output\obj\Libraries\bsp\bsp_cm.o
 .rela.text.bt_get_ext_link_info
                0x0000000010046321        0x0 Output\obj\Libraries\bsp\bsp_cm.o
 .rela.text.bt_put_ext_link_info
                0x0000000010046321        0x0 Output\obj\Libraries\bsp\bsp_cm.o
 .rela.text.bt_sync_link_info
                0x0000000010046321        0x0 Output\obj\Libraries\bsp\bsp_cm.o
 .rela.text.bsp_bt_hid_screen_left
                0x0000000010046321        0x0 Output\obj\Libraries\bsp\bsp_cm.o
 .rela.text.bsp_bt_hid_screen_right
                0x0000000010046321        0x0 Output\obj\Libraries\bsp\bsp_cm.o
 .rela.data     0x0000000010046321        0x0 Output\obj\Libraries\bsp\bsp_cm.o
 .rela.text.bt_init_lib
                0x0000000010046321        0x0 Output\obj\Libraries\bsp\bsp_cm.o
 .rela.text.spp_txpkt_init
                0x0000000010046321        0x0 Output\obj\Libraries\bsp\bsp_cm.o
 .rela.text.spp_connect_callback
                0x0000000010046321        0x0 Output\obj\Libraries\bsp\bsp_cm.o
 .rela.text.spp_disconnect_callback
                0x0000000010046321        0x0 Output\obj\Libraries\bsp\bsp_cm.o
 .rela.text.spp_rx_callback
                0x0000000010046321        0x0 Output\obj\Libraries\bsp\bsp_cm.o
 .rela.text.gpio_pic_config
                0x0000000010046321        0x0 Output\obj\Libraries\bsp\bsp_cm.o
 .rela.text.tmr_pic_config
                0x0000000010046321        0x0 Output\obj\Libraries\bsp\bsp_cm.o
 .rela.com_text.isr
                0x0000000010046321        0x0 Output\obj\Libraries\bsp\bsp_cm.o
 .rela.text.timer3_cap_init
                0x0000000010046321        0x0 Output\obj\Libraries\bsp\bsp_cm.o
 .rela.text.timer3_capture_example
                0x0000000010046321        0x0 Output\obj\Libraries\bsp\bsp_cm.o
 .rela.text.timer4_pwm_init
                0x0000000010046321        0x0 Output\obj\Libraries\bsp\bsp_cm.o
 .rela.text.getcfg_vddbt_sel
                0x0000000010046321        0x0 Output\obj\Libraries\bsp\bsp_cm.o
 .rela.text.getcfg_vddio_sel
                0x0000000010046321        0x0 Output\obj\Libraries\bsp\bsp_cm.o
 .rela.text.getcfg_vddbt_capless_en
                0x0000000010046321        0x0 Output\obj\Libraries\bsp\bsp_cm.o
 .rela.text.startup.main
                0x0000000010046321        0x0 Output\obj\Libraries\bsp\bsp_cm.o
 .rela.text.pll_vco_band_trimming
                0x0000000010046321        0x0 Output\obj\Libraries\bsp\bsp_cm.o
 .rela.com_text.dac
                0x0000000010046321        0x0 Output\obj\Libraries\bsp\bsp_cm.o
 .rela.text.adpll_divider_update_do
                0x0000000010046321        0x0 Output\obj\Libraries\bsp\bsp_cm.o
 .rela.text.adpll_divider_update
                0x0000000010046321        0x0 Output\obj\Libraries\bsp\bsp_cm.o
 .rela.text.adpll_init
                0x0000000010046321        0x0 Output\obj\Libraries\bsp\bsp_cm.o
 .rela.text.spires
                0x0000000010046321        0x0 Output\obj\Libraries\bsp\bsp_cm.o
 .rela.text.cm_loadpage
                0x0000000010046321        0x0 Output\obj\Libraries\bsp\bsp_cm.o
 .rela.text.cm_next_freepage
                0x0000000010046321        0x0 Output\obj\Libraries\bsp\bsp_cm.o
 .rela.text.cm_movepage
                0x0000000010046321        0x0 Output\obj\Libraries\bsp\bsp_cm.o
 .rela.text.cm_move_allpages
                0x0000000010046321        0x0 Output\obj\Libraries\bsp\bsp_cm.o
 .rela.text.cm_release
                0x0000000010046321        0x0 Output\obj\Libraries\bsp\bsp_cm.o
 .rela.text.cm_savepage
                0x0000000010046321        0x0 Output\obj\Libraries\bsp\bsp_cm.o
 .rela.text.cm_check_loadpage
                0x0000000010046321        0x0 Output\obj\Libraries\bsp\bsp_cm.o
 .rela.text.cm_sync
                0x0000000010046321        0x0 Output\obj\Libraries\bsp\bsp_cm.o
 .rela.text.cm_release_all
                0x0000000010046321        0x0 Output\obj\Libraries\bsp\bsp_cm.o
 .rela.text.cm_read
                0x0000000010046321        0x0 Output\obj\Libraries\bsp\bsp_cm.o
 .rela.text.cm_read8
                0x0000000010046321        0x0 Output\obj\Libraries\bsp\bsp_cm.o
 .rela.text.cm_read16
                0x0000000010046321        0x0 Output\obj\Libraries\bsp\bsp_cm.o
 .rela.text.cm_read32
                0x0000000010046321        0x0 Output\obj\Libraries\bsp\bsp_cm.o
 .rela.text.cm_write
                0x0000000010046321        0x0 Output\obj\Libraries\bsp\bsp_cm.o
 .rela.text.cm_write8
                0x0000000010046321        0x0 Output\obj\Libraries\bsp\bsp_cm.o
 .rela.text.cm_write16
                0x0000000010046321        0x0 Output\obj\Libraries\bsp\bsp_cm.o
 .rela.text.cm_write32
                0x0000000010046321        0x0 Output\obj\Libraries\bsp\bsp_cm.o
 .rela.text.cm_clear
                0x0000000010046321        0x0 Output\obj\Libraries\bsp\bsp_cm.o
 .rela.text.cm_init
                0x0000000010046321        0x0 Output\obj\Libraries\bsp\bsp_cm.o
 .rela.com_text.spiflash
                0x0000000010046321        0x0 Output\obj\Libraries\bsp\bsp_cm.o
 .rela.text.xcfg_init
                0x0000000010046321        0x0 Output\obj\Libraries\bsp\bsp_cm.o
 .rela.text.sd_disable_user
                0x0000000010046321        0x0 Output\obj\Libraries\bsp\bsp_cm.o
 .rela.text.device.init
                0x0000000010046321        0x0 Output\obj\Libraries\bsp\bsp_cm.o
 .rela.text.device
                0x0000000010046321        0x0 Output\obj\Libraries\bsp\bsp_cm.o
 .rela.com_text.sd.isr
                0x0000000010046321        0x0 Output\obj\Libraries\bsp\bsp_cm.o
 .rela.com_text.sd.api
                0x0000000010046321        0x0 Output\obj\Libraries\bsp\bsp_cm.o
 .rela.text.fs_lock
                0x0000000010046321        0x0 Output\obj\Libraries\bsp\bsp_cm.o
 .rela.text.fs_unlock
                0x0000000010046321        0x0 Output\obj\Libraries\bsp\bsp_cm.o
 .rela.com_text.exception.hook
                0x0000000010046321        0x0 Output\obj\Libraries\bsp\bsp_cm.o
 .rela.com_text.exception
                0x0000000010046321        0x0 Output\obj\Libraries\bsp\bsp_cm.o
 .rela.com_text.delay
                0x0000000010046321        0x0 Output\obj\Libraries\bsp\bsp_cm.o
 .rela.com_text.exception.do
                0x0000000010046321        0x0 Output\obj\Libraries\bsp\bsp_cm.o
 .rela.com_text.ledseg
                0x0000000010046321        0x0 Output\obj\Libraries\bsp\bsp_cm.o
 .rela.text.platform_main
                0x0000000010046321        0x0 Output\obj\Libraries\bsp\bsp_cm.o
 .rela.text.main_startup
                0x0000000010046321        0x0 Output\obj\Libraries\bsp\bsp_cm.o
 .rela.text.compiler
                0x0000000010046321        0x0 Output\obj\Libraries\bsp\bsp_cm.o
 .rela.com_text.irq
                0x0000000010046321        0x0 Output\obj\Libraries\bsp\bsp_cm.o
 .rela.text.sys_irq_init
                0x0000000010046321        0x0 Output\obj\Libraries\bsp\bsp_cm.o
 .rela.text.timer0_init
                0x0000000010046321        0x0 Output\obj\Libraries\bsp\bsp_cm.o
 .rela.text.soft_irq_init
                0x0000000010046321        0x0 Output\obj\Libraries\bsp\bsp_cm.o
 .rela.text.bthw_irq_init
                0x0000000010046321        0x0 Output\obj\Libraries\bsp\bsp_cm.o
 .rela.text.sd0_irq_init
                0x0000000010046321        0x0 Output\obj\Libraries\bsp\bsp_cm.o
 .rela.text.usb_irq_init
                0x0000000010046321        0x0 Output\obj\Libraries\bsp\bsp_cm.o
 .rela.text.timer1_irq_init
                0x0000000010046321        0x0 Output\obj\Libraries\bsp\bsp_cm.o
 .rela.com_text.tws.isr
                0x0000000010046321        0x0 Output\obj\Libraries\bsp\bsp_cm.o
 .rela.text.aubuf_irq_init
                0x0000000010046321        0x0 Output\obj\Libraries\bsp\bsp_cm.o
 .rela.text.huart_irq_init
                0x0000000010046321        0x0 Output\obj\Libraries\bsp\bsp_cm.o
 .rela.text.watch_point_set
                0x0000000010046321        0x0 Output\obj\Libraries\bsp\bsp_cm.o
 .rela.text.thread_main_entry
                0x0000000010046321        0x0 Output\obj\Libraries\bsp\bsp_cm.o
 .rela.text.thread_idle_create
                0x0000000010046321        0x0 Output\obj\Libraries\bsp\bsp_cm.o
 .rela.text.startup.init
                0x0000000010046321        0x0 Output\obj\Libraries\bsp\bsp_cm.o
 .rela.reset    0x0000000010046321        0x0 Output\obj\Libraries\bsp\bsp_cm.o
 .rela.vector   0x0000000010046321        0x0 Output\obj\Libraries\bsp\bsp_cm.o
 .rela.com_text.debug
                0x0000000010046321        0x0 Output\obj\Libraries\bsp\bsp_cm.o
 .rela.text.fot_init
                0x0000000010046321        0x0 Output\obj\Libraries\bsp\bsp_cm.o
 .rela.text.lock_code_bt_sleep
                0x0000000010046321        0x0 Output\obj\Libraries\bsp\bsp_cm.o
 .rela.text.lock_code_pwrsave
                0x0000000010046321        0x0 Output\obj\Libraries\bsp\bsp_cm.o
 .rela.text.lock_code_charge
                0x0000000010046321        0x0 Output\obj\Libraries\bsp\bsp_cm.o
 .rela.text.lock_code_usbdev
                0x0000000010046321        0x0 Output\obj\Libraries\bsp\bsp_cm.o
 .rela.text.load_code_btdec
                0x0000000010046321        0x0 Output\obj\Libraries\bsp\bsp_cm.o
 .rela.text.load_code_bt_voice
                0x0000000010046321        0x0 Output\obj\Libraries\bsp\bsp_cm.o
 .rela.text.lock_code_sniff
                0x0000000010046321        0x0 Output\obj\Libraries\bsp\bsp_cm.o
 .rela.text.lock_code_huart
                0x0000000010046321        0x0 Output\obj\Libraries\bsp\bsp_cm.o
 .rela.text.lock_code_bb_test
                0x0000000010046321        0x0 Output\obj\Libraries\bsp\bsp_cm.o
 .rela.text.load_code_fota
                0x0000000010046321        0x0 Output\obj\Libraries\bsp\bsp_cm.o
 .rela.text.patch_init
                0x0000000010046321        0x0 Output\obj\Libraries\bsp\bsp_cm.o
 .rela.text.vddio_voltage_configure
                0x0000000010046321        0x0 Output\obj\Libraries\bsp\bsp_cm.o
 .rela.text.vddbt_voltage_configure
                0x0000000010046321        0x0 Output\obj\Libraries\bsp\bsp_cm.o
 .rela.text.pmu_voltage_configure
                0x0000000010046321        0x0 Output\obj\Libraries\bsp\bsp_cm.o
 .rela.text.pmu_init
                0x0000000010046321        0x0 Output\obj\Libraries\bsp\bsp_cm.o
 .rela.com_text.voltage.trim
                0x0000000010046321        0x0 Output\obj\Libraries\bsp\bsp_cm.o
 .rela.text.sys_clk
                0x0000000010046321        0x0 Output\obj\Libraries\bsp\bsp_cm.o
 .rela.text.set_peripherals_clkdiv
                0x0000000010046321        0x0 Output\obj\Libraries\bsp\bsp_cm.o
 .rela.com_huart.text
                0x0000000010046321        0x0 Output\obj\Libraries\bsp\bsp_cm.o
 .rela.com_text.thread.usb
                0x0000000010046321        0x0 Output\obj\Libraries\bsp\bsp_cm.o
 .rela.bt_voice.plc
                0x0000000010046321        0x0 Output\obj\Libraries\bsp\bsp_cm.o
 .rela.text.stack.api
                0x0000000010046321        0x0 Output\obj\Libraries\bsp\bsp_cm.o
 .rela.com_text.stack.run_loop
                0x0000000010046321        0x0 Output\obj\Libraries\bsp\bsp_cm.o
 .rela.com_text.bb.bthw
                0x0000000010046321        0x0 Output\obj\Libraries\bsp\bsp_cm.o
 .rela.text     0x0000000010046321        0x0 Output\obj\Libraries\bsp\bsp_cm.o
 .rela.com_text.bb.nanos
                0x0000000010046321        0x0 Output\obj\Libraries\bsp\bsp_cm.o
 .rela.com_text.bb.patch
                0x0000000010046321        0x0 Output\obj\Libraries\bsp\bsp_cm.o
 .rela.com_text.ble.isr.con
                0x0000000010046321        0x0 Output\obj\Libraries\bsp\bsp_cm.o
 .rela.com_text.bb.isr.timer
                0x0000000010046321        0x0 Output\obj\Libraries\bsp\bsp_cm.o
 .rela.com_text.bb.isr
                0x0000000010046321        0x0 Output\obj\Libraries\bsp\bsp_cm.o
 .rela.sleep_text.bb
                0x0000000010046321        0x0 Output\obj\Libraries\bsp\bsp_cm.o
 .rela.com_text.bb.sleep
                0x0000000010046321        0x0 Output\obj\Libraries\bsp\bsp_cm.o
 .rela.com_text.bb.btisr
                0x0000000010046321        0x0 Output\obj\Libraries\bsp\bsp_cm.o
 .rela.rodata   0x0000000010046321        0x0 Output\obj\Libraries\bsp\bsp_cm.o
 .rela.com_text.pp.send_pkt
                0x0000000010046321        0x0 Output\obj\Libraries\bsp\bsp_cm.o
 .rela.com_text.spp.tx
                0x0000000010046321        0x0 Output\obj\Libraries\bsp\bsp_cm.o
 .rela.com_text.spp.send_req
                0x0000000010046321        0x0 Output\obj\Libraries\bsp\bsp_cm.o
 .rela.com_text.spp.event_send
                0x0000000010046321        0x0 Output\obj\Libraries\bsp\bsp_cm.o
 .rela.com_text.spp.rx_set_new_credit
                0x0000000010046321        0x0 Output\obj\Libraries\bsp\bsp_cm.o
 .rela.text.stack.spp.handler
                0x0000000010046321        0x0 Output\obj\Libraries\bsp\bsp_cm.o
 .rela.text.stack.sdp.util
                0x0000000010046321        0x0 Output\obj\Libraries\bsp\bsp_cm.o
 .rela.text.stack.sdp.server
                0x0000000010046321        0x0 Output\obj\Libraries\bsp\bsp_cm.o
 .rela.text.stack.setup
                0x0000000010046321        0x0 Output\obj\Libraries\bsp\bsp_cm.o
 .rela.text.stack.sdp.server_add
                0x0000000010046321        0x0 Output\obj\Libraries\bsp\bsp_cm.o
 .rela.text.stack.sdp.server_rmv
                0x0000000010046321        0x0 Output\obj\Libraries\bsp\bsp_cm.o
 .rela.text.stack.rfcomm
                0x0000000010046321        0x0 Output\obj\Libraries\bsp\bsp_cm.o
 .rela.text.stack.link_key
                0x0000000010046321        0x0 Output\obj\Libraries\bsp\bsp_cm.o
 .rela.text.stack.run_loop
                0x0000000010046321        0x0 Output\obj\Libraries\bsp\bsp_cm.o
 .rela.com_text.stack.ticks
                0x0000000010046321        0x0 Output\obj\Libraries\bsp\bsp_cm.o
 .rela.text.stack.memory
                0x0000000010046321        0x0 Output\obj\Libraries\bsp\bsp_cm.o
 .rela.text.stack.linkctrl
                0x0000000010046321        0x0 Output\obj\Libraries\bsp\bsp_cm.o
 .rela.com_text.ble.send_pkt
                0x0000000010046321        0x0 Output\obj\Libraries\bsp\bsp_cm.o
 .rela.text.att.r_cb
                0x0000000010046321        0x0 Output\obj\Libraries\bsp\bsp_cm.o
 .rela.text.att.w_cb
                0x0000000010046321        0x0 Output\obj\Libraries\bsp\bsp_cm.o
 .rela.com_text.stack.ble.mtu
                0x0000000010046321        0x0 Output\obj\Libraries\bsp\bsp_cm.o
 .rela.text.ble.notify_handle
                0x0000000010046321        0x0 Output\obj\Libraries\bsp\bsp_cm.o
 .rela.text.ble.att
                0x0000000010046321        0x0 Output\obj\Libraries\bsp\bsp_cm.o
 .rela.text.ble.hci
                0x0000000010046321        0x0 Output\obj\Libraries\bsp\bsp_cm.o
 .rela.text.stack.handler
                0x0000000010046321        0x0 Output\obj\Libraries\bsp\bsp_cm.o
 .rela.text.stack.ble.sm
                0x0000000010046321        0x0 Output\obj\Libraries\bsp\bsp_cm.o
 .rela.text.stack.ble.setup
                0x0000000010046321        0x0 Output\obj\Libraries\bsp\bsp_cm.o
 .rela.text.stack.status
                0x0000000010046321        0x0 Output\obj\Libraries\bsp\bsp_cm.o
 .rela.rodata.stack.api
                0x0000000010046321        0x0 Output\obj\Libraries\bsp\bsp_cm.o
 .rela.text.stack.api.hid_con
                0x0000000010046321        0x0 Output\obj\Libraries\bsp\bsp_cm.o
 .rela.text.stack.api.hid_disc
                0x0000000010046321        0x0 Output\obj\Libraries\bsp\bsp_cm.o
 .rela.text.stack.api.hid_send
                0x0000000010046321        0x0 Output\obj\Libraries\bsp\bsp_cm.o
 .rela.text.stack.le.api
                0x0000000010046321        0x0 Output\obj\Libraries\bsp\bsp_cm.o
 .rela.text.bb.vs.fcc
                0x0000000010046321        0x0 Output\obj\Libraries\bsp\bsp_cm.o
 .rela.com_text.isr.txrx
                0x0000000010046321        0x0 Output\obj\Libraries\bsp\bsp_cm.o
 .rela.com_text.bt21.isr
                0x0000000010046321        0x0 Output\obj\Libraries\bsp\bsp_cm.o
 .rela.text.ble.var.init
                0x0000000010046321        0x0 Output\obj\Libraries\bsp\bsp_cm.o
 .rela.text.bb.ble.adv0
                0x0000000010046321        0x0 Output\obj\Libraries\bsp\bsp_cm.o
 .rela.text.stk.l2cap.txreq
                0x0000000010046321        0x0 Output\obj\Libraries\bsp\bsp_cm.o
 .rela.text.stack.handler.l2cap
                0x0000000010046321        0x0 Output\obj\Libraries\bsp\bsp_cm.o
 .rela.text.stack.l2cap
                0x0000000010046321        0x0 Output\obj\Libraries\bsp\bsp_cm.o
 .rela.text.stack.hci
                0x0000000010046321        0x0 Output\obj\Libraries\bsp\bsp_cm.o
 .rela.text.stack.hci_init
                0x0000000010046321        0x0 Output\obj\Libraries\bsp\bsp_cm.o
 .rela.com_text.stack.hci
                0x0000000010046321        0x0 Output\obj\Libraries\bsp\bsp_cm.o
 .rela.text.stack.hci_send
                0x0000000010046321        0x0 Output\obj\Libraries\bsp\bsp_cm.o
 .rela.text.stack.hci.run
                0x0000000010046321        0x0 Output\obj\Libraries\bsp\bsp_cm.o
 .rela.text.stack.handler.event
                0x0000000010046321        0x0 Output\obj\Libraries\bsp\bsp_cm.o
 .rela.com_text.stack.hci_recv
                0x0000000010046321        0x0 Output\obj\Libraries\bsp\bsp_cm.o
 .rela.text.stack.hfp.api1
                0x0000000010046321        0x0 Output\obj\Libraries\bsp\bsp_cm.o
 .rela.text.bb.lm.inq.start
                0x0000000010046321        0x0 Output\obj\Libraries\bsp\bsp_cm.o
 .rela.text.le.ll_cntl
                0x0000000010046321        0x0 Output\obj\Libraries\bsp\bsp_cm.o
 .rela.text.le.ll_cntl.start
                0x0000000010046321        0x0 Output\obj\Libraries\bsp\bsp_cm.o
 .rela.text.le.ll_cntl.state
                0x0000000010046321        0x0 Output\obj\Libraries\bsp\bsp_cm.o
 .rela.text.le.ll_cntl.stop
                0x0000000010046321        0x0 Output\obj\Libraries\bsp\bsp_cm.o
 .rela.text.le.mgr
                0x0000000010046321        0x0 Output\obj\Libraries\bsp\bsp_cm.o
 .rela.rodata.le.mgr_cntl.tbl
                0x0000000010046321        0x0 Output\obj\Libraries\bsp\bsp_cm.o
 .rela.text.le.ll_scan
                0x0000000010046321        0x0 Output\obj\Libraries\bsp\bsp_cm.o
 .rela.text.le.ll_adv
                0x0000000010046321        0x0 Output\obj\Libraries\bsp\bsp_cm.o
 .rela.text.le.ll_adv.con
                0x0000000010046321        0x0 Output\obj\Libraries\bsp\bsp_cm.o
 .rela.com_rodata.bb.tbl
                0x0000000010046321        0x0 Output\obj\Libraries\bsp\bsp_cm.o
 .rela.rodata.le.ll_cntl.tbl
                0x0000000010046321        0x0 Output\obj\Libraries\bsp\bsp_cm.o
 .rela.text.le.ll_cntl.pdu
                0x0000000010046321        0x0 Output\obj\Libraries\bsp\bsp_cm.o
 .rela.text.le.ll_cntl.send
                0x0000000010046321        0x0 Output\obj\Libraries\bsp\bsp_cm.o
 .rela.com_text.usbdev
                0x0000000010046321        0x0 Output\obj\Libraries\bsp\bsp_cm.o
 .rela.usbdev.com
                0x0000000010046321        0x0 Output\obj\Libraries\bsp\bsp_cm.o
 .rela.com_text.bulkep
                0x0000000010046321        0x0 Output\obj\Libraries\bsp\bsp_cm.o
 .rela.text.udp_init
                0x0000000010046321        0x0 Output\obj\Libraries\bsp\bsp_cm.o
 .rela.text.usb_device_init
                0x0000000010046321        0x0 Output\obj\Libraries\bsp\bsp_cm.o
 .rela.text.usb_device_enter
                0x0000000010046321        0x0 Output\obj\Libraries\bsp\bsp_cm.o
 .rela.com_text.usb.device
                0x0000000010046321        0x0 Output\obj\Libraries\bsp\bsp_cm.o
 .rela.text.usb.host.init
                0x0000000010046321        0x0 Output\obj\Libraries\bsp\bsp_cm.o
 .rela.com_text.usb.host
                0x0000000010046321        0x0 Output\obj\Libraries\bsp\bsp_cm.o
 .rela.text.udisk_read
                0x0000000010046321        0x0 Output\obj\Libraries\bsp\bsp_cm.o
 .rela.text.udisk_write
                0x0000000010046321        0x0 Output\obj\Libraries\bsp\bsp_cm.o
 .rela.text.do_transfer
                0x0000000010046321        0x0 Output\obj\Libraries\bsp\bsp_cm.o
 .rela.text.do_receive
                0x0000000010046321        0x0 Output\obj\Libraries\bsp\bsp_cm.o
 .rela.text.uhs_start
                0x0000000010046321        0x0 Output\obj\Libraries\bsp\bsp_cm.o
 .rela.text.uhs_init
                0x0000000010046321        0x0 Output\obj\Libraries\bsp\bsp_cm.o
 .rela.text.usb_init
                0x0000000010046321        0x0 Output\obj\Libraries\bsp\bsp_cm.o
 .rela.text.usb_host_enter
                0x0000000010046321        0x0 Output\obj\Libraries\bsp\bsp_cm.o
 .rela.text.uhe_start
                0x0000000010046321        0x0 Output\obj\Libraries\bsp\bsp_cm.o
                0x0000000010046321        0x4 LONG 0x0
                0x0000000010046400                . = ALIGN (0x200)
 *fill*         0x0000000010046325       0xdb 

.stack          0x0000000000010800      0x400
                0x0000000000010800                __irq_stack_start = .
                0x0000000000000400                . = 0x400
 *fill*         0x0000000000010800      0x400 
                0x0000000000010c00                __irq_stack = .
                0x0000000000000400                __irq_stack_size = (__irq_stack - __irq_stack_start)

.bss            0x0000000000013c00     0x17a8
                0x0000000000013c00                __bss_start = .
 *(COMMON)
 COMMON         0x0000000000013c00       0x22 Output\obj\Libraries\bsp\bsp_fot.o
                0x0000000000013c00                fot_var
 *fill*         0x0000000000013c22        0x2 
 COMMON         0x0000000000013c24       0xb2 Output\obj\Libraries\bsp\bsp_sys.o
                0x0000000000013c24                ticks_50ms
                0x0000000000013c28                xcfg_cb
 *(.bss*)
 *fill*         0x0000000000013cd6        0x2 
 .bss           0x0000000000013cd8      0x22c ..\..\..\..\Libraries\libs\libplatform.a(cm.o)
 .bss           0x0000000000013f04       0xa0 ..\..\..\..\Libraries\libs\libplatform.a(main.o)
                0x0000000000013f04                cpu_gprs
                0x0000000000013f84                sys
 .bss.irq_tbl   0x0000000000013fa4       0x84 ..\..\..\..\Libraries\libs\libplatform.a(interrupt.o)
                0x0000000000013fa4                tbl_irq_vector
                0x0000000000014024                irq_mask
 .bss           0x0000000000014028       0x28 ..\..\..\..\Libraries\libs\libplatform.a(startup.o)
 .bss           0x0000000000014050       0x20 ..\..\..\..\Libraries\libs\libplatform.a(fot_update.o)
 .bss           0x0000000000014070       0x78 ..\..\..\..\Libraries\libs\libplatform.a(lock.o)
 .bss           0x00000000000140e8        0xc ..\..\..\..\Libraries\libs\libplatform.a(voltage_trim.o)
                0x00000000000140e8                sys_trim
 .bss           0x00000000000140f4        0x9 ..\..\..\..\Libraries\libs\libbtstack.a(bb.o)
                0x00000000000140f4                rf_api
 *fill*         0x00000000000140fd        0x3 
 .bss           0x0000000000014100       0x3e ..\..\..\..\Libraries\libs\libbtstack.a(btstack_link_key_db.o)
 *fill*         0x000000000001413e        0x2 
 .bss           0x0000000000014140      0x4fc ..\..\..\..\Libraries\libs\libbtstack.a(btstack_memory.o)
 .bss           0x000000000001463c       0x48 ..\..\..\..\Libraries\libs\libbtstack.a(btstack_api.o)
                0x000000000001463c                btstack_cb
                0x0000000000014648                btstack_st
 .bss           0x0000000000014684      0x184 ..\..\..\..\Libraries\libs\libbtstack.a(bb_sche.o)
                0x0000000000014684                ss_params
 .bss           0x0000000000014808        0xc ..\..\..\..\Libraries\libs\libbtstack.a(aes.o)
                0x0000000000014808                aes_env
 .bss           0x0000000000014814       0x24 ..\..\..\..\Libraries\libs\libbtstack.a(hct_tl.o)
 .bss           0x0000000000014838       0x26 ..\..\..\..\Libraries\libs\libbtstack.a(bc.o)
                0x0000000000014838                bc_env
 *fill*         0x000000000001485e        0x2 
 .bss           0x0000000000014860       0x40 ..\..\..\..\Libraries\libs\libbtstack.a(l2cap_test.o)
                0x0000000000014860                vd_tx
 .bss           0x00000000000148a0       0x10 ..\..\..\..\Libraries\libs\libbtstack.a(sm.o)
 .bss           0x00000000000148b0       0xc0 ..\..\..\..\Libraries\libs\libbtstack.a(lm_sp.o)
 .bss           0x0000000000014970      0x100 ..\..\..\..\Libraries\libs\libbtstack.a(ble_buf.o)
 .bss           0x0000000000014a70      0x21c ..\..\..\..\Libraries\libs\libbtstack.a(ll_proc.o)
 .bss           0x0000000000014c8c       0x24 ..\..\..\..\Libraries\libs\libdrivers.a(usb_device_ep.o)
                0x0000000000014c8c                eps
 *(.sbss*)
 .sbss          0x0000000000014cb0        0x4 Output\obj\Libraries\bsp\bsp_fot.o
 .sbss          0x0000000000014cb4       0x1e Output\obj\Libraries\BT\ble\ab_link\app.o
                0x0000000000014cb8                str
 .sbss          0x0000000000014cd2        0xc Output\obj\Libraries\BT\spp\bt.o
                0x0000000000014cd2                cfg_bt_hid_type
                0x0000000000014cd4                cfg_bt_support_codec
                0x0000000000014cd6                cfg_bt_simple_pair_mode
                0x0000000000014cd7                cfg_bt_scan_ctrl_mode
                0x0000000000014cd8                cfg_bt_work_mode
                0x0000000000014cd9                cfg_ble_page_rssi_thr
                0x0000000000014cda                cfg_ble_page_txpwr
                0x0000000000014cdb                cfg_bt_inq_txpwr
                0x0000000000014cdc                cfg_bt_page_txpwr
                0x0000000000014cdd                cfg_bt_rf_def_txpwr
 .sbss          0x0000000000014cde        0x2 Output\obj\Libraries\BT\spp\spp.o
                0x0000000000014cde                SPP_CreditCount
                0x0000000000014cdf                BtFlowControl_start
 .sbss          0x0000000000014ce0       0x18 Output\obj\Examples\TIMER\TIM_Capture\Source\timer_capture.o
                0x0000000000014cec                TMR3_CAP_VAL_L
                0x0000000000014cf0                TMR3_CAP_VAL_H
                0x0000000000014cf4                TMR3_CAP_STA
 .sbss          0x0000000000014cf8        0x8 ..\..\..\..\Libraries\libs\libplatform.a(audio.o)
                0x0000000000014cfc                aux_cur_gain
 .sbss          0x0000000000014d00        0x8 ..\..\..\..\Libraries\libs\libplatform.a(os_flash.o)
                0x0000000000014d00                spi_baud_w
                0x0000000000014d04                spi_baud_r
 .sbss          0x0000000000014d08        0xc ..\..\..\..\Libraries\libs\libplatform.a(interrupt.o)
                0x0000000000014d08                tmr5ms_cnt
                0x0000000000014d0c                ms_tick
                0x0000000000014d10                tmr0_counter
 .sbss          0x0000000000014d14       0x3c ..\..\..\..\Libraries\libs\libplatform.a(startup.o)
                0x0000000000014d14                user_timer_isr_en
                0x0000000000014d18                bt_timer_isr_en
                0x0000000000014d1c                pmutex_pff
                0x0000000000014d20                pmutex_bt_sta
                0x0000000000014d24                pmutex_math
                0x0000000000014d28                pmutex_dac
                0x0000000000014d2c                pmutex_uart
                0x0000000000014d30                pmutex_clk
                0x0000000000014d34                pmutex_cm
                0x0000000000014d38                pmq_usb
                0x0000000000014d3c                pmq_btstack
                0x0000000000014d40                psem_sd
                0x0000000000014d44                psem_aubuf
                0x0000000000014d48                psem_btstack
                0x0000000000014d4c                psem_bthw
 .sbss          0x0000000000014d50        0xc ..\..\..\..\Libraries\libs\libplatform.a(fot_update.o)
 .sbss          0x0000000000014d5c        0x4 ..\..\..\..\Libraries\libs\libplatform.a(bt.o)
                0x0000000000014d5c                bt_thread_res
 .sbss          0x0000000000014d60        0x1 ..\..\..\..\Libraries\libs\libbtstack.a(bb.o)
 .sbss          0x0000000000014d61        0x1 ..\..\..\..\Libraries\libs\libbtstack.a(platform.o)
                0x0000000000014d61                cfg_bt_spp_rx_flow_ctrl_en
 .sbss          0x0000000000014d62        0x6 ..\..\..\..\Libraries\libs\libbtstack.a(extern_tws.o)
                0x0000000000014d62                cfg_bt_tws_limit_pair_time
                0x0000000000014d64                cfg_bt_tws_feat
                0x0000000000014d66                cfg_bt_tws_pair_mode
 .sbss          0x0000000000014d68        0x9 ..\..\..\..\Libraries\libs\libbtstack.a(extern_bt.o)
                0x0000000000014d6a                cfg_bt_tws_mode
 *fill*         0x0000000000014d71        0x3 
 .sbss          0x0000000000014d74        0x4 ..\..\..\..\Libraries\libs\libbtstack.a(sdp_server.o)
 .sbss          0x0000000000014d78       0x13 ..\..\..\..\Libraries\libs\libbtstack.a(rfcomm.o)
                0x0000000000014d80                rfcomm_channels
                0x0000000000014d84                rfcomm_multiplexers
 *fill*         0x0000000000014d8b        0x1 
 .sbss          0x0000000000014d8c        0x5 ..\..\..\..\Libraries\libs\libbtstack.a(btstack_run_loop.o)
 *fill*         0x0000000000014d91        0x3 
 .sbss          0x0000000000014d94       0x20 ..\..\..\..\Libraries\libs\libbtstack.a(btstack_memory.o)
 .sbss          0x0000000000014db4       0x1f ..\..\..\..\Libraries\libs\libbtstack.a(att_server.o)
 *fill*         0x0000000000014dd3        0x1 
 .sbss          0x0000000000014dd4        0xc ..\..\..\..\Libraries\libs\libbtstack.a(att_dispatch.o)
 .sbss          0x0000000000014de0       0x10 ..\..\..\..\Libraries\libs\libbtstack.a(att_db.o)
 .sbss          0x0000000000014df0        0xd ..\..\..\..\Libraries\libs\libbtstack.a(btstack_main.o)
 *fill*         0x0000000000014dfd        0x3 
 .sbss          0x0000000000014e00        0x8 ..\..\..\..\Libraries\libs\libbtstack.a(hct_fc.o)
 .sbss          0x0000000000014e08        0xd ..\..\..\..\Libraries\libs\libbtstack.a(l2cap_test.o)
                0x0000000000014e08                vd_tx_cnt
                0x0000000000014e0c                vd_tx_w
                0x0000000000014e10                vd_tx_r
 *fill*         0x0000000000014e15        0x3 
 .sbss          0x0000000000014e18        0x5 ..\..\..\..\Libraries\libs\libbtstack.a(hci.o)
 *fill*         0x0000000000014e1d        0x3 
 .sbss          0x0000000000014e20        0x5 ..\..\..\..\Libraries\libs\libbtstack.a(hid_usage.o)
                0x0000000000014e20                ts_ctl
 *fill*         0x0000000000014e25        0x3 
 .sbss          0x0000000000014e28        0x9 ..\..\..\..\Libraries\libs\libbtstack.a(hfp_hf.o)
 *fill*         0x0000000000014e31        0x3 
 .sbss          0x0000000000014e34        0xf ..\..\..\..\Libraries\libs\libbtstack.a(sm.o)
 *fill*         0x0000000000014e43        0x1 
 .sbss          0x0000000000014e44        0x9 ..\..\..\..\Libraries\libs\libbtstack.a(hci_transport_hcic.o)
                0x0000000000014e48                p_hci_transport
 *fill*         0x0000000000014e4d        0x3 
 .sbss          0x0000000000014e50        0x2 ..\..\..\..\Libraries\libs\libbtstack.a(lc_proc.o)
                0x0000000000014e50                lc_state
 *fill*         0x0000000000014e52        0x2 
 .sbss          0x0000000000014e54        0x1 ..\..\..\..\Libraries\libs\libbtstack.a(mgr_proc.o)
 *fill*         0x0000000000014e55        0x3 
 .sbss          0x0000000000014e58        0x4 ..\..\..\..\Libraries\libs\libbtstack.a(ll_proc.o)
 *(.buf*)
 .buf.bsp.sys_cb
                0x0000000000014e5c       0x40 Output\obj\Libraries\bsp\bsp_sys.o
                0x0000000000014e5c                sys_cb
 .buf.device.cb
                0x0000000000014e9c       0x1b ..\..\..\..\Libraries\libs\libplatform.a(device.o)
                0x0000000000014e9c                dev_cb
 *fill*         0x0000000000014eb7        0x1 
 .buf.usb       0x0000000000014eb8      0x15c ..\..\..\..\Libraries\libs\libdrivers.a(usb_device_run_loop.o)
                0x0000000000014eb8                ude_0
                0x0000000000014ee0                udp_0
                0x0000000000014eec                epcb_printer_tx
                0x0000000000014f04                epcb_printer_rx
                0x0000000000014f1c                udh_0
                0x0000000000014f24                epcb3_tx
                0x0000000000014f3c                udu_0
                0x0000000000014f40                epcb_user
                0x0000000000014f58                uds_0
                0x0000000000014f8c                epcb2_rx
                0x0000000000014fa4                epcb2_tx
                0x0000000000014fbc                uda_0
                0x0000000000014fcc                epcb1_rx
                0x0000000000014fe4                epcb1_tx
                0x0000000000014ffc                lun_0
 *(.dac_obuf)
 *(.btmem.stack.sdp)
 .btmem.stack.sdp
                0x0000000000015014      0x18c ..\..\..\..\Libraries\libs\libbtstack.a(sdp_server.o)
 .btmem.stack.sdp
                0x00000000000151a0       0xba ..\..\..\..\Libraries\libs\libbtstack.a(sdp_client.o)
 *(.btmem.stack.spp)
 *fill*         0x000000000001525a        0x2 
 .btmem.stack.spp
                0x000000000001525c       0x58 ..\..\..\..\Libraries\libs\libbtstack.a(spp.o)
                0x000000000001525c                spp_connections
 *(.btmem.stack.l2cap)
 .btmem.stack.l2cap
                0x00000000000152b4       0xbc ..\..\..\..\Libraries\libs\libbtstack.a(l2cap.o)
                0x00000000000152dc                l2cap_channels
 *(.btmem.stack.hid)
 .btmem.stack.hid
                0x0000000000015370       0x38 ..\..\..\..\Libraries\libs\libbtstack.a(hid_device.o)
 *(.qtest_buf)
                0x00000000000153a8                __bss_end = .
                0x00000000000017a8                __bss_size = (__bss_end - __bss_start)

.heap           0x0000000000010c00     0x3000
 *(.mem_heap)
 .mem_heap      0x0000000000010c00     0x3000 ..\..\..\..\Libraries\libs\libplatform.a(startup.o)
                0x0000000000010c00                mem_heap

.bram           0x0000000000020000     0xb3a0
 *(.btmem.bthw)
 .btmem.bthw    0x0000000000020000     0x45f8 ..\..\..\..\Libraries\libs\libbtstack.a(bb.o)
                0x0000000000020000                bthw_mem
 *(.btmem*)
 .btmem.bb.buf  0x00000000000245f8       0x4c ..\..\..\..\Libraries\libs\libbtstack.a(nanos.o)
 .btmem.bt.sco  0x0000000000024644        0xa ..\..\..\..\Libraries\libs\libbtstack.a(bt_sco.o)
 *fill*         0x000000000002464e        0x2 
 .btmem.bt.acl  0x0000000000024650        0x8 ..\..\..\..\Libraries\libs\libbtstack.a(bt_acl.o)
                0x0000000000024650                bt_acl_env
 .btmem.bt.sco  0x0000000000024658        0x8 ..\..\..\..\Libraries\libs\libbtstack.a(bt_acl.o)
                0x0000000000024658                bt_sco_env
 .btmem.ble.con
                0x0000000000024660       0x14 ..\..\..\..\Libraries\libs\libbtstack.a(ble_con.o)
 .btmem.bb.env  0x0000000000024674       0x4c ..\..\..\..\Libraries\libs\libbtstack.a(bb_int.o)
                0x0000000000024674                bb_env
 .btmem.bb.buf  0x00000000000246c0     0x3278 ..\..\..\..\Libraries\libs\libbtstack.a(bb.o)
 .btmem.stack.util
                0x0000000000027938       0x12 ..\..\..\..\Libraries\libs\libbtstack.a(btstack_util.o)
 *fill*         0x000000000002794a        0x2 
 .btmem.stack   0x000000000002794c       0x14 ..\..\..\..\Libraries\libs\libbtstack.a(btstack_run_loop.o)
 .btmem.stack.linkctrl
                0x0000000000027960       0x58 ..\..\..\..\Libraries\libs\libbtstack.a(btstack_link_ctrl.o)
                0x0000000000027964                hci_link_max
 .btmem.ble.adv
                0x00000000000279b8       0x40 ..\..\..\..\Libraries\libs\libbtstack.a(btstack_main.o)
                0x00000000000279b8                scan_data
                0x00000000000279d7                scan_data_len
                0x00000000000279d8                adv_data
                0x00000000000279f7                adv_data_len
 .btmem.bb.vs   0x00000000000279f8        0xd ..\..\..\..\Libraries\libs\libbtstack.a(vs_proc.o)
                0x00000000000279f8                vs_env
                0x0000000000027a04                vs_state
 *fill*         0x0000000000027a05        0x3 
 .btmem.bb.rf   0x0000000000027a08        0x4 ..\..\..\..\Libraries\libs\libbtstack.a(rf_smart.o)
 .btmem.bb.hci  0x0000000000027a0c       0x62 ..\..\..\..\Libraries\libs\libbtstack.a(hct.o)
                0x0000000000027a0c                hci_env
 *fill*         0x0000000000027a6e        0x2 
 .btmem.bt.lm   0x0000000000027a70      0x1ac ..\..\..\..\Libraries\libs\libbtstack.a(lm.o)
                0x0000000000027a74                lm_env
 .btmem.bt.env  0x0000000000027c1c      0x1cc ..\..\..\..\Libraries\libs\libbtstack.a(bt_hal.o)
                0x0000000000027c1c                bt_env
 .btmem.bt.buf  0x0000000000027de8       0xdc ..\..\..\..\Libraries\libs\libbtstack.a(bt21.o)
 .btmem.ble.hal
                0x0000000000027ec4      0x130 ..\..\..\..\Libraries\libs\libbtstack.a(ble_hal.o)
                0x0000000000027ec8                ble_env
                0x0000000000027fec                ble_exp_sync_pos_tab
 .btmem.ble.adv
                0x0000000000027ff4       0x10 ..\..\..\..\Libraries\libs\libbtstack.a(ble_adv.o)
 .btmem.stack.hci
                0x0000000000028004      0xad1 ..\..\..\..\Libraries\libs\libbtstack.a(hci.o)
 *fill*         0x0000000000028ad5        0x3 
 .btmem.stack.hci_buf
                0x0000000000028ad8      0x3c4 ..\..\..\..\Libraries\libs\libbtstack.a(hci.o)
 .btmem.stack.hid.usage
                0x0000000000028e9c       0x12 ..\..\..\..\Libraries\libs\libbtstack.a(hid_usage.o)
                0x0000000000028e9c                hrpt_cb
                0x0000000000028ea4                hid_report_buf
 *fill*         0x0000000000028eae        0x2 
 .btmem.stack.hfp
                0x0000000000028eb0        0x5 ..\..\..\..\Libraries\libs\libbtstack.a(hfp.o)
                0x0000000000028eb0                hfp_connections
                0x0000000000028eb4                hfp_index
 *fill*         0x0000000000028eb5        0x3 
 .btmem.ble.adv
                0x0000000000028eb8       0x1f ..\..\..\..\Libraries\libs\libbtstack.a(btstack_adv0.o)
 *fill*         0x0000000000028ed7        0x1 
 .btmem.hci.transport
                0x0000000000028ed8       0x20 ..\..\..\..\Libraries\libs\libbtstack.a(hci_transport_hcic.o)
 .btmem.bt.lm   0x0000000000028ef8        0x1 ..\..\..\..\Libraries\libs\libbtstack.a(lm_proc.o)
                0x0000000000028ef8                lm_state
 *fill*         0x0000000000028ef9        0x3 
 .btmem.bt.lc   0x0000000000028efc        0x8 ..\..\..\..\Libraries\libs\libbtstack.a(lc.o)
                0x0000000000028efc                lc_env
 .btmem.ble.lm  0x0000000000028f04      0x24c ..\..\..\..\Libraries\libs\libbtstack.a(mgr.o)
                0x0000000000028f04                mgr_env
 .btmem.ble.lc  0x0000000000029150       0x10 ..\..\..\..\Libraries\libs\libbtstack.a(ll.o)
                0x0000000000029150                ll_env
 .btmem.ble.test
                0x0000000000029160        0x4 ..\..\..\..\Libraries\libs\libbtstack.a(ble_test.o)
 .btmem.ble.scan
                0x0000000000029164        0x8 ..\..\..\..\Libraries\libs\libbtstack.a(ble_scan.o)
 .btmem.ble.init
                0x000000000002916c        0x4 ..\..\..\..\Libraries\libs\libbtstack.a(ble_init.o)
 .btmem.ble.buf
                0x0000000000029170       0x30 ..\..\..\..\Libraries\libs\libbtstack.a(ble_buf.o)
 .btmem.bt.lm.sco
                0x00000000000291a0        0xf ..\..\..\..\Libraries\libs\libbtstack.a(lm_sco.o)
 *fill*         0x00000000000291af        0x1 
 .btmem.bt.lc.sniff
                0x00000000000291b0       0x68 ..\..\..\..\Libraries\libs\libbtstack.a(lc_sniff.o)
                0x00000000000291b0                lc_sniff_env
 .btmem.bt.lc.sco
                0x0000000000029218       0x12 ..\..\..\..\Libraries\libs\libbtstack.a(lc_sco.o)
 *(.ble_cache*)
 *fill*         0x000000000002922a        0x2 
 .ble_cache.att
                0x000000000002922c       0x10 ..\..\..\..\Libraries\libs\libbtstack.a(gatt_server.o)
                0x000000000002922c                notify_tx
 .ble_cache.att
                0x000000000002923c      0x458 ..\..\..\..\Libraries\libs\libbtstack.a(gatt_profile.o)
 .ble_cache.att
                0x0000000000029694       0x50 ..\..\..\..\Libraries\libs\libbtstack.a(ad_parser.o)
                0x0000000000029694                ad_param
 .ble_cache.sm  0x00000000000296e4      0x214 ..\..\..\..\Libraries\libs\libbtstack.a(sm.o)
 *(.ble_buf*)
 .ble_buf.stack.spp
                0x00000000000298f8       0x10 ..\..\..\..\Libraries\libs\libbtstack.a(spp.o)
                0x00000000000298f8                spp_tx
 .ble_buf.att   0x0000000000029908      0x138 ..\..\..\..\Libraries\libs\libbtstack.a(gatt_server.o)
                0x0000000000029908                att_attributes
 .ble_buf.att.buf
                0x0000000000029a40      0x400 ..\..\..\..\Libraries\libs\libbtstack.a(gatt_server.o)
                0x0000000000029a40                attribute_buf
 .ble_buf.queue.buf
                0x0000000000029e40       0xc0 ..\..\..\..\Libraries\libs\libbtstack.a(gatt_server.o)
                0x0000000000029e40                att_queue_buf
 .ble_buf.att   0x0000000000029f00      0x2e0 ..\..\..\..\Libraries\libs\libbtstack.a(att_server.o)
                0x0000000000029f00                att_connection
 .ble_buf.att   0x000000000002a1e0      0x180 ..\..\..\..\Libraries\libs\libbtstack.a(le_device_db_memory.o)
 *(.spp_tx_buff.*)
 .spp_tx_buff.spp_tx_pool
                0x000000000002a360     0x1040 Output\obj\Libraries\BT\spp\spp.o
                0x000000000002a360                spp_tx_pool
 *(.ble_tx_buff.*)

.aram           0x0000000000050000     0x1000
 *(.usb_buf*)
 .usb_buf.hid   0x0000000000050000        0x8 ..\..\..\..\Libraries\libs\libdrivers.a(usb_device_run_loop.o)
                0x0000000000050000                ep3_buf
 .usb_buf.user  0x0000000000050008      0x400 ..\..\..\..\Libraries\libs\libdrivers.a(usb_device_run_loop.o)
                0x0000000000050008                ep_user_buf
                0x0000000000001000                . = 0x1000
 *fill*         0x0000000000050408      0xbf8 

.fcc_buf        0x0000000000050000     0x1000
                0x0000000000001000                . = 0x1000
 *fill*         0x0000000000050000     0x1000 
 *(.fcc_buf.huart)

.aram_msc_stm   0x0000000000050000     0x1000
 *(.stm_buf)
                0x0000000000001000                . = 0x1000
 *fill*         0x0000000000050000     0x1000 

.cram_user
 *(.user.*)

.dram_upd       0x0000000000058000     0x4500
                0x0000000000003800                . = 0x3800
 *fill*         0x0000000000058000     0x3800 
 *(.upd_ota*)
 *(.upd_buf*)
                0x0000000000004500                . = 0x4500
 *fill*         0x000000000005b800      0xd00 

.eram_fot       0x0000000000054000      0xa00
 *(.fot_data.*)
 .fot_data.buf  0x0000000000054000      0x200 Output\obj\Libraries\bsp\bsp_fot.o
                0x0000000000054000                fot_data
 .fot_data.buf  0x0000000000054200      0x4e4 ..\..\..\..\Libraries\libs\libplatform.a(fot_update.o)
                0x0000000000054478                mac_ctl
                0x0000000000000a00                . = 0xa00
 *fill*         0x00000000000546e4      0x31c 
                0x0000000000042a00                __bank_size = SIZEOF (.flash)
                0x0000000010000200                __comm_lma = LOADADDR (.comm)
                0x0000000000003800                __comm_size = SIZEOF (.comm)
LOAD ..\..\..\..\Libraries\libs\libplatform.a
LOAD ..\..\..\..\Libraries\libs\libbtstack.a
LOAD ..\..\..\..\Libraries\libs\libdrivers.a
LOAD D:\×ÀÃæ\¼ÖÌìº½\×ªÕý¹¤×÷ÎÄ¼þ-2024\ÉÏ´«¹ÙÍøGW3323-¾«¼ò°æ\GW3323_SDK_V2.5_GW3323HGU6\Libraries\libs\libbtstack.a
LOAD D:\×ÀÃæ\¼ÖÌìº½\×ªÕý¹¤×÷ÎÄ¼þ-2024\ÉÏ´«¹ÙÍøGW3323-¾«¼ò°æ\GW3323_SDK_V2.5_GW3323HGU6\Libraries\libs\libbtstack_master.a
LOAD D:\×ÀÃæ\¼ÖÌìº½\×ªÕý¹¤×÷ÎÄ¼þ-2024\ÉÏ´«¹ÙÍøGW3323-¾«¼ò°æ\GW3323_SDK_V2.5_GW3323HGU6\Libraries\libs\libc.a
LOAD D:\×ÀÃæ\¼ÖÌìº½\×ªÕý¹¤×÷ÎÄ¼þ-2024\ÉÏ´«¹ÙÍøGW3323-¾«¼ò°æ\GW3323_SDK_V2.5_GW3323HGU6\Libraries\libs\libdrivers.a
LOAD D:\×ÀÃæ\¼ÖÌìº½\×ªÕý¹¤×÷ÎÄ¼þ-2024\ÉÏ´«¹ÙÍøGW3323-¾«¼ò°æ\GW3323_SDK_V2.5_GW3323HGU6\Libraries\libs\libgcc.a
LOAD D:\×ÀÃæ\¼ÖÌìº½\×ªÕý¹¤×÷ÎÄ¼þ-2024\ÉÏ´«¹ÙÍøGW3323-¾«¼ò°æ\GW3323_SDK_V2.5_GW3323HGU6\Libraries\libs\libm.a
LOAD D:\×ÀÃæ\¼ÖÌìº½\×ªÕý¹¤×÷ÎÄ¼þ-2024\ÉÏ´«¹ÙÍøGW3323-¾«¼ò°æ\GW3323_SDK_V2.5_GW3323HGU6\Libraries\libs\libplatform.a
OUTPUT(Output\bin\app.rv32 elf32-littleriscv)

.comment        0x0000000000000000       0x23
 .comment       0x0000000000000000       0x11 Output\obj\Libraries\bsp\bsp_cm.o
                                         0x12 (size before relaxing)
 .comment       0x0000000000000011       0x12 Output\obj\Libraries\bsp\bsp_fot.o
 .comment       0x0000000000000011       0x12 Output\obj\Libraries\bsp\bsp_param.o
 .comment       0x0000000000000011       0x12 Output\obj\Libraries\bsp\bsp_sys.o
 .comment       0x0000000000000011       0x12 Output\obj\Libraries\BT\ble\ab_link\app.o
 .comment       0x0000000000000011       0x12 Output\obj\Libraries\BT\ble\adv0.o
 .comment       0x0000000000000011       0x12 Output\obj\Libraries\BT\ble\ble.o
 .comment       0x0000000000000011       0x12 Output\obj\Libraries\BT\spp\bt.o
 .comment       0x0000000000000011       0x12 Output\obj\Libraries\BT\spp\profile.o
 .comment       0x0000000000000011       0x12 Output\obj\Libraries\BT\spp\spp.o
 .comment       0x0000000000000011       0x12 Output\obj\Libraries\Device\Source\gw3323_clk.o
 .comment       0x0000000000000011       0x12 Output\obj\Libraries\Device\Source\gw3323_gpio.o
 .comment       0x0000000000000011       0x12 Output\obj\Libraries\Device\Source\gw3323_tmr.o
 .comment       0x0000000000000011       0x12 Output\obj\Libraries\libs\strong_symbol.o
 .comment       0x0000000000000011       0x12 Output\obj\Examples\TIMER\TIM_Capture\Source\timer_capture.o
 .comment       0x0000000000000011       0x12 Output\obj\Examples\TIMER\TIM_Capture\Source\timer_pwm.o
 .comment       0x0000000000000011       0x12 Output\obj\Examples\TIMER\TIM_Capture\Project\config.o
 .comment       0x0000000000000011       0x12 Output\obj\Examples\TIMER\TIM_Capture\Project\main.o
 .comment       0x0000000000000011       0x12 ..\..\..\..\Libraries\libs\libplatform.a(audio.o)
                                         0x13 (size before relaxing)
 .comment       0x0000000000000023       0x13 ..\..\..\..\Libraries\libs\libplatform.a(cm.o)
 .comment       0x0000000000000023       0x13 ..\..\..\..\Libraries\libs\libplatform.a(os_flash.o)
 .comment       0x0000000000000023       0x13 ..\..\..\..\Libraries\libs\libplatform.a(xcfg.o)
 .comment       0x0000000000000023       0x13 ..\..\..\..\Libraries\libs\libplatform.a(device.o)
 .comment       0x0000000000000023       0x13 ..\..\..\..\Libraries\libs\libplatform.a(main.o)
 .comment       0x0000000000000023       0x13 ..\..\..\..\Libraries\libs\libplatform.a(interrupt.o)
 .comment       0x0000000000000023       0x13 ..\..\..\..\Libraries\libs\libplatform.a(startup.o)
 .comment       0x0000000000000023       0x13 ..\..\..\..\Libraries\libs\libplatform.a(sys_hook.o)
 .comment       0x0000000000000023       0x13 ..\..\..\..\Libraries\libs\libplatform.a(spiflash.o)
 .comment       0x0000000000000023       0x13 ..\..\..\..\Libraries\libs\libplatform.a(debug.o)
 .comment       0x0000000000000023       0x13 ..\..\..\..\Libraries\libs\libplatform.a(fot_update.o)
 .comment       0x0000000000000023       0x13 ..\..\..\..\Libraries\libs\libplatform.a(lock.o)
 .comment       0x0000000000000023       0x13 ..\..\..\..\Libraries\libs\libplatform.a(patch.o)
 .comment       0x0000000000000023       0x13 ..\..\..\..\Libraries\libs\libplatform.a(power.o)
 .comment       0x0000000000000023       0x13 ..\..\..\..\Libraries\libs\libplatform.a(rc.o)
 .comment       0x0000000000000023       0x13 ..\..\..\..\Libraries\libs\libplatform.a(sys.o)
 .comment       0x0000000000000023       0x13 ..\..\..\..\Libraries\libs\libplatform.a(sys_clk.o)
 .comment       0x0000000000000023       0x13 ..\..\..\..\Libraries\libs\libplatform.a(voltage_trim.o)
 .comment       0x0000000000000023       0x13 ..\..\..\..\Libraries\libs\libplatform.a(weak_symbol.o)
 .comment       0x0000000000000023       0x13 ..\..\..\..\Libraries\libs\libplatform.a(usb.o)
 .comment       0x0000000000000023       0x13 ..\..\..\..\Libraries\libs\libplatform.a(bt.o)
 .comment       0x0000000000000023       0x13 ..\..\..\..\Libraries\libs\libbtstack.a(nanos.o)
 .comment       0x0000000000000023       0x13 ..\..\..\..\Libraries\libs\libbtstack.a(patch.o)
 .comment       0x0000000000000023       0x13 ..\..\..\..\Libraries\libs\libbtstack.a(platform.o)
 .comment       0x0000000000000023       0x13 ..\..\..\..\Libraries\libs\libbtstack.a(bt_sco.o)
 .comment       0x0000000000000023       0x13 ..\..\..\..\Libraries\libs\libbtstack.a(bt_acl.o)
 .comment       0x0000000000000023       0x13 ..\..\..\..\Libraries\libs\libbtstack.a(ble_con.o)
 .comment       0x0000000000000023       0x13 ..\..\..\..\Libraries\libs\libbtstack.a(bb_utils.o)
 .comment       0x0000000000000023       0x13 ..\..\..\..\Libraries\libs\libbtstack.a(bb_int.o)
 .comment       0x0000000000000023       0x13 ..\..\..\..\Libraries\libs\libbtstack.a(bb.o)
 .comment       0x0000000000000023       0x13 ..\..\..\..\Libraries\libs\libbtstack.a(platform.o)
 .comment       0x0000000000000023       0x13 ..\..\..\..\Libraries\libs\libbtstack.a(extern_tws.o)
 .comment       0x0000000000000023       0x13 ..\..\..\..\Libraries\libs\libbtstack.a(extern_bt.o)
 .comment       0x0000000000000023       0x13 ..\..\..\..\Libraries\libs\libbtstack.a(extern.o)
 .comment       0x0000000000000023       0x13 ..\..\..\..\Libraries\libs\libbtstack.a(spp.o)
 .comment       0x0000000000000023       0x13 ..\..\..\..\Libraries\libs\libbtstack.a(sdp_util.o)
 .comment       0x0000000000000023       0x13 ..\..\..\..\Libraries\libs\libbtstack.a(sdp_tbl.o)
 .comment       0x0000000000000023       0x13 ..\..\..\..\Libraries\libs\libbtstack.a(sdp_server.o)
 .comment       0x0000000000000023       0x13 ..\..\..\..\Libraries\libs\libbtstack.a(sdp_client.o)
 .comment       0x0000000000000023       0x13 ..\..\..\..\Libraries\libs\libbtstack.a(rfcomm.o)
 .comment       0x0000000000000023       0x13 ..\..\..\..\Libraries\libs\libbtstack.a(btstack_link_key_db.o)
 .comment       0x0000000000000023       0x13 ..\..\..\..\Libraries\libs\libbtstack.a(btstack_util.o)
 .comment       0x0000000000000023       0x13 ..\..\..\..\Libraries\libs\libbtstack.a(btstack_txpkt.o)
 .comment       0x0000000000000023       0x13 ..\..\..\..\Libraries\libs\libbtstack.a(btstack_run_loop.o)
 .comment       0x0000000000000023       0x13 ..\..\..\..\Libraries\libs\libbtstack.a(btstack_memory.o)
 .comment       0x0000000000000023       0x13 ..\..\..\..\Libraries\libs\libbtstack.a(btstack_linked_list.o)
 .comment       0x0000000000000023       0x13 ..\..\..\..\Libraries\libs\libbtstack.a(btstack_link_ctrl.o)
 .comment       0x0000000000000023       0x13 ..\..\..\..\Libraries\libs\libbtstack.a(gatt_server.o)
 .comment       0x0000000000000023       0x13 ..\..\..\..\Libraries\libs\libbtstack.a(gatt_profile.o)
 .comment       0x0000000000000023       0x13 ..\..\..\..\Libraries\libs\libbtstack.a(att_server.o)
 .comment       0x0000000000000023       0x13 ..\..\..\..\Libraries\libs\libbtstack.a(att_dispatch.o)
 .comment       0x0000000000000023       0x13 ..\..\..\..\Libraries\libs\libbtstack.a(att_db.o)
 .comment       0x0000000000000023       0x13 ..\..\..\..\Libraries\libs\libbtstack.a(ad_parser.o)
 .comment       0x0000000000000023       0x13 ..\..\..\..\Libraries\libs\libbtstack.a(btstack_main.o)
 .comment       0x0000000000000023       0x13 ..\..\..\..\Libraries\libs\libbtstack.a(btstack_hal.o)
 .comment       0x0000000000000023       0x13 ..\..\..\..\Libraries\libs\libbtstack.a(btstack_api.o)
 .comment       0x0000000000000023       0x13 ..\..\..\..\Libraries\libs\libbtstack.a(bt_api.o)
 .comment       0x0000000000000023       0x13 ..\..\..\..\Libraries\libs\libbtstack.a(ble_api.o)
 .comment       0x0000000000000023       0x13 ..\..\..\..\Libraries\libs\libbtstack.a(bb_sche.o)
 .comment       0x0000000000000023       0x13 ..\..\..\..\Libraries\libs\libbtstack.a(bb_dbg.o)
 .comment       0x0000000000000023       0x13 ..\..\..\..\Libraries\libs\libbtstack.a(bb_clk.o)
 .comment       0x0000000000000023       0x13 ..\..\..\..\Libraries\libs\libbtstack.a(aes.o)
 .comment       0x0000000000000023       0x13 ..\..\..\..\Libraries\libs\libbtstack.a(vs_proc.o)
 .comment       0x0000000000000023       0x13 ..\..\..\..\Libraries\libs\libbtstack.a(vs_fcc.o)
 .comment       0x0000000000000023       0x13 ..\..\..\..\Libraries\libs\libbtstack.a(vs.o)
 .comment       0x0000000000000023       0x13 ..\..\..\..\Libraries\libs\libbtstack.a(rf_smart.o)
 .comment       0x0000000000000023       0x13 ..\..\..\..\Libraries\libs\libbtstack.a(rf.o)
 .comment       0x0000000000000023       0x13 ..\..\..\..\Libraries\libs\libbtstack.a(bt_hook.o)
 .comment       0x0000000000000023       0x13 ..\..\..\..\Libraries\libs\libbtstack.a(ble_hook.o)
 .comment       0x0000000000000023       0x13 ..\..\..\..\Libraries\libs\libbtstack.a(hct_tl.o)
 .comment       0x0000000000000023       0x13 ..\..\..\..\Libraries\libs\libbtstack.a(hct_msg.o)
 .comment       0x0000000000000023       0x13 ..\..\..\..\Libraries\libs\libbtstack.a(hct_fc.o)
 .comment       0x0000000000000023       0x13 ..\..\..\..\Libraries\libs\libbtstack.a(hct.o)
 .comment       0x0000000000000023       0x13 ..\..\..\..\Libraries\libs\libbtstack.a(tws_sco.o)
 .comment       0x0000000000000023       0x13 ..\..\..\..\Libraries\libs\libbtstack.a(tws_acl.o)
 .comment       0x0000000000000023       0x13 ..\..\..\..\Libraries\libs\libbtstack.a(lm.o)
 .comment       0x0000000000000023       0x13 ..\..\..\..\Libraries\libs\libbtstack.a(bt_hal.o)
 .comment       0x0000000000000023       0x13 ..\..\..\..\Libraries\libs\libbtstack.a(bt21.o)
 .comment       0x0000000000000023       0x13 ..\..\..\..\Libraries\libs\libbtstack.a(bc.o)
 .comment       0x0000000000000023       0x13 ..\..\..\..\Libraries\libs\libbtstack.a(ble_hal.o)
 .comment       0x0000000000000023       0x13 ..\..\..\..\Libraries\libs\libbtstack.a(ble_adv.o)
 .comment       0x0000000000000023       0x13 ..\..\..\..\Libraries\libs\libbtstack.a(ble.o)
 .comment       0x0000000000000023       0x13 ..\..\..\..\Libraries\libs\libbtstack.a(extern_ble.o)
 .comment       0x0000000000000023       0x13 ..\..\..\..\Libraries\libs\libbtstack.a(l2cap_test.o)
 .comment       0x0000000000000023       0x13 ..\..\..\..\Libraries\libs\libbtstack.a(l2cap.o)
 .comment       0x0000000000000023       0x13 ..\..\..\..\Libraries\libs\libbtstack.a(hci_sco.o)
 .comment       0x0000000000000023       0x13 ..\..\..\..\Libraries\libs\libbtstack.a(hci_dump.o)
 .comment       0x0000000000000023       0x13 ..\..\..\..\Libraries\libs\libbtstack.a(hci_cmd.o)
 .comment       0x0000000000000023       0x13 ..\..\..\..\Libraries\libs\libbtstack.a(hci.o)
 .comment       0x0000000000000023       0x13 ..\..\..\..\Libraries\libs\libbtstack.a(hid_usage.o)
 .comment       0x0000000000000023       0x13 ..\..\..\..\Libraries\libs\libbtstack.a(hid_device.o)
 .comment       0x0000000000000023       0x13 ..\..\..\..\Libraries\libs\libbtstack.a(hfp_hf.o)
 .comment       0x0000000000000023       0x13 ..\..\..\..\Libraries\libs\libbtstack.a(hfp.o)
 .comment       0x0000000000000023       0x13 ..\..\..\..\Libraries\libs\libbtstack.a(avdtp.o)
 .comment       0x0000000000000023       0x13 ..\..\..\..\Libraries\libs\libbtstack.a(a2dp.o)
 .comment       0x0000000000000023       0x13 ..\..\..\..\Libraries\libs\libbtstack.a(btstack_memory_pool.o)
 .comment       0x0000000000000023       0x13 ..\..\..\..\Libraries\libs\libbtstack.a(btstack_adv0.o)
 .comment       0x0000000000000023       0x13 ..\..\..\..\Libraries\libs\libbtstack.a(sm.o)
 .comment       0x0000000000000023       0x13 ..\..\..\..\Libraries\libs\libbtstack.a(le_device_db_memory.o)
 .comment       0x0000000000000023       0x13 ..\..\..\..\Libraries\libs\libbtstack.a(hci_transport_hcic.o)
 .comment       0x0000000000000023       0x13 ..\..\..\..\Libraries\libs\libbtstack.a(btstack_chipset_inner.o)
 .comment       0x0000000000000023       0x13 ..\..\..\..\Libraries\libs\libbtstack.a(lm_hook.o)
 .comment       0x0000000000000023       0x13 ..\..\..\..\Libraries\libs\libbtstack.a(lm_sp.o)
 .comment       0x0000000000000023       0x13 ..\..\..\..\Libraries\libs\libbtstack.a(lm_proc.o)
 .comment       0x0000000000000023       0x13 ..\..\..\..\Libraries\libs\libbtstack.a(lm_key.o)
 .comment       0x0000000000000023       0x13 ..\..\..\..\Libraries\libs\libbtstack.a(lc.o)
 .comment       0x0000000000000023       0x13 ..\..\..\..\Libraries\libs\libbtstack.a(mgr.o)
 .comment       0x0000000000000023       0x13 ..\..\..\..\Libraries\libs\libbtstack.a(ll.o)
 .comment       0x0000000000000023       0x13 ..\..\..\..\Libraries\libs\libbtstack.a(ble_test.o)
 .comment       0x0000000000000023       0x13 ..\..\..\..\Libraries\libs\libbtstack.a(ble_scan.o)
 .comment       0x0000000000000023       0x13 ..\..\..\..\Libraries\libs\libbtstack.a(ble_per_adv.o)
 .comment       0x0000000000000023       0x13 ..\..\..\..\Libraries\libs\libbtstack.a(ble_init.o)
 .comment       0x0000000000000023       0x13 ..\..\..\..\Libraries\libs\libbtstack.a(ble_buf.o)
 .comment       0x0000000000000023       0x13 ..\..\..\..\Libraries\libs\libbtstack.a(ble_adv0.o)
 .comment       0x0000000000000023       0x13 ..\..\..\..\Libraries\libs\libbtstack.a(extern_hfhs.o)
 .comment       0x0000000000000023       0x13 ..\..\..\..\Libraries\libs\libbtstack.a(l2cap_signaling.o)
 .comment       0x0000000000000023       0x13 ..\..\..\..\Libraries\libs\libbtstack.a(lc_hook.o)
 .comment       0x0000000000000023       0x13 ..\..\..\..\Libraries\libs\libbtstack.a(lm_sco.o)
 .comment       0x0000000000000023       0x13 ..\..\..\..\Libraries\libs\libbtstack.a(lc_util.o)
 .comment       0x0000000000000023       0x13 ..\..\..\..\Libraries\libs\libbtstack.a(lc_sniff.o)
 .comment       0x0000000000000023       0x13 ..\..\..\..\Libraries\libs\libbtstack.a(lc_sco.o)
 .comment       0x0000000000000023       0x13 ..\..\..\..\Libraries\libs\libbtstack.a(lc_proc.o)
 .comment       0x0000000000000023       0x13 ..\..\..\..\Libraries\libs\libbtstack.a(lc_lmppdu.o)
 .comment       0x0000000000000023       0x13 ..\..\..\..\Libraries\libs\libbtstack.a(mgr_proc.o)
 .comment       0x0000000000000023       0x13 ..\..\..\..\Libraries\libs\libbtstack.a(mgr_init.o)
 .comment       0x0000000000000023       0x13 ..\..\..\..\Libraries\libs\libbtstack.a(mgr_hci.o)
 .comment       0x0000000000000023       0x13 ..\..\..\..\Libraries\libs\libbtstack.a(ll_scan.o)
 .comment       0x0000000000000023       0x13 ..\..\..\..\Libraries\libs\libbtstack.a(ll_adv.o)
 .comment       0x0000000000000023       0x13 ..\..\..\..\Libraries\libs\libbtstack.a(ll_proc.o)
 .comment       0x0000000000000023       0x13 ..\..\..\..\Libraries\libs\libbtstack.a(ll_ping.o)
 .comment       0x0000000000000023       0x13 ..\..\..\..\Libraries\libs\libbtstack.a(ll_phy_upd.o)
 .comment       0x0000000000000023       0x13 ..\..\..\..\Libraries\libs\libbtstack.a(ll_past.o)
 .comment       0x0000000000000023       0x13 ..\..\..\..\Libraries\libs\libbtstack.a(ll_length.o)
 .comment       0x0000000000000023       0x13 ..\..\..\..\Libraries\libs\libbtstack.a(ll_feature.o)
 .comment       0x0000000000000023       0x13 ..\..\..\..\Libraries\libs\libbtstack.a(ll_encrypt.o)
 .comment       0x0000000000000023       0x13 ..\..\..\..\Libraries\libs\libbtstack.a(ll_disconnect.o)
 .comment       0x0000000000000023       0x13 ..\..\..\..\Libraries\libs\libbtstack.a(ll_con_upd.o)
 .comment       0x0000000000000023       0x13 ..\..\..\..\Libraries\libs\libbtstack.a(ll_cntl.o)
 .comment       0x0000000000000023       0x13 ..\..\..\..\Libraries\libs\libbtstack.a(ll_clk_acc.o)
 .comment       0x0000000000000023       0x13 ..\..\..\..\Libraries\libs\libbtstack.a(ll_chmap_upd.o)
 .comment       0x0000000000000023       0x13 ..\..\..\..\Libraries\libs\libbtstack.a(aes_rpa.o)
 .comment       0x0000000000000023       0x13 ..\..\..\..\Libraries\libs\libbtstack.a(scan_hook.o)
 .comment       0x0000000000000023       0x13 ..\..\..\..\Libraries\libs\libbtstack.a(adv_hook.o)
 .comment       0x0000000000000023       0x13 ..\..\..\..\Libraries\libs\libbtstack.a(ll_version.o)
 .comment       0x0000000000000023       0x13 ..\..\..\..\Libraries\libs\libbtstack.a(ll_pwr.o)
 .comment       0x0000000000000023       0x13 ..\..\..\..\Libraries\libs\libdrivers.a(usb_device_hid.o)
 .comment       0x0000000000000023       0x13 ..\..\..\..\Libraries\libs\libdrivers.a(usb_device_printer.o)
 .comment       0x0000000000000023       0x13 ..\..\..\..\Libraries\libs\libdrivers.a(usb_device_run_loop.o)
 .comment       0x0000000000000023       0x13 ..\..\..\..\Libraries\libs\libdrivers.a(usb_comm.o)
 .comment       0x0000000000000023       0x13 ..\..\..\..\Libraries\libs\libdrivers.a(usb_device_ep.o)

.riscv.attributes
                0x0000000000000000     0x1e12
 .riscv.attributes
                0x0000000000000000       0x32 ..\..\..\..\Libraries\libs\libplatform.a(audio.o)
 .riscv.attributes
                0x0000000000000032       0x32 ..\..\..\..\Libraries\libs\libplatform.a(cm.o)
 .riscv.attributes
                0x0000000000000064       0x32 ..\..\..\..\Libraries\libs\libplatform.a(os_flash.o)
 .riscv.attributes
                0x0000000000000096       0x32 ..\..\..\..\Libraries\libs\libplatform.a(xcfg.o)
 .riscv.attributes
                0x00000000000000c8       0x32 ..\..\..\..\Libraries\libs\libplatform.a(device.o)
 .riscv.attributes
                0x00000000000000fa       0x32 ..\..\..\..\Libraries\libs\libplatform.a(main.o)
 .riscv.attributes
                0x000000000000012c       0x32 ..\..\..\..\Libraries\libs\libplatform.a(interrupt.o)
 .riscv.attributes
                0x000000000000015e       0x32 ..\..\..\..\Libraries\libs\libplatform.a(startup.o)
 .riscv.attributes
                0x0000000000000190       0x32 ..\..\..\..\Libraries\libs\libplatform.a(sys_hook.o)
 .riscv.attributes
                0x00000000000001c2       0x34 ..\..\..\..\Libraries\libs\libplatform.a(reset.o)
 .riscv.attributes
                0x00000000000001f6       0x32 ..\..\..\..\Libraries\libs\libplatform.a(spiflash.o)
 .riscv.attributes
                0x0000000000000228       0x32 ..\..\..\..\Libraries\libs\libplatform.a(debug.o)
 .riscv.attributes
                0x000000000000025a       0x32 ..\..\..\..\Libraries\libs\libplatform.a(fot_update.o)
 .riscv.attributes
                0x000000000000028c       0x32 ..\..\..\..\Libraries\libs\libplatform.a(lock.o)
 .riscv.attributes
                0x00000000000002be       0x32 ..\..\..\..\Libraries\libs\libplatform.a(patch.o)
 .riscv.attributes
                0x00000000000002f0       0x32 ..\..\..\..\Libraries\libs\libplatform.a(power.o)
 .riscv.attributes
                0x0000000000000322       0x32 ..\..\..\..\Libraries\libs\libplatform.a(rc.o)
 .riscv.attributes
                0x0000000000000354       0x30 ..\..\..\..\Libraries\libs\libplatform.a(s_sys.o)
 .riscv.attributes
                0x0000000000000384       0x32 ..\..\..\..\Libraries\libs\libplatform.a(sys.o)
 .riscv.attributes
                0x00000000000003b6       0x32 ..\..\..\..\Libraries\libs\libplatform.a(sys_clk.o)
 .riscv.attributes
                0x00000000000003e8       0x32 ..\..\..\..\Libraries\libs\libplatform.a(voltage_trim.o)
 .riscv.attributes
                0x000000000000041a       0x32 ..\..\..\..\Libraries\libs\libplatform.a(weak_symbol.o)
 .riscv.attributes
                0x000000000000044c       0x32 ..\..\..\..\Libraries\libs\libplatform.a(usb.o)
 .riscv.attributes
                0x000000000000047e       0x32 ..\..\..\..\Libraries\libs\libplatform.a(bt.o)
 .riscv.attributes
                0x00000000000004b0       0x32 ..\..\..\..\Libraries\libs\libbtstack.a(nanos.o)
 .riscv.attributes
                0x00000000000004e2       0x32 ..\..\..\..\Libraries\libs\libbtstack.a(patch.o)
 .riscv.attributes
                0x0000000000000514       0x32 ..\..\..\..\Libraries\libs\libbtstack.a(platform.o)
 .riscv.attributes
                0x0000000000000546       0x32 ..\..\..\..\Libraries\libs\libbtstack.a(bt_sco.o)
 .riscv.attributes
                0x0000000000000578       0x32 ..\..\..\..\Libraries\libs\libbtstack.a(bt_acl.o)
 .riscv.attributes
                0x00000000000005aa       0x32 ..\..\..\..\Libraries\libs\libbtstack.a(ble_con.o)
 .riscv.attributes
                0x00000000000005dc       0x32 ..\..\..\..\Libraries\libs\libbtstack.a(bb_utils.o)
 .riscv.attributes
                0x000000000000060e       0x32 ..\..\..\..\Libraries\libs\libbtstack.a(bb_int.o)
 .riscv.attributes
                0x0000000000000640       0x32 ..\..\..\..\Libraries\libs\libbtstack.a(bb.o)
 .riscv.attributes
                0x0000000000000672       0x32 ..\..\..\..\Libraries\libs\libbtstack.a(platform.o)
 .riscv.attributes
                0x00000000000006a4       0x32 ..\..\..\..\Libraries\libs\libbtstack.a(extern_tws.o)
 .riscv.attributes
                0x00000000000006d6       0x32 ..\..\..\..\Libraries\libs\libbtstack.a(extern_bt.o)
 .riscv.attributes
                0x0000000000000708       0x32 ..\..\..\..\Libraries\libs\libbtstack.a(extern.o)
 .riscv.attributes
                0x000000000000073a       0x32 ..\..\..\..\Libraries\libs\libbtstack.a(spp.o)
 .riscv.attributes
                0x000000000000076c       0x32 ..\..\..\..\Libraries\libs\libbtstack.a(sdp_util.o)
 .riscv.attributes
                0x000000000000079e       0x32 ..\..\..\..\Libraries\libs\libbtstack.a(sdp_tbl.o)
 .riscv.attributes
                0x00000000000007d0       0x32 ..\..\..\..\Libraries\libs\libbtstack.a(sdp_server.o)
 .riscv.attributes
                0x0000000000000802       0x32 ..\..\..\..\Libraries\libs\libbtstack.a(sdp_client.o)
 .riscv.attributes
                0x0000000000000834       0x32 ..\..\..\..\Libraries\libs\libbtstack.a(rfcomm.o)
 .riscv.attributes
                0x0000000000000866       0x32 ..\..\..\..\Libraries\libs\libbtstack.a(btstack_link_key_db.o)
 .riscv.attributes
                0x0000000000000898       0x32 ..\..\..\..\Libraries\libs\libbtstack.a(btstack_util.o)
 .riscv.attributes
                0x00000000000008ca       0x32 ..\..\..\..\Libraries\libs\libbtstack.a(btstack_txpkt.o)
 .riscv.attributes
                0x00000000000008fc       0x32 ..\..\..\..\Libraries\libs\libbtstack.a(btstack_run_loop.o)
 .riscv.attributes
                0x000000000000092e       0x32 ..\..\..\..\Libraries\libs\libbtstack.a(btstack_memory.o)
 .riscv.attributes
                0x0000000000000960       0x32 ..\..\..\..\Libraries\libs\libbtstack.a(btstack_linked_list.o)
 .riscv.attributes
                0x0000000000000992       0x32 ..\..\..\..\Libraries\libs\libbtstack.a(btstack_link_ctrl.o)
 .riscv.attributes
                0x00000000000009c4       0x32 ..\..\..\..\Libraries\libs\libbtstack.a(gatt_server.o)
 .riscv.attributes
                0x00000000000009f6       0x32 ..\..\..\..\Libraries\libs\libbtstack.a(gatt_profile.o)
 .riscv.attributes
                0x0000000000000a28       0x32 ..\..\..\..\Libraries\libs\libbtstack.a(att_server.o)
 .riscv.attributes
                0x0000000000000a5a       0x32 ..\..\..\..\Libraries\libs\libbtstack.a(att_dispatch.o)
 .riscv.attributes
                0x0000000000000a8c       0x32 ..\..\..\..\Libraries\libs\libbtstack.a(att_db.o)
 .riscv.attributes
                0x0000000000000abe       0x32 ..\..\..\..\Libraries\libs\libbtstack.a(ad_parser.o)
 .riscv.attributes
                0x0000000000000af0       0x32 ..\..\..\..\Libraries\libs\libbtstack.a(btstack_main.o)
 .riscv.attributes
                0x0000000000000b22       0x32 ..\..\..\..\Libraries\libs\libbtstack.a(btstack_hal.o)
 .riscv.attributes
                0x0000000000000b54       0x32 ..\..\..\..\Libraries\libs\libbtstack.a(btstack_api.o)
 .riscv.attributes
                0x0000000000000b86       0x32 ..\..\..\..\Libraries\libs\libbtstack.a(bt_api.o)
 .riscv.attributes
                0x0000000000000bb8       0x32 ..\..\..\..\Libraries\libs\libbtstack.a(ble_api.o)
 .riscv.attributes
                0x0000000000000bea       0x32 ..\..\..\..\Libraries\libs\libbtstack.a(bb_sche.o)
 .riscv.attributes
                0x0000000000000c1c       0x30 ..\..\..\..\Libraries\libs\libbtstack.a(patch_asm.o)
 .riscv.attributes
                0x0000000000000c4c       0x32 ..\..\..\..\Libraries\libs\libbtstack.a(bb_dbg.o)
 .riscv.attributes
                0x0000000000000c7e       0x32 ..\..\..\..\Libraries\libs\libbtstack.a(bb_clk.o)
 .riscv.attributes
                0x0000000000000cb0       0x32 ..\..\..\..\Libraries\libs\libbtstack.a(aes.o)
 .riscv.attributes
                0x0000000000000ce2       0x32 ..\..\..\..\Libraries\libs\libbtstack.a(vs_proc.o)
 .riscv.attributes
                0x0000000000000d14       0x32 ..\..\..\..\Libraries\libs\libbtstack.a(vs_fcc.o)
 .riscv.attributes
                0x0000000000000d46       0x32 ..\..\..\..\Libraries\libs\libbtstack.a(vs.o)
 .riscv.attributes
                0x0000000000000d78       0x32 ..\..\..\..\Libraries\libs\libbtstack.a(rf_smart.o)
 .riscv.attributes
                0x0000000000000daa       0x32 ..\..\..\..\Libraries\libs\libbtstack.a(rf.o)
 .riscv.attributes
                0x0000000000000ddc       0x32 ..\..\..\..\Libraries\libs\libbtstack.a(bt_hook.o)
 .riscv.attributes
                0x0000000000000e0e       0x32 ..\..\..\..\Libraries\libs\libbtstack.a(ble_hook.o)
 .riscv.attributes
                0x0000000000000e40       0x32 ..\..\..\..\Libraries\libs\libbtstack.a(hct_tl.o)
 .riscv.attributes
                0x0000000000000e72       0x32 ..\..\..\..\Libraries\libs\libbtstack.a(hct_msg.o)
 .riscv.attributes
                0x0000000000000ea4       0x32 ..\..\..\..\Libraries\libs\libbtstack.a(hct_fc.o)
 .riscv.attributes
                0x0000000000000ed6       0x32 ..\..\..\..\Libraries\libs\libbtstack.a(hct.o)
 .riscv.attributes
                0x0000000000000f08       0x32 ..\..\..\..\Libraries\libs\libbtstack.a(tws_sco.o)
 .riscv.attributes
                0x0000000000000f3a       0x32 ..\..\..\..\Libraries\libs\libbtstack.a(tws_acl.o)
 .riscv.attributes
                0x0000000000000f6c       0x32 ..\..\..\..\Libraries\libs\libbtstack.a(lm.o)
 .riscv.attributes
                0x0000000000000f9e       0x32 ..\..\..\..\Libraries\libs\libbtstack.a(bt_hal.o)
 .riscv.attributes
                0x0000000000000fd0       0x32 ..\..\..\..\Libraries\libs\libbtstack.a(bt21.o)
 .riscv.attributes
                0x0000000000001002       0x32 ..\..\..\..\Libraries\libs\libbtstack.a(bc.o)
 .riscv.attributes
                0x0000000000001034       0x32 ..\..\..\..\Libraries\libs\libbtstack.a(ble_hal.o)
 .riscv.attributes
                0x0000000000001066       0x32 ..\..\..\..\Libraries\libs\libbtstack.a(ble_adv.o)
 .riscv.attributes
                0x0000000000001098       0x32 ..\..\..\..\Libraries\libs\libbtstack.a(ble.o)
 .riscv.attributes
                0x00000000000010ca       0x32 ..\..\..\..\Libraries\libs\libbtstack.a(extern_ble.o)
 .riscv.attributes
                0x00000000000010fc       0x32 ..\..\..\..\Libraries\libs\libbtstack.a(l2cap_test.o)
 .riscv.attributes
                0x000000000000112e       0x32 ..\..\..\..\Libraries\libs\libbtstack.a(l2cap.o)
 .riscv.attributes
                0x0000000000001160       0x32 ..\..\..\..\Libraries\libs\libbtstack.a(hci_sco.o)
 .riscv.attributes
                0x0000000000001192       0x32 ..\..\..\..\Libraries\libs\libbtstack.a(hci_dump.o)
 .riscv.attributes
                0x00000000000011c4       0x32 ..\..\..\..\Libraries\libs\libbtstack.a(hci_cmd.o)
 .riscv.attributes
                0x00000000000011f6       0x32 ..\..\..\..\Libraries\libs\libbtstack.a(hci.o)
 .riscv.attributes
                0x0000000000001228       0x32 ..\..\..\..\Libraries\libs\libbtstack.a(hid_usage.o)
 .riscv.attributes
                0x000000000000125a       0x32 ..\..\..\..\Libraries\libs\libbtstack.a(hid_device.o)
 .riscv.attributes
                0x000000000000128c       0x32 ..\..\..\..\Libraries\libs\libbtstack.a(hfp_hf.o)
 .riscv.attributes
                0x00000000000012be       0x32 ..\..\..\..\Libraries\libs\libbtstack.a(hfp.o)
 .riscv.attributes
                0x00000000000012f0       0x32 ..\..\..\..\Libraries\libs\libbtstack.a(avdtp.o)
 .riscv.attributes
                0x0000000000001322       0x32 ..\..\..\..\Libraries\libs\libbtstack.a(a2dp.o)
 .riscv.attributes
                0x0000000000001354       0x32 ..\..\..\..\Libraries\libs\libbtstack.a(btstack_memory_pool.o)
 .riscv.attributes
                0x0000000000001386       0x32 ..\..\..\..\Libraries\libs\libbtstack.a(btstack_adv0.o)
 .riscv.attributes
                0x00000000000013b8       0x32 ..\..\..\..\Libraries\libs\libbtstack.a(sm.o)
 .riscv.attributes
                0x00000000000013ea       0x32 ..\..\..\..\Libraries\libs\libbtstack.a(le_device_db_memory.o)
 .riscv.attributes
                0x000000000000141c       0x32 ..\..\..\..\Libraries\libs\libbtstack.a(hci_transport_hcic.o)
 .riscv.attributes
                0x000000000000144e       0x32 ..\..\..\..\Libraries\libs\libbtstack.a(btstack_chipset_inner.o)
 .riscv.attributes
                0x0000000000001480       0x32 ..\..\..\..\Libraries\libs\libbtstack.a(lm_hook.o)
 .riscv.attributes
                0x00000000000014b2       0x32 ..\..\..\..\Libraries\libs\libbtstack.a(lm_sp.o)
 .riscv.attributes
                0x00000000000014e4       0x32 ..\..\..\..\Libraries\libs\libbtstack.a(lm_proc.o)
 .riscv.attributes
                0x0000000000001516       0x32 ..\..\..\..\Libraries\libs\libbtstack.a(lm_key.o)
 .riscv.attributes
                0x0000000000001548       0x32 ..\..\..\..\Libraries\libs\libbtstack.a(lc.o)
 .riscv.attributes
                0x000000000000157a       0x32 ..\..\..\..\Libraries\libs\libbtstack.a(mgr.o)
 .riscv.attributes
                0x00000000000015ac       0x32 ..\..\..\..\Libraries\libs\libbtstack.a(ll.o)
 .riscv.attributes
                0x00000000000015de       0x32 ..\..\..\..\Libraries\libs\libbtstack.a(ble_test.o)
 .riscv.attributes
                0x0000000000001610       0x32 ..\..\..\..\Libraries\libs\libbtstack.a(ble_scan.o)
 .riscv.attributes
                0x0000000000001642       0x32 ..\..\..\..\Libraries\libs\libbtstack.a(ble_per_adv.o)
 .riscv.attributes
                0x0000000000001674       0x32 ..\..\..\..\Libraries\libs\libbtstack.a(ble_init.o)
 .riscv.attributes
                0x00000000000016a6       0x32 ..\..\..\..\Libraries\libs\libbtstack.a(ble_buf.o)
 .riscv.attributes
                0x00000000000016d8       0x32 ..\..\..\..\Libraries\libs\libbtstack.a(ble_adv0.o)
 .riscv.attributes
                0x000000000000170a       0x32 ..\..\..\..\Libraries\libs\libbtstack.a(extern_hfhs.o)
 .riscv.attributes
                0x000000000000173c       0x32 ..\..\..\..\Libraries\libs\libbtstack.a(l2cap_signaling.o)
 .riscv.attributes
                0x000000000000176e       0x32 ..\..\..\..\Libraries\libs\libbtstack.a(lc_hook.o)
 .riscv.attributes
                0x00000000000017a0       0x32 ..\..\..\..\Libraries\libs\libbtstack.a(lm_sco.o)
 .riscv.attributes
                0x00000000000017d2       0x32 ..\..\..\..\Libraries\libs\libbtstack.a(lc_util.o)
 .riscv.attributes
                0x0000000000001804       0x32 ..\..\..\..\Libraries\libs\libbtstack.a(lc_sniff.o)
 .riscv.attributes
                0x0000000000001836       0x32 ..\..\..\..\Libraries\libs\libbtstack.a(lc_sco.o)
 .riscv.attributes
                0x0000000000001868       0x32 ..\..\..\..\Libraries\libs\libbtstack.a(lc_proc.o)
 .riscv.attributes
                0x000000000000189a       0x32 ..\..\..\..\Libraries\libs\libbtstack.a(lc_lmppdu.o)
 .riscv.attributes
                0x00000000000018cc       0x32 ..\..\..\..\Libraries\libs\libbtstack.a(mgr_proc.o)
 .riscv.attributes
                0x00000000000018fe       0x32 ..\..\..\..\Libraries\libs\libbtstack.a(mgr_init.o)
 .riscv.attributes
                0x0000000000001930       0x32 ..\..\..\..\Libraries\libs\libbtstack.a(mgr_hci.o)
 .riscv.attributes
                0x0000000000001962       0x32 ..\..\..\..\Libraries\libs\libbtstack.a(ll_scan.o)
 .riscv.attributes
                0x0000000000001994       0x32 ..\..\..\..\Libraries\libs\libbtstack.a(ll_adv.o)
 .riscv.attributes
                0x00000000000019c6       0x32 ..\..\..\..\Libraries\libs\libbtstack.a(ll_proc.o)
 .riscv.attributes
                0x00000000000019f8       0x32 ..\..\..\..\Libraries\libs\libbtstack.a(ll_ping.o)
 .riscv.attributes
                0x0000000000001a2a       0x32 ..\..\..\..\Libraries\libs\libbtstack.a(ll_phy_upd.o)
 .riscv.attributes
                0x0000000000001a5c       0x32 ..\..\..\..\Libraries\libs\libbtstack.a(ll_past.o)
 .riscv.attributes
                0x0000000000001a8e       0x32 ..\..\..\..\Libraries\libs\libbtstack.a(ll_length.o)
 .riscv.attributes
                0x0000000000001ac0       0x32 ..\..\..\..\Libraries\libs\libbtstack.a(ll_feature.o)
 .riscv.attributes
                0x0000000000001af2       0x32 ..\..\..\..\Libraries\libs\libbtstack.a(ll_encrypt.o)
 .riscv.attributes
                0x0000000000001b24       0x32 ..\..\..\..\Libraries\libs\libbtstack.a(ll_disconnect.o)
 .riscv.attributes
                0x0000000000001b56       0x32 ..\..\..\..\Libraries\libs\libbtstack.a(ll_con_upd.o)
 .riscv.attributes
                0x0000000000001b88       0x32 ..\..\..\..\Libraries\libs\libbtstack.a(ll_cntl.o)
 .riscv.attributes
                0x0000000000001bba       0x32 ..\..\..\..\Libraries\libs\libbtstack.a(ll_clk_acc.o)
 .riscv.attributes
                0x0000000000001bec       0x32 ..\..\..\..\Libraries\libs\libbtstack.a(ll_chmap_upd.o)
 .riscv.attributes
                0x0000000000001c1e       0x32 ..\..\..\..\Libraries\libs\libbtstack.a(aes_rpa.o)
 .riscv.attributes
                0x0000000000001c50       0x32 ..\..\..\..\Libraries\libs\libbtstack.a(scan_hook.o)
 .riscv.attributes
                0x0000000000001c82       0x32 ..\..\..\..\Libraries\libs\libbtstack.a(adv_hook.o)
 .riscv.attributes
                0x0000000000001cb4       0x32 ..\..\..\..\Libraries\libs\libbtstack.a(ll_version.o)
 .riscv.attributes
                0x0000000000001ce6       0x32 ..\..\..\..\Libraries\libs\libbtstack.a(ll_pwr.o)
 .riscv.attributes
                0x0000000000001d18       0x32 ..\..\..\..\Libraries\libs\libdrivers.a(usb_device_hid.o)
 .riscv.attributes
                0x0000000000001d4a       0x32 ..\..\..\..\Libraries\libs\libdrivers.a(usb_device_printer.o)
 .riscv.attributes
                0x0000000000001d7c       0x32 ..\..\..\..\Libraries\libs\libdrivers.a(usb_device_run_loop.o)
 .riscv.attributes
                0x0000000000001dae       0x32 ..\..\..\..\Libraries\libs\libdrivers.a(usb_comm.o)
 .riscv.attributes
                0x0000000000001de0       0x32 ..\..\..\..\Libraries\libs\libdrivers.a(usb_device_ep.o)
